 cgamex86

 Timestamp is 4839b7c2 (Sun May 25 23:02:26 2008)

 Preferred load address is 30000000

 Start         Length     Name                   Class
 0001:00000000 00056194H .text                   CODE
 0002:00000000 0000014cH .idata$5                DATA
 0002:00000150 0000953aH .rdata                  DATA
 0002:0000968c 00000056H .rdata$debug            DATA
 0002:000096e4 00000004H .rtc$IAA                DATA
 0002:000096e8 00000004H .rtc$IZZ                DATA
 0002:000096ec 00000004H .rtc$TAA                DATA
 0002:000096f0 00000004H .rtc$TZZ                DATA
 0002:000096f4 00000014H .idata$2                DATA
 0002:00009708 00000014H .idata$3                DATA
 0002:0000971c 0000014cH .idata$4                DATA
 0002:00009868 000005f2H .idata$6                DATA
 0002:00009e60 00000059H .edata                  DATA
 0003:00000000 00000004H .CRT$XCA                DATA
 0003:00000004 00000004H .CRT$XCAA               DATA
 0003:00000008 00000004H .CRT$XCZ                DATA
 0003:0000000c 00000004H .CRT$XIA                DATA
 0003:00000010 00000010H .CRT$XIC                DATA
 0003:00000020 00000004H .CRT$XIZ                DATA
 0003:00000024 00000004H .CRT$XPA                DATA
 0003:00000028 00000004H .CRT$XPX                DATA
 0003:0000002c 00000004H .CRT$XPZ                DATA
 0003:00000030 00000004H .CRT$XTA                DATA
 0003:00000034 00000004H .CRT$XTZ                DATA
 0003:00000040 00003ef0H .data                   DATA
 0003:00003f40 0050ea54H .bss                    DATA

  Address         Publics by Value              Rva+Base     Lib:Object

 0000:00000000       ___safe_se_handler_table   00000000     <absolute>
 0000:00000000       __except_list              00000000     <absolute>
 0000:00000000       ___safe_se_handler_count   00000000     <absolute>
 0001:00000000       _BG_FindItemForPowerup     30001000 f   bg_misc.obj
 0001:00000080       _BG_FindItemForHoldable    30001080 f   bg_misc.obj
 0001:000000f0       _BG_FindItemForWeapon      300010f0 f   bg_misc.obj
 0001:00000150       _BG_FindItem               30001150 f   bg_misc.obj
 0001:000001a0       _BG_PlayerTouchesItem      300011a0 f   bg_misc.obj
 0001:00000260       _BG_CanItemBeGrabbed       30001260 f   bg_misc.obj
 0001:00000490       _BG_EvaluateTrajectory     30001490 f   bg_misc.obj
 0001:000006f0       _BG_EvaluateTrajectoryDelta 300016f0 f   bg_misc.obj
 0001:000008b0       _BG_AddPredictableEventToPlayerstate 300018b0 f   bg_misc.obj
 0001:00000960       _BG_TouchJumpPad           30001960 f   bg_misc.obj
 0001:00000a50       _BG_PlayerStateToEntityState 30001a50 f   bg_misc.obj
 0001:00000db0       _BG_PlayerStateToEntityStateExtraPolate 30001db0 f   bg_misc.obj
 0001:00001120       _PM_AddEvent               30002120 f   bg_pmove.obj
 0001:00001150       _PM_AddTouchEnt            30002150 f   bg_pmove.obj
 0001:000011e0       _PM_ClipVelocity           300021e0 f   bg_pmove.obj
 0001:00001280       _PM_UpdateViewAngles       30002280 f   bg_pmove.obj
 0001:00001380       _PmoveSingle               30002380 f   bg_pmove.obj
 0001:00004740       _Pmove                     30005740 f   bg_pmove.obj
 0001:00004830       _PM_SlideMove              30005830 f   bg_slidemove.obj
 0001:000050d0       _PM_StepSlideMove          300060d0 f   bg_slidemove.obj
 0001:000054f0       _CG_TargetCommand_f        300064f0 f   cg_consolecmds.obj
 0001:00005950       _CG_ConsoleCommand         30006950 f   cg_consolecmds.obj
 0001:000059c0       _CG_InitConsoleCommands    300069c0 f   cg_consolecmds.obj
 0001:00005b60       _CG_Draw3DModel            30006b60 f   cg_draw.obj
 0001:00005cc0       _CG_DrawHead               30006cc0 f   cg_draw.obj
 0001:00005e10       _CG_DrawFlagModel          30006e10 f   cg_draw.obj
 0001:00005fb0       _CG_DrawTeamBackground     30006fb0 f   cg_draw.obj
 0001:00006050       _CG_AddLagometerFrameInfo  30007050 f   cg_draw.obj
 0001:00006090       _CG_AddLagometerSnapshotInfo 30007090 f   cg_draw.obj
 0001:00006100       _CG_CenterPrint            30007100 f   cg_draw.obj
 0001:00006180       _CG_DrawActive             30007180 f   cg_draw.obj
 0001:00009860       _CG_AdjustFrom640          3000a860 f   cg_drawtools.obj
 0001:000098b0       _CG_FillRect               3000a8b0 f   cg_drawtools.obj
 0001:00009920       _CG_DrawSides              3000a920 f   cg_drawtools.obj
 0001:000099b0       _CG_DrawTopBottom          3000a9b0 f   cg_drawtools.obj
 0001:00009a40       _CG_DrawRect               3000aa40 f   cg_drawtools.obj
 0001:00009aa0       _CG_DrawPic                3000aaa0 f   cg_drawtools.obj
 0001:00009b00       _CG_DrawChar               3000ab00 f   cg_drawtools.obj
 0001:00009bd0       _CG_DrawStringExt          3000abd0 f   cg_drawtools.obj
 0001:00009dc0       _CG_DrawBigString          3000adc0 f   cg_drawtools.obj
 0001:00009e10       _CG_DrawBigStringColor     3000ae10 f   cg_drawtools.obj
 0001:00009e50       _CG_DrawSmallString        3000ae50 f   cg_drawtools.obj
 0001:00009ea0       _CG_DrawSmallStringColor   3000aea0 f   cg_drawtools.obj
 0001:00009ee0       _CG_DrawStrlen             3000aee0 f   cg_drawtools.obj
 0001:00009f60       _CG_TileClear              3000af60 f   cg_drawtools.obj
 0001:0000a0f0       _CG_FadeColor              3000b0f0 f   cg_drawtools.obj
 0001:0000a180       _CG_TeamColor              3000b180 f   cg_drawtools.obj
 0001:0000a1d0       _CG_GetColorForHealth      3000b1d0 f   cg_drawtools.obj
 0001:0000a2e0       _CG_ColorForHealth         3000b2e0 f   cg_drawtools.obj
 0001:0000a320       _UI_DrawBannerString       3000b320 f   cg_drawtools.obj
 0001:0000a5b0       _UI_ProportionalStringWidth 3000b5b0 f   cg_drawtools.obj
 0001:0000a630       _UI_ProportionalSizeScale  3000b630 f   cg_drawtools.obj
 0001:0000a660       _UI_DrawProportionalString 3000b660 f   cg_drawtools.obj
 0001:0000aa20       _CG_BubbleTrail            3000ba20 f   cg_effects.obj
 0001:0000ace0       _CG_SmokePuff              3000bce0 f   cg_effects.obj
 0001:0000af10       _CG_SpawnEffect            3000bf10 f   cg_effects.obj
 0001:0000b030       _CG_ScorePlum              3000c030 f   cg_effects.obj
 0001:0000b1b0       _CG_MakeExplosion          3000c1b0 f   cg_effects.obj
 0001:0000b3c0       _CG_Bleed                  3000c3c0 f   cg_effects.obj
 0001:0000b4b0       _CG_LaunchGib              3000c4b0 f   cg_effects.obj
 0001:0000b5f0       _CG_GibPlayer              3000c5f0 f   cg_effects.obj
 0001:0000bcf0       _CG_LaunchExplode          3000ccf0 f   cg_effects.obj
 0001:0000be30       _CG_BigExplode             3000ce30 f   cg_effects.obj
 0001:0000c1d0       _CG_PositionEntityOnTag    3000d1d0 f   cg_ents.obj
 0001:0000c2e0       _CG_PositionRotatedEntityOnTag 3000d2e0 f   cg_ents.obj
 0001:0000c400       _CG_SetEntitySoundPosition 3000d400 f   cg_ents.obj
 0001:0000c4a0       _CG_Beam                   3000d4a0 f   cg_ents.obj
 0001:0000c550       _CG_AdjustPositionForMover 3000d550 f   cg_ents.obj
 0001:0000c6a0       _CG_AddPacketEntities      3000d6a0 f   cg_ents.obj
 0001:0000dd00       _CG_PlaceString            3000ed00 f   cg_event.obj
 0001:0000de50       _CG_PainEvent              3000ee50 f   cg_event.obj
 0001:0000df00       _CG_EntityEvent            3000ef00 f   cg_event.obj
 0001:0000fc00       _CG_CheckEvents            30010c00 f   cg_event.obj
 0001:0000fcf0       _CG_LoadingString          30010cf0 f   cg_info.obj
 0001:0000fd20       _CG_LoadingItem            30010d20 f   cg_info.obj
 0001:0000fd90       _CG_LoadingClient          30010d90 f   cg_info.obj
 0001:0000ff70       _CG_DrawInformation        30010f70 f   cg_info.obj
 0001:00010500       _CG_InitLocalEntities      30011500 f   cg_localents.obj
 0001:00010580       _CG_FreeLocalEntity        30011580 f   cg_localents.obj
 0001:000105e0       _CG_AllocLocalEntity       300115e0 f   cg_localents.obj
 0001:00010660       _CG_BloodTrail             30011660 f   cg_localents.obj
 0001:00010720       _CG_FragmentBounceMark     30011720 f   cg_localents.obj
 0001:00010830       _CG_FragmentBounceSound    30011830 f   cg_localents.obj
 0001:000108b0       _CG_ReflectVelocity        300118b0 f   cg_localents.obj
 0001:00010a30       _CG_AddFragment            30011a30 f   cg_localents.obj
 0001:00010c70       _CG_AddFadeRGB             30011c70 f   cg_localents.obj
 0001:00010d10       _CG_AddScorePlum           30011d10 f   cg_localents.obj
 0001:000111a0       _CG_AddLocalEntities       300121a0 f   cg_localents.obj
 0001:00011880       _vmMain                    30012880 f   cg_main.obj
 0001:00011970       _CG_RegisterCvars          30012970 f   cg_main.obj
 0001:00011a70       _CG_UpdateCvars            30012a70 f   cg_main.obj
 0001:00011ba0       _CG_CrosshairPlayer        30012ba0 f   cg_main.obj
 0001:00011bd0       _CG_LastAttacker           30012bd0 f   cg_main.obj
 0001:00011c00       _CG_Printf                 30012c00 f   cg_main.obj
 0001:00011c50       _CG_Error                  30012c50 f   cg_main.obj
 0001:00011ca0       _Com_Error                 30012ca0 f   cg_main.obj
 0001:00011cf0       _Com_Printf                30012cf0 f   cg_main.obj
 0001:00011d40       _CG_Argv                   30012d40 f   cg_main.obj
 0001:00011d70       _CG_BuildSpectatorString   30012d70 f   cg_main.obj
 0001:00011e30       _CG_ConfigString           30012e30 f   cg_main.obj
 0001:00011e70       _CG_StartMusic             30012e70 f   cg_main.obj
 0001:00011ee0       _CG_Init                   30012ee0 f   cg_main.obj
 0001:00013400       _CG_Shutdown               30014400 f   cg_main.obj
 0001:00013410       _CG_EventHandling          30014410 f   cg_main.obj
 0001:00013420       _CG_KeyEvent               30014420 f   cg_main.obj
 0001:00013430       _CG_MouseEvent             30014430 f   cg_main.obj
 0001:00013440       _CG_InitMarkPolys          30014440 f   cg_marks.obj
 0001:000134c0       _CG_FreeMarkPoly           300144c0 f   cg_marks.obj
 0001:00013520       _CG_AllocMark              30014520 f   cg_marks.obj
 0001:000135c0       _CG_ImpactMark             300145c0 f   cg_marks.obj
 0001:00013aa0       _CG_AddMarks               30014aa0 f   cg_marks.obj
 0001:00013ce0       _CG_ClearParticles         30014ce0 f   cg_marks.obj
 0001:00013e10       _CG_AddParticleToScene     30014e10 f   cg_marks.obj
 0001:00016100       _CG_AddParticles           30017100 f   cg_marks.obj
 0001:000164f0       _CG_ParticleSnowFlurry     300174f0 f   cg_marks.obj
 0001:000167a0       _CG_ParticleSnow           300177a0 f   cg_marks.obj
 0001:000169f0       _CG_ParticleBubble         300179f0 f   cg_marks.obj
 0001:00016c90       _CG_ParticleSmoke          30017c90 f   cg_marks.obj
 0001:00016e60       _CG_ParticleBulletDebris   30017e60 f   cg_marks.obj
 0001:00016fc0       _CG_ParticleExplosion      30017fc0 f   cg_marks.obj
 0001:000171b0       _CG_AddParticleShrapnel    300181b0 f   cg_marks.obj
 0001:000171c0       _CG_NewParticleArea        300181c0 f   cg_marks.obj
 0001:000173d0       _CG_SnowLink               300183d0 f   cg_marks.obj
 0001:00017450       _CG_ParticleImpactSmokePuff 30018450 f   cg_marks.obj
 0001:00017610       _CG_Particle_Bleed         30018610 f   cg_marks.obj
 0001:000177b0       _CG_Particle_OilParticle   300187b0 f   cg_marks.obj
 0001:00017970       _CG_Particle_OilSlick      30018970 f   cg_marks.obj
 0001:00017bc0       _CG_OilSlickRemove         30018bc0 f   cg_marks.obj
 0001:00017c50       _ValidBloodPool            30018c50 f   cg_marks.obj
 0001:00017e30       _CG_BloodPool              30018e30 f   cg_marks.obj
 0001:00018010       _CG_ParticleBloodCloud     30019010 f   cg_marks.obj
 0001:00018280       _CG_ParticleSparks         30019280 f   cg_marks.obj
 0001:00018510       _CG_ParticleDust           30019510 f   cg_marks.obj
 0001:00018900       _CG_ParticleMisc           30019900 f   cg_marks.obj
 0001:00018a20       _CG_CustomSound            30019a20 f   cg_players.obj
 0001:00018ae0       _CG_NewClientInfo          30019ae0 f   cg_players.obj
 0001:0001acf0       _CG_LoadDeferredPlayers    3001bcf0 f   cg_players.obj
 0001:0001ad80       _CG_AddRefEntityWithPowerups 3001bd80 f   cg_players.obj
 0001:0001ae70       _CG_LightVerts             3001be70 f   cg_players.obj
 0001:0001aff0       _CG_Player                 3001bff0 f   cg_players.obj
 0001:0001cd20       _CG_ResetPlayerEntity      3001dd20 f   cg_players.obj
 0001:0001cf90       _CG_CheckAmmo              3001df90 f   cg_playerstate.obj
 0001:0001d090       _CG_DamageFeedback         3001e090 f   cg_playerstate.obj
 0001:0001d3b0       _CG_Respawn                3001e3b0 f   cg_playerstate.obj
 0001:0001d3f0       _CG_CheckPlayerstateEvents 3001e3f0 f   cg_playerstate.obj
 0001:0001d540       _CG_CheckChangedPredictableEvents 3001e540 f   cg_playerstate.obj
 0001:0001d630       _CG_CheckLocalSounds       3001e630 f   cg_playerstate.obj
 0001:0001dc40       _CG_TransitionPlayerState  3001ec40 f   cg_playerstate.obj
 0001:0001dd70       _CG_BuildSolidList         3001ed70 f   cg_predict.obj
 0001:0001de80       _CG_Trace                  3001ee80 f   cg_predict.obj
 0001:0001e130       _CG_PointContents          3001f130 f   cg_predict.obj
 0001:0001e1f0       _CG_PredictPlayerState     3001f1f0 f   cg_predict.obj
 0001:0001ed10       _CG_DrawOldScoreboard      3001fd10 f   cg_scoreboard.obj
 0001:0001fa60       _CG_DrawOldTourneyScoreboard 30020a60 f   cg_scoreboard.obj
 0001:0001fdd0       _CG_ParseServerinfo        30020dd0 f   cg_servercmds.obj
 0001:0001ff80       _CG_SetConfigValues        30020f80 f   cg_servercmds.obj
 0001:00020030       _CG_ShaderStateChanged     30021030 f   cg_servercmds.obj
 0001:000201f0       _CG_ParseVoiceChats        300211f0 f   cg_servercmds.obj
 0001:000206a0       _CG_LoadVoiceChats         300216a0 f   cg_servercmds.obj
 0001:00020770       _CG_HeadModelVoiceChats    30021770 f   cg_servercmds.obj
 0001:000208b0       _CG_GetVoiceChat           300218b0 f   cg_servercmds.obj
 0001:00020980       _CG_VoiceChatListForClient 30021980 f   cg_servercmds.obj
 0001:00020d20       _CG_PlayVoiceChat          30021d20 f   cg_servercmds.obj
 0001:00020d30       _CG_PlayBufferedVoiceChats 30021d30 f   cg_servercmds.obj
 0001:00020d40       _CG_AddBufferedVoiceChat   30021d40 f   cg_servercmds.obj
 0001:00020d50       _CG_VoiceChatLocal         30021d50 f   cg_servercmds.obj
 0001:00020d60       _CG_VoiceChat              30021d60 f   cg_servercmds.obj
 0001:00020d70       _CG_ExecuteNewServerCommands 30021d70 f   cg_servercmds.obj
 0001:00021c50       _CG_SetInitialSnapshot     30022c50 f   cg_snapshot.obj
 0001:00021e10       _CG_ProcessSnapshots       30022e10 f   cg_snapshot.obj
 0001:000223e0       _dllEntry                  300233e0 f   cg_syscalls.obj
 0001:00022400       _PASSFLOAT                 30023400 f   cg_syscalls.obj
 0001:00022420       _trap_Print                30023420 f   cg_syscalls.obj
 0001:00022440       _trap_Error                30023440 f   cg_syscalls.obj
 0001:00022460       _trap_Milliseconds         30023460 f   cg_syscalls.obj
 0001:00022480       _trap_Cvar_Register        30023480 f   cg_syscalls.obj
 0001:000224b0       _trap_Cvar_Update          300234b0 f   cg_syscalls.obj
 0001:000224d0       _trap_Cvar_Set             300234d0 f   cg_syscalls.obj
 0001:00022500       _trap_Cvar_VariableStringBuffer 30023500 f   cg_syscalls.obj
 0001:00022530       _trap_Argc                 30023530 f   cg_syscalls.obj
 0001:00022550       _trap_Argv                 30023550 f   cg_syscalls.obj
 0001:00022580       _trap_Args                 30023580 f   cg_syscalls.obj
 0001:000225b0       _trap_FS_FOpenFile         300235b0 f   cg_syscalls.obj
 0001:000225e0       _trap_FS_Read              300235e0 f   cg_syscalls.obj
 0001:00022610       _trap_FS_Write             30023610 f   cg_syscalls.obj
 0001:00022640       _trap_FS_FCloseFile        30023640 f   cg_syscalls.obj
 0001:00022660       _trap_FS_Seek              30023660 f   cg_syscalls.obj
 0001:00022690       _trap_SendConsoleCommand   30023690 f   cg_syscalls.obj
 0001:000226b0       _trap_AddCommand           300236b0 f   cg_syscalls.obj
 0001:000226d0       _trap_RemoveCommand        300236d0 f   cg_syscalls.obj
 0001:000226f0       _trap_SendClientCommand    300236f0 f   cg_syscalls.obj
 0001:00022710       _trap_UpdateScreen         30023710 f   cg_syscalls.obj
 0001:00022730       _trap_CM_LoadMap           30023730 f   cg_syscalls.obj
 0001:00022750       _trap_CM_NumInlineModels   30023750 f   cg_syscalls.obj
 0001:00022770       _trap_CM_InlineModel       30023770 f   cg_syscalls.obj
 0001:00022790       _trap_CM_TempBoxModel      30023790 f   cg_syscalls.obj
 0001:000227c0       _trap_CM_TempCapsuleModel  300237c0 f   cg_syscalls.obj
 0001:000227f0       _trap_CM_PointContents     300237f0 f   cg_syscalls.obj
 0001:00022820       _trap_CM_TransformedPointContents 30023820 f   cg_syscalls.obj
 0001:00022850       _trap_CM_BoxTrace          30023850 f   cg_syscalls.obj
 0001:00022890       _trap_CM_CapsuleTrace      30023890 f   cg_syscalls.obj
 0001:000228d0       _trap_CM_TransformedBoxTrace 300238d0 f   cg_syscalls.obj
 0001:00022910       _trap_CM_TransformedCapsuleTrace 30023910 f   cg_syscalls.obj
 0001:00022950       _trap_CM_MarkFragments     30023950 f   cg_syscalls.obj
 0001:00022990       _trap_S_StartSound         30023990 f   cg_syscalls.obj
 0001:000229c0       _trap_S_StartLocalSound    300239c0 f   cg_syscalls.obj
 0001:000229f0       _trap_S_ClearLoopingSounds 300239f0 f   cg_syscalls.obj
 0001:00022a10       _trap_S_AddLoopingSound    30023a10 f   cg_syscalls.obj
 0001:00022a40       _trap_S_AddRealLoopingSound 30023a40 f   cg_syscalls.obj
 0001:00022a70       _trap_S_StopLoopingSound   30023a70 f   cg_syscalls.obj
 0001:00022a90       _trap_S_UpdateEntityPosition 30023a90 f   cg_syscalls.obj
 0001:00022ac0       _trap_S_Respatialize       30023ac0 f   cg_syscalls.obj
 0001:00022af0       _trap_S_RegisterSound      30023af0 f   cg_syscalls.obj
 0001:00022b20       _trap_S_StartBackgroundTrack 30023b20 f   cg_syscalls.obj
 0001:00022b50       _trap_R_LoadWorldMap       30023b50 f   cg_syscalls.obj
 0001:00022b70       _trap_R_RegisterModel      30023b70 f   cg_syscalls.obj
 0001:00022b90       _trap_R_RegisterSkin       30023b90 f   cg_syscalls.obj
 0001:00022bb0       _trap_R_RegisterShader     30023bb0 f   cg_syscalls.obj
 0001:00022bd0       _trap_R_RegisterShaderNoMip 30023bd0 f   cg_syscalls.obj
 0001:00022bf0       _trap_R_RegisterFont       30023bf0 f   cg_syscalls.obj
 0001:00022c20       _trap_R_ClearScene         30023c20 f   cg_syscalls.obj
 0001:00022c40       _trap_R_AddRefEntityToScene 30023c40 f   cg_syscalls.obj
 0001:00022c60       _trap_R_AddPolyToScene     30023c60 f   cg_syscalls.obj
 0001:00022c90       _trap_R_AddPolysToScene    30023c90 f   cg_syscalls.obj
 0001:00022cc0       _trap_R_LightForPoint      30023cc0 f   cg_syscalls.obj
 0001:00022cf0       _trap_R_AddLightToScene    30023cf0 f   cg_syscalls.obj
 0001:00022d50       _trap_R_AddAdditiveLightToScene 30023d50 f   cg_syscalls.obj
 0001:00022db0       _trap_R_RenderScene        30023db0 f   cg_syscalls.obj
 0001:00022dd0       _trap_R_SetColor           30023dd0 f   cg_syscalls.obj
 0001:00022df0       _trap_R_DrawStretchPic     30023df0 f   cg_syscalls.obj
 0001:00022e80       _trap_R_ModelBounds        30023e80 f   cg_syscalls.obj
 0001:00022eb0       _trap_R_LerpTag            30023eb0 f   cg_syscalls.obj
 0001:00022ef0       _trap_R_RemapShader        30023ef0 f   cg_syscalls.obj
 0001:00022f20       _trap_GetGlconfig          30023f20 f   cg_syscalls.obj
 0001:00022f40       _trap_GetGameState         30023f40 f   cg_syscalls.obj
 0001:00022f60       _trap_GetCurrentSnapshotNumber 30023f60 f   cg_syscalls.obj
 0001:00022f90       _trap_GetSnapshot          30023f90 f   cg_syscalls.obj
 0001:00022fc0       _trap_GetServerCommand     30023fc0 f   cg_syscalls.obj
 0001:00022fe0       _trap_GetCurrentCmdNumber  30023fe0 f   cg_syscalls.obj
 0001:00023000       _trap_GetUserCmd           30024000 f   cg_syscalls.obj
 0001:00023030       _trap_SetUserCmdValue      30024030 f   cg_syscalls.obj
 0001:00023060       _testPrintInt              30024060 f   cg_syscalls.obj
 0001:00023090       _testPrintFloat            30024090 f   cg_syscalls.obj
 0001:000230c0       _trap_MemoryRemaining      300240c0 f   cg_syscalls.obj
 0001:000230e0       _trap_Key_IsDown           300240e0 f   cg_syscalls.obj
 0001:00023100       _trap_Key_GetCatcher       30024100 f   cg_syscalls.obj
 0001:00023120       _trap_Key_SetCatcher       30024120 f   cg_syscalls.obj
 0001:00023140       _trap_Key_GetKey           30024140 f   cg_syscalls.obj
 0001:00023160       _trap_PC_AddGlobalDefine   30024160 f   cg_syscalls.obj
 0001:00023180       _trap_PC_LoadSource        30024180 f   cg_syscalls.obj
 0001:000231a0       _trap_PC_FreeSource        300241a0 f   cg_syscalls.obj
 0001:000231c0       _trap_PC_ReadToken         300241c0 f   cg_syscalls.obj
 0001:000231f0       _trap_PC_SourceFileAndLine 300241f0 f   cg_syscalls.obj
 0001:00023220       _trap_S_StopBackgroundTrack 30024220 f   cg_syscalls.obj
 0001:00023240       _trap_RealTime             30024240 f   cg_syscalls.obj
 0001:00023260       _trap_SnapVector           30024260 f   cg_syscalls.obj
 0001:00023280       _trap_CIN_PlayCinematic    30024280 f   cg_syscalls.obj
 0001:000232c0       _trap_CIN_StopCinematic    300242c0 f   cg_syscalls.obj
 0001:000232e0       _trap_CIN_RunCinematic     300242e0 f   cg_syscalls.obj
 0001:00023300       _trap_CIN_DrawCinematic    30024300 f   cg_syscalls.obj
 0001:00023320       _trap_CIN_SetExtents       30024320 f   cg_syscalls.obj
 0001:00023350       _trap_GetEntityToken       30024350 f   cg_syscalls.obj
 0001:00023380       _trap_R_inPVS              30024380 f   cg_syscalls.obj
 0001:000233b0       _CG_TestModel_f            300243b0 f   cg_view.obj
 0001:000234f0       _CG_TestGun_f              300244f0 f   cg_view.obj
 0001:00023520       _CG_TestModelNextFrame_f   30024520 f   cg_view.obj
 0001:00023550       _CG_TestModelPrevFrame_f   30024550 f   cg_view.obj
 0001:00023590       _CG_TestModelNextSkin_f    30024590 f   cg_view.obj
 0001:000235c0       _CG_TestModelPrevSkin_f    300245c0 f   cg_view.obj
 0001:00023600       _CG_ZoomDown_f             30024600 f   cg_view.obj
 0001:00023630       _CG_ZoomUp_f               30024630 f   cg_view.obj
 0001:00023660       _CG_AddBufferedSound       30024660 f   cg_view.obj
 0001:000236c0       _CG_DrawActiveFrame        300246c0 f   cg_view.obj
 0001:00024b10       _CG_RailTrail              30025b10 f   cg_weapons.obj
 0001:00025250       _CG_GrappleTrail           30026250 f   cg_weapons.obj
 0001:00025470       _CG_RegisterWeapon         30026470 f   cg_weapons.obj
 0001:00026a50       _CG_RegisterItemVisuals    30027a50 f   cg_weapons.obj
 0001:00026b60       _CG_AddPlayerWeapon        30027b60 f   cg_weapons.obj
 0001:00027770       _CG_AddViewWeapon          30028770 f   cg_weapons.obj
 0001:00027d00       _CG_DrawWeaponSelect       30028d00 f   cg_weapons.obj
 0001:00027f20       _CG_NextWeapon_f           30028f20 f   cg_weapons.obj
 0001:00028020       _CG_PrevWeapon_f           30029020 f   cg_weapons.obj
 0001:000280d0       _CG_Weapon_f               300290d0 f   cg_weapons.obj
 0001:00028150       _CG_OutOfAmmoChange        30029150 f   cg_weapons.obj
 0001:000281a0       _CG_FireWeapon             300291a0 f   cg_weapons.obj
 0001:000282e0       _CG_MissileHitWall         300292e0 f   cg_weapons.obj
 0001:000287a0       _CG_MissileHitPlayer       300297a0 f   cg_weapons.obj
 0001:000287f0       _CG_ShotgunFire            300297f0 f   cg_weapons.obj
 0001:00028c40       _CG_Tracer                 30029c40 f   cg_weapons.obj
 0001:00029020       _CG_Bullet                 3002a020 f   cg_weapons.obj
 0001:00029340       _Q_rand                    3002a340 f   q_math.obj
 0001:00029370       _Q_random                  3002a370 f   q_math.obj
 0001:000293a0       _Q_crandom                 3002a3a0 f   q_math.obj
 0001:000293d0       _ClampChar                 3002a3d0 f   q_math.obj
 0001:00029400       _ClampShort                3002a400 f   q_math.obj
 0001:00029440       _DirToByte                 3002a440 f   q_math.obj
 0001:000294e0       _ByteToDir                 3002a4e0 f   q_math.obj
 0001:00029560       _ColorBytes3               3002a560 f   q_math.obj
 0001:000295b0       _ColorBytes4               3002a5b0 f   q_math.obj
 0001:00029610       _NormalizeColor            3002a610 f   q_math.obj
 0001:000296c0       _PlaneFromPoints           3002a6c0 f   q_math.obj
 0001:00029800       _RotatePointAroundVector   3002a800 f   q_math.obj
 0001:00029a30       _RotateAroundDirection     3002aa30 f   q_math.obj
 0001:00029ac0       _vectoangles               3002aac0 f   q_math.obj
 0001:00029c40       _AnglesToAxis              3002ac40 f   q_math.obj
 0001:00029ca0       _AxisClear                 3002aca0 f   q_math.obj
 0001:00029d10       _AxisCopy                  3002ad10 f   q_math.obj
 0001:00029d90       _ProjectPointOnPlane       3002ad90 f   q_math.obj
 0001:00029e90       _MakeNormalVectors         3002ae90 f   q_math.obj
 0001:00029f60       _VectorRotate              3002af60 f   q_math.obj
 0001:0002a000       _Q_rsqrt                   3002b000 f   q_math.obj
 0001:0002a060       _Q_fabs                    3002b060 f   q_math.obj
 0001:0002a090       _LerpAngle                 3002b090 f   q_math.obj
 0001:0002a0f0       _AngleSubtract             3002b0f0 f   q_math.obj
 0001:0002a150       _AnglesSubtract            3002b150 f   q_math.obj
 0001:0002a1c0       _AngleMod                  3002b1c0 f   q_math.obj
 0001:0002a200       _AngleNormalize360         3002b200 f   q_math.obj
 0001:0002a240       _AngleNormalize180         3002b240 f   q_math.obj
 0001:0002a280       _AngleDelta                3002b280 f   q_math.obj
 0001:0002a2b0       _SetPlaneSignbits          3002b2b0 f   q_math.obj
 0001:0002a310       _BoxOnPlaneSide            3002b310 f   q_math.obj
 0001:0002a550       _RadiusFromBounds          3002b550 f   q_math.obj
 0001:0002a630       _ClearBounds               3002b630 f   q_math.obj
 0001:0002a680       _AddPointToBounds          3002b680 f   q_math.obj
 0001:0002a750       _VectorNormalize           3002b750 f   q_math.obj
 0001:0002a7f0       _VectorNormalize2          3002b7f0 f   q_math.obj
 0001:0002a8b0       __VectorMA                 3002b8b0 f   q_math.obj
 0001:0002a900       __DotProduct               3002b900 f   q_math.obj
 0001:0002a940       __VectorSubtract           3002b940 f   q_math.obj
 0001:0002a990       __VectorAdd                3002b990 f   q_math.obj
 0001:0002a9e0       __VectorCopy               3002b9e0 f   q_math.obj
 0001:0002aa20       __VectorScale              3002ba20 f   q_math.obj
 0001:0002aa60       _Vector4Scale              3002ba60 f   q_math.obj
 0001:0002aab0       _Q_log2                    3002bab0 f   q_math.obj
 0001:0002aaf0       _MatrixMultiply            3002baf0 f   q_math.obj
 0001:0002aca0       _AngleVectors              3002bca0 f   q_math.obj
 0001:0002ae90       _PerpendicularVector       3002be90 f   q_math.obj
 0001:0002af50       _Com_Clamp                 3002bf50 f   q_shared.obj
 0001:0002af90       _COM_SkipPath              3002bf90 f   q_shared.obj
 0001:0002afe0       _COM_StripExtension        3002bfe0 f   q_shared.obj
 0001:0002b030       _COM_DefaultExtension      3002c030 f   q_shared.obj
 0001:0002b0c0       _ShortSwap                 3002c0c0 f   q_shared.obj
 0001:0002b100       _ShortNoSwap               3002c100 f   q_shared.obj
 0001:0002b120       _LongSwap                  3002c120 f   q_shared.obj
 0001:0002b190       _LongNoSwap                3002c190 f   q_shared.obj
 0001:0002b1b0       _Long64Swap                3002c1b0 f   q_shared.obj
 0001:0002b200       _Long64NoSwap              3002c200 f   q_shared.obj
 0001:0002b220       _FloatSwap                 3002c220 f   q_shared.obj
 0001:0002b250       _FloatNoSwap               3002c250 f   q_shared.obj
 0001:0002b270       _COM_BeginParseSession     3002c270 f   q_shared.obj
 0001:0002b2b0       _COM_GetCurrentParseLine   3002c2b0 f   q_shared.obj
 0001:0002b2d0       _COM_Parse                 3002c2d0 f   q_shared.obj
 0001:0002b2f0       _COM_ParseError            3002c2f0 f   q_shared.obj
 0001:0002b340       _COM_ParseWarning          3002c340 f   q_shared.obj
 0001:0002b390       _COM_Compress              3002c390 f   q_shared.obj
 0001:0002b590       _COM_ParseExt              3002c590 f   q_shared.obj
 0001:0002b820       _COM_MatchToken            3002c820 f   q_shared.obj
 0001:0002b870       _SkipBracedSection         3002c870 f   q_shared.obj
 0001:0002b8e0       _SkipRestOfLine            3002c8e0 f   q_shared.obj
 0001:0002b930       _Parse1DMatrix             3002c930 f   q_shared.obj
 0001:0002b9b0       _Parse2DMatrix             3002c9b0 f   q_shared.obj
 0001:0002ba20       _Parse3DMatrix             3002ca20 f   q_shared.obj
 0001:0002baa0       _Q_isprint                 3002caa0 f   q_shared.obj
 0001:0002bad0       _Q_islower                 3002cad0 f   q_shared.obj
 0001:0002bb00       _Q_isupper                 3002cb00 f   q_shared.obj
 0001:0002bb30       _Q_isalpha                 3002cb30 f   q_shared.obj
 0001:0002bb70       _Q_strrchr                 3002cb70 f   q_shared.obj
 0001:0002bbd0       _Q_strncpyz                3002cbd0 f   q_shared.obj
 0001:0002bc40       _Q_stricmpn                3002cc40 f   q_shared.obj
 0001:0002bd10       _Q_strncmp                 3002cd10 f   q_shared.obj
 0001:0002bd80       _Q_stricmp                 3002cd80 f   q_shared.obj
 0001:0002bdc0       _Q_strlwr                  3002cdc0 f   q_shared.obj
 0001:0002be10       _Q_strupr                  3002ce10 f   q_shared.obj
 0001:0002be60       _Q_strcat                  3002ce60 f   q_shared.obj
 0001:0002beb0       _Q_PrintStrlen             3002ceb0 f   q_shared.obj
 0001:0002bf30       _Q_CleanStr                3002cf30 f   q_shared.obj
 0001:0002bfc0       _Com_sprintf               3002cfc0 f   q_shared.obj
 0001:0002c050       _va                        3002d050 f   q_shared.obj
 0001:0002c0b0       _Info_ValueForKey          3002d0b0 f   q_shared.obj
 0001:0002c230       _Info_NextPair             3002d230 f   q_shared.obj
 0001:0002c310       _Info_RemoveKey            3002d310 f   q_shared.obj
 0001:0002c480       _Info_RemoveKey_Big        3002d480 f   q_shared.obj
 0001:0002c5f0       _Info_Validate             3002d5f0 f   q_shared.obj
 0001:0002c640       _Info_SetValueForKey       3002d640 f   q_shared.obj
 0001:0002c7c0       _Info_SetValueForKey_Big   3002d7c0 f   q_shared.obj
 0001:0002c930       _UI_Alloc                  3002d930 f   ui_shared.obj
 0001:0002c9b0       _UI_InitMemory             3002d9b0 f   ui_shared.obj
 0001:0002c9e0       _UI_OutOfMemory            3002d9e0 f   ui_shared.obj
 0001:0002ca00       _String_Alloc              3002da00 f   ui_shared.obj
 0001:0002cbd0       _String_Report             3002dbd0 f   ui_shared.obj
 0001:0002cc80       _String_Init               3002dc80 f   ui_shared.obj
 0001:0002cd10       _PC_SourceWarning          3002dd10 f   ui_shared.obj
 0001:0002cd90       _PC_SourceError            3002dd90 f   ui_shared.obj
 0001:0002ce10       _LerpColor                 3002de10 f   ui_shared.obj
 0001:0002ceb0       _Float_Parse               3002deb0 f   ui_shared.obj
 0001:0002cf00       _PC_Float_Parse            3002df00 f   ui_shared.obj
 0001:0002cfc0       _Color_Parse               3002dfc0 f   ui_shared.obj
 0001:0002d020       _PC_Color_Parse            3002e020 f   ui_shared.obj
 0001:0002d080       _Int_Parse                 3002e080 f   ui_shared.obj
 0001:0002d0d0       _PC_Int_Parse              3002e0d0 f   ui_shared.obj
 0001:0002d190       _Rect_Parse                3002e190 f   ui_shared.obj
 0001:0002d210       _PC_Rect_Parse             3002e210 f   ui_shared.obj
 0001:0002d290       _String_Parse              3002e290 f   ui_shared.obj
 0001:0002d2e0       _PC_String_Parse           3002e2e0 f   ui_shared.obj
 0001:0002d330       _PC_Script_Parse           3002e330 f   ui_shared.obj
 0001:0002d470       _Init_Display              3002e470 f   ui_shared.obj
 0001:0002d490       _GradientBar_Paint         3002e490 f   ui_shared.obj
 0001:0002d4f0       _Window_Init               3002e4f0 f   ui_shared.obj
 0001:0002d550       _Fade                      3002e550 f   ui_shared.obj
 0001:0002d610       _Window_Paint              3002e610 f   ui_shared.obj
 0001:0002db00       _Item_SetScreenCoords      3002eb00 f   ui_shared.obj
 0001:0002db90       _Item_UpdatePosition       3002eb90 f   ui_shared.obj
 0001:0002dc10       _Menu_UpdatePosition       3002ec10 f   ui_shared.obj
 0001:0002dca0       _Menu_PostParse            3002eca0 f   ui_shared.obj
 0001:0002dd00       _Menu_ClearFocus           3002ed00 f   ui_shared.obj
 0001:0002dde0       _IsVisible                 3002ede0 f   ui_shared.obj
 0001:0002de20       _Rect_ContainsPoint        3002ee20 f   ui_shared.obj
 0001:0002de90       _Menu_ItemsMatchingGroup   3002ee90 f   ui_shared.obj
 0001:0002df30       _Menu_GetMatchingItemByNumber 3002ef30 f   ui_shared.obj
 0001:0002dff0       _Script_SetColor           3002eff0 f   ui_shared.obj
 0001:0002e0f0       _Script_SetAsset           3002f0f0 f   ui_shared.obj
 0001:0002e110       _Script_SetBackground      3002f110 f   ui_shared.obj
 0001:0002e150       _Menu_FindItemByName       3002f150 f   ui_shared.obj
 0001:0002e1d0       _Script_SetTeamColor       3002f1d0 f   ui_shared.obj
 0001:0002e230       _Script_SetItemColor       3002f230 f   ui_shared.obj
 0001:0002e3a0       _Menu_ShowItemByName       3002f3a0 f   ui_shared.obj
 0001:0002e450       _Menu_FadeItemByName       3002f450 f   ui_shared.obj
 0001:0002e4f0       _Menus_FindByName          3002f4f0 f   ui_shared.obj
 0001:0002e560       _Menus_ShowByName          3002f560 f   ui_shared.obj
 0001:0002e5a0       _Menus_OpenByName          3002f5a0 f   ui_shared.obj
 0001:0002e5c0       _Menus_CloseByName         3002f5c0 f   ui_shared.obj
 0001:0002e660       _Menus_CloseAll            3002f660 f   ui_shared.obj
 0001:0002e6d0       _Script_Show               3002f6d0 f   ui_shared.obj
 0001:0002e710       _Script_Hide               3002f710 f   ui_shared.obj
 0001:0002e750       _Script_FadeIn             3002f750 f   ui_shared.obj
 0001:0002e790       _Script_FadeOut            3002f790 f   ui_shared.obj
 0001:0002e7d0       _Script_Open               3002f7d0 f   ui_shared.obj
 0001:0002e800       _Script_ConditionalOpen    3002f800 f   ui_shared.obj
 0001:0002e890       _Script_Close              3002f890 f   ui_shared.obj
 0001:0002e8c0       _Menu_TransitionItemByName 3002f8c0 f   ui_shared.obj
 0001:0002ea10       _Script_Transition         3002fa10 f   ui_shared.obj
 0001:0002eaf0       _Menu_OrbitItemByName      3002faf0 f   ui_shared.obj
 0001:0002eba0       _Script_Orbit              3002fba0 f   ui_shared.obj
 0001:0002ec60       _Script_SetFocus           3002fc60 f   ui_shared.obj
 0001:0002ed30       _Script_SetPlayerModel     3002fd30 f   ui_shared.obj
 0001:0002ed70       _Script_SetPlayerHead      3002fd70 f   ui_shared.obj
 0001:0002edb0       _Script_SetCvar            3002fdb0 f   ui_shared.obj
 0001:0002ee00       _Script_Exec               3002fe00 f   ui_shared.obj
 0001:0002ee50       _Script_Play               3002fe50 f   ui_shared.obj
 0001:0002eea0       _Script_playLooped         3002fea0 f   ui_shared.obj
 0001:0002eef0       _Item_RunScript            3002fef0 f   ui_shared.obj
 0001:0002f050       _Item_EnableShowViaCvar    30030050 f   ui_shared.obj
 0001:0002f1e0       _Item_SetFocus             300301e0 f   ui_shared.obj
 0001:0002f410       _Item_ListBox_MaxScroll    30030410 f   ui_shared.obj
 0001:0002f4a0       _Item_ListBox_ThumbPosition 300304a0 f   ui_shared.obj
 0001:0002f5b0       _Item_ListBox_ThumbDrawPosition 300305b0 f   ui_shared.obj
 0001:0002f730       _Item_Slider_ThumbPosition 30030730 f   ui_shared.obj
 0001:0002f820       _Item_Slider_OverSlider    30030820 f   ui_shared.obj
 0001:0002f890       _Item_ListBox_OverLB       30030890 f   ui_shared.obj
 0001:0002fb40       _Item_ListBox_MouseEnter   30030b40 f   ui_shared.obj
 0001:0002fce0       _Item_MouseEnter           30030ce0 f   ui_shared.obj
 0001:0002fe80       _Item_MouseLeave           30030e80 f   ui_shared.obj
 0001:0002ff00       _Menu_HitTest              30030f00 f   ui_shared.obj
 0001:0002ff70       _Item_SetMouseOver         30030f70 f   ui_shared.obj
 0001:0002ffb0       _Item_OwnerDraw_HandleKey  30030fb0 f   ui_shared.obj
 0001:00030000       _Item_ListBox_HandleKey    30031000 f   ui_shared.obj
 0001:000307e0       _Item_YesNo_HandleKey      300317e0 f   ui_shared.obj
 0001:000308d0       _Item_Multi_CountSettings  300318d0 f   ui_shared.obj
 0001:00030900       _Item_Multi_FindCvarByValue 30031900 f   ui_shared.obj
 0001:00030a30       _Item_Multi_Setting        30031a30 f   ui_shared.obj
 0001:00030b70       _Item_Multi_HandleKey      30031b70 f   ui_shared.obj
 0001:00030d10       _Item_TextField_HandleKey  30031d10 f   ui_shared.obj
 0001:00031340       _Item_StartCapture         30032340 f   ui_shared.obj
 0001:00031980       _Item_StopCapture          30032980 f   ui_shared.obj
 0001:00031990       _Item_Slider_HandleKey     30032990 f   ui_shared.obj
 0001:00031b50       _Item_HandleKey            30032b50 f   ui_shared.obj
 0001:00031cd0       _Item_Action               30032cd0 f   ui_shared.obj
 0001:00031d00       _Menu_SetPrevCursorItem    30032d00 f   ui_shared.obj
 0001:00031e50       _Menu_SetNextCursorItem    30032e50 f   ui_shared.obj
 0001:00031fa0       _Menus_Activate            30032fa0 f   ui_shared.obj
 0001:00032180       _Display_VisibleMenuCount  30033180 f   ui_shared.obj
 0001:000321e0       _Menus_HandleOOBClick      300331e0 f   ui_shared.obj
 0001:00032350       _Menu_HandleKey            30033350 f   ui_shared.obj
 0001:00032980       _ToWindowCoords            30033980 f   ui_shared.obj
 0001:000329e0       _Rect_ToWindowCoords       300339e0 f   ui_shared.obj
 0001:00032a10       _Item_SetTextExtents       30033a10 f   ui_shared.obj
 0001:00032c80       _Item_TextColor            30033c80 f   ui_shared.obj
 0001:00032ed0       _Item_Text_AutoWrapped_Paint 30033ed0 f   ui_shared.obj
 0001:00033260       _Item_Text_Wrapped_Paint   30034260 f   ui_shared.obj
 0001:00033490       _Item_Text_Paint           30034490 f   ui_shared.obj
 0001:000335d0       _Item_TextField_Paint      300345d0 f   ui_shared.obj
 0001:000338a0       _Item_YesNo_Paint          300348a0 f   ui_shared.obj
 0001:00033ab0       _Item_Multi_Paint          30034ab0 f   ui_shared.obj
 0001:00033c50       _Controls_GetConfig        30034c50 f   ui_shared.obj
 0001:00033d70       _Controls_SetConfig        30034d70 f   ui_shared.obj
 0001:00033e30       _Controls_SetDefaults      30034e30 f   ui_shared.obj
 0001:00033e90       _BindingIDFromName         30034e90 f   ui_shared.obj
 0001:00033ef0       _BindingFromName           30034ef0 f   ui_shared.obj
 0001:00034000       _Item_Slider_Paint         30035000 f   ui_shared.obj
 0001:000341e0       _Item_Bind_Paint           300351e0 f   ui_shared.obj
 0001:00034420       _Display_KeyBindPending    30035420 f   ui_shared.obj
 0001:00034440       _Item_Bind_HandleKey       30035440 f   ui_shared.obj
 0001:00034790       _AdjustFrom640             30035790 f   ui_shared.obj
 0001:00034800       _Item_Model_Paint          30035800 f   ui_shared.obj
 0001:00034b70       _Item_Image_Paint          30035b70 f   ui_shared.obj
 0001:00034be0       _Item_ListBox_Paint        30035be0 f   ui_shared.obj
 0001:00035480       _Item_OwnerDraw_Paint      30036480 f   ui_shared.obj
 0001:00035930       _Item_Paint                30036930 f   ui_shared.obj
 0001:00035f80       _Menu_Init                 30036f80 f   ui_shared.obj
 0001:00036000       _Menu_GetFocusedItem       30037000 f   ui_shared.obj
 0001:00036060       _Menu_GetFocused           30037060 f   ui_shared.obj
 0001:000360d0       _Menu_ScrollFeeder         300370d0 f   ui_shared.obj
 0001:00036160       _Menu_SetFeederSelection   30037160 f   ui_shared.obj
 0001:00036270       _Menus_AnyFullScreenVisible 30037270 f   ui_shared.obj
 0001:000362d0       _Menus_ActivateByName      300372d0 f   ui_shared.obj
 0001:000363b0       _Item_Init                 300373b0 f   ui_shared.obj
 0001:000363f0       _Menu_HandleMouseMove      300373f0 f   ui_shared.obj
 0001:00036630       _Menu_Paint                30037630 f   ui_shared.obj
 0001:00036790       _Item_ValidateTypeData     30037790 f   ui_shared.obj
 0001:000368e0       _KeywordHash_Key           300378e0 f   ui_shared.obj
 0001:00036990       _KeywordHash_Add           30037990 f   ui_shared.obj
 0001:000369d0       _KeywordHash_Find          300379d0 f   ui_shared.obj
 0001:00036a30       _ItemParse_name            30037a30 f   ui_shared.obj
 0001:00036a60       _ItemParse_focusSound      30037a60 f   ui_shared.obj
 0001:00036ab0       _ItemParse_text            30037ab0 f   ui_shared.obj
 0001:00036af0       _ItemParse_group           30037af0 f   ui_shared.obj
 0001:00036b20       _ItemParse_asset_model     30037b20 f   ui_shared.obj
 0001:00036b90       _ItemParse_asset_shader    30037b90 f   ui_shared.obj
 0001:00036be0       _ItemParse_model_origin    30037be0 f   ui_shared.obj
 0001:00036c60       _ItemParse_model_fovx      30037c60 f   ui_shared.obj
 0001:00036cb0       _ItemParse_model_fovy      30037cb0 f   ui_shared.obj
 0001:00036d00       _ItemParse_model_rotation  30037d00 f   ui_shared.obj
 0001:00036d50       _ItemParse_model_angle     30037d50 f   ui_shared.obj
 0001:00036da0       _ItemParse_rect            30037da0 f   ui_shared.obj
 0001:00036dd0       _ItemParse_style           30037dd0 f   ui_shared.obj
 0001:00036e00       _ItemParse_decoration      30037e00 f   ui_shared.obj
 0001:00036e30       _ItemParse_notselectable   30037e30 f   ui_shared.obj
 0001:00036e80       _ItemParse_wrapped         30037e80 f   ui_shared.obj
 0001:00036eb0       _ItemParse_autowrapped     30037eb0 f   ui_shared.obj
 0001:00036ee0       _ItemParse_horizontalscroll 30037ee0 f   ui_shared.obj
 0001:00036f10       _ItemParse_type            30037f10 f   ui_shared.obj
 0001:00036f50       _ItemParse_elementwidth    30037f50 f   ui_shared.obj
 0001:00036fa0       _ItemParse_elementheight   30037fa0 f   ui_shared.obj
 0001:00036ff0       _ItemParse_feeder          30037ff0 f   ui_shared.obj
 0001:00037030       _ItemParse_elementtype     30038030 f   ui_shared.obj
 0001:00037090       _ItemParse_columns         30038090 f   ui_shared.obj
 0001:000371a0       _ItemParse_border          300381a0 f   ui_shared.obj
 0001:000371d0       _ItemParse_bordersize      300381d0 f   ui_shared.obj
 0001:00037200       _ItemParse_visible         30038200 f   ui_shared.obj
 0001:00037250       _ItemParse_ownerdraw       30038250 f   ui_shared.obj
 0001:00037290       _ItemParse_align           30038290 f   ui_shared.obj
 0001:000372d0       _ItemParse_textalign       300382d0 f   ui_shared.obj
 0001:00037310       _ItemParse_textalignx      30038310 f   ui_shared.obj
 0001:00037350       _ItemParse_textaligny      30038350 f   ui_shared.obj
 0001:00037390       _ItemParse_textscale       30038390 f   ui_shared.obj
 0001:000373d0       _ItemParse_textstyle       300383d0 f   ui_shared.obj
 0001:00037410       _ItemParse_backcolor       30038410 f   ui_shared.obj
 0001:00037470       _ItemParse_forecolor       30038470 f   ui_shared.obj
 0001:000374e0       _ItemParse_bordercolor     300384e0 f   ui_shared.obj
 0001:00037540       _ItemParse_outlinecolor    30038540 f   ui_shared.obj
 0001:00037580       _ItemParse_background      30038580 f   ui_shared.obj
 0001:000375d0       _ItemParse_cinematic       300385d0 f   ui_shared.obj
 0001:00037600       _ItemParse_doubleClick     30038600 f   ui_shared.obj
 0001:00037660       _ItemParse_onFocus         30038660 f   ui_shared.obj
 0001:000376a0       _ItemParse_leaveFocus      300386a0 f   ui_shared.obj
 0001:000376e0       _ItemParse_mouseEnter      300386e0 f   ui_shared.obj
 0001:00037720       _ItemParse_mouseExit       30038720 f   ui_shared.obj
 0001:00037760       _ItemParse_mouseEnterText  30038760 f   ui_shared.obj
 0001:000377a0       _ItemParse_mouseExitText   300387a0 f   ui_shared.obj
 0001:000377e0       _ItemParse_action          300387e0 f   ui_shared.obj
 0001:00037820       _ItemParse_special         30038820 f   ui_shared.obj
 0001:00037860       _ItemParse_cvarTest        30038860 f   ui_shared.obj
 0001:000378a0       _ItemParse_cvar            300388a0 f   ui_shared.obj
 0001:00037920       _ItemParse_maxChars        30038920 f   ui_shared.obj
 0001:00037980       _ItemParse_maxPaintChars   30038980 f   ui_shared.obj
 0001:000379e0       _ItemParse_cvarFloat       300389e0 f   ui_shared.obj
 0001:00037a80       _ItemParse_cvarStrList     30038a80 f   ui_shared.obj
 0001:00037c30       _ItemParse_cvarFloatList   30038c30 f   ui_shared.obj
 0001:00037dc0       _ItemParse_addColorRange   30038dc0 f   ui_shared.obj
 0001:00037e60       _ItemParse_ownerdrawFlag   30038e60 f   ui_shared.obj
 0001:00037ea0       _ItemParse_enableCvar      30038ea0 f   ui_shared.obj
 0001:00037ee0       _ItemParse_disableCvar     30038ee0 f   ui_shared.obj
 0001:00037f20       _ItemParse_showCvar        30038f20 f   ui_shared.obj
 0001:00037f60       _ItemParse_hideCvar        30038f60 f   ui_shared.obj
 0001:00037fa0       _Item_SetupKeywordHash     30038fa0 f   ui_shared.obj
 0001:00038000       _Item_Parse                30039000 f   ui_shared.obj
 0001:00038110       _Item_InitControls         30039110 f   ui_shared.obj
 0001:00038180       _MenuParse_font            30039180 f   ui_shared.obj
 0001:00038200       _MenuParse_name            30039200 f   ui_shared.obj
 0001:00038250       _MenuParse_fullscreen      30039250 f   ui_shared.obj
 0001:00038290       _MenuParse_rect            30039290 f   ui_shared.obj
 0001:000382d0       _MenuParse_style           300392d0 f   ui_shared.obj
 0001:00038310       _MenuParse_visible         30039310 f   ui_shared.obj
 0001:00038360       _MenuParse_onOpen          30039360 f   ui_shared.obj
 0001:000383a0       _MenuParse_onClose         300393a0 f   ui_shared.obj
 0001:000383e0       _MenuParse_onESC           300393e0 f   ui_shared.obj
 0001:00038420       _MenuParse_border          30039420 f   ui_shared.obj
 0001:00038460       _MenuParse_borderSize      30039460 f   ui_shared.obj
 0001:000384a0       _MenuParse_backcolor       300394a0 f   ui_shared.obj
 0001:00038500       _MenuParse_forecolor       30039500 f   ui_shared.obj
 0001:00038570       _MenuParse_bordercolor     30039570 f   ui_shared.obj
 0001:000385d0       _MenuParse_focuscolor      300395d0 f   ui_shared.obj
 0001:00038630       _MenuParse_disablecolor    30039630 f   ui_shared.obj
 0001:00038690       _MenuParse_outlinecolor    30039690 f   ui_shared.obj
 0001:000386d0       _MenuParse_background      300396d0 f   ui_shared.obj
 0001:00038720       _MenuParse_cinematic       30039720 f   ui_shared.obj
 0001:00038760       _MenuParse_ownerdrawFlag   30039760 f   ui_shared.obj
 0001:000387b0       _MenuParse_ownerdraw       300397b0 f   ui_shared.obj
 0001:000387f0       _MenuParse_popup           300397f0 f   ui_shared.obj
 0001:00038820       _MenuParse_outOfBounds     30039820 f   ui_shared.obj
 0001:00038850       _MenuParse_soundLoop       30039850 f   ui_shared.obj
 0001:00038890       _MenuParse_fadeClamp       30039890 f   ui_shared.obj
 0001:000388d0       _MenuParse_fadeAmount      300398d0 f   ui_shared.obj
 0001:00038910       _MenuParse_fadeCycle       30039910 f   ui_shared.obj
 0001:00038950       _MenuParse_itemDef         30039950 f   ui_shared.obj
 0001:00038a30       _Menu_SetupKeywordHash     30039a30 f   ui_shared.obj
 0001:00038a90       _Menu_Parse                30039a90 f   ui_shared.obj
 0001:00038bc0       _Menu_New                  30039bc0 f   ui_shared.obj
 0001:00038c30       _Menu_Count                30039c30 f   ui_shared.obj
 0001:00038c50       _Menu_PaintAll             30039c50 f   ui_shared.obj
 0001:00038d20       _Menu_Reset                30039d20 f   ui_shared.obj
 0001:00038d40       _Display_GetContext        30039d40 f   ui_shared.obj
 0001:00038d60       _Display_CaptureItem       30039d60 f   ui_shared.obj
 0001:00038dd0       _Display_MouseMove         30039dd0 f   ui_shared.obj
 0001:00038ea0       _Display_CursorType        30039ea0 f   ui_shared.obj
 0001:00038f40       _Display_HandleKey         30039f40 f   ui_shared.obj
 0001:00038f90       _Display_CacheAll          30039f90 f   ui_shared.obj
 0001:00039240       __fpmath                   3003a240 f   LIBCMTD:fpinit.obj
 0001:00039270       __fpclear                  3003a270 f   LIBCMTD:fpinit.obj
 0001:00039280       __cfltcvt_init             3003a280 f   LIBCMTD:fpinit.obj
 0001:000392d0       ___setfflag                3003a2d0 f   LIBCMTD:fpinit.obj
 0001:000392f0       __CIsin                    3003a2f0 f   LIBCMTD:sin.obj
 0001:00039304       _sin                       3003a304     LIBCMTD:sin.obj
 0001:000393a0       __CIcos                    3003a3a0 f   LIBCMTD:cos.obj
 0001:000393b4       _cos                       3003a3b4     LIBCMTD:cos.obj
 0001:00039450       _atof                      3003a450 f   LIBCMTD:atof.obj
 0001:000394a0       _fabs                      3003a4a0 f   LIBCMTD:fabs.obj
 0001:00039598       __ftol2                    3003a598 f   LIBCMTD:ftol2.obj
 0001:00039610       _memset                    3003a610 f   LIBCMTD:memset.obj
 0001:00039670       _abs                       3003a670 f   LIBCMTD:abs.obj
 0001:000396a0       __abs64                    3003a6a0 f   LIBCMTD:abs.obj
 0001:000396e0       __CIsqrt                   3003a6e0 f   LIBCMTD:sqrt.obj
 0001:000396f4       _sqrt                      3003a6f4     LIBCMTD:sqrt.obj
 0001:000397a0       _atol                      3003a7a0 f   LIBCMTD:atox.obj
 0001:000398b0       _atoi                      3003a8b0 f   LIBCMTD:atox.obj
 0001:000398d0       __atoi64                   3003a8d0 f   LIBCMTD:atox.obj
 0001:00039a10       _strlen                    3003aa10 f   LIBCMTD:strlen.obj
 0001:00039aa0       _srand                     3003aaa0 f   LIBCMTD:rand.obj
 0001:00039ab0       _rand                      3003aab0 f   LIBCMTD:rand.obj
 0001:00039af0       _memcpy                    3003aaf0 f   LIBCMTD:memcpy.obj
 0001:00039e30       _strcpy                    3003ae30 f   LIBCMTD:strcat.obj
 0001:00039e40       _strcat                    3003ae40 f   LIBCMTD:strcat.obj
 0001:00039f30       _vsprintf                  3003af30 f   LIBCMTD:vsprintf.obj
 0001:0003a020       __vscprintf                3003b020 f   LIBCMTD:vsprintf.obj
 0001:0003a0a0       _strcmp                    3003b0a0 f   LIBCMTD:strcmp.obj
 0001:0003a130       __alloca_probe             3003b130     LIBCMTD:chkstk.obj
 0001:0003a130       __chkstk                   3003b130 f   LIBCMTD:chkstk.obj
 0001:0003a170       _floor                     3003b170 f   LIBCMTD:floor_pentium4.obj
 0001:0003a1b0       __floor_pentium4           3003b1b0 f   LIBCMTD:floor_pentium4.obj
 0001:0003a2b0       _strchr                    3003b2b0 f   LIBCMTD:strchr.obj
 0001:0003a2b6       ___from_strstr_to_strchr   3003b2b6     LIBCMTD:strchr.obj
 0001:0003a370       __CIacos                   3003b370 f   LIBCMTD:acos.obj
 0001:0003a384       _acos                      3003b384     LIBCMTD:acos.obj
 0001:0003a440       _strncpy                   3003b440 f   LIBCMTD:strncpy.obj
 0001:0003a570       _strstr                    3003b570 f   LIBCMTD:strstr.obj
 0001:0003a600       _atan2                     3003b600 f   LIBCMTD:87ctriga.obj
 0001:0003a60a       __CIatan2                  3003b60a f   LIBCMTD:87ctriga.obj
 0001:0003a620       __CItan                    3003b620 f   LIBCMTD:tan.obj
 0001:0003a634       _tan                       3003b634     LIBCMTD:tan.obj
 0001:0003a6e0       __assert                   3003b6e0 f   LIBCMTD:assert.obj
 0001:0003ace0       __tolower                  3003bce0 f   LIBCMTD:tolower.obj
 0001:0003acf0       _tolower                   3003bcf0 f   LIBCMTD:tolower.obj
 0001:0003ad30       ___tolower_mt              3003bd30 f   LIBCMTD:tolower.obj
 0001:0003ae70       __toupper                  3003be70 f   LIBCMTD:toupper.obj
 0001:0003ae80       _toupper                   3003be80 f   LIBCMTD:toupper.obj
 0001:0003aec0       ___toupper_mt              3003bec0 f   LIBCMTD:toupper.obj
 0001:0003b000       _memmove                   3003c000 f   LIBCMTD:memmove.obj
 0001:0003b340       __CRT_INIT@12              3003c340 f   LIBCMTD:dllcrt0.obj
 0001:0003b590       __DllMainCRTStartup@12     3003c590 f   LIBCMTD:dllcrt0.obj
 0001:0003b710       __amsg_exit                3003c710 f   LIBCMTD:dllcrt0.obj
 0001:0003b750       __setdefaultprecision      3003c750 f   LIBCMTD:fp8.obj
 0001:0003b770       __ms_p5_test_fdiv          3003c770 f   LIBCMTD:testfdiv.obj
 0001:0003b7c0       __ms_p5_mp_test_fdiv       3003c7c0 f   LIBCMTD:testfdiv.obj
 0001:0003b810       __forcdecpt                3003c810 f   LIBCMTD:cvt.obj
 0001:0003b890       __cropzeros                3003c890 f   LIBCMTD:cvt.obj
 0001:0003b970       __positive                 3003c970 f   LIBCMTD:cvt.obj
 0001:0003b9a0       __fassign                  3003c9a0 f   LIBCMTD:cvt.obj
 0001:0003b9f0       __cftoe                    3003c9f0 f   LIBCMTD:cvt.obj
 0001:0003bbf0       __cftof                    3003cbf0 f   LIBCMTD:cvt.obj
 0001:0003bdb0       __cftog                    3003cdb0 f   LIBCMTD:cvt.obj
 0001:0003beb0       __cfltcvt                  3003ceb0 f   LIBCMTD:cvt.obj
 0001:0003bf40       __trandisp1                3003cf40 f   LIBCMTD:87disp.obj
 0001:0003bfa7       __trandisp2                3003cfa7 f   LIBCMTD:87disp.obj
 0001:0003c033       __rttospopde               3003d033     LIBCMTD:87disp.obj
 0001:0003c038       __rttospop                 3003d038     LIBCMTD:87disp.obj
 0001:0003c03a       __rtnospop                 3003d03a     LIBCMTD:87disp.obj
 0001:0003c03c       __rttosnpop                3003d03c     LIBCMTD:87disp.obj
 0001:0003c03d       __rtnospopde               3003d03d     LIBCMTD:87disp.obj
 0001:0003c044       __rtzeropop                3003d044     LIBCMTD:87disp.obj
 0001:0003c046       __rtzeronpop               3003d046     LIBCMTD:87disp.obj
 0001:0003c04b       __rtonepop                 3003d04b     LIBCMTD:87disp.obj
 0001:0003c04d       __rtonenpop                3003d04d     LIBCMTD:87disp.obj
 0001:0003c052       __tosnan1                  3003d052     LIBCMTD:87disp.obj
 0001:0003c07d       __nosnan2                  3003d07d     LIBCMTD:87disp.obj
 0001:0003c07f       __tosnan2                  3003d07f     LIBCMTD:87disp.obj
 0001:0003c0a7       __nan2                     3003d0a7     LIBCMTD:87disp.obj
 0001:0003c0e6       __rtindfpop                3003d0e6     LIBCMTD:87disp.obj
 0001:0003c0e8       __rtindfnpop               3003d0e8     LIBCMTD:87disp.obj
 0001:0003c0f9       __rttosnpopde              3003d0f9     LIBCMTD:87disp.obj
 0001:0003c103       __rtchsifneg               3003d103     LIBCMTD:87disp.obj
 0001:0003c110       __twoToTOS                 3003d110 f   LIBCMTD:common.obj
 0001:0003c125       __load_CW                  3003d125 f   LIBCMTD:common.obj
 0001:0003c13c       __convertTOStoQNaN         3003d13c f   LIBCMTD:common.obj
 0001:0003c155       __fload_withFB             3003d155 f   LIBCMTD:common.obj
 0001:0003c198       __checkTOS_withFB          3003d198 f   LIBCMTD:common.obj
 0001:0003c1ae       __fast_exit                3003d1ae f   LIBCMTD:common.obj
 0001:0003c1bb       __math_exit                3003d1bb f   LIBCMTD:common.obj
 0001:0003c1e5       __check_overflow_exit      3003d1e5 f   LIBCMTD:common.obj
 0001:0003c1f9       __check_range_exit         3003d1f9 f   LIBCMTD:common.obj
 0001:0003c2a0       __startTwoArgErrorHandling 3003d2a0 f   LIBCMTD:genexcep.obj
 0001:0003c2b7       __startOneArgErrorHandling 3003d2b7 f   LIBCMTD:genexcep.obj
 0001:0003c300       __fltin2                   3003d300 f   LIBCMTD:cfin.obj
 0001:0003c3e0       _isalpha                   3003d3e0 f   LIBCMTD:_ctype.obj
 0001:0003c450       _isupper                   3003d450 f   LIBCMTD:_ctype.obj
 0001:0003c4b0       _islower                   3003d4b0 f   LIBCMTD:_ctype.obj
 0001:0003c510       _isdigit                   3003d510 f   LIBCMTD:_ctype.obj
 0001:0003c570       _isxdigit                  3003d570 f   LIBCMTD:_ctype.obj
 0001:0003c5e0       _isspace                   3003d5e0 f   LIBCMTD:_ctype.obj
 0001:0003c640       _ispunct                   3003d640 f   LIBCMTD:_ctype.obj
 0001:0003c6a0       _isalnum                   3003d6a0 f   LIBCMTD:_ctype.obj
 0001:0003c710       _isprint                   3003d710 f   LIBCMTD:_ctype.obj
 0001:0003c780       _isgraph                   3003d780 f   LIBCMTD:_ctype.obj
 0001:0003c7f0       _iscntrl                   3003d7f0 f   LIBCMTD:_ctype.obj
 0001:0003c850       ___isascii                 3003d850 f   LIBCMTD:_ctype.obj
 0001:0003c860       ___toascii                 3003d860 f   LIBCMTD:_ctype.obj
 0001:0003c870       ___iscsymf                 3003d870 f   LIBCMTD:_ctype.obj
 0001:0003c8b0       ___iscsym                  3003d8b0 f   LIBCMTD:_ctype.obj
 0001:0003c8f0       __handle_qnan1             3003d8f0 f   LIBCMTD:fpexcept.obj
 0001:0003c950       __handle_qnan2             3003d950 f   LIBCMTD:fpexcept.obj
 0001:0003c9c0       __except1                  3003d9c0 f   LIBCMTD:fpexcept.obj
 0001:0003cac0       __except2                  3003dac0 f   LIBCMTD:fpexcept.obj
 0001:0003cbd0       __raise_exc                3003dbd0 f   LIBCMTD:fpexcept.obj
 0001:0003d080       __handle_exc               3003e080 f   LIBCMTD:fpexcept.obj
 0001:0003d3a0       __umatherr                 3003e3a0 f   LIBCMTD:fpexcept.obj
 0001:0003d440       __set_errno                3003e440 f   LIBCMTD:fpexcept.obj
 0001:0003d4c0       __errcode                  3003e4c0 f   LIBCMTD:fpexcept.obj
 0001:0003d530       __set_exp                  3003e530 f   LIBCMTD:util.obj
 0001:0003d570       __get_exp                  3003e570 f   LIBCMTD:util.obj
 0001:0003d5a0       __add_exp                  3003e5a0 f   LIBCMTD:util.obj
 0001:0003d5d0       __set_bexp                 3003e5d0 f   LIBCMTD:util.obj
 0001:0003d600       __sptype                   3003e600 f   LIBCMTD:util.obj
 0001:0003d680       __decomp                   3003e680 f   LIBCMTD:util.obj
 0001:0003d7b0       __statfp                   3003e7b0 f   LIBCMTD:fpctrl.obj
 0001:0003d7c0       __clrfp                    3003e7c0 f   LIBCMTD:fpctrl.obj
 0001:0003d7e0       __ctrlfp                   3003e7e0 f   LIBCMTD:fpctrl.obj
 0001:0003d810       __set_statfp               3003e810 f   LIBCMTD:fpctrl.obj
 0001:0003d880       __chvalidator              3003e880 f   LIBCMTD:isctype.obj
 0001:0003d8c0       __chvalidator_mt           3003e8c0 f   LIBCMTD:isctype.obj
 0001:0003d900       __isctype                  3003e900 f   LIBCMTD:isctype.obj
 0001:0003d940       ___isctype_mt              3003e940 f   LIBCMTD:isctype.obj
 0001:0003da00       ____setlc_active_func      3003ea00 f   LIBCMTD:setlocal.obj
 0001:0003da10       ____unguarded_readlc_active_add_func 3003ea10 f   LIBCMTD:setlocal.obj
 0001:0003da20       ___freetlocinfo            3003ea20 f   LIBCMTD:setlocal.obj
 0001:0003dba0       ___updatetlocinfo          3003eba0 f   LIBCMTD:setlocal.obj
 0001:0003dde0       _setlocale                 3003ede0 f   LIBCMTD:setlocal.obj
 0001:0003e890       __expandlocale             3003f890 f   LIBCMTD:setlocal.obj
 0001:0003ea70       ___init_dummy              3003fa70 f   LIBCMTD:setlocal.obj
 0001:0003ea80       __strcats                  3003fa80 f   LIBCMTD:setlocal.obj
 0001:0003ead0       ___lc_strtolc              3003fad0 f   LIBCMTD:setlocal.obj
 0001:0003ec40       ___lc_lctostr              3003fc40 f   LIBCMTD:setlocal.obj
 0001:0003ecb0       ___crtTlsAlloc@4           3003fcb0 f   LIBCMTD:tidtable.obj
 0001:0003ecc0       __mtinit                   3003fcc0 f   LIBCMTD:tidtable.obj
 0001:0003ee10       __mtterm                   3003fe10 f   LIBCMTD:tidtable.obj
 0001:0003ee40       __initptd                  3003fe40 f   LIBCMTD:tidtable.obj
 0001:0003ee60       __getptd                   3003fe60 f   LIBCMTD:tidtable.obj
 0001:0003ef00       __freefls@4                3003ff00 f   LIBCMTD:tidtable.obj
 0001:0003f180       __freeptd                  30040180 f   LIBCMTD:tidtable.obj
 0001:0003f1c0       ___threadid                300401c0 f   LIBCMTD:tidtable.obj
 0001:0003f1d0       ___threadhandle            300401d0 f   LIBCMTD:tidtable.obj
 0001:0003f1e0       __allmul                   300401e0 f   LIBCMTD:llmul.obj
 0001:0003f220       __flsbuf                   30040220 f   LIBCMTD:_flsbuf.obj
 0001:0003f480       __output                   30040480 f   LIBCMTD:output.obj
 0001:00040400       __CrtDbgBreak              30041400 f   LIBCMTD:dbgrpt.obj
 0001:00040410       __CrtSetReportMode         30041410 f   LIBCMTD:dbgrpt.obj
 0001:00040470       __CrtSetReportFile         30041470 f   LIBCMTD:dbgrpt.obj
 0001:000404f0       __CrtSetReportHook         300414f0 f   LIBCMTD:dbgrpt.obj
 0001:00040510       __CrtSetReportHook2        30041510 f   LIBCMTD:dbgrpt.obj
 0001:00040760       __CrtDbgReport             30041760 f   LIBCMTD:dbgrpt.obj
 0001:00040ed0       ___libm_error_support      30041ed0 f   LIBCMTD:libm_error.obj
 0001:000418e0       ___sse2_available_init     300428e0 f   LIBCMTD:cpu_disp.obj
 0001:00041a70       __set_SSE2_enable          30042a70 f   LIBCMTD:cpu_disp.obj
 0001:00041a90       __floor_default            30042a90 f   LIBCMTD:floor.obj
 0001:00041bec       __fFATN2                   30042bec     LIBCMTD:87triga.obj
 0001:00041c3c       __rtpiby2                  30042c3c     LIBCMTD:87triga.obj
 0001:00041c80       __cintrindisp2             30042c80 f   LIBCMTD:87cdisp.obj
 0001:00041cbe       __cintrindisp1             30042cbe f   LIBCMTD:87cdisp.obj
 0001:00041cfb       __ctrandisp2               30042cfb f   LIBCMTD:87cdisp.obj
 0001:00041e91       __ctrandisp1               30042e91 f   LIBCMTD:87cdisp.obj
 0001:00041ec4       __fload                    30042ec4 f   LIBCMTD:87cdisp.obj
 0001:00041f00       _abort                     30042f00 f   LIBCMTD:abort.obj
 0001:00041f20       __cinit                    30042f20 f   LIBCMTD:crt0dat.obj
 0001:00041f80       _exit                      30042f80 f   LIBCMTD:crt0dat.obj
 0001:00041fa0       __exit                     30042fa0 f   LIBCMTD:crt0dat.obj
 0001:00041fc0       __cexit                    30042fc0 f   LIBCMTD:crt0dat.obj
 0001:00041fe0       __c_exit                   30042fe0 f   LIBCMTD:crt0dat.obj
 0001:00042130       ___crtExitProcess          30043130 f   LIBCMTD:crt0dat.obj
 0001:00042180       __lockexit                 30043180 f   LIBCMTD:crt0dat.obj
 0001:00042190       __unlockexit               30043190 f   LIBCMTD:crt0dat.obj
 0001:00042210       _signal                    30043210 f   LIBCMTD:winsig.obj
 0001:00042550       _raise                     30043550 f   LIBCMTD:winsig.obj
 0001:00042810       ___fpecode                 30043810 f   LIBCMTD:winsig.obj
 0001:00042820       ___pxcptinfoptrs           30043820 f   LIBCMTD:winsig.obj
 0001:00042830       ___crtMessageBoxA          30043830 f   LIBCMTD:crtmbox.obj
 0001:000429a0       __itoa                     300439a0 f   LIBCMTD:xtoa.obj
 0001:00042ac0       __ltoa                     30043ac0 f   LIBCMTD:xtoa.obj
 0001:00042b00       __ultoa                    30043b00 f   LIBCMTD:xtoa.obj
 0001:00042b20       __i64toa                   30043b20 f   LIBCMTD:xtoa.obj
 0001:00042c70       __ui64toa                  30043c70 f   LIBCMTD:xtoa.obj
 0001:00042c90       _strncat                   30043c90 f   LIBCMTD:strncat.obj
 0001:00042dd0       _fflush                    30043dd0 f   LIBCMTD:fflush.obj
 0001:00042e60       __fflush_lk                30043e60 f   LIBCMTD:fflush.obj
 0001:00042ea0       __flush                    30043ea0 f   LIBCMTD:fflush.obj
 0001:00042f60       __flushall                 30043f60 f   LIBCMTD:fflush.obj
 0001:00043100       _fprintf                   30044100 f   LIBCMTD:fprintf.obj
 0001:000431f0       _setvbuf                   300441f0 f   LIBCMTD:setvbuf.obj
 0001:00043390       ___iob_func                30044390 f   LIBCMTD:_file.obj
 0001:000433a0       ___initstdio               300443a0 f   LIBCMTD:_file.obj
 0001:000434d0       ___endstdio                300444d0 f   LIBCMTD:_file.obj
 0001:000434f0       __lock_file                300444f0 f   LIBCMTD:_file.obj
 0001:00043530       __lock_file2               30044530 f   LIBCMTD:_file.obj
 0001:00043560       __unlock_file              30044560 f   LIBCMTD:_file.obj
 0001:000435a0       __unlock_file2             300445a0 f   LIBCMTD:_file.obj
 0001:000435d0       @__security_check_cookie@4 300445d0 f   LIBCMTD:secchk.obj
 0001:00043650       ___crtLCMapStringA         30044650 f   LIBCMTD:a_map.obj
 0001:00043c10       _malloc                    30044c10 f   LIBCMTD:dbgheap.obj
 0001:00043c40       __malloc_dbg               30044c40 f   LIBCMTD:dbgheap.obj
 0001:00043c70       __nh_malloc                30044c70 f   LIBCMTD:dbgheap.obj
 0001:00043c90       __nh_malloc_dbg            30044c90 f   LIBCMTD:dbgheap.obj
 0001:00043d30       __heap_alloc               30044d30 f   LIBCMTD:dbgheap.obj
 0001:00043d50       __heap_alloc_dbg           30044d50 f   LIBCMTD:dbgheap.obj
 0001:00044070       _calloc                    30045070 f   LIBCMTD:dbgheap.obj
 0001:000440a0       __calloc_dbg               300450a0 f   LIBCMTD:dbgheap.obj
 0001:00044100       _realloc                   30045100 f   LIBCMTD:dbgheap.obj
 0001:00044130       __realloc_dbg              30045130 f   LIBCMTD:dbgheap.obj
 0001:000446d0       __expand                   300456d0 f   LIBCMTD:dbgheap.obj
 0001:00044700       __expand_dbg               30045700 f   LIBCMTD:dbgheap.obj
 0001:00044790       _free                      30045790 f   LIBCMTD:dbgheap.obj
 0001:000447b0       __free_lk                  300457b0 f   LIBCMTD:dbgheap.obj
 0001:000447d0       __free_dbg                 300457d0 f   LIBCMTD:dbgheap.obj
 0001:00044840       __free_dbg_lk              30045840 f   LIBCMTD:dbgheap.obj
 0001:00044c50       __msize                    30045c50 f   LIBCMTD:dbgheap.obj
 0001:00044c70       __msize_dbg                30045c70 f   LIBCMTD:dbgheap.obj
 0001:00044de0       __CrtSetBreakAlloc         30045de0 f   LIBCMTD:dbgheap.obj
 0001:00044e00       __CrtSetDbgBlockType       30045e00 f   LIBCMTD:dbgheap.obj
 0001:00044ee0       __CrtSetAllocHook          30045ee0 f   LIBCMTD:dbgheap.obj
 0001:00044f50       __CrtCheckMemory           30045f50 f   LIBCMTD:dbgheap.obj
 0001:000452c0       __CrtSetDbgFlag            300462c0 f   LIBCMTD:dbgheap.obj
 0001:00045370       __CrtDoForAllClientObjects 30046370 f   LIBCMTD:dbgheap.obj
 0001:00045420       __CrtIsValidPointer        30046420 f   LIBCMTD:dbgheap.obj
 0001:00045470       __CrtIsValidHeapPointer    30046470 f   LIBCMTD:dbgheap.obj
 0001:00045520       __CrtIsMemoryBlock         30046520 f   LIBCMTD:dbgheap.obj
 0001:00045650       __CrtReportBlockType       30046650 f   LIBCMTD:dbgheap.obj
 0001:00045680       __CrtSetDumpClient         30046680 f   LIBCMTD:dbgheap.obj
 0001:000456a0       __CrtMemCheckpoint         300466a0 f   LIBCMTD:dbgheap.obj
 0001:00045840       __CrtMemDifference         30046840 f   LIBCMTD:dbgheap.obj
 0001:00045960       __CrtMemDumpAllObjectsSince 30046960 f   LIBCMTD:dbgheap.obj
 0001:00045d60       __CrtDumpMemoryLeaks       30046d60 f   LIBCMTD:dbgheap.obj
 0001:00045dd0       __CrtMemDumpStatistics     30046dd0 f   LIBCMTD:dbgheap.obj
 0001:00045e80       __aligned_malloc           30046e80 f   LIBCMTD:dbgheap.obj
 0001:00045ea0       __aligned_malloc_dbg       30046ea0 f   LIBCMTD:dbgheap.obj
 0001:00045ec0       __aligned_realloc          30046ec0 f   LIBCMTD:dbgheap.obj
 0001:00045ee0       __aligned_realloc_dbg      30046ee0 f   LIBCMTD:dbgheap.obj
 0001:00045f10       __aligned_offset_malloc    30046f10 f   LIBCMTD:dbgheap.obj
 0001:00045f30       __aligned_offset_malloc_dbg 30046f30 f   LIBCMTD:dbgheap.obj
 0001:00046070       __aligned_offset_realloc   30047070 f   LIBCMTD:dbgheap.obj
 0001:000460a0       __aligned_offset_realloc_dbg 300470a0 f   LIBCMTD:dbgheap.obj
 0001:00046300       __aligned_free             30047300 f   LIBCMTD:dbgheap.obj
 0001:00046320       __aligned_free_dbg         30047320 f   LIBCMTD:dbgheap.obj
 0001:000463d0       __ioinit                   300473d0 f   LIBCMTD:ioinit.obj
 0001:00046760       __ioterm                   30047760 f   LIBCMTD:ioinit.obj
 0001:00046800       __setenvp                  30047800 f   LIBCMTD:stdenvp.obj
 0001:00046980       __setargv                  30047980 f   LIBCMTD:stdargv.obj
 0001:00046de0       ___crtGetEnvironmentStringsA 30047de0 f   LIBCMTD:a_env.obj
 0001:00047000       __RTC_Initialize           30048000 f   LIBCMTD:initsect.obj
 0001:00047080       __RTC_Terminate            30048080 f   LIBCMTD:initsect.obj
 0001:00047100       ___heap_select             30048100 f   LIBCMTD:heapinit.obj
 0001:00047130       __heap_init                30048130 f   LIBCMTD:heapinit.obj
 0001:000471a0       __heap_term                300481a0 f   LIBCMTD:heapinit.obj
 0001:00047250       __get_heap_handle          30048250 f   LIBCMTD:heapinit.obj
 0001:00047260       ___CppXcptFilter           30048260 f   LIBCMTD:winxfltr.obj
 0001:00047290       __XcptFilter               30048290 f   LIBCMTD:winxfltr.obj
 0001:000474b0       _DllMain@12                300484b0 f   LIBCMTD:dllmain.obj
 0001:000474bc       __global_unwind2           300484bc f   LIBCMTD:exsup.obj
 0001:000474fe       __local_unwind2            300484fe f   LIBCMTD:exsup.obj
 0001:00047556       __NLG_Return2              30048556     LIBCMTD:exsup.obj
 0001:00047566       __abnormal_termination     30048566 f   LIBCMTD:exsup.obj
 0001:00047589       __NLG_Notify1              30048589 f   LIBCMTD:exsup.obj
 0001:00047592       __NLG_Notify               30048592 f   LIBCMTD:exsup.obj
 0001:000475a5       __NLG_Dispatch             300485a5     LIBCMTD:exsup.obj
 0001:000475b4       __except_handler3          300485b4 f   LIBCMTD:exsup3.obj
 0001:0004769a       __seh_longjmp_unwind@4     3004869a f   LIBCMTD:exsup3.obj
 0001:000476c0       __FF_MSGBANNER             300486c0 f   LIBCMTD:crt0msg.obj
 0001:00047710       __NMSG_WRITE               30048710 f   LIBCMTD:crt0msg.obj
 0001:00047920       __GET_RTERRMSG             30048920 f   LIBCMTD:crt0msg.obj
 0001:00047970       __statusfp                 30048970 f   LIBCMTD:ieee87.obj
 0001:00047990       __clearfp                  30048990 f   LIBCMTD:ieee87.obj
 0001:000479b0       __control87                300489b0 f   LIBCMTD:ieee87.obj
 0001:00047a00       __controlfp                30048a00 f   LIBCMTD:ieee87.obj
 0001:00047a20       __fpreset                  30048a20 f   LIBCMTD:ieee87.obj
 0001:00047db0       __ZeroTail                 30048db0 f   LIBCMTD:intrncvt.obj
 0001:00047e40       __IncMan                   30048e40 f   LIBCMTD:intrncvt.obj
 0001:00047ef0       __RoundMan                 30048ef0 f   LIBCMTD:intrncvt.obj
 0001:00047fd0       __CopyMan                  30048fd0 f   LIBCMTD:intrncvt.obj
 0001:00048020       __FillZeroMan              30049020 f   LIBCMTD:intrncvt.obj
 0001:00048050       __IsZeroMan                30049050 f   LIBCMTD:intrncvt.obj
 0001:00048090       __ShrMan                   30049090 f   LIBCMTD:intrncvt.obj
 0001:00048180       __ld12cvt                  30049180 f   LIBCMTD:intrncvt.obj
 0001:000483c0       __ld12tod                  300493c0 f   LIBCMTD:intrncvt.obj
 0001:000483e0       __ld12tof                  300493e0 f   LIBCMTD:intrncvt.obj
 0001:00048400       __ld12told                 30049400 f   LIBCMTD:intrncvt.obj
 0001:000484b0       __atodbl                   300494b0 f   LIBCMTD:intrncvt.obj
 0001:00048500       __atoldbl                  30049500 f   LIBCMTD:intrncvt.obj
 0001:00048550       __atoflt                   30049550 f   LIBCMTD:intrncvt.obj
 0001:000485a0       __fptostr                  300495a0 f   LIBCMTD:_fptostr.obj
 0001:000486a0       __fltout2                  300496a0 f   LIBCMTD:cfout.obj
 0001:00048730       ___dtold                   30049730 f   LIBCMTD:cfout.obj
 0001:00048880       __fptrap                   30049880 f   LIBCMTD:crt0fp.obj
 0001:00048890       __87except                 30049890 f   LIBCMTD:87except.obj
 0001:00048a40       ___strgtold12              30049a40 f   LIBCMTD:strgtold.obj
 0001:00049440       ___STRINGTOLD              3004a440 f   LIBCMTD:strgtold.obj
 0001:000494a0       __dosmaperr                3004a4a0 f   LIBCMTD:dosmap.obj
 0001:00049540       __errno                    3004a540 f   LIBCMTD:dosmap.obj
 0001:00049550       ___doserrno                3004a550 f   LIBCMTD:dosmap.obj
 0001:00049560       __matherr                  3004a560 f   LIBCMTD:matherr.obj
 0001:00049570       ___pwctype_func            3004a570 f   LIBCMTD:ctype.obj
 0001:00049580       ___pctype_func             3004a580 f   LIBCMTD:ctype.obj
 0001:00049590       ___crtGetStringTypeA       3004a590 f   LIBCMTD:a_str.obj
 0001:00049830       __Getdays                  3004a830 f   LIBCMTD:strftime.obj
 0001:00049960       __Getmonths                3004a960 f   LIBCMTD:strftime.obj
 0001:00049a90       __Gettnames                3004aa90 f   LIBCMTD:strftime.obj
 0001:00049e20       _strftime                  3004ae20 f   LIBCMTD:strftime.obj
 0001:00049e40       __Strftime                 3004ae40 f   LIBCMTD:strftime.obj
 0001:00049e90       __Strftime_mt              3004ae90 f   LIBCMTD:strftime.obj
 0001:0004b0b0       _localeconv                3004c0b0 f   LIBCMTD:lconv.obj
 0001:0004b0c0       ___init_time               3004c0c0 f   LIBCMTD:inittime.obj
 0001:0004b6d0       ___free_lc_time            3004c6d0 f   LIBCMTD:inittime.obj
 0001:0004b9e0       ___init_numeric            3004c9e0 f   LIBCMTD:initnum.obj
 0001:0004bd20       ___free_lconv_num          3004cd20 f   LIBCMTD:initnum.obj
 0001:0004bdc0       ___init_monetary           3004cdc0 f   LIBCMTD:initmon.obj
 0001:0004c1c0       ___free_lconv_mon          3004d1c0 f   LIBCMTD:initmon.obj
 0001:0004c320       ___init_ctype              3004d320 f   LIBCMTD:initctyp.obj
 0001:0004c5e0       ____mb_cur_max_func        3004d5e0 f   LIBCMTD:initctyp.obj
 0001:0004c5f0       ____lc_codepage_func       3004d5f0 f   LIBCMTD:initctyp.obj
 0001:0004c620       ____lc_collate_cp_func     3004d620 f   LIBCMTD:initctyp.obj
 0001:0004c650       ____lc_handle_func         3004d650 f   LIBCMTD:initctyp.obj
 0001:0004c680       ___init_collate            3004d680 f   LIBCMTD:initcoll.obj
 0001:0004c690       __mtinitlocks              3004d690 f   LIBCMTD:mlock.obj
 0001:0004c720       __mtdeletelocks            3004d720 f   LIBCMTD:mlock.obj
 0001:0004c7e0       __mtinitlocknum            3004d7e0 f   LIBCMTD:mlock.obj
 0001:0004c900       __lock                     3004d900 f   LIBCMTD:mlock.obj
 0001:0004c940       __unlock                   3004d940 f   LIBCMTD:mlock.obj
 0001:0004c960       __lockerr_exit             3004d960 f   LIBCMTD:mlock.obj
 0001:0004c980       _strcspn                   3004d980 f   LIBCMTD:strcspn.obj
 0001:0004c9d0       _strncmp                   3004d9d0 f   LIBCMTD:strncmp.obj
 0001:0004ca10       _strpbrk                   3004da10 f   LIBCMTD:strpbrk.obj
 0001:0004ca50       _memcmp                    3004da50 f   LIBCMTD:memcmp.obj
 0001:0004cb10       ___get_qualified_locale    3004db10 f   LIBCMTD:getqloc.obj
 0001:0004d940       ___updatetmbcinfo          3004e940 f   LIBCMTD:mbctype.obj
 0001:0004da10       __setmbcp                  3004ea10 f   LIBCMTD:mbctype.obj
 0001:0004e350       __getmbcp                  3004f350 f   LIBCMTD:mbctype.obj
 0001:0004e370       ___initmbctable            3004f370 f   LIBCMTD:mbctype.obj
 0001:0004e3a0       __lseek                    3004f3a0 f   LIBCMTD:lseek.obj
 0001:0004e4b0       __lseek_lk                 3004f4b0 f   LIBCMTD:lseek.obj
 0001:0004e570       __write                    3004f570 f   LIBCMTD:write.obj
 0001:0004e680       __write_lk                 3004f680 f   LIBCMTD:write.obj
 0001:0004e970       __getbuf                   3004f970 f   LIBCMTD:_getbuf.obj
 0001:0004ea30       __isatty                   3004fa30 f   LIBCMTD:isatty.obj
 0001:0004ea70       _wctomb                    3004fa70 f   LIBCMTD:wctomb.obj
 0001:0004eab0       ___wctomb_mt               3004fab0 f   LIBCMTD:wctomb.obj
 0001:0004eb50       __aulldiv                  3004fb50 f   LIBCMTD:ulldiv.obj
 0001:0004ebc0       __aullrem                  3004fbc0 f   LIBCMTD:ullrem.obj
 0001:0004ec40       __snprintf                 3004fc40 f   LIBCMTD:snprintf.obj
 0001:0004ed30       __vsnprintf                3004fd30 f   LIBCMTD:vsnprint.obj
 0001:0004ee00       __frnd                     3004fe00 f   LIBCMTD:frnd.obj
 0001:0004ee20       __onexit                   3004fe20 f   LIBCMTD:onexit.obj
 0001:0004ef80       _atexit                    3004ff80 f   LIBCMTD:onexit.obj
 0001:0004efa0       ___onexitinit              3004ffa0 f   LIBCMTD:onexit.obj
 0001:0004eff0       __commit                   3004fff0 f   LIBCMTD:commit.obj
 0001:0004f100       __stbuf                    30050100 f   LIBCMTD:_sftbuf.obj
 0001:0004f250       __ftbuf                    30050250 f   LIBCMTD:_sftbuf.obj
 0001:0004f2e0       __freebuf                  300502e0 f   LIBCMTD:_freebuf.obj
 0001:0004f370       __fcloseall                30050370 f   LIBCMTD:closeall.obj
 0001:0004f490       ___security_init_cookie    30050490 f   LIBCMTD:seccinit.obj
 0001:0004f530       ___security_error_handler  30050530 f   LIBCMTD:secfail.obj
 0001:0004f760       __set_security_error_handler 30050760 f   LIBCMTD:secfail.obj
 0001:0004f780       ___buffer_overrun          30050780 f   LIBCMTD:secfail.obj
 0001:0004f7a0       ___set_buffer_overrun_handler 300507a0 f   LIBCMTD:secfail.obj
 0001:0004f7c0       __resetstkoflw             300507c0 f   LIBCMTD:resetstk.obj
 0001:0004f910       ___ansicp                  30050910 f   LIBCMTD:convrtcp.obj
 0001:0004f970       ___convertcp               30050970 f   LIBCMTD:convrtcp.obj
 0001:0004fc10       ?_set_new_handler@@YAP6AHI@ZP6AHI@Z@Z 30050c10 f   LIBCMTD:handler.obj
 0001:0004fc40       ?_query_new_handler@@YAP6AHI@ZXZ 30050c40 f   LIBCMTD:handler.obj
 0001:0004fc50       __callnewh                 30050c50 f   LIBCMTD:handler.obj
 0001:0004fc80       __malloc_base              30050c80 f   LIBCMTD:malloc.obj
 0001:0004fca0       __nh_malloc_base           30050ca0 f   LIBCMTD:malloc.obj
 0001:0004fd00       __heap_alloc_base          30050d00 f   LIBCMTD:malloc.obj
 0001:0004fdd0       __CrtDefaultAllocHook      30050dd0 f   LIBCMTD:dbghook.obj
 0001:0004fde0       __expand_base              30050de0 f   LIBCMTD:expand.obj
 0001:0004ff00       __realloc_base             30050f00 f   LIBCMTD:realloc.obj
 0001:000501b0       __free_base                300511b0 f   LIBCMTD:free.obj
 0001:00050280       __heapchk                  30051280 f   LIBCMTD:heapchk.obj
 0001:00050340       __heapset                  30051340 f   LIBCMTD:heapchk.obj
 0001:00050350       __get_sbh_threshold        30051350 f   LIBCMTD:sbheap.obj
 0001:00050370       __set_sbh_threshold        30051370 f   LIBCMTD:sbheap.obj
 0001:000503e0       ___sbh_heap_init           300513e0 f   LIBCMTD:sbheap.obj
 0001:00050450       ___sbh_find_block          30051450 f   LIBCMTD:sbheap.obj
 0001:000504b0       ___sbh_verify_block        300514b0 f   LIBCMTD:sbheap.obj
 0001:00050510       ___sbh_free_block          30051510 f   LIBCMTD:sbheap.obj
 0001:00050ad0       ___sbh_alloc_block         30051ad0 f   LIBCMTD:sbheap.obj
 0001:00050ff0       ___sbh_alloc_new_region    30051ff0 f   LIBCMTD:sbheap.obj
 0001:00051100       ___sbh_alloc_new_group     30052100 f   LIBCMTD:sbheap.obj
 0001:000512f0       ___sbh_resize_block        300522f0 f   LIBCMTD:sbheap.obj
 0001:000518c0       ___sbh_heapmin             300528c0 f   LIBCMTD:sbheap.obj
 0001:000519f0       ___sbh_heap_check          300529f0 f   LIBCMTD:sbheap.obj
 0001:00051f00       _sprintf                   30052f00 f   LIBCMTD:sprintf.obj
 0001:00051ff0       __scprintf                 30052ff0 f   LIBCMTD:sprintf.obj
 0001:00052070       ___crtInitCritSecAndSpinCount 30053070 f   LIBCMTD:initcrit.obj
 0001:00052190       __ValidateEH3RN            30053190 f   LIBCMTD:eh3valid.obj
 0001:00052580       ___addl                    30053580 f   LIBCMTD:mantold.obj
 0001:000525c0       ___add_12                  300535c0 f   LIBCMTD:mantold.obj
 0001:00052670       ___shl_12                  30053670 f   LIBCMTD:mantold.obj
 0001:000526d0       ___shr_12                  300536d0 f   LIBCMTD:mantold.obj
 0001:00052740       ___mtold12                 30053740 f   LIBCMTD:mantold.obj
 0001:00052890       _$I10_OUTPUT               30053890 f   LIBCMTD:x10fout.obj
 0001:00052d70       ___ld12mul                 30053d70 f   LIBCMTD:tenpow.obj
 0001:00053160       ___multtenpow12            30054160 f   LIBCMTD:tenpow.obj
 0001:00053230       ___tzset                   30054230 f   LIBCMTD:tzset.obj
 0001:000532c0       __tzset                    300542c0 f   LIBCMTD:tzset.obj
 0001:00053750       __isindst                  30054750 f   LIBCMTD:tzset.obj
 0001:00053d30       ___ascii_stricmp           30054d30 f   LIBCMTD:_stricmp.obj
 0001:00053d80       ___getlocaleinfo           30054d80 f   LIBCMTD:inithelp.obj
 0001:00053fe0       __stricmp                  30054fe0 f   LIBCMTD:stricmp.obj
 0001:00054090       __strnicmp                 30055090 f   LIBCMTD:strnicmp.obj
 0001:00054150       __alloc_osfhnd             30055150 f   LIBCMTD:osfinfo.obj
 0001:000543d0       __set_osfhnd               300553d0 f   LIBCMTD:osfinfo.obj
 0001:00054490       __free_osfhnd              30055490 f   LIBCMTD:osfinfo.obj
 0001:00054570       __get_osfhandle            30055570 f   LIBCMTD:osfinfo.obj
 0001:000545e0       __open_osfhandle           300555e0 f   LIBCMTD:osfinfo.obj
 0001:00054730       __lock_fhandle             30055730 f   LIBCMTD:osfinfo.obj
 0001:00054820       __unlock_fhandle           30055820 f   LIBCMTD:osfinfo.obj
 0001:00054850       __lseeki64                 30055850 f   LIBCMTD:lseeki64.obj
 0001:00054970       __lseeki64_lk              30055970 f   LIBCMTD:lseeki64.obj
 0001:00054a40       _fclose                    30055a40 f   LIBCMTD:fclose.obj
 0001:00054b00       __fclose_lk                30055b00 f   LIBCMTD:fclose.obj
 0001:00054bb0       _getenv                    30055bb0 f   LIBCMTD:getenv.obj
 0001:00054c20       __getenv_lk                30055c20 f   LIBCMTD:getenv.obj
 0001:00054cf0       ___crtGetLocaleInfoW       30055cf0 f   LIBCMTD:w_loc.obj
 0001:00054ed0       ___crtGetLocaleInfoA       30055ed0 f   LIBCMTD:a_loc.obj
 0001:000550c0       ___ascii_strnicmp          300560c0 f   LIBCMTD:_strnicm.obj
 0001:00055130       __close                    30056130 f   LIBCMTD:close.obj
 0001:00055220       __close_lk                 30056220 f   LIBCMTD:close.obj
 0001:000552d0       __mbsnbicoll               300562d0 f   LIBCMTD:mbsnbico.obj
 0001:00055340       ___wtomb_environ           30056340 f   LIBCMTD:wtombenv.obj
 0001:00055430       ___crtCompareStringA       30056430 f   LIBCMTD:a_cmp.obj
 0001:000559f0       ___crtsetenv               300569f0 f   LIBCMTD:setenv.obj
 0001:00055ee0       __mbschr                   30056ee0 f   LIBCMTD:mbschr.obj
 0001:00055fa8       _GetModuleFileNameA@12     30056fa8 f   kernel32:KERNEL32.dll
 0001:00055fae       _GetCurrentThreadId@0      30056fae f   kernel32:KERNEL32.dll
 0001:00055fb4       _GetCommandLineA@0         30056fb4 f   kernel32:KERNEL32.dll
 0001:00055fba       _GetVersionExA@4           30056fba f   kernel32:KERNEL32.dll
 0001:00055fc0       _GetProcAddress@8          30056fc0 f   kernel32:KERNEL32.dll
 0001:00055fc6       _GetModuleHandleA@4        30056fc6 f   kernel32:KERNEL32.dll
 0001:00055fcc       _RaiseException@16         30056fcc f   kernel32:KERNEL32.dll
 0001:00055fd2       _TlsAlloc@0                30056fd2 f   kernel32:KERNEL32.dll
 0001:00055fd8       _TlsFree@4                 30056fd8 f   kernel32:KERNEL32.dll
 0001:00055fde       _TlsSetValue@8             30056fde f   kernel32:KERNEL32.dll
 0001:00055fe4       _TlsGetValue@4             30056fe4 f   kernel32:KERNEL32.dll
 0001:00055fea       _SetLastError@4            30056fea f   kernel32:KERNEL32.dll
 0001:00055ff0       _GetLastError@0            30056ff0 f   kernel32:KERNEL32.dll
 0001:00055ff6       _GetCurrentThread@0        30056ff6 f   kernel32:KERNEL32.dll
 0001:00055ffc       _DebugBreak@0              30056ffc f   kernel32:KERNEL32.dll
 0001:00056002       _GetStdHandle@4            30057002 f   kernel32:KERNEL32.dll
 0001:00056008       _WriteFile@20              30057008 f   kernel32:KERNEL32.dll
 0001:0005600e       _InterlockedDecrement@4    3005700e f   kernel32:KERNEL32.dll
 0001:00056014       _OutputDebugStringA@4      30057014 f   kernel32:KERNEL32.dll
 0001:0005601a       _LoadLibraryA@4            3005701a f   kernel32:KERNEL32.dll
 0001:00056020       _InterlockedIncrement@4    30057020 f   kernel32:KERNEL32.dll
 0001:00056026       _TerminateProcess@8        30057026 f   kernel32:KERNEL32.dll
 0001:0005602c       _GetCurrentProcess@0       3005702c f   kernel32:KERNEL32.dll
 0001:00056032       _ExitProcess@4             30057032 f   kernel32:KERNEL32.dll
 0001:00056038       _SetConsoleCtrlHandler@8   30057038 f   kernel32:KERNEL32.dll
 0001:0005603e       _EnterCriticalSection@4    3005703e f   kernel32:KERNEL32.dll
 0001:00056044       _LeaveCriticalSection@4    30057044 f   kernel32:KERNEL32.dll
 0001:0005604a       _WideCharToMultiByte@32    3005704a f   kernel32:KERNEL32.dll
 0001:00056050       _MultiByteToWideChar@24    30057050 f   kernel32:KERNEL32.dll
 0001:00056056       _LCMapStringA@24           30057056 f   kernel32:KERNEL32.dll
 0001:0005605c       _LCMapStringW@24           3005705c f   kernel32:KERNEL32.dll
 0001:00056062       _IsBadWritePtr@8           30057062 f   kernel32:KERNEL32.dll
 0001:00056068       _IsBadReadPtr@8            30057068 f   kernel32:KERNEL32.dll
 0001:0005606e       _HeapValidate@12           3005706e f   kernel32:KERNEL32.dll
 0001:00056074       _SetHandleCount@4          30057074 f   kernel32:KERNEL32.dll
 0001:0005607a       _GetFileType@4             3005707a f   kernel32:KERNEL32.dll
 0001:00056080       _GetStartupInfoA@4         30057080 f   kernel32:KERNEL32.dll
 0001:00056086       _DeleteCriticalSection@4   30057086 f   kernel32:KERNEL32.dll
 0001:0005608c       _FreeEnvironmentStringsA@4 3005708c f   kernel32:KERNEL32.dll
 0001:00056092       _GetEnvironmentStrings@0   30057092 f   kernel32:KERNEL32.dll
 0001:00056098       _FreeEnvironmentStringsW@4 30057098 f   kernel32:KERNEL32.dll
 0001:0005609e       _GetEnvironmentStringsW@0  3005709e f   kernel32:KERNEL32.dll
 0001:000560a4       _HeapDestroy@4             300570a4 f   kernel32:KERNEL32.dll
 0001:000560aa       _HeapCreate@12             300570aa f   kernel32:KERNEL32.dll
 0001:000560b0       _HeapFree@12               300570b0 f   kernel32:KERNEL32.dll
 0001:000560b6       _VirtualFree@12            300570b6 f   kernel32:KERNEL32.dll
 0001:000560bc       _UnhandledExceptionFilter@4 300570bc f   kernel32:KERNEL32.dll
 0001:000560c2       _RtlUnwind@16              300570c2 f   kernel32:KERNEL32.dll
 0001:000560c8       _GetStringTypeA@20         300570c8 f   kernel32:KERNEL32.dll
 0001:000560ce       _GetStringTypeW@16         300570ce f   kernel32:KERNEL32.dll
 0001:000560d4       _GetTimeFormatA@24         300570d4 f   kernel32:KERNEL32.dll
 0001:000560da       _GetDateFormatA@24         300570da f   kernel32:KERNEL32.dll
 0001:000560e0       _GetCPInfo@8               300570e0 f   kernel32:KERNEL32.dll
 0001:000560e6       _FatalAppExitA@8           300570e6 f   kernel32:KERNEL32.dll
 0001:000560ec       _IsValidLocale@8           300570ec f   kernel32:KERNEL32.dll
 0001:000560f2       _IsValidCodePage@4         300570f2 f   kernel32:KERNEL32.dll
 0001:000560f8       _GetLocaleInfoA@16         300570f8 f   kernel32:KERNEL32.dll
 0001:000560fe       _EnumSystemLocalesA@8      300570fe f   kernel32:KERNEL32.dll
 0001:00056104       _GetUserDefaultLCID@0      30057104 f   kernel32:KERNEL32.dll
 0001:0005610a       _GetACP@0                  3005710a f   kernel32:KERNEL32.dll
 0001:00056110       _GetOEMCP@0                30057110 f   kernel32:KERNEL32.dll
 0001:00056116       _SetFilePointer@16         30057116 f   kernel32:KERNEL32.dll
 0001:0005611c       _FlushFileBuffers@4        3005711c f   kernel32:KERNEL32.dll
 0001:00056122       _QueryPerformanceCounter@4 30057122 f   kernel32:KERNEL32.dll
 0001:00056128       _GetTickCount@0            30057128 f   kernel32:KERNEL32.dll
 0001:0005612e       _GetCurrentProcessId@0     3005712e f   kernel32:KERNEL32.dll
 0001:00056134       _GetSystemTimeAsFileTime@4 30057134 f   kernel32:KERNEL32.dll
 0001:0005613a       _VirtualProtect@16         3005713a f   kernel32:KERNEL32.dll
 0001:00056140       _VirtualAlloc@16           30057140 f   kernel32:KERNEL32.dll
 0001:00056146       _GetSystemInfo@4           30057146 f   kernel32:KERNEL32.dll
 0001:0005614c       _VirtualQuery@12           3005714c f   kernel32:KERNEL32.dll
 0001:00056152       _HeapAlloc@12              30057152 f   kernel32:KERNEL32.dll
 0001:00056158       _HeapReAlloc@16            30057158 f   kernel32:KERNEL32.dll
 0001:0005615e       _InitializeCriticalSection@4 3005715e f   kernel32:KERNEL32.dll
 0001:00056164       _InterlockedExchange@8     30057164 f   kernel32:KERNEL32.dll
 0001:0005616a       _GetTimeZoneInformation@4  3005716a f   kernel32:KERNEL32.dll
 0001:00056170       _SetStdHandle@8            30057170 f   kernel32:KERNEL32.dll
 0001:00056176       _GetLocaleInfoW@16         30057176 f   kernel32:KERNEL32.dll
 0001:0005617c       _CloseHandle@4             3005717c f   kernel32:KERNEL32.dll
 0001:00056182       _CompareStringA@24         30057182 f   kernel32:KERNEL32.dll
 0001:00056188       _CompareStringW@24         30057188 f   kernel32:KERNEL32.dll
 0001:0005618e       _SetEnvironmentVariableA@8 3005718e f   kernel32:KERNEL32.dll
 0002:00000000       __imp__GetModuleFileNameA@12 30058000     kernel32:KERNEL32.dll
 0002:00000004       __imp__GetCurrentThreadId@0 30058004     kernel32:KERNEL32.dll
 0002:00000008       __imp__GetCommandLineA@0   30058008     kernel32:KERNEL32.dll
 0002:0000000c       __imp__GetVersionExA@4     3005800c     kernel32:KERNEL32.dll
 0002:00000010       __imp__GetProcAddress@8    30058010     kernel32:KERNEL32.dll
 0002:00000014       __imp__GetModuleHandleA@4  30058014     kernel32:KERNEL32.dll
 0002:00000018       __imp__RaiseException@16   30058018     kernel32:KERNEL32.dll
 0002:0000001c       __imp__TlsAlloc@0          3005801c     kernel32:KERNEL32.dll
 0002:00000020       __imp__TlsFree@4           30058020     kernel32:KERNEL32.dll
 0002:00000024       __imp__TlsSetValue@8       30058024     kernel32:KERNEL32.dll
 0002:00000028       __imp__TlsGetValue@4       30058028     kernel32:KERNEL32.dll
 0002:0000002c       __imp__SetLastError@4      3005802c     kernel32:KERNEL32.dll
 0002:00000030       __imp__GetLastError@0      30058030     kernel32:KERNEL32.dll
 0002:00000034       __imp__GetCurrentThread@0  30058034     kernel32:KERNEL32.dll
 0002:00000038       __imp__DebugBreak@0        30058038     kernel32:KERNEL32.dll
 0002:0000003c       __imp__GetStdHandle@4      3005803c     kernel32:KERNEL32.dll
 0002:00000040       __imp__WriteFile@20        30058040     kernel32:KERNEL32.dll
 0002:00000044       __imp__InterlockedDecrement@4 30058044     kernel32:KERNEL32.dll
 0002:00000048       __imp__OutputDebugStringA@4 30058048     kernel32:KERNEL32.dll
 0002:0000004c       __imp__LoadLibraryA@4      3005804c     kernel32:KERNEL32.dll
 0002:00000050       __imp__InterlockedIncrement@4 30058050     kernel32:KERNEL32.dll
 0002:00000054       __imp__TerminateProcess@8  30058054     kernel32:KERNEL32.dll
 0002:00000058       __imp__GetCurrentProcess@0 30058058     kernel32:KERNEL32.dll
 0002:0000005c       __imp__ExitProcess@4       3005805c     kernel32:KERNEL32.dll
 0002:00000060       __imp__SetConsoleCtrlHandler@8 30058060     kernel32:KERNEL32.dll
 0002:00000064       __imp__EnterCriticalSection@4 30058064     kernel32:KERNEL32.dll
 0002:00000068       __imp__LeaveCriticalSection@4 30058068     kernel32:KERNEL32.dll
 0002:0000006c       __imp__WideCharToMultiByte@32 3005806c     kernel32:KERNEL32.dll
 0002:00000070       __imp__MultiByteToWideChar@24 30058070     kernel32:KERNEL32.dll
 0002:00000074       __imp__LCMapStringA@24     30058074     kernel32:KERNEL32.dll
 0002:00000078       __imp__LCMapStringW@24     30058078     kernel32:KERNEL32.dll
 0002:0000007c       __imp__IsBadWritePtr@8     3005807c     kernel32:KERNEL32.dll
 0002:00000080       __imp__IsBadReadPtr@8      30058080     kernel32:KERNEL32.dll
 0002:00000084       __imp__HeapValidate@12     30058084     kernel32:KERNEL32.dll
 0002:00000088       __imp__SetHandleCount@4    30058088     kernel32:KERNEL32.dll
 0002:0000008c       __imp__GetFileType@4       3005808c     kernel32:KERNEL32.dll
 0002:00000090       __imp__GetStartupInfoA@4   30058090     kernel32:KERNEL32.dll
 0002:00000094       __imp__DeleteCriticalSection@4 30058094     kernel32:KERNEL32.dll
 0002:00000098       __imp__FreeEnvironmentStringsA@4 30058098     kernel32:KERNEL32.dll
 0002:0000009c       __imp__GetEnvironmentStrings@0 3005809c     kernel32:KERNEL32.dll
 0002:000000a0       __imp__FreeEnvironmentStringsW@4 300580a0     kernel32:KERNEL32.dll
 0002:000000a4       __imp__GetEnvironmentStringsW@0 300580a4     kernel32:KERNEL32.dll
 0002:000000a8       __imp__HeapDestroy@4       300580a8     kernel32:KERNEL32.dll
 0002:000000ac       __imp__HeapCreate@12       300580ac     kernel32:KERNEL32.dll
 0002:000000b0       __imp__HeapFree@12         300580b0     kernel32:KERNEL32.dll
 0002:000000b4       __imp__VirtualFree@12      300580b4     kernel32:KERNEL32.dll
 0002:000000b8       __imp__UnhandledExceptionFilter@4 300580b8     kernel32:KERNEL32.dll
 0002:000000bc       __imp__RtlUnwind@16        300580bc     kernel32:KERNEL32.dll
 0002:000000c0       __imp__GetStringTypeA@20   300580c0     kernel32:KERNEL32.dll
 0002:000000c4       __imp__GetStringTypeW@16   300580c4     kernel32:KERNEL32.dll
 0002:000000c8       __imp__GetTimeFormatA@24   300580c8     kernel32:KERNEL32.dll
 0002:000000cc       __imp__GetDateFormatA@24   300580cc     kernel32:KERNEL32.dll
 0002:000000d0       __imp__GetCPInfo@8         300580d0     kernel32:KERNEL32.dll
 0002:000000d4       __imp__FatalAppExitA@8     300580d4     kernel32:KERNEL32.dll
 0002:000000d8       __imp__IsValidLocale@8     300580d8     kernel32:KERNEL32.dll
 0002:000000dc       __imp__IsValidCodePage@4   300580dc     kernel32:KERNEL32.dll
 0002:000000e0       __imp__GetLocaleInfoA@16   300580e0     kernel32:KERNEL32.dll
 0002:000000e4       __imp__EnumSystemLocalesA@8 300580e4     kernel32:KERNEL32.dll
 0002:000000e8       __imp__GetUserDefaultLCID@0 300580e8     kernel32:KERNEL32.dll
 0002:000000ec       __imp__GetACP@0            300580ec     kernel32:KERNEL32.dll
 0002:000000f0       __imp__GetOEMCP@0          300580f0     kernel32:KERNEL32.dll
 0002:000000f4       __imp__SetFilePointer@16   300580f4     kernel32:KERNEL32.dll
 0002:000000f8       __imp__FlushFileBuffers@4  300580f8     kernel32:KERNEL32.dll
 0002:000000fc       __imp__QueryPerformanceCounter@4 300580fc     kernel32:KERNEL32.dll
 0002:00000100       __imp__GetTickCount@0      30058100     kernel32:KERNEL32.dll
 0002:00000104       __imp__GetCurrentProcessId@0 30058104     kernel32:KERNEL32.dll
 0002:00000108       __imp__GetSystemTimeAsFileTime@4 30058108     kernel32:KERNEL32.dll
 0002:0000010c       __imp__VirtualProtect@16   3005810c     kernel32:KERNEL32.dll
 0002:00000110       __imp__VirtualAlloc@16     30058110     kernel32:KERNEL32.dll
 0002:00000114       __imp__GetSystemInfo@4     30058114     kernel32:KERNEL32.dll
 0002:00000118       __imp__VirtualQuery@12     30058118     kernel32:KERNEL32.dll
 0002:0000011c       __imp__HeapAlloc@12        3005811c     kernel32:KERNEL32.dll
 0002:00000120       __imp__HeapReAlloc@16      30058120     kernel32:KERNEL32.dll
 0002:00000124       __imp__InitializeCriticalSection@4 30058124     kernel32:KERNEL32.dll
 0002:00000128       __imp__InterlockedExchange@8 30058128     kernel32:KERNEL32.dll
 0002:0000012c       __imp__GetTimeZoneInformation@4 3005812c     kernel32:KERNEL32.dll
 0002:00000130       __imp__SetStdHandle@8      30058130     kernel32:KERNEL32.dll
 0002:00000134       __imp__GetLocaleInfoW@16   30058134     kernel32:KERNEL32.dll
 0002:00000138       __imp__CloseHandle@4       30058138     kernel32:KERNEL32.dll
 0002:0000013c       __imp__CompareStringA@24   3005813c     kernel32:KERNEL32.dll
 0002:00000140       __imp__CompareStringW@24   30058140     kernel32:KERNEL32.dll
 0002:00000144       __imp__SetEnvironmentVariableA@8 30058144     kernel32:KERNEL32.dll
 0002:00000148       \177KERNEL32_NULL_THUNK_DATA 30058148     kernel32:KERNEL32.dll
 0002:0000016c       ??_C@_08GBKLDCBE@EV_TAUNT?$AA@ 3005816c     bg_misc.obj
 0002:00000178       ??_C@_0BE@OHJHDFJH@EV_STOPLOOPINGSOUND?$AA@ 30058178     bg_misc.obj
 0002:0000018c       ??_C@_0O@PBPAKHP@EV_DEBUG_LINE?$AA@ 3005818c     bg_misc.obj
 0002:0000019c       ??_C@_0BB@HHACOGHI@EV_LIGHTNINGBOLT?$AA@ 3005819c     bg_misc.obj
 0002:000001b0       ??_C@_09GLJGDJEJ@EV_JUICED?$AA@ 300581b0     bg_misc.obj
 0002:000001bc       ??_C@_0BA@NHKGBGBA@EV_INVUL_IMPACT?$AA@ 300581bc     bg_misc.obj
 0002:000001cc       ??_C@_0BC@LMKNBBLF@EV_OBELISKEXPLODE?$AA@ 300581cc     bg_misc.obj
 0002:000001e0       ??_C@_0M@KACLGFEA@EV_KAMIKAZE?$AA@ 300581e0     bg_misc.obj
 0002:000001ec       ??_C@_0BK@PIFCIJEJ@EV_PROXIMITY_MINE_TRIGGER?$AA@ 300581ec     bg_misc.obj
 0002:00000208       ??_C@_0BI@KNJAKDGK@EV_PROXIMITY_MINE_STICK?$AA@ 30058208     bg_misc.obj
 0002:00000220       ??_C@_0N@GAJBP@EV_SCOREPLUM?$AA@ 30058220     bg_misc.obj
 0002:00000230       ??_C@_0O@JLGFLKBE@EV_GIB_PLAYER?$AA@ 30058230     bg_misc.obj
 0002:00000240       ??_C@_0BB@EGIJIDAN@EV_POWERUP_REGEN?$AA@ 30058240     bg_misc.obj
 0002:00000254       ??_C@_0BG@CHAMNADK@EV_POWERUP_BATTLESUIT?$AA@ 30058254     bg_misc.obj
 0002:0000026c       ??_C@_0BA@HLHGHIIE@EV_POWERUP_QUAD?$AA@ 3005826c     bg_misc.obj
 0002:0000027c       ??_C@_0M@PPLCDPP@EV_OBITUARY?$AA@ 3005827c     bg_misc.obj
 0002:00000288       ??_C@_09KNGHBIAK@EV_DEATH3?$AA@ 30058288     bg_misc.obj
 0002:00000294       ??_C@_09LEHMCJEL@EV_DEATH2?$AA@ 30058294     bg_misc.obj
 0002:000002a0       ??_C@_09JPFBHKII@EV_DEATH1?$AA@ 300582a0     bg_misc.obj
 0002:000002ac       ??_C@_07EMHHKOOH@EV_PAIN?$AA@ 300582ac     bg_misc.obj
 0002:000002b4       ??_C@_09ICDIPKFJ@EV_BULLET?$AA@ 300582b4     bg_misc.obj
 0002:000002c0       ??_C@_0L@LHBIHDML@EV_SHOTGUN?$AA@ 300582c0     bg_misc.obj
 0002:000002cc       ??_C@_0N@HMLLJFGF@EV_RAILTRAIL?$AA@ 300582cc     bg_misc.obj
 0002:000002dc       ??_C@_0BG@LPAHEABB@EV_MISSILE_MISS_METAL?$AA@ 300582dc     bg_misc.obj
 0002:000002f4       ??_C@_0BA@CAHALNAE@EV_MISSILE_MISS?$AA@ 300582f4     bg_misc.obj
 0002:00000304       ??_C@_0P@JFMFNBMO@EV_MISSILE_HIT?$AA@ 30058304     bg_misc.obj
 0002:00000314       ??_C@_0BD@MFLMCLPN@EV_BULLET_HIT_WALL?$AA@ 30058314     bg_misc.obj
 0002:00000328       ??_C@_0BE@KBABEJMP@EV_BULLET_HIT_FLESH?$AA@ 30058328     bg_misc.obj
 0002:0000033c       ??_C@_0BF@DDOIKLHD@EV_GLOBAL_TEAM_SOUND?$AA@ 3005833c     bg_misc.obj
 0002:00000354       ??_C@_0BA@JAMKLOPJ@EV_GLOBAL_SOUND?$AA@ 30058354     bg_misc.obj
 0002:00000364       ??_C@_0BB@LJGGMAII@EV_GENERAL_SOUND?$AA@ 30058364     bg_misc.obj
 0002:00000378       ??_C@_0BC@ECIIAFLJ@EV_GRENADE_BOUNCE?$AA@ 30058378     bg_misc.obj
 0002:0000038c       ??_C@_0BH@FNNILPIN@EV_PLAYER_TELEPORT_OUT?$AA@ 3005838c     bg_misc.obj
 0002:000003a4       ??_C@_0BG@HBBJKNDP@EV_PLAYER_TELEPORT_IN?$AA@ 300583a4     bg_misc.obj
 0002:000003bc       ??_C@_0M@ECGFPIMP@EV_ITEM_POP?$AA@ 300583bc     bg_misc.obj
 0002:000003c8       ??_C@_0BA@GJNCODNG@EV_ITEM_RESPAWN?$AA@ 300583c8     bg_misc.obj
 0002:000003d8       ??_C@_0O@HHGOLJPJ@EV_USE_ITEM15?$AA@ 300583d8     bg_misc.obj
 0002:000003e8       ??_C@_0O@GOHFIILI@EV_USE_ITEM14?$AA@ 300583e8     bg_misc.obj
 0002:000003f8       ??_C@_0O@CBDEBOHP@EV_USE_ITEM13?$AA@ 300583f8     bg_misc.obj
 0002:00000408       ??_C@_0O@DICPCPDO@EV_USE_ITEM12?$AA@ 30058408     bg_misc.obj
 0002:00000418       ??_C@_0O@BDACHMPN@EV_USE_ITEM11?$AA@ 30058418     bg_misc.obj
 0002:00000428       ??_C@_0O@KBJENLM@EV_USE_ITEM10?$AA@ 30058428     bg_misc.obj
 0002:00000438       ??_C@_0N@PHODCBCK@EV_USE_ITEM9?$AA@ 30058438     bg_misc.obj
 0002:00000448       ??_C@_0N@OOPIBAGL@EV_USE_ITEM8?$AA@ 30058448     bg_misc.obj
 0002:00000458       ??_C@_0N@GJGAAMKE@EV_USE_ITEM7?$AA@ 30058458     bg_misc.obj
 0002:00000468       ??_C@_0N@HAHLDNOF@EV_USE_ITEM6?$AA@ 30058468     bg_misc.obj
 0002:00000478       ??_C@_0N@FLFGGOCG@EV_USE_ITEM5?$AA@ 30058478     bg_misc.obj
 0002:00000488       ??_C@_0N@ECENFPGH@EV_USE_ITEM4?$AA@ 30058488     bg_misc.obj
 0002:00000498       ??_C@_0N@NAMMJKA@EV_USE_ITEM3?$AA@ 30058498     bg_misc.obj
 0002:000004a8       ??_C@_0N@BEBHPIOB@EV_USE_ITEM2?$AA@ 300584a8     bg_misc.obj
 0002:000004b8       ??_C@_0N@DPDKKLCC@EV_USE_ITEM1?$AA@ 300584b8     bg_misc.obj
 0002:000004c8       ??_C@_0N@CGCBJKGD@EV_USE_ITEM0?$AA@ 300584c8     bg_misc.obj
 0002:000004d8       ??_C@_0P@PFJPAFGH@EV_FIRE_WEAPON?$AA@ 300584d8     bg_misc.obj
 0002:000004e8       ??_C@_0BB@ENKPHJLP@EV_CHANGE_WEAPON?$AA@ 300584e8     bg_misc.obj
 0002:000004fc       ??_C@_09NMIICG@EV_NOAMMO?$AA@ 300584fc     bg_misc.obj
 0002:00000508       ??_C@_0BG@KFILGAMN@EV_GLOBAL_ITEM_PICKUP?$AA@ 30058508     bg_misc.obj
 0002:00000520       ??_C@_0P@BGIOEPCB@EV_ITEM_PICKUP?$AA@ 30058520     bg_misc.obj
 0002:00000530       ??_C@_0P@NIPCJOBG@EV_WATER_CLEAR?$AA@ 30058530     bg_misc.obj
 0002:00000540       ??_C@_0P@MIAIODEJ@EV_WATER_UNDER?$AA@ 30058540     bg_misc.obj
 0002:00000550       ??_C@_0P@LHDMOIIG@EV_WATER_LEAVE?$AA@ 30058550     bg_misc.obj
 0002:00000560       ??_C@_0P@GCDBKPMP@EV_WATER_TOUCH?$AA@ 30058560     bg_misc.obj
 0002:00000570       ??_C@_07GKBEHGAP@EV_JUMP?$AA@ 30058570     bg_misc.obj
 0002:00000578       ??_C@_0M@BPNFGBOJ@EV_JUMP_PAD?$AA@ 30058578     bg_misc.obj
 0002:00000584       ??_C@_0M@LKJJNJOM@EV_FALL_FAR?$AA@ 30058584     bg_misc.obj
 0002:00000590       ??_C@_0P@MGFLMCKC@EV_FALL_MEDIUM?$AA@ 30058590     bg_misc.obj
 0002:000005a0       ??_C@_0O@EAFDHAJM@EV_FALL_SHORT?$AA@ 300585a0     bg_misc.obj
 0002:000005b0       ??_C@_0L@HOOIOPKF@EV_STEP_16?$AA@ 300585b0     bg_misc.obj
 0002:000005bc       ??_C@_0L@BKIECKKB@EV_STEP_12?$AA@ 300585bc     bg_misc.obj
 0002:000005c8       ??_C@_09EHOLDGNN@EV_STEP_8?$AA@ 300585c8     bg_misc.obj
 0002:000005d4       ??_C@_09OLFOHJNB@EV_STEP_4?$AA@ 300585d4     bg_misc.obj
 0002:000005e0       ??_C@_07FFIIIPLH@EV_SWIM?$AA@ 300585e0     bg_misc.obj
 0002:000005e8       ??_C@_0M@NPJBGELA@EV_FOOTWADE?$AA@ 300585e8     bg_misc.obj
 0002:000005f4       ??_C@_0O@HLJHKIDH@EV_FOOTSPLASH?$AA@ 300585f4     bg_misc.obj
 0002:00000604       ??_C@_0BC@DIJMAMMI@EV_FOOTSTEP_METAL?$AA@ 30058604     bg_misc.obj
 0002:00000618       ??_C@_0M@HLKBOJPO@EV_FOOTSTEP?$AA@ 30058618     bg_misc.obj
 0002:00000624       ??_C@_07JFMDDPHJ@EV_NONE?$AA@ 30058624     bg_misc.obj
 0002:0000062c       ??_C@_09MDBFHCAB@Blue?5Flag?$AA@ 3005862c     bg_misc.obj
 0002:00000638       ??_C@_0BB@EMIIAFKA@icons?1iconf_blu1?$AA@ 30058638     bg_misc.obj
 0002:0000064c       ??_C@_0BI@FKICCNIF@models?1flags?1b_flag?4md3?$AA@ 3005864c     bg_misc.obj
 0002:00000664       ??_C@_0BC@NLKCOFAB@team_CTF_blueflag?$AA@ 30058664     bg_misc.obj
 0002:00000678       ??_C@_08GAOGPIJL@Red?5Flag?$AA@ 30058678     bg_misc.obj
 0002:00000684       ??_C@_0BB@EMIEBEOP@icons?1iconf_red1?$AA@ 30058684     bg_misc.obj
 0002:00000698       ??_C@_0BI@PEHEOJEO@models?1flags?1r_flag?4md3?$AA@ 30058698     bg_misc.obj
 0002:000006b0       ??_C@_0BB@JNMMCIHG@team_CTF_redflag?$AA@ 300586b0     bg_misc.obj
 0002:000006c4       ??_C@_06FDKFDAP@Flight?$AA@ 300586c4     bg_misc.obj
 0002:000006cc       ??_C@_0N@GLEPEEPG@icons?1flight?$AA@ 300586cc     bg_misc.obj
 0002:000006dc       ??_C@_0CI@IADFFEDP@models?1powerups?1instant?1flight_r@ 300586dc     bg_misc.obj
 0002:00000704       ??_C@_0CD@MKDGJOMG@models?1powerups?1instant?1flight?4m@ 30058704     bg_misc.obj
 0002:00000728       ??_C@_0BH@COLFHEAE@sound?1items?1flight?4wav?$AA@ 30058728     bg_misc.obj
 0002:00000740       ??_C@_0M@MBNKEMMH@item_flight?$AA@ 30058740     bg_misc.obj
 0002:0000074c       ??_C@_0BG@LHDLOKKN@sound?1items?1regen?4wav?$AA@ 3005874c     bg_misc.obj
 0002:00000764       ??_C@_0N@CBPBLBHG@Regeneration?$AA@ 30058764     bg_misc.obj
 0002:00000774       ??_C@_0M@FDCLJBFC@icons?1regen?$AA@ 30058774     bg_misc.obj
 0002:00000780       ??_C@_0CH@FANACKJM@models?1powerups?1instant?1regen_ri@ 30058780     bg_misc.obj
 0002:000007a8       ??_C@_0CC@OEAPIKIN@models?1powerups?1instant?1regen?4md@ 300587a8     bg_misc.obj
 0002:000007cc       ??_C@_0BN@OBGKHNFF@sound?1items?1regeneration?4wav?$AA@ 300587cc     bg_misc.obj
 0002:000007ec       ??_C@_0L@MMGPPPDM@item_regen?$AA@ 300587ec     bg_misc.obj
 0002:000007f8       ??_C@_0N@LCCEENAK@Invisibility?$AA@ 300587f8     bg_misc.obj
 0002:00000808       ??_C@_0M@FDDJPHJJ@icons?1invis?$AA@ 30058808     bg_misc.obj
 0002:00000814       ??_C@_0CH@IMIHJDNC@models?1powerups?1instant?1invis_ri@ 30058814     bg_misc.obj
 0002:0000083c       ??_C@_0CC@HBONCEML@models?1powerups?1instant?1invis?4md@ 3005883c     bg_misc.obj
 0002:00000860       ??_C@_0BN@OJBEBLGB@sound?1items?1invisibility?4wav?$AA@ 30058860     bg_misc.obj
 0002:00000880       ??_C@_0L@MMHNJJPH@item_invis?$AA@ 30058880     bg_misc.obj
 0002:0000088c       ??_C@_05HOIAGEJD@Speed?$AA@ 3005888c     bg_misc.obj
 0002:00000894       ??_C@_0M@CFINMGCL@icons?1haste?$AA@ 30058894     bg_misc.obj
 0002:000008a0       ??_C@_0CH@KKDDKNEF@models?1powerups?1instant?1haste_ri@ 300588a0     bg_misc.obj
 0002:000008c8       ??_C@_0CC@NKPAJCMI@models?1powerups?1instant?1haste?4md@ 300588c8     bg_misc.obj
 0002:000008ec       ??_C@_0BG@IJMEPCOI@sound?1items?1haste?4wav?$AA@ 300588ec     bg_misc.obj
 0002:00000904       ??_C@_0L@LKMJKIEF@item_haste?$AA@ 30058904     bg_misc.obj
 0002:00000910       ??_C@_0DA@OCPACKGN@sound?1items?1airout?4wav?5sound?1ite@ 30058910     bg_misc.obj
 0002:00000940       ??_C@_0M@ONKEJEFE@Battle?5Suit?$AA@ 30058940     bg_misc.obj
 0002:0000094c       ??_C@_0BB@MGICBJOH@icons?1envirosuit?$AA@ 3005894c     bg_misc.obj
 0002:00000960       ??_C@_0CI@KAEDJDGE@models?1powerups?1instant?1enviro_r@ 30058960     bg_misc.obj
 0002:00000988       ??_C@_0CD@JLGNIGLA@models?1powerups?1instant?1enviro?4m@ 30058988     bg_misc.obj
 0002:000009ac       ??_C@_0BI@DEKBIKDD@sound?1items?1protect?4wav?$AA@ 300589ac     bg_misc.obj
 0002:000009c4       ??_C@_0M@HBCGNAN@item_enviro?$AA@ 300589c4     bg_misc.obj
 0002:000009d0       ??_C@_0DA@PPPPKFJI@sound?1items?1damage2?4wav?5sound?1it@ 300589d0     bg_misc.obj
 0002:00000a00       ??_C@_0M@KOJLOALK@Quad?5Damage?$AA@ 30058a00     bg_misc.obj
 0002:00000a0c       ??_C@_0L@DICHEOBB@icons?1quad?$AA@ 30058a0c     bg_misc.obj
 0002:00000a18       ??_C@_0CG@JNMBMLHJ@models?1powerups?1instant?1quad_rin@ 30058a18     bg_misc.obj
 0002:00000a40       ??_C@_0CB@HIFGFDGN@models?1powerups?1instant?1quad?4md3@ 30058a40     bg_misc.obj
 0002:00000a64       ??_C@_0BL@GLEJLOCA@sound?1items?1quaddamage?4wav?$AA@ 30058a64     bg_misc.obj
 0002:00000a80       ??_C@_09MDKNIFFH@item_quad?$AA@ 30058a80     bg_misc.obj
 0002:00000a8c       ??_C@_0BL@GLIFPGGG@sound?1items?1use_medkit?4wav?$AA@ 30058a8c     bg_misc.obj
 0002:00000aa8       ??_C@_06JDLGEHAD@Medkit?$AA@ 30058aa8     bg_misc.obj
 0002:00000ab0       ??_C@_0N@PNMDFAPK@icons?1medkit?$AA@ 30058ab0     bg_misc.obj
 0002:00000ac0       ??_C@_0CL@LOBKLABC@models?1powerups?1holdable?1medkit_@ 30058ac0     bg_misc.obj
 0002:00000aec       ??_C@_0CE@NKMJILL@models?1powerups?1holdable?1medkit?4@ 30058aec     bg_misc.obj
 0002:00000b10       ??_C@_0BA@PDDMBOCP@holdable_medkit?$AA@ 30058b10     bg_misc.obj
 0002:00000b20       ??_C@_0BE@PCKJDFFA@Personal?5Teleporter?$AA@ 30058b20     bg_misc.obj
 0002:00000b34       ??_C@_0BB@HCFICFKF@icons?1teleporter?$AA@ 30058b34     bg_misc.obj
 0002:00000b48       ??_C@_0CI@FHEOFFOB@models?1powerups?1holdable?1telepor@ 30058b48     bg_misc.obj
 0002:00000b70       ??_C@_0BJ@PNIOAJDI@sound?1items?1holdable?4wav?$AA@ 30058b70     bg_misc.obj
 0002:00000b8c       ??_C@_0BE@GNEKBMLB@holdable_teleporter?$AA@ 30058b8c     bg_misc.obj
 0002:00000ba0       ??_C@_08LIBOGPIN@Bfg?5Ammo?$AA@ 30058ba0     bg_misc.obj
 0002:00000bac       ??_C@_0BA@NIKNDLKG@icons?1icona_bfg?$AA@ 30058bac     bg_misc.obj
 0002:00000bbc       ??_C@_0BP@BOBKFIKJ@models?1powerups?1ammo?1bfgam?4md3?$AA@ 30058bbc     bg_misc.obj
 0002:00000bdc       ??_C@_08EHEJHGBG@ammo_bfg?$AA@ 30058bdc     bg_misc.obj
 0002:00000be8       ??_C@_05INIOBJHH@Slugs?$AA@ 30058be8     bg_misc.obj
 0002:00000bf0       ??_C@_0BE@DPOADFL@icons?1icona_railgun?$AA@ 30058bf0     bg_misc.obj
 0002:00000c04       ??_C@_0CD@CAJEPMME@models?1powerups?1ammo?1railgunam?4m@ 30058c04     bg_misc.obj
 0002:00000c28       ??_C@_0L@JEFOIHIM@ammo_slugs?$AA@ 30058c28     bg_misc.obj
 0002:00000c34       ??_C@_07MLLADOAB@Rockets?$AA@ 30058c34     bg_misc.obj
 0002:00000c3c       ??_C@_0BD@BFBJLPJK@icons?1icona_rocket?$AA@ 30058c3c     bg_misc.obj
 0002:00000c50       ??_C@_0CC@KCOEDLFM@models?1powerups?1ammo?1rocketam?4md@ 30058c50     bg_misc.obj
 0002:00000c74       ??_C@_0N@CLEPKBOE@ammo_rockets?$AA@ 30058c74     bg_misc.obj
 0002:00000c84       ??_C@_09JCCOMJEA@Lightning?$AA@ 30058c84     bg_misc.obj
 0002:00000c90       ??_C@_0BG@MEGMAGOM@icons?1icona_lightning?$AA@ 30058c90     bg_misc.obj
 0002:00000ca8       ??_C@_0CF@HDAADIIL@models?1powerups?1ammo?1lightningam@ 30058ca8     bg_misc.obj
 0002:00000cd0       ??_C@_0P@NBJHKAMD@ammo_lightning?$AA@ 30058cd0     bg_misc.obj
 0002:00000ce0       ??_C@_05KCAMIOGJ@Cells?$AA@ 30058ce0     bg_misc.obj
 0002:00000ce8       ??_C@_0BD@NCNJEHKB@icons?1icona_plasma?$AA@ 30058ce8     bg_misc.obj
 0002:00000cfc       ??_C@_0CC@FGLALJGN@models?1powerups?1ammo?1plasmaam?4md@ 30058cfc     bg_misc.obj
 0002:00000d20       ??_C@_0L@LLNMBAJC@ammo_cells?$AA@ 30058d20     bg_misc.obj
 0002:00000d2c       ??_C@_08PMBIADEN@Grenades?$AA@ 30058d2c     bg_misc.obj
 0002:00000d38       ??_C@_0BE@LHOKGGAM@icons?1icona_grenade?$AA@ 30058d38     bg_misc.obj
 0002:00000d4c       ??_C@_0CD@HNOBKKLC@models?1powerups?1ammo?1grenadeam?4m@ 30058d4c     bg_misc.obj
 0002:00000d70       ??_C@_0O@CMJIOKCF@ammo_grenades?$AA@ 30058d70     bg_misc.obj
 0002:00000d80       ??_C@_07DHNDKCGP@Bullets?$AA@ 30058d80     bg_misc.obj
 0002:00000d88       ??_C@_0BH@HMOAGCNP@icons?1icona_machinegun?$AA@ 30058d88     bg_misc.obj
 0002:00000da0       ??_C@_0CG@OLENEOKN@models?1powerups?1ammo?1machineguna@ 30058da0     bg_misc.obj
 0002:00000dc8       ??_C@_0N@NHCMDNIK@ammo_bullets?$AA@ 30058dc8     bg_misc.obj
 0002:00000dd8       ??_C@_06PBPEPGGL@Shells?$AA@ 30058dd8     bg_misc.obj
 0002:00000de0       ??_C@_0BE@NMAFHJEI@icons?1icona_shotgun?$AA@ 30058de0     bg_misc.obj
 0002:00000df4       ??_C@_0CD@MBAGJHDE@models?1powerups?1ammo?1shotgunam?4m@ 30058df4     bg_misc.obj
 0002:00000e18       ??_C@_0BH@DPAADLFH@sound?1misc?1am_pkup?4wav?$AA@ 30058e18     bg_misc.obj
 0002:00000e30       ??_C@_0M@NLICANGB@ammo_shells?$AA@ 30058e30     bg_misc.obj
 0002:00000e3c       ??_C@_0P@CFJPDDC@Grappling?5Hook?$AA@ 30058e3c     bg_misc.obj
 0002:00000e4c       ??_C@_0BE@DPKNJNBE@icons?1iconw_grapple?$AA@ 30058e4c     bg_misc.obj
 0002:00000e60       ??_C@_0CE@LFAGANA@models?1weapons2?1grapple?1grapple?4@ 30058e60     bg_misc.obj
 0002:00000e84       ??_C@_0BF@MEMGGPGH@weapon_grapplinghook?$AA@ 30058e84     bg_misc.obj
 0002:00000e9c       ??_C@_06PNKEMFGD@BFG10K?$AA@ 30058e9c     bg_misc.obj
 0002:00000ea4       ??_C@_0BA@NCCNKCA@icons?1iconw_bfg?$AA@ 30058ea4     bg_misc.obj
 0002:00000eb4       ??_C@_0BM@HHDGGOHP@models?1weapons2?1bfg?1bfg?4md3?$AA@ 30058eb4     bg_misc.obj
 0002:00000ed0       ??_C@_0L@JBGNLNGG@weapon_bfg?$AA@ 30058ed0     bg_misc.obj
 0002:00000edc       ??_C@_0L@JFFCGJF@Plasma?5Gun?$AA@ 30058edc     bg_misc.obj
 0002:00000ee8       ??_C@_0BD@NADHMFK@icons?1iconw_plasma?$AA@ 30058ee8     bg_misc.obj
 0002:00000efc       ??_C@_0CC@EHGHEDND@models?1weapons2?1plasma?1plasma?4md@ 30058efc     bg_misc.obj
 0002:00000f20       ??_C@_0BB@LBHAKENA@weapon_plasmagun?$AA@ 30058f20     bg_misc.obj
 0002:00000f34       ??_C@_07NMJDHEIK@Railgun?$AA@ 30058f34     bg_misc.obj
 0002:00000f3c       ??_C@_0BE@CJEOPCPE@icons?1iconw_railgun?$AA@ 30058f3c     bg_misc.obj
 0002:00000f50       ??_C@_0CE@JHJFFEBE@models?1weapons2?1railgun?1railgun?4@ 30058f50     bg_misc.obj
 0002:00000f74       ??_C@_0P@FEPBKEBF@weapon_railgun?$AA@ 30058f74     bg_misc.obj
 0002:00000f84       ??_C@_0O@HOCKKNKE@Lightning?5Gun?$AA@ 30058f84     bg_misc.obj
 0002:00000f94       ??_C@_0BG@CHEJEOPA@icons?1iconw_lightning?$AA@ 30058f94     bg_misc.obj
 0002:00000fac       ??_C@_0CI@MNAFJDPO@models?1weapons2?1lightning?1lightn@ 30058fac     bg_misc.obj
 0002:00000fd4       ??_C@_0BB@OCCEAFCD@weapon_lightning?$AA@ 30058fd4     bg_misc.obj
 0002:00000fe8       ??_C@_0BA@DJIGCIDL@Rocket?5Launcher?$AA@ 30058fe8     bg_misc.obj
 0002:00000ff8       ??_C@_0BD@MKMDIEGB@icons?1iconw_rocket?$AA@ 30058ff8     bg_misc.obj
 0002:0000100c       ??_C@_0CE@GGGFLKKE@models?1weapons2?1rocketl?1rocketl?4@ 3005900c     bg_misc.obj
 0002:00001030       ??_C@_0BG@HJKONAJE@weapon_rocketlauncher?$AA@ 30059030     bg_misc.obj
 0002:00001048       ??_C@_0EG@LFEMOCGK@sound?1weapons?1grenade?1hgrenb1a?4w@ 30059048     bg_misc.obj
 0002:00001090       ??_C@_0BB@GIEOMMBO@Grenade?5Launcher?$AA@ 30059090     bg_misc.obj
 0002:000010a4       ??_C@_0BE@JNFKJHKD@icons?1iconw_grenade?$AA@ 300590a4     bg_misc.obj
 0002:000010b8       ??_C@_0CG@INCGOMDL@models?1weapons2?1grenadel?1grenade@ 300590b8     bg_misc.obj
 0002:000010e0       ??_C@_0BH@DGCCJPLM@weapon_grenadelauncher?$AA@ 300590e0     bg_misc.obj
 0002:000010f8       ??_C@_0L@KDNGMPND@Machinegun?$AA@ 300590f8     bg_misc.obj
 0002:00001104       ??_C@_0BH@GIACBLNI@icons?1iconw_machinegun?$AA@ 30059104     bg_misc.obj
 0002:0000111c       ??_C@_0CK@BBPFNIFO@models?1weapons2?1machinegun?1machi@ 3005911c     bg_misc.obj
 0002:00001148       ??_C@_0BC@HHBNPFPN@weapon_machinegun?$AA@ 30059148     bg_misc.obj
 0002:0000115c       ??_C@_07DGIAOJJ@Shotgun?$AA@ 3005915c     bg_misc.obj
 0002:00001164       ??_C@_0BE@PGLFIIOH@icons?1iconw_shotgun?$AA@ 30059164     bg_misc.obj
 0002:00001178       ??_C@_0CE@CJGCHKCN@models?1weapons2?1shotgun?1shotgun?4@ 30059178     bg_misc.obj
 0002:0000119c       ??_C@_0P@ILAKNOAG@weapon_shotgun?$AA@ 3005919c     bg_misc.obj
 0002:000011ac       ??_C@_08ELAHAPJB@Gauntlet?$AA@ 300591ac     bg_misc.obj
 0002:000011b8       ??_C@_0BF@PMEPIOCM@icons?1iconw_gauntlet?$AA@ 300591b8     bg_misc.obj
 0002:000011d0       ??_C@_0CG@PFPPJBAC@models?1weapons2?1gauntlet?1gauntle@ 300591d0     bg_misc.obj
 0002:000011f8       ??_C@_0BG@BBKFHONL@sound?1misc?1w_pkup?4wav?$AA@ 300591f8     bg_misc.obj
 0002:00001210       ??_C@_0BA@CLDPODJE@weapon_gauntlet?$AA@ 30059210     bg_misc.obj
 0002:00001220       ??_C@_0M@IOJDMPNO@Mega?5Health?$AA@ 30059220     bg_misc.obj
 0002:0000122c       ??_C@_0BB@EGPGIMOM@icons?1iconh_mega?$AA@ 3005922c     bg_misc.obj
 0002:00001240       ??_C@_0CH@NEGHBKPB@models?1powerups?1health?1mega_sphe@ 30059240     bg_misc.obj
 0002:00001268       ??_C@_0CG@PDJMMGME@models?1powerups?1health?1mega_cros@ 30059268     bg_misc.obj
 0002:00001290       ??_C@_0BJ@FGLGEHNG@sound?1items?1m_health?4wav?$AA@ 30059290     bg_misc.obj
 0002:000012ac       ??_C@_0BB@PBGAONGH@item_health_mega?$AA@ 300592ac     bg_misc.obj
 0002:000012c0       ??_C@_09EBELOOOD@50?5Health?$AA@ 300592c0     bg_misc.obj
 0002:000012cc       ??_C@_0BA@IGNANAGL@icons?1iconh_red?$AA@ 300592cc     bg_misc.obj
 0002:000012dc       ??_C@_0CI@CEEMEFNH@models?1powerups?1health?1large_sph@ 300592dc     bg_misc.obj
 0002:00001304       ??_C@_0CH@NHFAKEFE@models?1powerups?1health?1large_cro@ 30059304     bg_misc.obj
 0002:0000132c       ??_C@_0BJ@ILCAJOFD@sound?1items?1l_health?4wav?$AA@ 3005932c     bg_misc.obj
 0002:00001348       ??_C@_0BC@JGDLKFIO@item_health_large?$AA@ 30059348     bg_misc.obj
 0002:0000135c       ??_C@_09OJAALANF@25?5Health?$AA@ 3005935c     bg_misc.obj
 0002:00001368       ??_C@_0BD@CDBLAHCA@icons?1iconh_yellow?$AA@ 30059368     bg_misc.obj
 0002:0000137c       ??_C@_0CJ@NCCPDHOD@models?1powerups?1health?1medium_sp@ 3005937c     bg_misc.obj
 0002:000013a8       ??_C@_0CI@NAEMLIB@models?1powerups?1health?1medium_cr@ 300593a8     bg_misc.obj
 0002:000013d0       ??_C@_0BJ@OLHMCLBI@sound?1items?1n_health?4wav?$AA@ 300593d0     bg_misc.obj
 0002:000013ec       ??_C@_0M@KCNAKNNL@item_health?$AA@ 300593ec     bg_misc.obj
 0002:000013f8       ??_C@_08IAIFJOAI@5?5Health?$AA@ 300593f8     bg_misc.obj
 0002:00001404       ??_C@_0BC@IMNPBGFF@icons?1iconh_green?$AA@ 30059404     bg_misc.obj
 0002:00001418       ??_C@_0CI@MPAPPIIE@models?1powerups?1health?1small_sph@ 30059418     bg_misc.obj
 0002:00001440       ??_C@_0CH@JKNLMIJB@models?1powerups?1health?1small_cro@ 30059440     bg_misc.obj
 0002:00001468       ??_C@_0BJ@BIFHONLM@sound?1items?1s_health?4wav?$AA@ 30059468     bg_misc.obj
 0002:00001484       ??_C@_0BC@DOHAFEBI@item_health_small?$AA@ 30059484     bg_misc.obj
 0002:00001498       ??_C@_0M@ICCAHGAD@Heavy?5Armor?$AA@ 30059498     bg_misc.obj
 0002:000014a4       ??_C@_0BA@CEJNPBJG@icons?1iconr_red?$AA@ 300594a4     bg_misc.obj
 0002:000014b4       ??_C@_0CE@EGJFDJJK@models?1powerups?1armor?1armor_red?4@ 300594b4     bg_misc.obj
 0002:000014d8       ??_C@_0BA@EKKMHIH@item_armor_body?$AA@ 300594d8     bg_misc.obj
 0002:000014e8       ??_C@_05JOOFIMIN@Armor?$AA@ 300594e8     bg_misc.obj
 0002:000014f0       ??_C@_0BD@BKPFMPMP@icons?1iconr_yellow?$AA@ 300594f0     bg_misc.obj
 0002:00001504       ??_C@_0CE@PHKMKHKB@models?1powerups?1armor?1armor_yel?4@ 30059504     bg_misc.obj
 0002:00001528       ??_C@_0BI@KNMPECGK@sound?1misc?1ar2_pkup?4wav?$AA@ 30059528     bg_misc.obj
 0002:00001540       ??_C@_0BC@FPPLPJIL@item_armor_combat?$AA@ 30059540     bg_misc.obj
 0002:00001554       ??_C@_0M@PJIPIDNH@Armor?5Shard?$AA@ 30059554     bg_misc.obj
 0002:00001560       ??_C@_0BC@LPFHDODA@icons?1iconr_shard?$AA@ 30059560     bg_misc.obj
 0002:00001574       ??_C@_0CH@NEKDLKN@models?1powerups?1armor?1shard_sphe@ 30059574     bg_misc.obj
 0002:0000159c       ??_C@_0CA@NOFOCCIK@models?1powerups?1armor?1shard?4md3?$AA@ 3005959c     bg_misc.obj
 0002:000015bc       ??_C@_0BI@DECNCEGL@sound?1misc?1ar1_pkup?4wav?$AA@ 300595bc     bg_misc.obj
 0002:000015d4       ??_C@_0BB@DDGIAABK@item_armor_shard?$AA@ 300595d4     bg_misc.obj
 0002:000015e5       ??_C@_00CNPNBAHC@?$AA@     300595e5     bg_misc.obj
 0002:000015e8       ??_C@_0BH@MFGKJDLM@HoldableItem?5not?5found?$AA@ 300595e8     bg_misc.obj
 0002:00001600       ??_C@_0CB@DEACFJO@Couldn?8t?5find?5item?5for?5weapon?5?$CFi@ 30059600     bg_misc.obj
 0002:00001624       __real@c2100000            30059624     bg_misc.obj
 0002:00001628       __real@42100000            30059628     bg_misc.obj
 0002:0000162c       __real@c2480000            3005962c     bg_misc.obj
 0002:00001630       __real@42300000            30059630     bg_misc.obj
 0002:00001634       ??_C@_0CG@HNLFCMEK@BG_CanItemBeGrabbed?3?5unknown?5enu@ 30059634     bg_misc.obj
 0002:0000165c       ??_C@_0BM@NECGLAIF@BG_CanItemBeGrabbed?3?5IT_BAD?$AA@ 3005965c     bg_misc.obj
 0002:00001678       ??_C@_0CI@MFONMA@BG_CanItemBeGrabbed?3?5index?5out?5o@ 30059678     bg_misc.obj
 0002:000016a0       ??_C@_0CK@DNBGNAED@BG_EvaluateTrajectory?3?5unknown?5t@ 300596a0     bg_misc.obj
 0002:000016d0       __real@4079000000000000    300596d0     bg_misc.obj
 0002:000016d8       __real@00000000            300596d8     bg_misc.obj
 0002:000016dc       __real@40490fdb            300596dc     bg_misc.obj
 0002:000016e0       __real@3f50624dd2f1a9fc    300596e0     bg_misc.obj
 0002:000016e8       ??_C@_0CP@MCFPOIMF@BG_EvaluateTrajectoryDelta?3?5unkn@ 300596e8     bg_misc.obj
 0002:00001718       __real@44480000            30059718     bg_misc.obj
 0002:00001720       __real@3fe0000000000000    30059720     bg_misc.obj
 0002:00001728       ??_C@_0DA@KOPJLGJF@Cgame?5event?5svt?5?$CF5d?5?9?$DO?5?$CF5d?3?5num?5@ 30059728     bg_misc.obj
 0002:00001758       __real@0000000000000000    30059758     bg_misc.obj
 0002:00001760       ??_C@_0L@MNPDPHLD@showevents?$AA@ 30059760     bg_misc.obj
 0002:0000176c       __real@42340000            3005976c     bg_misc.obj
 0002:00001770       __real@3f76800000000000    30059770     bg_pmove.obj
 0002:00001778       __real@3f800000            30059778     bg_pmove.obj
 0002:00001780       __real@405fc00000000000    30059780     bg_pmove.obj
 0002:00001788       __real@43480000            30059788     bg_pmove.obj
 0002:0000178c       __real@41800000            3005978c     bg_pmove.obj
 0002:00001790       __real@40800000            30059790     bg_pmove.obj
 0002:00001794       __real@41f00000            30059794     bg_pmove.obj
 0002:00001798       __real@41200000            30059798     bg_pmove.obj
 0002:0000179c       __real@42c80000            3005979c     bg_pmove.obj
 0002:000017a0       __real@c1800000            300597a0     bg_pmove.obj
 0002:000017a8       __real@3ff0000000000000    300597a8     bg_pmove.obj
 0002:000017b0       __real@4008000000000000    300597b0     bg_pmove.obj
 0002:000017b8       __real@41a00000            300597b8     bg_pmove.obj
 0002:000017c0       __real@3ff8000000000000    300597c0     bg_pmove.obj
 0002:000017c8       __real@c3480000            300597c8     bg_pmove.obj
 0002:000017cc       ??_C@_08KACHPCJN@?$CFi?3Land?6?$AA@ 300597cc     bg_pmove.obj
 0002:000017d8       ??_C@_09OPMLNNOA@?$CFi?3steep?6?$AA@ 300597d8     bg_pmove.obj
 0002:000017e4       __real@3f333333            300597e4     bg_pmove.obj
 0002:000017e8       ??_C@_0M@CKJFDFGH@?$CFi?3kickoff?6?$AA@ 300597e8     bg_pmove.obj
 0002:000017f8       __real@3fd0000000000000    300597f8     bg_pmove.obj
 0002:00001800       __real@40e00000            30059800     bg_pmove.obj
 0002:00001804       __real@42200000            30059804     bg_pmove.obj
 0002:00001808       __real@42700000            30059808     bg_pmove.obj
 0002:00001810       __real@3f1a36e2eb1c432d    30059810     bg_pmove.obj
 0002:00001818       __real@40000000            30059818     bg_pmove.obj
 0002:0000181c       ??_C@_0N@KJCNHCBK@?$CFi?3allsolid?6?$AA@ 3005981c     bg_pmove.obj
 0002:0000182c       __real@42800000            3005982c     bg_pmove.obj
 0002:00001830       ??_C@_08EOGJDHPF@?$CFi?3lift?6?$AA@ 30059830     bg_pmove.obj
 0002:0000183c       __real@c1c00000            3005983c     bg_pmove.obj
 0002:00001840       __real@40a00000            30059840     bg_pmove.obj
 0002:00001848       __real@3ff4cccccccccccd    30059848     bg_pmove.obj
 0002:00001850       __real@3fb999999999999a    30059850     bg_slidemove.obj
 0002:00001858       __real@3fefae147ae147ae    30059858     bg_slidemove.obj
 0002:00001860       ??_C@_0M@CDHDENEF@?$CFi?3stepped?6?$AA@ 30059860     bg_slidemove.obj
 0002:0000186c       __real@41700000            3005986c     bg_slidemove.obj
 0002:00001870       __real@41300000            30059870     bg_slidemove.obj
 0002:00001874       ??_C@_0BE@FLPNHHPN@?$CFi?3bend?5can?8t?5step?6?$AA@ 30059874     bg_slidemove.obj
 0002:00001888       __real@3fe6666666666666    30059888     bg_slidemove.obj
 0002:00001890       __real@41900000            30059890     bg_slidemove.obj
 0002:00001894       ??_C@_0N@FDCACBMC@loaddeferred?$AA@ 30059894     cg_consolecmds.obj
 0002:000018a4       ??_C@_0L@FBDGNAPC@startOrbit?$AA@ 300598a4     cg_consolecmds.obj
 0002:000018b0       ??_C@_04FNICOANA@tcmd?$AA@ 300598b0     cg_consolecmds.obj
 0002:000018b8       ??_C@_0P@KDBBCIM@vtell_attacker?$AA@ 300598b8     cg_consolecmds.obj
 0002:000018c8       ??_C@_0N@OKPMAMBK@vtell_target?$AA@ 300598c8     cg_consolecmds.obj
 0002:000018d8       ??_C@_0O@CIPPGGPC@tell_attacker?$AA@ 300598d8     cg_consolecmds.obj
 0002:000018e8       ??_C@_0M@IEEMCPKO@tell_target?$AA@ 300598e8     cg_consolecmds.obj
 0002:000018f4       ??_C@_06GEPNGEJI@weapon?$AA@ 300598f4     cg_consolecmds.obj
 0002:000018fc       ??_C@_08DMEBPOGB@weapprev?$AA@ 300598fc     cg_consolecmds.obj
 0002:00001908       ??_C@_08IJHOKAF@weapnext?$AA@ 30059908     cg_consolecmds.obj
 0002:00001914       ??_C@_08KKGKLAHJ@sizedown?$AA@ 30059914     cg_consolecmds.obj
 0002:00001920       ??_C@_06FCHHJILH@sizeup?$AA@ 30059920     cg_consolecmds.obj
 0002:00001928       ??_C@_05LGPAMOHI@?9zoom?$AA@ 30059928     cg_consolecmds.obj
 0002:00001930       ??_C@_05GAKJCNGF@?$CLzoom?$AA@ 30059930     cg_consolecmds.obj
 0002:00001938       ??_C@_07DLBEELCG@?9scores?$AA@ 30059938     cg_consolecmds.obj
 0002:00001940       ??_C@_07PNHLECKB@?$CLscores?$AA@ 30059940     cg_consolecmds.obj
 0002:00001948       ??_C@_07NBKBBFDF@viewpos?$AA@ 30059948     cg_consolecmds.obj
 0002:00001950       ??_C@_08ONPIGPGM@prevskin?$AA@ 30059950     cg_consolecmds.obj
 0002:0000195c       ??_C@_08LEEFJCLI@nextskin?$AA@ 3005995c     cg_consolecmds.obj
 0002:00001968       ??_C@_09KFHKLKJD@prevframe?$AA@ 30059968     cg_consolecmds.obj
 0002:00001974       ??_C@_09CEJNBBKD@nextframe?$AA@ 30059974     cg_consolecmds.obj
 0002:00001980       ??_C@_09FDMDKFOH@testmodel?$AA@ 30059980     cg_consolecmds.obj
 0002:0000198c       ??_C@_07OFBIMGPG@testgun?$AA@ 3005998c     cg_consolecmds.obj
 0002:00001994       ??_C@_08FJOFODJK@gc?5?$CFi?5?$CFi?$AA@ 30059994     cg_consolecmds.obj
 0002:000019a0       ??_C@_0M@NABCNGBA@cg_viewsize?$AA@ 300599a0     cg_consolecmds.obj
 0002:000019ac       ??_C@_02IKAHHCAI@?$CFi?$AA@ 300599ac     cg_consolecmds.obj
 0002:000019b0       ??_C@_0BB@MJMOCNNN@?$CI?$CFi?5?$CFi?5?$CFi?$CJ?5?3?5?$CFi?6?$AA@ 300599b0     cg_consolecmds.obj
 0002:000019c4       ??_C@_05DBKDOICH@score?$AA@ 300599c4     cg_consolecmds.obj
 0002:000019cc       ??_C@_0L@EGAGNODH@tell?5?$CFi?5?$CFs?$AA@ 300599cc     cg_consolecmds.obj
 0002:000019d8       ??_C@_0M@JNCDINKA@vtell?5?$CFi?5?$CFs?$AA@ 300599d8     cg_consolecmds.obj
 0002:000019e4       ??_C@_0BE@FKFEAA@cg_thirdPersonRange?$AA@ 300599e4     cg_consolecmds.obj
 0002:000019f8       ??_C@_03GNABGMEE@100?$AA@  300599f8     cg_consolecmds.obj
 0002:000019fc       ??_C@_0BE@HGBFBDIP@cg_thirdPersonAngle?$AA@ 300599fc     cg_consolecmds.obj
 0002:00001a10       ??_C@_01HIHLOKLC@1?$AA@    30059a10     cg_consolecmds.obj
 0002:00001a14       ??_C@_01BMBHCPLG@5?$AA@    30059a14     cg_consolecmds.obj
 0002:00001a18       ??_C@_0P@OPFJLCMG@cg_thirdPerson?$AA@ 30059a18     cg_consolecmds.obj
 0002:00001a28       ??_C@_0P@GDCMABHL@cg_cameraOrbit?$AA@ 30059a28     cg_consolecmds.obj
 0002:00001a38       ??_C@_01GBGANLPD@0?$AA@    30059a38     cg_consolecmds.obj
 0002:00001a3c       ??_C@_09DNECJBKD@developer?$AA@ 30059a3c     cg_consolecmds.obj
 0002:00001a48       ??_C@_0M@NJBPNDAH@loaddefered?$AA@ 30059a48     cg_consolecmds.obj
 0002:00001a54       ??_C@_08OKGPDOIO@teamtask?$AA@ 30059a54     cg_consolecmds.obj
 0002:00001a60       ??_C@_05BLKJBNOD@stats?$AA@ 30059a60     cg_consolecmds.obj
 0002:00001a68       ??_C@_08OLLMCBNG@teamvote?$AA@ 30059a68     cg_consolecmds.obj
 0002:00001a74       ??_C@_0N@JDBKAFAM@callteamvote?$AA@ 30059a74     cg_consolecmds.obj
 0002:00001a84       ??_C@_04GHHIKFLG@vote?$AA@ 30059a84     cg_consolecmds.obj
 0002:00001a8c       ??_C@_08NNMLCPB@callvote?$AA@ 30059a8c     cg_consolecmds.obj
 0002:00001a98       ??_C@_0L@CCEFBCKP@setviewpos?$AA@ 30059a98     cg_consolecmds.obj
 0002:00001aa4       ??_C@_06CJHCPEHG@addbot?$AA@ 30059aa4     cg_consolecmds.obj
 0002:00001aac       ??_C@_09EFOFPGPE@levelshot?$AA@ 30059aac     cg_consolecmds.obj
 0002:00001ab8       ??_C@_06HNJAFFAK@follow?$AA@ 30059ab8     cg_consolecmds.obj
 0002:00001ac0       ??_C@_04KADBPNCB@team?$AA@ 30059ac0     cg_consolecmds.obj
 0002:00001ac8       ??_C@_06IHODGGMJ@noclip?$AA@ 30059ac8     cg_consolecmds.obj
 0002:00001ad0       ??_C@_08HPLPOCJL@notarget?$AA@ 30059ad0     cg_consolecmds.obj
 0002:00001adc       ??_C@_03DKFAMNOH@god?$AA@  30059adc     cg_consolecmds.obj
 0002:00001ae0       ??_C@_04BMBHJADG@give?$AA@ 30059ae0     cg_consolecmds.obj
 0002:00001ae8       ??_C@_06JMKGCPMO@votell?$AA@ 30059ae8     cg_consolecmds.obj
 0002:00001af0       ??_C@_0L@GKKIAMHC@vosay_team?$AA@ 30059af0     cg_consolecmds.obj
 0002:00001afc       ??_C@_05EGEGDMMG@vosay?$AA@ 30059afc     cg_consolecmds.obj
 0002:00001b04       ??_C@_06IMDBNOMM@vtaunt?$AA@ 30059b04     cg_consolecmds.obj
 0002:00001b0c       ??_C@_05BLGJOHFB@vtell?$AA@ 30059b0c     cg_consolecmds.obj
 0002:00001b14       ??_C@_09CPIJOHHK@vsay_team?$AA@ 30059b14     cg_consolecmds.obj
 0002:00001b20       ??_C@_04IBCNHBFH@vsay?$AA@ 30059b20     cg_consolecmds.obj
 0002:00001b28       ??_C@_04LBPCFPDD@tell?$AA@ 30059b28     cg_consolecmds.obj
 0002:00001b30       ??_C@_08NBFNGOHN@say_team?$AA@ 30059b30     cg_consolecmds.obj
 0002:00001b3c       ??_C@_03BANJEMDJ@say?$AA@  30059b3c     cg_consolecmds.obj
 0002:00001b40       ??_C@_04BJJEOANI@kill?$AA@ 30059b40     cg_consolecmds.obj
 0002:00001b48       __real@3fd126e978d4fdf4    30059b48     cg_draw.obj
 0002:00001b50       __real@bfe0000000000000    30059b50     cg_draw.obj
 0002:00001b58       __real@404e000000000000    30059b58     cg_draw.obj
 0002:00001b60       __real@409f400000000000    30059b60     cg_draw.obj
 0002:00001b68       ??_C@_0CE@GNKHIBFA@CG_DrawActive?3?5Undefined?5stereoV@ 30059b68     cg_draw.obj
 0002:00001b90       __real@40a0000000000000    30059b90     cg_draw.obj
 0002:00001b98       __real@4056800000000000    30059b98     cg_draw.obj
 0002:00001ba0       __real@4034000000000000    30059ba0     cg_draw.obj
 0002:00001ba8       __real@408f400000000000    30059ba8     cg_draw.obj
 0002:00001bb0       __real@43f00000            30059bb0     cg_draw.obj
 0002:00001bb4       __real@40400000            30059bb4     cg_draw.obj
 0002:00001bb8       __real@44fa0000            30059bb8     cg_draw.obj
 0002:00001bc0       __real@4014000000000000    30059bc0     cg_draw.obj
 0002:00001bc8       __real@4066800000000000    30059bc8     cg_draw.obj
 0002:00001bd0       __real@400921fb60000000    30059bd0     cg_draw.obj
 0002:00001bd8       __real@46fffe00            30059bd8     cg_draw.obj
 0002:00001bdc       __real@43340000            30059bdc     cg_draw.obj
 0002:00001be0       __real@43fa0000            30059be0     cg_draw.obj
 0002:00001be4       ??_C@_01EFFIKLCJ@n?$AA@    30059be4     cg_draw.obj
 0002:00001be8       __real@44200000            30059be8     cg_draw.obj
 0002:00001bec       ??_C@_0BH@OGHHEKME@time?3?$CFi?5snap?3?$CFi?5cmd?3?$CFi?$AA@ 30059bec     cg_draw.obj
 0002:00001c04       ??_C@_05MDNADFFP@?$CFifps?$AA@ 30059c04     cg_draw.obj
 0002:00001c0c       ??_C@_07FFDCCNEB@?$CFi?3?$CFi?$CFi?$AA@ 30059c0c     cg_draw.obj
 0002:00001c14       __real@41000000            30059c14     cg_draw.obj
 0002:00001c18       ??_C@_07FJAEFGNG@?$CF3i?5?$CF3i?$AA@ 30059c18     cg_draw.obj
 0002:00001c20       ??_C@_07CIFAGBMG@unknown?$AA@ 30059c20     cg_draw.obj
 0002:00001c28       ??_C@_03NKIHJOPP@?$CF2i?$AA@ 30059c28     cg_draw.obj
 0002:00001c2c       __real@41c00000            30059c2c     cg_draw.obj
 0002:00001c30       __real@4048000000000000    30059c30     cg_draw.obj
 0002:00001c38       __real@447a0000            30059c38     cg_draw.obj
 0002:00001c3c       __real@42400000            30059c3c     cg_draw.obj
 0002:00001c40       ??_C@_02DPKJAMEF@?$CFd?$AA@ 30059c40     cg_draw.obj
 0002:00001c44       ??_C@_03KLKIPBNP@snc?$AA@  30059c44     cg_draw.obj
 0002:00001c48       __real@44610000            30059c48     cg_draw.obj
 0002:00001c4c       __real@43960000            30059c4c     cg_draw.obj
 0002:00001c50       ??_C@_0P@NNJCDNEK@gfx?12d?1net?4tga?$AA@ 30059c50     cg_draw.obj
 0002:00001c60       ??_C@_0BH@HFDDJIMF@Connection?5Interrupted?$AA@ 30059c60     cg_draw.obj
 0002:00001c78       __real@43a00000            30059c78     cg_draw.obj
 0002:00001c7c       __real@3f000000            30059c7c     cg_draw.obj
 0002:00001c80       __real@48000000            30059c80     cg_draw.obj
 0002:00001c84       ??_C@_0CI@GGHFPFB@press?5ESC?5and?5use?5the?5JOIN?5menu?5@ 30059c84     cg_draw.obj
 0002:00001cac       ??_C@_0BA@PJMJBMDH@waiting?5to?5play?$AA@ 30059cac     cg_draw.obj
 0002:00001cbc       ??_C@_09GNDCBOBP@SPECTATOR?$AA@ 30059cbc     cg_draw.obj
 0002:00001cc8       ??_C@_0BJ@JAENOHOK@VOTE?$CI?$CFi?$CJ?3?$CFs?5yes?3?$CFi?5no?3?$CFi?$AA@ 30059cc8     cg_draw.obj
 0002:00001ce4       ??_C@_0BN@CPIJHJOL@TEAMVOTE?$CI?$CFi?$CJ?3?$CFs?5yes?3?$CFi?5no?3?$CFi?$AA@ 30059ce4     cg_draw.obj
 0002:00001d04       ??_C@_09BEIPBMDN@following?$AA@ 30059d04     cg_draw.obj
 0002:00001d10       ??_C@_0BB@IAFHNAPI@LOW?5AMMO?5WARNING?$AA@ 30059d10     cg_draw.obj
 0002:00001d24       ??_C@_0M@COLOONJC@OUT?5OF?5AMMO?$AA@ 30059d24     cg_draw.obj
 0002:00001d30       ??_C@_0O@DIOKDBHN@Starts?5in?3?5?$CFi?$AA@ 30059d30     cg_draw.obj
 0002:00001d40       __real@3f8ccccd            30059d40     cg_draw.obj
 0002:00001d44       ??_C@_0BB@OOIHNFAG@Capture?5the?5Flag?$AA@ 30059d44     cg_draw.obj
 0002:00001d58       ??_C@_0BA@KHHNIIJE@Team?5Deathmatch?$AA@ 30059d58     cg_draw.obj
 0002:00001d68       ??_C@_0N@PCEMCJC@Free?5For?5All?$AA@ 30059d68     cg_draw.obj
 0002:00001d78       __real@3fc00000            30059d78     cg_draw.obj
 0002:00001d7c       ??_C@_08MFFNPGJB@?$CFs?5vs?5?$CFs?$AA@ 30059d7c     cg_draw.obj
 0002:00001d88       ??_C@_0BE@JNOOFOAO@Waiting?5for?5players?$AA@ 30059d88     cg_draw.obj
 0002:00001da0       __real@3fb0000000000000    30059da0     cg_drawtools.obj
 0002:00001da8       __real@4050000000000000    30059da8     cg_drawtools.obj
 0002:00001db0       __real@4069000000000000    30059db0     cg_drawtools.obj
 0002:00001db8       __real@403e000000000000    30059db8     cg_drawtools.obj
 0002:00001dc0       __real@4040800000000000    30059dc0     cg_drawtools.obj
 0002:00001dc8       __real@3fd5c28f5c28f5c2    30059dc8     cg_drawtools.obj
 0002:00001dd0       __real@3fe51eb851eb851f    30059dd0     cg_drawtools.obj
 0002:00001dd8       __real@43800000            30059dd8     cg_drawtools.obj
 0002:00001ddc       __real@3f400000            30059ddc     cg_drawtools.obj
 0002:00001de0       __real@3fe999999999999a    30059de0     cg_drawtools.obj
 0002:00001de8       __real@41d80000            30059de8     cg_drawtools.obj
 0002:00001df0       __real@4018000000000000    30059df0     cg_effects.obj
 0002:00001df8       __real@437a0000            30059df8     cg_effects.obj
 0002:00001dfc       __real@437f0000            30059dfc     cg_effects.obj
 0002:00001e00       __real@43b40000            30059e00     cg_effects.obj
 0002:00001e04       ??_C@_0BM@FJKGAFKH@CG_MakeExplosion?3?5msec?5?$DN?5?$CFi?$AA@ 30059e04     cg_effects.obj
 0002:00001e20       __real@453b8000            30059e20     cg_effects.obj
 0002:00001e28       __real@406f400000000000    30059e28     cg_effects.obj
 0002:00001e30       __real@45bb8000            30059e30     cg_effects.obj
 0002:00001e38       __real@4004000000000000    30059e38     cg_effects.obj
 0002:00001e40       __real@4062c00000000000    30059e40     cg_effects.obj
 0002:00001e48       __real@4059000000000000    30059e48     cg_effects.obj
 0002:00001e50       __real@44800000            30059e50     cg_ents.obj
 0002:00001e54       ??_C@_0DB@OLDIELNC@CG_InterpoateEntityPosition?3?5cg?4@ 30059e54     cg_ents.obj
 0002:00001e88       ??_C@_0BF@NGFHFBLN@Bad?5entity?5type?3?5?$CFi?6?$AA@ 30059e88     cg_ents.obj
 0002:00001ea0       __real@c4800000            30059ea0     cg_ents.obj
 0002:00001ea4       __real@41400000            30059ea4     cg_ents.obj
 0002:00001ea8       __real@4010000000000000    30059ea8     cg_ents.obj
 0002:00001eb0       __real@3f747ae147ae147b    30059eb0     cg_ents.obj
 0002:00001eb8       __real@3ee4f8b588e368f1    30059eb8     cg_ents.obj
 0002:00001ec0       ??_C@_0BM@DFPOGHOF@Bad?5item?5index?5?$CFi?5on?5entity?$AA@ 30059ec0     cg_ents.obj
 0002:00001ee0       __real@4076800000000000    30059ee0     cg_ents.obj
 0002:00001ee8       __real@4070000000000000    30059ee8     cg_ents.obj
 0002:00001ef0       ??_C@_04HDOCAJNK@?$CFs?$CFs?$AA@ 30059ef0     cg_event.obj
 0002:00001ef8       ??_C@_04IIAODBDM@?$CFith?$AA@ 30059ef8     cg_event.obj
 0002:00001f00       ??_C@_04CADGACIC@?$CFird?$AA@ 30059f00     cg_event.obj
 0002:00001f08       ??_C@_04DFAKFIJG@?$CFind?$AA@ 30059f08     cg_event.obj
 0002:00001f10       ??_C@_04GLDGHKOE@?$CFist?$AA@ 30059f10     cg_event.obj
 0002:00001f18       ??_C@_04LJNOOPLI@13th?$AA@ 30059f18     cg_event.obj
 0002:00001f20       ??_C@_04BGCIINN@12th?$AA@  30059f20     cg_event.obj
 0002:00001f28       ??_C@_04BDNHCHDD@11th?$AA@ 30059f28     cg_event.obj
 0002:00001f30       ??_C@_07GHHLNL@?$FO33rd?$FO7?$AA@ 30059f30     cg_event.obj
 0002:00001f38       ??_C@_07PJLEMDNE@?$FO12nd?$FO7?$AA@ 30059f38     cg_event.obj
 0002:00001f40       ??_C@_07OFHBJKHB@?$FO41st?$FO7?$AA@ 30059f40     cg_event.obj
 0002:00001f48       ??_C@_09LNCLIHP@Tied?5for?5?$AA@ 30059f48     cg_event.obj
 0002:00001f54       ??_C@_0P@MHKKKFHB@?$CKpain100_1?4wav?$AA@ 30059f54     cg_event.obj
 0002:00001f64       ??_C@_0O@PJAMCPJF@?$CKpain75_1?4wav?$AA@ 30059f64     cg_event.obj
 0002:00001f74       ??_C@_0O@JPBKAJHH@?$CKpain50_1?4wav?$AA@ 30059f74     cg_event.obj
 0002:00001f84       ??_C@_0O@LDJLGKNK@?$CKpain25_1?4wav?$AA@ 30059f84     cg_event.obj
 0002:00001f94       ??_C@_0BC@OKELKAPM@Unknown?5event?3?5?$CFi?$AA@ 30059f94     cg_event.obj
 0002:00001fa8       ??_C@_08GCOIMFOL@UNKNOWN?6?$AA@ 30059fa8     cg_event.obj
 0002:00001fb4       ??_C@_0P@DKFKJLCN@EV_DEBUG_LINE?6?$AA@ 30059fb4     cg_event.obj
 0002:00001fc4       ??_C@_0BF@JEGDHJFI@EV_STOPLOOPINGSOUND?6?$AA@ 30059fc4     cg_event.obj
 0002:00001fdc       ??_C@_0P@OAKOFJEN@EV_GIB_PLAYER?6?$AA@ 30059fdc     cg_event.obj
 0002:00001fec       ??_C@_0BC@IEBIBNLE@EV_POWERUP_REGEN?6?$AA@ 30059fec     cg_event.obj
 0002:00002000       ??_C@_0BH@DMMEDNOI@EV_POWERUP_BATTLESUIT?6?$AA@ 3005a000     cg_event.obj
 0002:00002018       ??_C@_0BB@BAEBNJML@EV_POWERUP_QUAD?6?$AA@ 3005a018     cg_event.obj
 0002:0000202c       ??_C@_0N@NHOCPMCE@EV_OBITUARY?6?$AA@ 3005a02c     cg_event.obj
 0002:0000203c       ??_C@_0N@OJAOIBLE@?$CKdeath?$CFi?4wav?$AA@ 3005a03c     cg_event.obj
 0002:0000204c       ??_C@_0L@GGFIAEKN@EV_DEATHx?6?$AA@ 3005a04c     cg_event.obj
 0002:00002058       ??_C@_08MEMNOIPP@EV_PAIN?6?$AA@ 3005a058     cg_event.obj
 0002:00002064       ??_C@_0BG@DDNACAKH@EV_GLOBAL_TEAM_SOUND?6?$AA@ 3005a064     cg_event.obj
 0002:0000207c       ??_C@_0BB@DOBOGIIM@EV_GLOBAL_SOUND?6?$AA@ 3005a07c     cg_event.obj
 0002:00002090       ??_C@_0BC@BJDFIFFI@EV_GENERAL_SOUND?6?$AA@ 3005a090     cg_event.obj
 0002:000020a4       ??_C@_0M@PGOOOLMB@EV_SHOTGUN?6?$AA@ 3005a0a4     cg_event.obj
 0002:000020b0       ??_C@_0BF@PBJFDGOC@EV_BULLET_HIT_FLESH?6?$AA@ 3005a0b0     cg_event.obj
 0002:000020c8       ??_C@_0BE@DJCGNKAA@EV_BULLET_HIT_WALL?6?$AA@ 3005a0c8     cg_event.obj
 0002:000020dc       ??_C@_0O@MHELMGMI@EV_RAILTRAIL?6?$AA@ 3005a0dc     cg_event.obj
 0002:000020ec       ??_C@_0BH@JAOAMPDI@EV_MISSILE_MISS_METAL?6?$AA@ 3005a0ec     cg_event.obj
 0002:00002104       ??_C@_0BB@PNKCFMCO@EV_MISSILE_MISS?6?$AA@ 3005a104     cg_event.obj
 0002:00002118       ??_C@_0BA@IGKGMCOM@EV_MISSILE_HIT?6?$AA@ 3005a118     cg_event.obj
 0002:00002128       ??_C@_0O@HHOHODHG@EV_SCOREPLUM?6?$AA@ 3005a128     cg_event.obj
 0002:00002138       ??_C@_0BD@EIBAGLKH@EV_GRENADE_BOUNCE?6?$AA@ 3005a138     cg_event.obj
 0002:0000214c       ??_C@_0BB@JFDGENII@EV_ITEM_RESPAWN?6?$AA@ 3005a14c     cg_event.obj
 0002:00002160       ??_C@_0N@PBHGFCFD@EV_ITEM_POP?6?$AA@ 3005a160     cg_event.obj
 0002:00002170       ??_C@_0BI@GJLLMPKI@EV_PLAYER_TELEPORT_OUT?6?$AA@ 3005a170     cg_event.obj
 0002:00002188       ??_C@_0BH@EMPINMBK@EV_PLAYER_TELEPORT_IN?6?$AA@ 3005a188     cg_event.obj
 0002:000021a0       ??_C@_0P@DPDLKGLM@EV_USE_ITEM14?6?$AA@ 3005a1a0     cg_event.obj
 0002:000021b0       ??_C@_0P@DKHELADJ@EV_USE_ITEM13?6?$AA@ 3005a1b0     cg_event.obj
 0002:000021c0       ??_C@_0P@DLLGNKAO@EV_USE_ITEM12?6?$AA@ 3005a1c0     cg_event.obj
 0002:000021d0       ??_C@_0P@DJPAGEFH@EV_USE_ITEM11?6?$AA@ 3005a1d0     cg_event.obj
 0002:000021e0       ??_C@_0P@DIDCAOGA@EV_USE_ITEM10?6?$AA@ 3005a1e0     cg_event.obj
 0002:000021f0       ??_C@_0O@CBKDMCHN@EV_USE_ITEM9?6?$AA@ 3005a1f0     cg_event.obj
 0002:00002200       ??_C@_0O@CAGBKIEK@EV_USE_ITEM8?6?$AA@ 3005a200     cg_event.obj
 0002:00002210       ??_C@_0O@CLDNOPHH@EV_USE_ITEM7?6?$AA@ 3005a210     cg_event.obj
 0002:00002220       ??_C@_0O@CKPPIFEA@EV_USE_ITEM6?6?$AA@ 3005a220     cg_event.obj
 0002:00002230       ??_C@_0O@CILJDLBJ@EV_USE_ITEM5?6?$AA@ 3005a230     cg_event.obj
 0002:00002240       ??_C@_0O@CJHLFBCO@EV_USE_ITEM4?6?$AA@ 3005a240     cg_event.obj
 0002:00002250       ??_C@_0O@CMDEEHKL@EV_USE_ITEM3?6?$AA@ 3005a250     cg_event.obj
 0002:00002260       ??_C@_0O@CNPGCNJM@EV_USE_ITEM2?6?$AA@ 3005a260     cg_event.obj
 0002:00002270       ??_C@_0O@CPLAJDMF@EV_USE_ITEM1?6?$AA@ 3005a270     cg_event.obj
 0002:00002280       ??_C@_0O@COHCPJPC@EV_USE_ITEM0?6?$AA@ 3005a280     cg_event.obj
 0002:00002290       ??_C@_0BA@CJMMIDHE@EV_FIRE_WEAPON?6?$AA@ 3005a290     cg_event.obj
 0002:000022a0       ??_C@_0BC@KBHMOJOO@EV_CHANGE_WEAPON?6?$AA@ 3005a2a0     cg_event.obj
 0002:000022b4       ??_C@_0L@CIOCLBPP@EV_NOAMMO?6?$AA@ 3005a2b4     cg_event.obj
 0002:000022c0       ??_C@_0BH@BPJPNNOH@EV_GLOBAL_ITEM_PICKUP?6?$AA@ 3005a2c0     cg_event.obj
 0002:000022d8       ??_C@_0BA@LGJAHGJL@EV_ITEM_PICKUP?6?$AA@ 3005a2d8     cg_event.obj
 0002:000022e8       ??_C@_09OICPJII@?$CKgasp?4wav?$AA@ 3005a2e8     cg_event.obj
 0002:000022f4       ??_C@_0BA@OODKPEF@EV_WATER_CLEAR?6?$AA@ 3005a2f4     cg_event.obj
 0002:00002304       ??_C@_0BA@PFCHBJFN@EV_WATER_UNDER?6?$AA@ 3005a304     cg_event.obj
 0002:00002314       ??_C@_0BA@POIDPCHH@EV_WATER_LEAVE?6?$AA@ 3005a314     cg_event.obj
 0002:00002324       ??_C@_0BA@PBFGAGAE@EV_WATER_TOUCH?6?$AA@ 3005a324     cg_event.obj
 0002:00002334       ??_C@_0L@FDBCLIPJ@?$CKtaunt?4wav?$AA@ 3005a334     cg_event.obj
 0002:00002340       ??_C@_09OAFEJHMF@EV_TAUNT?6?$AA@ 3005a340     cg_event.obj
 0002:0000234c       ??_C@_08GKDKOBGN@EV_JUMP?6?$AA@ 3005a34c     cg_event.obj
 0002:00002358       ??_C@_0L@FMHDEMAN@?$CKjump1?4wav?$AA@ 3005a358     cg_event.obj
 0002:00002364       ??_C@_0N@CDCGGHDH@EV_JUMP_PAD?6?$AA@ 3005a364     cg_event.obj
 0002:00002374       __real@42000000            3005a374     cg_event.obj
 0002:00002378       ??_C@_08LGDHLDGB@EV_STEP?6?$AA@ 3005a378     cg_event.obj
 0002:00002384       ??_C@_0L@NLLHEJNK@?$CKfall1?4wav?$AA@ 3005a384     cg_event.obj
 0002:00002390       ??_C@_0N@FDOJNPAA@EV_FALL_FAR?6?$AA@ 3005a390     cg_event.obj
 0002:000023a0       ??_C@_0BA@MCPBHBIM@EV_FALL_MEDIUM?6?$AA@ 3005a3a0     cg_event.obj
 0002:000023b0       ??_C@_0P@DBGGEJF@EV_FALL_SHORT?6?$AA@ 3005a3b0     cg_event.obj
 0002:000023c0       ??_C@_08KPLPEGCK@EV_SWIM?6?$AA@ 3005a3c0     cg_event.obj
 0002:000023cc       ??_C@_0N@DBFBMKGC@EV_FOOTWADE?6?$AA@ 3005a3cc     cg_event.obj
 0002:000023dc       ??_C@_0P@ECCJNKCN@EV_FOOTSPLASH?6?$AA@ 3005a3dc     cg_event.obj
 0002:000023ec       ??_C@_0BD@GPGIDOAE@EV_FOOTSTEP_METAL?6?$AA@ 3005a3ec     cg_event.obj
 0002:00002400       ??_C@_0N@KAJBJGHI@EV_FOOTSTEP?6?$AA@ 3005a400     cg_event.obj
 0002:00002410       ??_C@_0L@GMIFJJAD@ZEROEVENT?6?$AA@ 3005a410     cg_event.obj
 0002:0000241c       ??_C@_0BE@HGIJDIOP@ent?3?$CF3i?5?5event?3?$CF3i?5?$AA@ 3005a41c     cg_event.obj
 0002:00002430       ??_C@_09PIPBOPDG@?$CFs?5died?4?6?$AA@ 3005a430     cg_event.obj
 0002:0000243c       ??_C@_0M@NLIGKFEM@?$CFs?5?$CFs?5?$CFs?$CFs?6?$AA@ 3005a43c     cg_event.obj
 0002:00002448       ??_C@_0O@JEEJCGAD@was?5killed?5by?$AA@ 3005a448     cg_event.obj
 0002:00002458       ??_C@_0BC@CJMFGHKA@?8s?5personal?5space?$AA@ 3005a458     cg_event.obj
 0002:0000246c       ??_C@_0BA@CBNEPGEH@tried?5to?5invade?$AA@ 3005a46c     cg_event.obj
 0002:0000247c       ??_C@_06NOMMMPPO@?8s?5BFG?$AA@ 3005a47c     cg_event.obj
 0002:00002484       ??_C@_0P@CIDIINED@was?5blasted?5by?$AA@ 3005a484     cg_event.obj
 0002:00002494       ??_C@_0BE@IJJLPGGN@was?5electrocuted?5by?$AA@ 3005a494     cg_event.obj
 0002:000024a8       ??_C@_0O@LMMKCAFN@was?5railed?5by?$AA@ 3005a4a8     cg_event.obj
 0002:000024b8       ??_C@_0N@HJJMNEOJ@?8s?5plasmagun?$AA@ 3005a4b8     cg_event.obj
 0002:000024c8       ??_C@_0O@CLFCHHPJ@was?5melted?5by?$AA@ 3005a4c8     cg_event.obj
 0002:000024d8       ??_C@_0O@JENMCGOI@almost?5dodged?$AA@ 3005a4d8     cg_event.obj
 0002:000024e8       ??_C@_09DEADKGEN@?8s?5rocket?$AA@ 3005a4e8     cg_event.obj
 0002:000024f4       ??_C@_0M@BHBOCILJ@?8s?5shrapnel?$AA@ 3005a4f4     cg_event.obj
 0002:00002500       ??_C@_0BA@LIKKPCIN@was?5shredded?5by?$AA@ 3005a500     cg_event.obj
 0002:00002510       ??_C@_0L@KPHMDLGC@?8s?5grenade?$AA@ 3005a510     cg_event.obj
 0002:0000251c       ??_C@_03BGFDOPOL@ate?$AA@  3005a51c     cg_event.obj
 0002:00002520       ??_C@_0BD@MKJCHKPL@was?5gunned?5down?5by?$AA@ 3005a520     cg_event.obj
 0002:00002534       ??_C@_0BF@PGKPLAEB@was?5machinegunned?5by?$AA@ 3005a534     cg_event.obj
 0002:0000254c       ??_C@_0BA@DIGOJPDF@was?5pummeled?5by?$AA@ 3005a54c     cg_event.obj
 0002:0000255c       ??_C@_0O@IBMLDOEJ@was?5caught?5by?$AA@ 3005a55c     cg_event.obj
 0002:0000256c       ??_C@_06LNKFDEGN@noname?$AA@ 3005a56c     cg_event.obj
 0002:00002574       ??_C@_0P@IOLDCJGB@You?5fragged?5?$CFs?$AA@ 3005a574     cg_event.obj
 0002:00002584       ??_C@_0CA@EJEIBOAF@You?5fragged?5?$CFs?6?$CFs?5place?5with?5?$CFi?$AA@ 3005a584     cg_event.obj
 0002:000025a4       ??_C@_07EJPAKPEC@?$CFs?5?$CFs?4?6?$AA@ 3005a5a4     cg_event.obj
 0002:000025ac       ??_C@_0P@DNKIPMGE@killed?5himself?$AA@ 3005a5ac     cg_event.obj
 0002:000025bc       ??_C@_0O@JCBLJPFM@killed?5itself?$AA@ 3005a5bc     cg_event.obj
 0002:000025cc       ??_C@_0P@IIICGFO@killed?5herself?$AA@ 3005a5cc     cg_event.obj
 0002:000025dc       ??_C@_0BP@DBEBPALD@should?5have?5used?5a?5smaller?5gun?$AA@ 3005a5dc     cg_event.obj
 0002:000025fc       ??_C@_0P@DPLDCCLJ@melted?5himself?$AA@ 3005a5fc     cg_event.obj
 0002:0000260c       ??_C@_0O@OEFGEIJP@melted?5itself?$AA@ 3005a60c     cg_event.obj
 0002:0000261c       ??_C@_0P@KJDPIID@melted?5herself?$AA@ 3005a61c     cg_event.obj
 0002:0000262c       ??_C@_0BA@FIENEKJD@blew?5himself?5up?$AA@ 3005a62c     cg_event.obj
 0002:0000263c       ??_C@_0P@GOLBOBGC@blew?5itself?5up?$AA@ 3005a63c     cg_event.obj
 0002:0000264c       ??_C@_0BA@DBAICHLN@blew?5herself?5up?$AA@ 3005a64c     cg_event.obj
 0002:0000265c       ??_C@_0BL@BJDCDLDL@tripped?5on?5his?5own?5grenade?$AA@ 3005a65c     cg_event.obj
 0002:00002678       ??_C@_0BL@PDGEHOJ@tripped?5on?5its?5own?5grenade?$AA@ 3005a678     cg_event.obj
 0002:00002694       ??_C@_0BL@MBMIHDKJ@tripped?5on?5her?5own?5grenade?$AA@ 3005a694     cg_event.obj
 0002:000026b0       ??_C@_0BH@GICEGFFN@was?5in?5the?5wrong?5place?$AA@ 3005a6b0     cg_event.obj
 0002:000026c8       ??_C@_0O@LCLMFGAB@saw?5the?5light?$AA@ 3005a6c8     cg_event.obj
 0002:000026d8       ??_C@_0BP@NAHBLPBA@does?5a?5back?5flip?5into?5the?5lava?$AA@ 3005a6d8     cg_event.obj
 0002:000026f8       ??_C@_06CHNJJJKC@melted?$AA@ 3005a6f8     cg_event.obj
 0002:00002700       ??_C@_0BB@IPCHCEIC@sank?5like?5a?5rock?$AA@ 3005a700     cg_event.obj
 0002:00002714       ??_C@_0N@JLHEPJHP@was?5squished?$AA@ 3005a714     cg_event.obj
 0002:00002724       ??_C@_08PAHGPPBJ@cratered?$AA@ 3005a724     cg_event.obj
 0002:00002730       ??_C@_08MOEOKJOB@suicides?$AA@ 3005a730     cg_event.obj
 0002:0000273c       ??_C@_02PGJLIFGD@?$FO7?$AA@ 3005a73c     cg_event.obj
 0002:00002740       ??_C@_0CB@LLKCBBGA@CG_Obituary?3?5target?5out?5of?5range@ 3005a740     cg_event.obj
 0002:00002764       ??_C@_06FFLMGAMD@Use?5?$CFs?$AA@ 3005a764     cg_event.obj
 0002:0000276c       ??_C@_0P@MMJPCMLF@No?5item?5to?5use?$AA@ 3005a76c     cg_event.obj
 0002:0000277c       ??_C@_0BN@PBJAICBL@sound?1player?1announce?1?$CFs?4wav?$AA@ 3005a77c     cg_info.obj
 0002:0000279c       ??_C@_05PDPNFFJO@sarge?$AA@ 3005a79c     cg_info.obj
 0002:000027a4       ??_C@_0CJ@KFDGMKIH@models?1players?1characters?1?$CFs?1ico@ 3005a7a4     cg_info.obj
 0002:000027d0       ??_C@_0BO@BHADLJEM@models?1players?1?$CFs?1icon_?$CFs?4tga?$AA@ 3005a7d0     cg_info.obj
 0002:000027f0       ??_C@_07DLHCIBDH@default?$AA@ 3005a7f0     cg_info.obj
 0002:000027f8       ??_C@_05NCCFOPHA@model?$AA@ 3005a7f8     cg_info.obj
 0002:00002800       ??_C@_0BA@NDPDGDCC@capturelimit?5?$CFi?$AA@ 3005a800     cg_info.obj
 0002:00002810       ??_C@_0N@FCAHJCDA@capturelimit?$AA@ 3005a810     cg_info.obj
 0002:00002820       ??_C@_0N@KCDNPCCH@fraglimit?5?$CFi?$AA@ 3005a820     cg_info.obj
 0002:00002830       ??_C@_09GCIEGDDN@fraglimit?$AA@ 3005a830     cg_info.obj
 0002:0000283c       ??_C@_0N@FADOKLO@timelimit?5?$CFi?$AA@ 3005a83c     cg_info.obj
 0002:0000284c       ??_C@_09KPHKOKCC@timelimit?$AA@ 3005a84c     cg_info.obj
 0002:00002858       ??_C@_0BB@DMLMKGKN@Unknown?5Gametype?$AA@ 3005a858     cg_info.obj
 0002:0000286c       ??_C@_0BB@GMHGFHKF@Capture?5The?5Flag?$AA@ 3005a86c     cg_info.obj
 0002:00002880       ??_C@_0L@FENDKKGN@Tournament?$AA@ 3005a880     cg_info.obj
 0002:0000288c       ??_C@_0O@NNAOEDOE@Single?5Player?$AA@ 3005a88c     cg_info.obj
 0002:0000289c       ??_C@_0BD@HCPEKLFD@CHEATS?5ARE?5ENABLED?$AA@ 3005a89c     cg_info.obj
 0002:000028b0       ??_C@_09NFOPKLIK@sv_cheats?$AA@ 3005a8b0     cg_info.obj
 0002:000028bc       ??_C@_0M@POENFNKG@Pure?5Server?$AA@ 3005a8bc     cg_info.obj
 0002:000028c8       ??_C@_07CAKOHKGL@sv_pure?$AA@ 3005a8c8     cg_info.obj
 0002:000028d0       ??_C@_0M@NHCIKFPA@sv_hostname?$AA@ 3005a8d0     cg_info.obj
 0002:000028dc       ??_C@_0L@MPAGGMDN@sv_running?$AA@ 3005a8dc     cg_info.obj
 0002:000028e8       ??_C@_0BF@NHPKANBN@Awaiting?5snapshot?4?4?4?$AA@ 3005a8e8     cg_info.obj
 0002:00002900       ??_C@_0O@BKHPEAJO@Loading?4?4?4?5?$CFs?$AA@ 3005a900     cg_info.obj
 0002:00002910       ??_C@_0BA@LBOAECOK@levelShotDetail?$AA@ 3005a910     cg_info.obj
 0002:00002920       ??_C@_0BE@JCMNICLJ@menu?1art?1unknownmap?$AA@ 3005a920     cg_info.obj
 0002:00002934       ??_C@_0BC@PIIMIPAI@levelshots?1?$CFs?4tga?$AA@ 3005a934     cg_info.obj
 0002:00002948       ??_C@_07KMNEBLH@mapname?$AA@ 3005a948     cg_info.obj
 0002:00002950       ??_C@_0BP@HOJADAKE@CG_FreeLocalEntity?3?5not?5active?$AA@ 3005a950     cg_localents.obj
 0002:00002970       __real@c0000000            3005a970     cg_localents.obj
 0002:00002978       __real@4030000000000000    3005a978     cg_localents.obj
 0002:00002980       __real@c024000000000000    3005a980     cg_localents.obj
 0002:00002988       __real@42dc0000            3005a988     cg_localents.obj
 0002:0000298c       __real@447f0000            3005a98c     cg_localents.obj
 0002:00002990       ??_C@_0P@JBCHHKP@Bad?5leType?3?5?$CFi?$AA@ 3005a990     cg_localents.obj
 0002:000029a0       __real@4020000000000000    3005a9a0     cg_localents.obj
 0002:000029a8       __real@4045000000000000    3005a9a8     cg_localents.obj
 0002:000029b0       __real@3fd51eb851eb851f    3005a9b0     cg_localents.obj
 0002:000029b8       ??_C@_0BJ@PPCBGHDL@gfx?12d?1numbers?1minus_32b?$AA@ 3005a9b8     cg_main.obj
 0002:000029d4       ??_C@_0BI@HJFCMICO@gfx?12d?1numbers?1nine_32b?$AA@ 3005a9d4     cg_main.obj
 0002:000029ec       ??_C@_0BJ@OILFPBFC@gfx?12d?1numbers?1eight_32b?$AA@ 3005a9ec     cg_main.obj
 0002:00002a08       ??_C@_0BJ@FHLKICGB@gfx?12d?1numbers?1seven_32b?$AA@ 3005aa08     cg_main.obj
 0002:00002a24       ??_C@_0BH@DOOFJAPO@gfx?12d?1numbers?1six_32b?$AA@ 3005aa24     cg_main.obj
 0002:00002a3c       ??_C@_0BI@JGLLLIJP@gfx?12d?1numbers?1five_32b?$AA@ 3005aa3c     cg_main.obj
 0002:00002a54       ??_C@_0BI@HPOPJJKG@gfx?12d?1numbers?1four_32b?$AA@ 3005aa54     cg_main.obj
 0002:00002a6c       ??_C@_0BJ@KKKEIAHG@gfx?12d?1numbers?1three_32b?$AA@ 3005aa6c     cg_main.obj
 0002:00002a88       ??_C@_0BH@BNBCEMFH@gfx?12d?1numbers?1two_32b?$AA@ 3005aa88     cg_main.obj
 0002:00002aa0       ??_C@_0BH@GPBOJLFB@gfx?12d?1numbers?1one_32b?$AA@ 3005aaa0     cg_main.obj
 0002:00002ab8       ??_C@_0BI@NODEBLMA@gfx?12d?1numbers?1zero_32b?$AA@ 3005aab8     cg_main.obj
 0002:00002ad0       ??_C@_03MDAFIFFL@0?40?$AA@ 3005aad0     cg_main.obj
 0002:00002ad4       ??_C@_0BB@DCJMDHFD@cg_trueLightning?$AA@ 3005aad4     cg_main.obj
 0002:00002ae8       ??_C@_0N@IHPGFFAI@cg_oldPlasma?$AA@ 3005aae8     cg_main.obj
 0002:00002af8       ??_C@_0N@EADGKNDD@cg_oldRocket?$AA@ 3005aaf8     cg_main.obj
 0002:00002b08       ??_C@_0L@FKCBCOIH@cg_oldRail?$AA@ 3005ab08     cg_main.obj
 0002:00002b14       ??_C@_0L@LPOJJAMJ@ui_bigFont?$AA@ 3005ab14     cg_main.obj
 0002:00002b20       ??_C@_04FNMPJLCB@0?425?$AA@ 3005ab20     cg_main.obj
 0002:00002b28       ??_C@_0N@CLDCAIAI@ui_smallFont?$AA@ 3005ab28     cg_main.obj
 0002:00002b38       ??_C@_0BF@IHAIMPIG@cg_noProjectileTrail?$AA@ 3005ab38     cg_main.obj
 0002:00002b50       ??_C@_0L@BNLHLPGL@cg_noTaunt?$AA@ 3005ab50     cg_main.obj
 0002:00002b5c       ??_C@_01KJLJFBPL@8?$AA@    3005ab5c     cg_main.obj
 0002:00002b60       ??_C@_0L@JLBEBBAD@pmove_msec?$AA@ 3005ab60     cg_main.obj
 0002:00002b6c       ??_C@_0M@HOGKGHBI@pmove_fixed?$AA@ 3005ab6c     cg_main.obj
 0002:00002b78       ??_C@_0P@EIAPFKBF@com_cameraMode?$AA@ 3005ab78     cg_main.obj
 0002:00002b88       ??_C@_0BB@EPNKMEEL@cg_smoothClients?$AA@ 3005ab88     cg_main.obj
 0002:00002b9c       ??_C@_0O@ECBGLFLJ@cg_scorePlums?$AA@ 3005ab9c     cg_main.obj
 0002:00002bac       ??_C@_09IIOBMIO@timescale?$AA@ 3005abac     cg_main.obj
 0002:00002bb8       ??_C@_0BG@HODAAIBP@cg_timescaleFadeSpeed?$AA@ 3005abb8     cg_main.obj
 0002:00002bd0       ??_C@_0BE@INLNOCBP@cg_timescaleFadeEnd?$AA@ 3005abd0     cg_main.obj
 0002:00002be4       ??_C@_02PNFIDHGF@50?$AA@   3005abe4     cg_main.obj
 0002:00002be8       ??_C@_0BE@EKDKKKAP@cg_cameraOrbitDelay?$AA@ 3005abe8     cg_main.obj
 0002:00002bfc       ??_C@_0BF@LICFCALK@g_synchronousClients?$AA@ 3005abfc     cg_main.obj
 0002:00002c14       ??_C@_09DKNLLEN@com_blood?$AA@ 3005ac14     cg_main.obj
 0002:00002c20       ??_C@_09DIABHAFB@cl_paused?$AA@ 3005ac20     cg_main.obj
 0002:00002c2c       ??_C@_0BA@MOHNLIKA@com_buildScript?$AA@ 3005ac2c     cg_main.obj
 0002:00002c3c       ??_C@_0P@HEADOJJM@cg_noVoiceText?$AA@ 3005ac3c     cg_main.obj
 0002:00002c4c       ??_C@_0BA@DGINBIDE@cg_noVoiceChats?$AA@ 3005ac4c     cg_main.obj
 0002:00002c5c       ??_C@_0BB@GFOCPFOA@cg_teamChatsOnly?$AA@ 3005ac5c     cg_main.obj
 0002:00002c70       ??_C@_0O@KGJIDOMN@cg_drawFriend?$AA@ 3005ac70     cg_main.obj
 0002:00002c80       ??_C@_08CGDPCFHD@cg_stats?$AA@ 3005ac80     cg_main.obj
 0002:00002c8c       ??_C@_0M@IKKMOBIP@teamoverlay?$AA@ 3005ac8c     cg_main.obj
 0002:00002c98       ??_C@_0BD@BNGDPIGC@cg_drawTeamOverlay?$AA@ 3005ac98     cg_main.obj
 0002:00002cac       ??_C@_0BA@PFOJHBKN@cg_deferPlayers?$AA@ 3005acac     cg_main.obj
 0002:00002cbc       ??_C@_0BA@PKAEEJJB@cg_predictItems?$AA@ 3005acbc     cg_main.obj
 0002:00002ccc       ??_C@_0O@LJBBKNGE@cg_forceModel?$AA@ 3005accc     cg_main.obj
 0002:00002cdc       ??_C@_0BC@JPKKPJNB@cg_teamChatHeight?$AA@ 3005acdc     cg_main.obj
 0002:00002cf0       ??_C@_04NEFKOBHG@3000?$AA@ 3005acf0     cg_main.obj
 0002:00002cf8       ??_C@_0BA@FOMJOJCG@cg_teamChatTime?$AA@ 3005acf8     cg_main.obj
 0002:00002d08       ??_C@_02PMJKFNFC@40?$AA@   3005ad08     cg_main.obj
 0002:00002d0c       ??_C@_0BA@CAFKIKHE@cg_tracerlength?$AA@ 3005ad0c     cg_main.obj
 0002:00002d1c       ??_C@_0P@ENCNJBFG@cg_tracerwidth?$AA@ 3005ad1c     cg_main.obj
 0002:00002d2c       ??_C@_0BA@DJBDPKKA@cg_tracerchance?$AA@ 3005ad2c     cg_main.obj
 0002:00002d3c       ??_C@_0N@GHAOKDNB@cg_footsteps?$AA@ 3005ad3c     cg_main.obj
 0002:00002d4c       ??_C@_0M@DOMGGLDE@cg_showmiss?$AA@ 3005ad4c     cg_main.obj
 0002:00002d58       ??_C@_0BB@HOMHKKFN@cg_noplayeranims?$AA@ 3005ad58     cg_main.obj
 0002:00002d6c       ??_C@_0N@BMAKLHMK@cg_nopredict?$AA@ 3005ad6c     cg_main.obj
 0002:00002d7c       ??_C@_0O@MAANEMBM@cg_errordecay?$AA@ 3005ad7c     cg_main.obj
 0002:00002d8c       ??_C@_0P@NKGOJNHN@cg_debugevents?$AA@ 3005ad8c     cg_main.obj
 0002:00002d9c       ??_C@_0BB@PNGPLJB@cg_debugposition?$AA@ 3005ad9c     cg_main.obj
 0002:00002db0       ??_C@_0N@OLFHJPEJ@cg_debuganim?$AA@ 3005adb0     cg_main.obj
 0002:00002dc0       ??_C@_0N@EMGODPLM@cg_animspeed?$AA@ 3005adc0     cg_main.obj
 0002:00002dd0       ??_C@_03OICINGJI@0?43?$AA@ 3005add0     cg_main.obj
 0002:00002dd4       ??_C@_0O@NLMPFCHA@cg_swingSpeed?$AA@ 3005add4     cg_main.obj
 0002:00002de4       ??_C@_0L@BEAFIAK@cg_bobroll?$AA@ 3005ade4     cg_main.obj
 0002:00002df0       ??_C@_0M@BBIJCEAP@cg_bobpitch?$AA@ 3005adf0     cg_main.obj
 0002:00002dfc       ??_C@_08MBNPMEME@cg_bobup?$AA@ 3005adfc     cg_main.obj
 0002:00002e08       ??_C@_05ECMHBHBD@0?4005?$AA@ 3005ae08     cg_main.obj
 0002:00002e10       ??_C@_0L@MJJHGKNK@cg_runroll?$AA@ 3005ae10     cg_main.obj
 0002:00002e1c       ??_C@_05NIGIBNE@0?4002?$AA@ 3005ae1c     cg_main.obj
 0002:00002e24       ??_C@_0M@JHJCCBOJ@cg_runpitch?$AA@ 3005ae24     cg_main.obj
 0002:00002e30       ??_C@_01EKENIIDA@3?$AA@    3005ae30     cg_main.obj
 0002:00002e34       ??_C@_0O@CMEJDJHP@cg_centertime?$AA@ 3005ae34     cg_main.obj
 0002:00002e44       ??_C@_07CJOOHIA@cg_gunZ?$AA@ 3005ae44     cg_main.obj
 0002:00002e4c       ??_C@_07CJLDLEED@cg_gunY?$AA@ 3005ae4c     cg_main.obj
 0002:00002e54       ??_C@_07DAKIIFAC@cg_gunX?$AA@ 3005ae54     cg_main.obj
 0002:00002e5c       ??_C@_03FKNPJMHG@400?$AA@  3005ae5c     cg_main.obj
 0002:00002e60       ??_C@_0BB@PPFMMLIA@cg_railTrailTime?$AA@ 3005ae60     cg_main.obj
 0002:00002e74       ??_C@_0N@IBNNIGPC@cg_lagometer?$AA@ 3005ae74     cg_main.obj
 0002:00002e84       ??_C@_08OCDFECFG@cg_marks?$AA@ 3005ae84     cg_main.obj
 0002:00002e90       ??_C@_0P@CCFIBNOJ@cg_simpleItems?$AA@ 3005ae90     cg_main.obj
 0002:00002ea0       ??_C@_04NOOEDIPE@2500?$AA@ 3005aea0     cg_main.obj
 0002:00002ea8       ??_C@_0N@GADGJPHJ@cg_brassTime?$AA@ 3005aea8     cg_main.obj
 0002:00002eb8       ??_C@_0O@JOEPLDPN@cg_crosshairY?$AA@ 3005aeb8     cg_main.obj
 0002:00002ec8       ??_C@_0O@IHFEICLM@cg_crosshairX?$AA@ 3005aec8     cg_main.obj
 0002:00002ed8       ??_C@_0BD@JJIJCGAH@cg_crosshairHealth?$AA@ 3005aed8     cg_main.obj
 0002:00002eec       ??_C@_02JMHLOEOE@24?$AA@   3005aeec     cg_main.obj
 0002:00002ef0       ??_C@_0BB@NJOFJDCL@cg_crosshairSize?$AA@ 3005aef0     cg_main.obj
 0002:00002f04       ??_C@_0P@GNHKLMJL@cg_drawRewards?$AA@ 3005af04     cg_main.obj
 0002:00002f14       ??_C@_0BG@PFLNOEEN@cg_drawCrosshairNames?$AA@ 3005af14     cg_main.obj
 0002:00002f2c       ??_C@_01FAMBOPH@4?$AA@     3005af2c     cg_main.obj
 0002:00002f30       ??_C@_0BB@KBADOJHA@cg_drawCrosshair?$AA@ 3005af30     cg_main.obj
 0002:00002f44       ??_C@_0BA@HDEFAPDO@cg_drawAttacker?$AA@ 3005af44     cg_main.obj
 0002:00002f54       ??_C@_0BD@FJPGADGN@cg_drawAmmoWarning?$AA@ 3005af54     cg_main.obj
 0002:00002f68       ??_C@_0N@BEDCNPCC@cg_drawIcons?$AA@ 3005af68     cg_main.obj
 0002:00002f78       ??_C@_0P@DMBICICD@cg_draw3dIcons?$AA@ 3005af78     cg_main.obj
 0002:00002f88       ??_C@_0BA@MIPMDAEB@cg_drawSnapshot?$AA@ 3005af88     cg_main.obj
 0002:00002f98       ??_C@_0L@CHMHIHCB@cg_drawFPS?$AA@ 3005af98     cg_main.obj
 0002:00002fa4       ??_C@_0N@FOINMAON@cg_drawTimer?$AA@ 3005afa4     cg_main.obj
 0002:00002fb4       ??_C@_0O@IIACNNIF@cg_drawStatus?$AA@ 3005afb4     cg_main.obj
 0002:00002fc4       ??_C@_09EKPCJMOG@cg_draw2D?$AA@ 3005afc4     cg_main.obj
 0002:00002fd0       ??_C@_07FFANGJCI@cg_gibs?$AA@ 3005afd0     cg_main.obj
 0002:00002fd8       ??_C@_0L@MAOLAFLC@cg_shadows?$AA@ 3005afd8     cg_main.obj
 0002:00002fe4       ??_C@_03KHGJEAFP@0?44?$AA@ 3005afe4     cg_main.obj
 0002:00002fe8       ??_C@_0BE@EMBJACLB@cg_stereoSeparation?$AA@ 3005afe8     cg_main.obj
 0002:00002ffc       ??_C@_02PEECMOAB@90?$AA@   3005affc     cg_main.obj
 0002:00003000       ??_C@_06FDNMOLLD@cg_fov?$AA@ 3005b000     cg_main.obj
 0002:00003008       ??_C@_04CIPMHKHC@22?45?$AA@ 3005b008     cg_main.obj
 0002:00003010       ??_C@_0L@DPFDGKBB@cg_zoomfov?$AA@ 3005b010     cg_main.obj
 0002:0000301c       ??_C@_0L@MLBFCMPB@cg_drawGun?$AA@ 3005b01c     cg_main.obj
 0002:00003028       ??_C@_0O@JKEEFDLF@cg_autoswitch?$AA@ 3005b028     cg_main.obj
 0002:00003038       ??_C@_09JDMGBOIM@cg_ignore?$AA@ 3005b038     cg_main.obj
 0002:00003044       ??_C@_0BL@MDCOCEP@vmMain?3?5unknown?5command?5?$CFi?$AA@ 3005b044     cg_main.obj
 0002:00003060       ??_C@_0P@JMIBMNM@team_headmodel?$AA@ 3005b060     cg_main.obj
 0002:00003070       ??_C@_0L@KEDOKIKJ@team_model?$AA@ 3005b070     cg_main.obj
 0002:0000307c       ??_C@_09DHBBGOBJ@headmodel?$AA@ 3005b07c     cg_main.obj
 0002:00003088       ??_C@_02DKCKIIND@?$CFs?$AA@ 3005b088     cg_main.obj
 0002:0000308c       ??_C@_07DNFNGBFM@?$CFs?5?5?5?5?5?$AA@ 3005b08c     cg_main.obj
 0002:00003094       ??_C@_0BP@KAAOENNK@CG_ConfigString?3?5bad?5index?3?5?$CFi?$AA@ 3005b094     cg_main.obj
 0002:000030b4       ??_C@_07HKJFGNHJ@clients?$AA@ 3005b0b4     cg_main.obj
 0002:000030bc       ??_C@_08EIINAAAI@graphics?$AA@ 3005b0bc     cg_main.obj
 0002:000030c8       ??_C@_06OHLGPBPO@sounds?$AA@ 3005b0c8     cg_main.obj
 0002:000030d0       ??_C@_0O@IKDCOHPA@collision?5map?$AA@ 3005b0d0     cg_main.obj
 0002:000030e0       ??_C@_0CD@GOCPBDLD@Client?1Server?5game?5mismatch?3?5?$CFs?1@ 3005b0e0     cg_main.obj
 0002:00003104       ??_C@_08CCHPPKDI@baseq3?91?$AA@ 3005b104     cg_main.obj
 0002:00003110       __real@407e000000000000    3005b110     cg_main.obj
 0002:00003118       __real@4084000000000000    3005b118     cg_main.obj
 0002:00003120       ??_C@_0BI@EFKAEII@menu?1art?1font2_prop?4tga?$AA@ 3005b120     cg_main.obj
 0002:00003138       ??_C@_0BM@PPJDNIIP@menu?1art?1font1_prop_glo?4tga?$AA@ 3005b138     cg_main.obj
 0002:00003154       ??_C@_0BI@JNLIGCIJ@menu?1art?1font1_prop?4tga?$AA@ 3005b154     cg_main.obj
 0002:0000316c       ??_C@_05PMAELIEO@white?$AA@ 3005b16c     cg_main.obj
 0002:00003174       ??_C@_0BA@FILGFBEK@gfx?12d?1bigchars?$AA@ 3005b174     cg_main.obj
 0002:00003184       ??_C@_0CD@EBGCAAHF@sound?1weapons?1grenade?1hgrenb2a?4w@ 3005b184     cg_main.obj
 0002:000031a8       ??_C@_0CD@HAIKBKOI@sound?1weapons?1grenade?1hgrenb1a?4w@ 3005b1a8     cg_main.obj
 0002:000031cc       ??_C@_0BJ@CANBBPKF@sound?1items?1protect3?4wav?$AA@ 3005b1cc     cg_main.obj
 0002:000031e8       ??_C@_0CC@JCODPDKN@sound?1weapons?1plasma?1plasmx1a?4wa@ 3005b1e8     cg_main.obj
 0002:0000320c       ??_C@_0CC@GHLEALEG@sound?1weapons?1rocket?1rocklx1a?4wa@ 3005b20c     cg_main.obj
 0002:00003230       ??_C@_0CD@BFPOBJCL@sound?1weapons?1railgun?1railgf1a?4w@ 3005b230     cg_main.obj
 0002:00003254       ??_C@_0CC@BJBGICBG@sound?1weapons?1machinegun?1ric3?4wa@ 3005b254     cg_main.obj
 0002:00003278       ??_C@_0CC@NCEKFBLD@sound?1weapons?1machinegun?1ric2?4wa@ 3005b278     cg_main.obj
 0002:0000329c       ??_C@_0CC@FENOCDBN@sound?1weapons?1machinegun?1ric1?4wa@ 3005b29c     cg_main.obj
 0002:000032c0       ??_C@_0BI@NNKBCBOK@sound?1items?1damage3?4wav?$AA@ 3005b2c0     cg_main.obj
 0002:000032d8       ??_C@_0CD@CPOICIJI@sound?1player?1footsteps?1clank?$CFi?4w@ 3005b2d8     cg_main.obj
 0002:000032fc       ??_C@_0CE@GNHKDPID@sound?1player?1footsteps?1splash?$CFi?4@ 3005b2fc     cg_main.obj
 0002:00003320       ??_C@_0CE@GKFIFOMA@sound?1player?1footsteps?1energy?$CFi?4@ 3005b320     cg_main.obj
 0002:00003344       ??_C@_0CC@FFJILBOO@sound?1player?1footsteps?1mech?$CFi?4wa@ 3005b344     cg_main.obj
 0002:00003368       ??_C@_0CD@GNKAFNDH@sound?1player?1footsteps?1flesh?$CFi?4w@ 3005b368     cg_main.obj
 0002:0000338c       ??_C@_0CC@BMGCACJB@sound?1player?1footsteps?1boot?$CFi?4wa@ 3005b38c     cg_main.obj
 0002:000033b0       ??_C@_0CC@LNDAOHOB@sound?1player?1footsteps?1step?$CFi?4wa@ 3005b3b0     cg_main.obj
 0002:000033d4       ??_C@_0BI@DGLBHPLI@sound?1world?1jumppad?4wav?$AA@ 3005b3d4     cg_main.obj
 0002:000033ec       ??_C@_0BJ@ILNOCJIO@sound?1player?1watr_un?4wav?$AA@ 3005b3ec     cg_main.obj
 0002:00003408       ??_C@_0BK@PEBHADE@sound?1player?1watr_out?4wav?$AA@ 3005b408     cg_main.obj
 0002:00003424       ??_C@_0BJ@CLKANPDE@sound?1player?1watr_in?4wav?$AA@ 3005b424     cg_main.obj
 0002:00003440       ??_C@_0BM@LNOOLHLA@sound?1feedback?1lostlead?4wav?$AA@ 3005b440     cg_main.obj
 0002:0000345c       ??_C@_0BM@NNDKOIIH@sound?1feedback?1tiedlead?4wav?$AA@ 3005b45c     cg_main.obj
 0002:00003478       ??_C@_0BN@PBCHFDJF@sound?1feedback?1takenlead?4wav?$AA@ 3005b478     cg_main.obj
 0002:00003498       ??_C@_0BL@BAGIPNBG@sound?1feedback?1defense?4wav?$AA@ 3005b498     cg_main.obj
 0002:000034b4       ??_C@_0BK@HOPMGIJN@sound?1feedback?1assist?4wav?$AA@ 3005b4b4     cg_main.obj
 0002:000034d0       ??_C@_0BP@GOCIBAEN@sound?1feedback?1humiliation?4wav?$AA@ 3005b4d0     cg_main.obj
 0002:000034f0       ??_C@_0BK@HPEMDLDJ@sound?1feedback?1denied?4wav?$AA@ 3005b4f0     cg_main.obj
 0002:0000350c       ??_C@_0BN@MOGPPGAM@sound?1feedback?1excellent?4wav?$AA@ 3005b50c     cg_main.obj
 0002:0000352c       ??_C@_0BO@HFFLOFKH@sound?1feedback?1impressive?4wav?$AA@ 3005b52c     cg_main.obj
 0002:0000354c       ??_C@_0BH@PPLJNIIB@sound?1feedback?1hit?4wav?$AA@ 3005b54c     cg_main.obj
 0002:00003564       ??_C@_0BH@BPJFFDHG@sound?1player?1land1?4wav?$AA@ 3005b564     cg_main.obj
 0002:0000357c       ??_C@_0BG@MOPKJEGA@sound?1player?1talk?4wav?$AA@ 3005b57c     cg_main.obj
 0002:00003594       ??_C@_0BJ@OHOJGDLI@sound?1weapons?1noammo?4wav?$AA@ 3005b594     cg_main.obj
 0002:000035b0       ??_C@_0BJ@LOHBFELN@sound?1items?1respawn1?4wav?$AA@ 3005b5b0     cg_main.obj
 0002:000035cc       ??_C@_0BI@EBCHHAFA@sound?1world?1teleout?4wav?$AA@ 3005b5cc     cg_main.obj
 0002:000035e4       ??_C@_0BH@EJCDOPNG@sound?1world?1telein?4wav?$AA@ 3005b5e4     cg_main.obj
 0002:000035fc       ??_C@_0BJ@BMOAGILK@sound?1player?1gibimp3?4wav?$AA@ 3005b5fc     cg_main.obj
 0002:00003618       ??_C@_0BJ@NHLMLLBP@sound?1player?1gibimp2?4wav?$AA@ 3005b618     cg_main.obj
 0002:00003634       ??_C@_0BJ@FBCIMJLB@sound?1player?1gibimp1?4wav?$AA@ 3005b634     cg_main.obj
 0002:00003650       ??_C@_0BK@DOOOBPFM@sound?1player?1gibsplt1?4wav?$AA@ 3005b650     cg_main.obj
 0002:0000366c       ??_C@_0BM@OECMCAJK@sound?1items?1use_nothing?4wav?$AA@ 3005b66c     cg_main.obj
 0002:00003688       ??_C@_0BI@CHMBGLDC@sound?1items?1wearoff?4wav?$AA@ 3005b688     cg_main.obj
 0002:000036a0       ??_C@_0BJ@EFMFEOAN@sound?1weapons?1change?4wav?$AA@ 3005b6a0     cg_main.obj
 0002:000036bc       ??_C@_0CG@FIPFLECJ@sound?1weapons?1machinegun?1buletby@ 3005b6bc     cg_main.obj
 0002:000036e4       ??_C@_0CD@KNAADEBC@sound?1teamplay?1voc_enemy_1flag?4w@ 3005b6e4     cg_main.obj
 0002:00003708       ??_C@_0CC@MDHGHHAG@sound?1teamplay?1voc_team_1flag?4wa@ 3005b708     cg_main.obj
 0002:0000372c       ??_C@_0CA@JIIPPEEH@sound?1feedback?1voc_holyshit?4wav?$AA@ 3005b72c     cg_main.obj
 0002:0000374c       ??_C@_0CA@HNMMFEAI@sound?1teamplay?1voc_you_flag?4wav?$AA@ 3005b74c     cg_main.obj
 0002:0000376c       ??_C@_0CB@NCMOABK@sound?1teamplay?1voc_team_flag?4wav@ 3005b76c     cg_main.obj
 0002:00003790       ??_C@_0CC@BAGJBDIN@sound?1teamplay?1voc_enemy_flag?4wa@ 3005b790     cg_main.obj
 0002:000037b4       ??_C@_0CF@INHHAMNB@sound?1teamplay?1voc_blue_returned@ 3005b7b4     cg_main.obj
 0002:000037dc       ??_C@_0CE@LLBNHHJG@sound?1teamplay?1voc_red_returned?4@ 3005b7dc     cg_main.obj
 0002:00003800       ??_C@_0CG@NNLCDPOA@sound?1teamplay?1flagtaken_opponen@ 3005b800     cg_main.obj
 0002:00003828       ??_C@_0CG@PPKEHJCF@sound?1teamplay?1flagtaken_yourtea@ 3005b828     cg_main.obj
 0002:00003850       ??_C@_0CH@ENNMPOJM@sound?1teamplay?1flagreturn_oppone@ 3005b850     cg_main.obj
 0002:00003878       ??_C@_0CH@GPMKLIFJ@sound?1teamplay?1flagreturn_yourte@ 3005b878     cg_main.obj
 0002:000038a0       ??_C@_0CI@NELGEHON@sound?1teamplay?1flagcapture_oppon@ 3005b8a0     cg_main.obj
 0002:000038c8       ??_C@_0CD@KLDPFGFG@sound?1teamplay?1voc_blue_scores?4w@ 3005b8c8     cg_main.obj
 0002:000038ec       ??_C@_0CC@JMEMACMF@sound?1teamplay?1voc_red_scores?4wa@ 3005b8ec     cg_main.obj
 0002:00003910       ??_C@_0CA@NGJNFJDA@sound?1feedback?1hit_teammate?4wav?$AA@ 3005b910     cg_main.obj
 0002:00003930       ??_C@_0BN@HMCOLEK@sound?1feedback?1teamstied?4wav?$AA@ 3005b930     cg_main.obj
 0002:00003950       ??_C@_0BN@KNKFAPML@sound?1feedback?1blueleads?4wav?$AA@ 3005b950     cg_main.obj
 0002:00003970       ??_C@_0BM@MOIOEAMK@sound?1feedback?1redleads?4wav?$AA@ 3005b970     cg_main.obj
 0002:0000398c       ??_C@_0CI@PGKAABCI@sound?1teamplay?1flagcapture_yourt@ 3005b98c     cg_main.obj
 0002:000039b4       ??_C@_0BL@OKIMFPPI@sound?1feedback?1prepare?4wav?$AA@ 3005b9b4     cg_main.obj
 0002:000039d0       ??_C@_0BJ@LFENOPFJ@sound?1feedback?1fight?4wav?$AA@ 3005b9d0     cg_main.obj
 0002:000039ec       ??_C@_0BH@PIFBDOCI@sound?1feedback?1one?4wav?$AA@ 3005b9ec     cg_main.obj
 0002:00003a04       ??_C@_0BH@IKFNOJCO@sound?1feedback?1two?4wav?$AA@ 3005ba04     cg_main.obj
 0002:00003a1c       ??_C@_0BJ@BMGLCFHO@sound?1feedback?1three?4wav?$AA@ 3005ba1c     cg_main.obj
 0002:00003a38       ??_C@_0BL@MFNBDJEC@sound?1feedback?13_frags?4wav?$AA@ 3005ba38     cg_main.obj
 0002:00003a54       ??_C@_0BL@FOHEHFCN@sound?1feedback?12_frags?4wav?$AA@ 3005ba54     cg_main.obj
 0002:00003a70       ??_C@_0BK@OBKGIBHG@sound?1feedback?11_frag?4wav?$AA@ 3005ba70     cg_main.obj
 0002:00003a8c       ??_C@_0CA@MIDPIFA@sound?1feedback?1sudden_death?4wav?$AA@ 3005ba8c     cg_main.obj
 0002:00003aac       ??_C@_0BM@KFPPCANJ@sound?1feedback?15_minute?4wav?$AA@ 3005baac     cg_main.obj
 0002:00003ac8       ??_C@_0BM@GFEGEKEP@sound?1feedback?11_minute?4wav?$AA@ 3005bac8     cg_main.obj
 0002:00003ae4       ??_C@_03BICDMHKB@wav?$AA@  3005bae4     cg_main.obj
 0002:00003ae8       ??_C@_0CJ@CMOPAMCG@PrecacheItem?3?5?$CFs?5has?5bad?5precach@ 3005bae8     cg_main.obj
 0002:00003b14       ??_C@_03JLINDLFM@?$CK?$CFi?$AA@ 3005bb14     cg_main.obj
 0002:00003b18       ??_C@_09GGOFPAOP@bloodMark?$AA@ 3005bb18     cg_main.obj
 0002:00003b24       ??_C@_04KNLNBPHI@wake?$AA@ 3005bb24     cg_main.obj
 0002:00003b2c       ??_C@_0L@KHLAIOEE@markShadow?$AA@ 3005bb2c     cg_main.obj
 0002:00003b38       ??_C@_0BG@EGMLCGNC@gfx?1damage?1plasma_mrk?$AA@ 3005bb38     cg_main.obj
 0002:00003b50       ??_C@_0BH@NJDKADCK@gfx?1damage?1hole_lg_mrk?$AA@ 3005bb50     cg_main.obj
 0002:00003b68       ??_C@_0BI@HAJPOEDB@gfx?1damage?1burn_med_mrk?$AA@ 3005bb68     cg_main.obj
 0002:00003b80       ??_C@_0BG@FPMKOIGF@gfx?1damage?1bullet_mrk?$AA@ 3005bb80     cg_main.obj
 0002:00003b98       ??_C@_0O@LNEKLMGE@medal_capture?$AA@ 3005bb98     cg_main.obj
 0002:00003ba8       ??_C@_0N@KEBDHBDI@medal_assist?$AA@ 3005bba8     cg_main.obj
 0002:00003bb8       ??_C@_0N@JPEODKCB@medal_defend?$AA@ 3005bbb8     cg_main.obj
 0002:00003bc8       ??_C@_0P@CBAOAFEF@medal_gauntlet?$AA@ 3005bbc8     cg_main.obj
 0002:00003bd8       ??_C@_0BA@PLFOJPJ@medal_excellent?$AA@ 3005bbd8     cg_main.obj
 0002:00003be8       ??_C@_0BB@OCKBIFDG@medal_impressive?$AA@ 3005bbe8     cg_main.obj
 0002:00003bfc       ??_C@_0CC@ICGGEAGG@models?1powerups?1shield?1shield?4md@ 3005bbfc     cg_main.obj
 0002:00003c20       ??_C@_0P@HDJNFJNH@teleportEffect?$AA@ 3005bc20     cg_main.obj
 0002:00003c30       ??_C@_0BG@MIEMONNI@models?1misc?1telep?4md3?$AA@ 3005bc30     cg_main.obj
 0002:00003c48       ??_C@_0BL@ECHNCMPC@models?1weaphits?1boom01?4md3?$AA@ 3005bc48     cg_main.obj
 0002:00003c64       ??_C@_0BL@OBLKOCFL@models?1weaphits?1ring02?4md3?$AA@ 3005bc64     cg_main.obj
 0002:00003c80       ??_C@_0BL@KJKOFMEH@models?1weaphits?1bullet?4md3?$AA@ 3005bc80     cg_main.obj
 0002:00003c9c       ??_C@_0P@JNFBEAMD@bloodExplosion?$AA@ 3005bc9c     cg_main.obj
 0002:00003cac       ??_C@_0BB@NCNCDGDJ@sprites?1balloon3?$AA@ 3005bcac     cg_main.obj
 0002:00003cc0       ??_C@_0BG@ENKCMADE@models?1gibs?1brain?4md3?$AA@ 3005bcc0     cg_main.obj
 0002:00003cd8       ??_C@_0BG@GCKMGPLF@models?1gibs?1skull?4md3?$AA@ 3005bcd8     cg_main.obj
 0002:00003cf0       ??_C@_0BE@PBDAJPPM@models?1gibs?1leg?4md3?$AA@ 3005bcf0     cg_main.obj
 0002:00003d04       ??_C@_0BK@EGFHPFIO@models?1gibs?1intestine?4md3?$AA@ 3005bd04     cg_main.obj
 0002:00003d20       ??_C@_0BI@NDPGKIHD@models?1gibs?1forearm?4md3?$AA@ 3005bd20     cg_main.obj
 0002:00003d38       ??_C@_0BF@NBCNENBO@models?1gibs?1foot?4md3?$AA@ 3005bd38     cg_main.obj
 0002:00003d50       ??_C@_0BF@LHDMLCCD@models?1gibs?1fist?4md3?$AA@ 3005bd50     cg_main.obj
 0002:00003d68       ??_C@_0BG@HOCHIPGC@models?1gibs?1chest?4md3?$AA@ 3005bd68     cg_main.obj
 0002:00003d80       ??_C@_0BE@GJNHALAL@models?1gibs?1arm?4md3?$AA@ 3005bd80     cg_main.obj
 0002:00003d94       ??_C@_0BI@KACGLCGL@models?1gibs?1abdomen?4md3?$AA@ 3005bd94     cg_main.obj
 0002:00003dac       ??_C@_0CD@FGDIHLFA@models?1weapons2?1shells?1s_shell?4m@ 3005bdac     cg_main.obj
 0002:00003dd0       ??_C@_0CD@LDBBEFLC@models?1weapons2?1shells?1m_shell?4m@ 3005bdd0     cg_main.obj
 0002:00003df4       ??_C@_0BE@MEJHIMJO@gfx?12d?1colorbar?4tga?$AA@ 3005bdf4     cg_main.obj
 0002:00003e08       ??_C@_0BC@PBFIMOJD@powerups?1blueflag?$AA@ 3005be08     cg_main.obj
 0002:00003e1c       ??_C@_0M@FBFPNKIP@sprites?1foe?$AA@ 3005be1c     cg_main.obj
 0002:00003e28       ??_C@_0BB@HOLOGHCC@icons?1iconf_blu3?$AA@ 3005be28     cg_main.obj
 0002:00003e3c       ??_C@_0BB@GHKFFGGD@icons?1iconf_blu2?$AA@ 3005be3c     cg_main.obj
 0002:00003e50       ??_C@_0BB@HOLCHGGN@icons?1iconf_red3?$AA@ 3005be50     cg_main.obj
 0002:00003e64       ??_C@_0BB@GHKJEHCM@icons?1iconf_red2?$AA@ 3005be64     cg_main.obj
 0002:00003e78       ??_C@_0BB@BCGKNBJH@icons?1skull_blue?$AA@ 3005be78     cg_main.obj
 0002:00003e8c       ??_C@_0BA@OMPBBNIO@icons?1skull_red?$AA@ 3005be8c     cg_main.obj
 0002:00003e9c       ??_C@_0BO@CMJEFEFK@models?1powerups?1orb?1b_orb?4md3?$AA@ 3005be9c     cg_main.obj
 0002:00003ebc       ??_C@_0BO@LDKNFLC@models?1powerups?1orb?1r_orb?4md3?$AA@ 3005bebc     cg_main.obj
 0002:00003edc       ??_C@_0P@IJPLAABH@hasteSmokePuff?$AA@ 3005bedc     cg_main.obj
 0002:00003eec       ??_C@_0P@NKEDBBDN@powerups?1regen?$AA@ 3005beec     cg_main.obj
 0002:00003efc       ??_C@_0BG@BGIMBFCE@powerups?1invisibility?$AA@ 3005befc     cg_main.obj
 0002:00003f14       ??_C@_0BG@GANDEAKN@powerups?1battleWeapon?$AA@ 3005bf14     cg_main.obj
 0002:00003f2c       ??_C@_0BE@NKPPFPFJ@powerups?1battleSuit?$AA@ 3005bf2c     cg_main.obj
 0002:00003f40       ??_C@_0BE@KLLJIGAB@powerups?1quadWeapon?$AA@ 3005bf40     cg_main.obj
 0002:00003f54       ??_C@_0O@IDIMMBII@powerups?1quad?$AA@ 3005bf54     cg_main.obj
 0002:00003f64       ??_C@_0N@COAENKOL@icons?1noammo?$AA@ 3005bf64     cg_main.obj
 0002:00003f74       ??_C@_0BA@PJMLIFEA@gfx?12d?1backtile?$AA@ 3005bf74     cg_main.obj
 0002:00003f84       ??_C@_0BD@PPPBDMEH@gfx?12d?1crosshair?$CFc?$AA@ 3005bf84     cg_main.obj
 0002:00003f98       ??_C@_0O@MHPONILH@gfx?12d?1select?$AA@ 3005bf98     cg_main.obj
 0002:00003fa8       ??_C@_0BA@LPLLBJPM@gfx?1misc?1tracer?$AA@ 3005bfa8     cg_main.obj
 0002:00003fb8       ??_C@_0M@OBGACBNG@waterBubble?$AA@ 3005bfb8     cg_main.obj
 0002:00003fc4       ??_C@_0N@GGGDBMDO@disconnected?$AA@ 3005bfc4     cg_main.obj
 0002:00003fd4       ??_C@_09GJJGLCPD@lagometer?$AA@ 3005bfd4     cg_main.obj
 0002:00003fe0       ??_C@_0L@LLCKKMKM@bloodTrail?$AA@ 3005bfe0     cg_main.obj
 0002:00003fec       ??_C@_0BA@PMLAEFDB@sprites?1plasma1?$AA@ 3005bfec     cg_main.obj
 0002:00003ffc       ??_C@_0BB@FPJBCPAO@shotgunSmokePuff?$AA@ 3005bffc     cg_main.obj
 0002:00004010       ??_C@_0BB@LHMIJHPJ@smokePuffRagePro?$AA@ 3005c010     cg_main.obj
 0002:00004024       ??_C@_09GPGLBPNG@smokePuff?$AA@ 3005c024     cg_main.obj
 0002:00004030       ??_C@_0BC@LIBCKFBH@menu?1tab?1time?4tga?$AA@ 3005c030     cg_main.obj
 0002:00004044       ??_C@_0BD@DJDOFAFI@menu?1tab?1score?4tga?$AA@ 3005c044     cg_main.obj
 0002:00004058       ??_C@_0BC@JJNOEPIN@menu?1tab?1ping?4tga?$AA@ 3005c058     cg_main.obj
 0002:0000406c       ??_C@_0BC@FCBJHGEN@menu?1tab?1name?4tga?$AA@ 3005c06c     cg_main.obj
 0002:00004080       ??_C@_0BB@OIENEINL@gfx?12d?1defer?4tga?$AA@ 3005c080     cg_main.obj
 0002:00004094       ??_C@_0P@IMGKCNMO@viewBloodBlend?$AA@ 3005c094     cg_main.obj
 0002:000040a4       ??_C@_0BE@KBEMACEB@menu?1art?1skill5?4tga?$AA@ 3005c0a4     cg_main.obj
 0002:000040b8       ??_C@_0BE@GKBANBOE@menu?1art?1skill4?4tga?$AA@ 3005c0b8     cg_main.obj
 0002:000040cc       ??_C@_0BE@HHBFOBFM@menu?1art?1skill3?4tga?$AA@ 3005c0cc     cg_main.obj
 0002:000040e0       ??_C@_0BE@LMEJDCPJ@menu?1art?1skill2?4tga?$AA@ 3005c0e0     cg_main.obj
 0002:000040f4       ??_C@_0BE@DKNNEAFH@menu?1art?1skill1?4tga?$AA@ 3005c0f4     cg_main.obj
 0002:00004108       ??_C@_0L@EDDEHNPC@game?5media?$AA@ 3005c108     cg_main.obj
 0002:00004114       ??_C@_08MEIODECE@explode1?$AA@ 3005c114     cg_marks.obj
 0002:00004120       __real@c1a00000            3005c120     cg_marks.obj
 0002:00004124       ??_C@_0CG@NBPMFGF@CG_ImpactMark?5called?5with?5?$DM?$DN?50?5r@ 3005c124     cg_marks.obj
 0002:00004150       __real@407c200000000000    3005c150     cg_marks.obj
 0002:00004158       __real@40a7700000000000    3005c158     cg_marks.obj
 0002:00004160       ??_C@_04MDMPPDAB@?$CFs?$CFi?$AA@ 3005c160     cg_marks.obj
 0002:00004168       __real@4000000000000000    3005c168     cg_marks.obj
 0002:00004170       __real@45800000            3005c170     cg_marks.obj
 0002:00004178       __real@3feccccccccccccd    3005c178     cg_marks.obj
 0002:00004180       ??_C@_0CI@CKGHJCDF@CG_ParticleSnowFlurry?5pshader?5?$DN?$DN@ 3005c180     cg_marks.obj
 0002:000041a8       ??_C@_0CC@DIFPPKPM@CG_ParticleSnow?5pshader?5?$DN?$DN?5ZERO?$CB@ 3005c1a8     cg_marks.obj
 0002:000041d0       __real@4049000000000000    3005c1d0     cg_marks.obj
 0002:000041d8       __real@4024000000000000    3005c1d8     cg_marks.obj
 0002:000041e0       __real@bf800000            3005c1e0     cg_marks.obj
 0002:000041e4       ??_C@_0BL@MLDGCJII@CG_ParticleSmoke?5?$DN?$DN?5ZERO?$CB?6?$AA@ 3005c1e4     cg_marks.obj
 0002:00004200       __real@4066600000000000    3005c200     cg_marks.obj
 0002:00004208       ??_C@_0DE@LHPJKLJP@CG_ParticleExplosion?3?5unknown?5an@ 3005c208     cg_marks.obj
 0002:00004240       ??_C@_0EI@EKMNKCC@CG_ParticleExplosion?3?5animStr?5is@ 3005c240     cg_marks.obj
 0002:00004288       ??_C@_0CN@HAOPCKBM@CG_ParticleImpactSmokePuff?5pshad@ 3005c288     cg_marks.obj
 0002:000042b8       ??_C@_0CE@FDMOADGI@CG_Particle_Bleed?5pshader?5?$DN?$DN?5ZER@ 3005c2b8     cg_marks.obj
 0002:000042dc       ??_C@_0CC@KJEJNONH@CG_Particle_OilParticle?5?$DN?$DN?5ZERO?$CB@ 3005c2dc     cg_marks.obj
 0002:00004300       __real@3fe199999999999a    3005c300     cg_marks.obj
 0002:00004308       ??_C@_0BP@LFCJGJJN@CG_Particle_OilSlick?5?$DN?$DN?5ZERO?$CB?6?$AA@ 3005c308     cg_marks.obj
 0002:00004328       ??_C@_0BL@DDKPPMGF@CG_OilSlickRevove?5NULL?5id?6?$AA@ 3005c328     cg_marks.obj
 0002:00004348       __real@bff0000000000000    3005c348     cg_marks.obj
 0002:00004350       __real@3fd999999999999a    3005c350     cg_marks.obj
 0002:00004358       __real@3fe3333333333333    3005c358     cg_marks.obj
 0002:00004360       ??_C@_0BP@PNDEBGI@CG_BloodPool?5pshader?5?$DN?$DN?5ZERO?$CB?6?$AA@ 3005c360     cg_marks.obj
 0002:00004380       __real@3e4ccccd            3005c380     cg_marks.obj
 0002:00004388       __real@407f400000000000    3005c388     cg_marks.obj
 0002:00004390       __real@40ab580000000000    3005c390     cg_marks.obj
 0002:00004398       ??_C@_0L@FMIBJCKG@?$CKdrown?4wav?$AA@ 3005c398     cg_players.obj
 0002:000043a4       ??_C@_0O@LBBMLEKM@?$CKfalling1?4wav?$AA@ 3005c3a4     cg_players.obj
 0002:000043b4       ??_C@_0M@EADDCLKM@?$CKdeath3?4wav?$AA@ 3005c3b4     cg_players.obj
 0002:000043c0       ??_C@_0M@ILGPPIAJ@?$CKdeath2?4wav?$AA@ 3005c3c0     cg_players.obj
 0002:000043cc       ??_C@_0M@NPLIKKH@?$CKdeath1?4wav?$AA@ 3005c3cc     cg_players.obj
 0002:000043d8       ??_C@_0BJ@HBJEEGKP@Unknown?5custom?5sound?3?5?$CFs?$AA@ 3005c3d8     cg_players.obj
 0002:000043f4       ??_C@_0CH@OIHGELEA@Memory?5is?5low?4?5?5Using?5deferred?5m@ 3005c3f4     cg_players.obj
 0002:0000441c       ??_C@_06EGNCJDCP@hmodel?$AA@ 3005c41c     cg_players.obj
 0002:00004424       ??_C@_0L@CPNMJIBN@g_blueteam?$AA@ 3005c424     cg_players.obj
 0002:00004430       ??_C@_09LPNHELAH@g_redteam?$AA@ 3005c430     cg_players.obj
 0002:0000443c       ??_C@_02JKAOMCMK@tl?$AA@   3005c43c     cg_players.obj
 0002:00004440       ??_C@_02BIBFFKJD@tt?$AA@   3005c440     cg_players.obj
 0002:00004444       ??_C@_01PFHFFBPC@t?$AA@    3005c444     cg_players.obj
 0002:00004448       ??_C@_01HHGOMJKL@l?$AA@    3005c448     cg_players.obj
 0002:0000444c       ??_C@_01NOFIACDB@w?$AA@    3005c44c     cg_players.obj
 0002:00004450       ??_C@_02IKKIEBB@hc?$AA@    3005c450     cg_players.obj
 0002:00004454       ??_C@_05ODMCMJAJ@skill?$AA@ 3005c454     cg_players.obj
 0002:0000445c       ??_C@_02KHFPAHOF@c2?$AA@   3005c45c     cg_players.obj
 0002:00004460       ??_C@_02IMHCFECG@c1?$AA@   3005c460     cg_players.obj
 0002:00004464       ??_C@_0BD@NDLIHGFC@sound?1player?1?$CFs?1?$CFs?$AA@ 3005c464     cg_players.obj
 0002:00004478       ??_C@_08BPBKIHMF@tag_flag?$AA@ 3005c478     cg_players.obj
 0002:00004484       ??_C@_0CG@NFMPGJHJ@DEFAULT_MODEL?5?$CI?$CFs?$CJ?5failed?5to?5reg@ 3005c484     cg_players.obj
 0002:000044ac       ??_C@_0DF@GJHBNGJF@DEFAULT_TEAM_MODEL?5?1?5skin?5?$CI?$CFs?1?$CFs@ 3005c4ac     cg_players.obj
 0002:000044e4       ??_C@_07OLKAFEPH@Stroggs?$AA@ 3005c4e4     cg_players.obj
 0002:000044ec       ??_C@_06GMDNOCON@Pagans?$AA@ 3005c4ec     cg_players.obj
 0002:000044f4       ??_C@_0DH@DLIOIGIN@CG_RegisterClientModelname?$CI?5?$CFs?0?5@ 3005c4f4     cg_players.obj
 0002:0000452c       ??_C@_03LJIJAGL@tga?$AA@   3005c52c     cg_players.obj
 0002:00004530       ??_C@_04DMJJIPAH@icon?$AA@ 3005c530     cg_players.obj
 0002:00004538       ??_C@_04NHPAFEHJ@skin?$AA@ 3005c538     cg_players.obj
 0002:00004540       ??_C@_0CC@BDJGDBLP@Failed?5to?5load?5animation?5file?5?$CFs@ 3005c540     cg_players.obj
 0002:00004564       ??_C@_0CL@CKIMBAJB@models?1players?1characters?1?$CFs?1ani@ 3005c564     cg_players.obj
 0002:00004590       ??_C@_0CA@MLIOIMKH@models?1players?1?$CFs?1animation?4cfg?$AA@ 3005c590     cg_players.obj
 0002:000045b0       ??_C@_0CM@NJHANNLM@Failed?5to?5load?5skin?5file?3?5?$CFs?5?3?5?$CF@ 3005c5b0     cg_players.obj
 0002:000045dc       ??_C@_03NPMJBIL@?$CFs?1?$AA@ 3005c5dc     cg_players.obj
 0002:000045e0       ??_C@_0DB@JFHOKPOB@Failed?5to?5load?5skin?5file?3?5?$CFs?5?3?5?$CF@ 3005c5e0     cg_players.obj
 0002:00004614       ??_C@_0BL@MHNDFDC@models?1players?1?$CFs?1head?4md3?$AA@ 3005c614     cg_players.obj
 0002:00004630       ??_C@_0BP@KFHLABFJ@models?1players?1heads?1?$CFs?1?$CFs?4md3?$AA@ 3005c630     cg_players.obj
 0002:00004650       ??_C@_0CH@BOIMLMJA@models?1players?1characters?1?$CFs?1upp@ 3005c650     cg_players.obj
 0002:00004678       ??_C@_0BM@GODFODEI@models?1players?1?$CFs?1upper?4md3?$AA@ 3005c678     cg_players.obj
 0002:00004694       ??_C@_0BO@KKNKOPB@Failed?5to?5load?5model?5file?5?$CFs?6?$AA@ 3005c694     cg_players.obj
 0002:000046b4       ??_C@_0CH@LMILJCAL@models?1players?1characters?1?$CFs?1low@ 3005c6b4     cg_players.obj
 0002:000046dc       ??_C@_0BM@MMDCMNND@models?1players?1?$CFs?1lower?4md3?$AA@ 3005c6dc     cg_players.obj
 0002:000046f8       ??_C@_0CB@CMKGLJDL@Error?5parsing?5animation?5file?3?5?$CFs@ 3005c6f8     cg_players.obj
 0002:0000471c       ??_C@_0BK@CGODILEM@unknown?5token?5?8?$CFs?8?5is?5?$CFs?6?$AA@ 3005c71c     cg_players.obj
 0002:00004738       ??_C@_0L@FDFHPMAL@fixedtorso?$AA@ 3005c738     cg_players.obj
 0002:00004744       ??_C@_09BMKCBKIH@fixedlegs?$AA@ 3005c744     cg_players.obj
 0002:00004750       ??_C@_03OMLNFKE@sex?$AA@   3005c750     cg_players.obj
 0002:00004754       ??_C@_0L@JPPMCFBB@headoffset?$AA@ 3005c754     cg_players.obj
 0002:00004760       ??_C@_0BO@KPCLPKFJ@Bad?5footsteps?5parm?5in?5?$CFs?3?5?$CFs?6?$AA@ 3005c760     cg_players.obj
 0002:00004780       ??_C@_06KKGCKCNJ@energy?$AA@ 3005c780     cg_players.obj
 0002:00004788       ??_C@_04LDDCCIPJ@mech?$AA@ 3005c788     cg_players.obj
 0002:00004790       ??_C@_05DLDJBIMA@flesh?$AA@ 3005c790     cg_players.obj
 0002:00004798       ??_C@_04LBLCPLHF@boot?$AA@ 3005c798     cg_players.obj
 0002:000047a0       ??_C@_06IKLLLDHL@normal?$AA@ 3005c7a0     cg_players.obj
 0002:000047a8       ??_C@_09IPEFJHNA@footsteps?$AA@ 3005c7a8     cg_players.obj
 0002:000047b4       ??_C@_0BC@NFDFKMPA@File?5?$CFs?5too?5long?6?$AA@ 3005c7b4     cg_players.obj
 0002:000047c8       ??_C@_0BN@EDIIPDOB@models?1players?1?$CFs?$CFs?1?$CFs_?$CFs?4?$CFs?$AA@ 3005c7c8     cg_players.obj
 0002:000047e8       ??_C@_0BP@EDGPHBII@models?1players?1?$CFs?$CFs?1?$CFs?$CFs_?$CFs?4?$CFs?$AA@ 3005c7e8     cg_players.obj
 0002:00004808       ??_C@_0CA@LCPNCLIM@models?1players?1?$CFs?$CFs?1?$CFs?1?$CFs_?$CFs?4?$CFs?$AA@ 3005c808     cg_players.obj
 0002:00004828       ??_C@_0CC@BLDEMPPB@models?1players?1?$CFs?$CFs?1?$CFs?1?$CFs?$CFs_?$CFs?4?$CF@ 3005c828     cg_players.obj
 0002:0000484c       ??_C@_06NGEOGMCH@heads?1?$AA@ 3005c84c     cg_players.obj
 0002:00004854       ??_C@_03FAAAOPJM@red?$AA@  3005c854     cg_players.obj
 0002:00004858       ??_C@_04OBGPFBCN@blue?$AA@ 3005c858     cg_players.obj
 0002:00004860       ??_C@_0BM@CECLOEIL@Head?5skin?5load?5failure?3?5?$CFs?6?$AA@ 3005c860     cg_players.obj
 0002:0000487c       ??_C@_04NEODDMOL@head?$AA@ 3005c87c     cg_players.obj
 0002:00004884       ??_C@_0BN@BAPBAPJE@Torso?5skin?5load?5failure?3?5?$CFs?6?$AA@ 3005c884     cg_players.obj
 0002:000048a4       ??_C@_05NECKJAMC@upper?$AA@ 3005c8a4     cg_players.obj
 0002:000048ac       ??_C@_0BL@NBGPNFJF@Leg?5skin?5load?5failure?3?5?$CFs?6?$AA@ 3005c8ac     cg_players.obj
 0002:000048c8       ??_C@_05IPJEPLHL@lower?$AA@ 3005c8c8     cg_players.obj
 0002:000048d0       ??_C@_0M@DDGCLDMM@characters?1?$AA@ 3005c8d0     cg_players.obj
 0002:000048dc       ??_C@_0CA@EELEKOBE@models?1players?1?$CFs?$CFs?1?$CFs_?$CFs_?$CFs?4?$CFs?$AA@ 3005c8dc     cg_players.obj
 0002:000048fc       ??_C@_0CC@DEGJNDKJ@models?1players?1?$CFs?$CFs?1?$CFs?$CFs_?$CFs_?$CFs?4?$CF@ 3005c8fc     cg_players.obj
 0002:00004920       ??_C@_0CN@PBDGFPPP@CG_SetDeferredClientInfo?3?5no?5val@ 3005c920     cg_players.obj
 0002:00004950       ??_C@_08PGAPCFON@tag_head?$AA@ 3005c950     cg_players.obj
 0002:0000495c       ??_C@_09FJEJHBEN@tag_torso?$AA@ 3005c95c     cg_players.obj
 0002:00004968       ??_C@_0BP@EEHJJPLA@Bad?5clientNum?5on?5player?5entity?$AA@ 3005c968     cg_players.obj
 0002:00004988       ??_C@_0BF@IBAKKNBL@Clamp?5lf?9?$DOframeTime?6?$AA@ 3005c988     cg_players.obj
 0002:000049a0       ??_C@_09JCEMHLHC@Anim?3?5?$CFi?6?$AA@ 3005c9a0     cg_players.obj
 0002:000049ac       ??_C@_0BJ@OHDPKGG@Bad?5animation?5number?3?5?$CFi?$AA@ 3005c9ac     cg_players.obj
 0002:000049c8       __real@3d4ccccd            3005c9c8     cg_players.obj
 0002:000049cc       __real@c3b40000            3005c9cc     cg_players.obj
 0002:000049d0       ??_C@_0BK@GAIDHALI@Bad?5player?5movement?5angle?$AA@ 3005c9d0     cg_players.obj
 0002:000049ec       __real@42b40000            3005c9ec     cg_players.obj
 0002:000049f0       __real@43000000            3005c9f0     cg_players.obj
 0002:000049f4       ??_C@_0BN@FKDGBGEH@?$CFi?5ResetPlayerEntity?5yaw?$DN?$CFi?6?$AA@ 3005c9f4     cg_players.obj
 0002:00004a18       __real@406fe00000000000    3005ca18     cg_playerstate.obj
 0002:00004a20       __real@4044000000000000    3005ca20     cg_playerstate.obj
 0002:00004a28       ??_C@_0CC@NIDOAJN@WARNING?3?5changed?5predicted?5event@ 3005ca28     cg_playerstate.obj
 0002:00004a4c       ??_C@_0BH@JOJLKMBP@WARNING?3?5double?5event?6?$AA@ 3005ca4c     cg_predict.obj
 0002:00004a64       ??_C@_0BI@ELMKHMCD@WARNING?3?5dropped?5event?6?$AA@ 3005ca64     cg_predict.obj
 0002:00004a7c       ??_C@_0L@DOJHFFNN@not?5moved?6?$AA@ 3005ca7c     cg_predict.obj
 0002:00004a88       ??_C@_0L@NKHFPHNI@?$FL?$CFi?5?3?5?$CFi?$FN?5?$AA@ 3005ca88     cg_predict.obj
 0002:00004a94       ??_C@_0BN@HNLMAFPF@Double?5prediction?5decay?3?5?$CFf?6?$AA@ 3005ca94     cg_predict.obj
 0002:00004ab4       ??_C@_0BF@BBGFLFIG@Prediction?5miss?3?5?$CFf?6?$AA@ 3005cab4     cg_predict.obj
 0002:00004acc       ??_C@_0BC@GIKLPGML@prediction?5error?6?$AA@ 3005cacc     cg_predict.obj
 0002:00004ae0       ??_C@_0BE@DPKKIGLP@PredictionTeleport?6?$AA@ 3005cae0     cg_predict.obj
 0002:00004af4       ??_C@_02NCPIBIBE@33?$AA@   3005caf4     cg_predict.obj
 0002:00004af8       ??_C@_0CE@JCAHPAJ@exceeded?5PACKET_BACKUP?5on?5comman@ 3005caf8     cg_predict.obj
 0002:00004b1c       ??_C@_0BE@IPIDHCFO@Blue?5leads?5?$CFi?5to?5?$CFi?$AA@ 3005cb1c     cg_scoreboard.obj
 0002:00004b30       ??_C@_0BD@KNNGDKPF@Red?5leads?5?$CFi?5to?5?$CFi?$AA@ 3005cb30     cg_scoreboard.obj
 0002:00004b44       ??_C@_0BF@GPCPNFAF@Teams?5are?5tied?5at?5?$CFi?$AA@ 3005cb44     cg_scoreboard.obj
 0002:00004b5c       ??_C@_0BB@IIGPLNFH@?$CFs?5place?5with?5?$CFi?$AA@ 3005cb5c     cg_scoreboard.obj
 0002:00004b70       ??_C@_0O@BCAEDBLM@Fragged?5by?5?$CFs?$AA@ 3005cb70     cg_scoreboard.obj
 0002:00004b80       ??_C@_05KACKNMMA@READY?$AA@ 3005cb80     cg_scoreboard.obj
 0002:00004b88       ??_C@_0P@LOMDEOFI@?$CF5i?5?$CF4i?5?$CF4i?5?$CFs?$AA@ 3005cb88     cg_scoreboard.obj
 0002:00004b98       ??_C@_0BC@HAIDHOJD@?5SPECT?5?$CF3i?5?$CF4i?5?$CFs?$AA@ 3005cb98     cg_scoreboard.obj
 0002:00004bac       ??_C@_0BC@EIJNNBMO@?5connecting?5?5?5?5?$CFs?$AA@ 3005cbac     cg_scoreboard.obj
 0002:00004bc0       ??_C@_05PPJGDEGI@?$CFi?1?$CFi?$AA@ 3005cbc0     cg_scoreboard.obj
 0002:00004bc8       ??_C@_0BH@DLHNHBEG@Bad?5score?9?$DOclient?3?5?$CFi?6?$AA@ 3005cbc8     cg_scoreboard.obj
 0002:00004be0       ??_C@_09FONCBBOD@Blue?5Team?$AA@ 3005cbe0     cg_scoreboard.obj
 0002:00004bec       ??_C@_08PNCBJLHJ@Red?5Team?$AA@ 3005cbec     cg_scoreboard.obj
 0002:00004bf8       ??_C@_0L@HAPFDNKJ@Scoreboard?$AA@ 3005cbf8     cg_scoreboard.obj
 0002:00004c54       ??_C@_0BC@HILCMIJJ@followflagcarrier?$AA@ 3005cc54     cg_servercmds.obj
 0002:00004c68       ??_C@_0L@BCFFODB@returnflag?$AA@ 3005cc68     cg_servercmds.obj
 0002:00004c74       ??_C@_08LJGLPHPA@followme?$AA@ 3005cc74     cg_servercmds.obj
 0002:00004c80       ??_C@_04LOFLEJM@camp?$AA@  3005cc80     cg_servercmds.obj
 0002:00004c88       ??_C@_06KPEKKPL@patrol?$AA@ 3005cc88     cg_servercmds.obj
 0002:00004c90       ??_C@_0L@LIAONOLJ@defendflag?$AA@ 3005cc90     cg_servercmds.obj
 0002:00004c9c       ??_C@_06BMABBLML@defend?$AA@ 3005cc9c     cg_servercmds.obj
 0002:00004ca4       ??_C@_07GBMLDGPP@offense?$AA@ 3005cca4     cg_servercmds.obj
 0002:00004cac       ??_C@_07NOFDDIA@getflag?$AA@ 3005ccac     cg_servercmds.obj
 0002:00004cb4       ??_C@_0L@OOBNLHBJ@g_blueTeam?$AA@ 3005ccb4     cg_servercmds.obj
 0002:00004cc0       ??_C@_09HOBGGEAD@g_redTeam?$AA@ 3005ccc0     cg_servercmds.obj
 0002:00004ccc       ??_C@_0M@DKNJHPLK@maps?1?$CFs?4bsp?$AA@ 3005cccc     cg_servercmds.obj
 0002:00004cd8       ??_C@_0O@OCOCOONB@sv_maxclients?$AA@ 3005ccd8     cg_servercmds.obj
 0002:00004ce8       ??_C@_09ELHMOKHN@teamflags?$AA@ 3005cce8     cg_servercmds.obj
 0002:00004cf4       ??_C@_07GMGCLCAP@dmflags?$AA@ 3005ccf4     cg_servercmds.obj
 0002:00004cfc       ??_C@_0L@GFINLBEC@g_gametype?$AA@ 3005ccfc     cg_servercmds.obj
 0002:00004d08       ??_C@_01EOFPKCAF@?$EA?$AA@ 3005cd08     cg_servercmds.obj
 0002:00004d0c       ??_C@_01JLIPDDHJ@?3?$AA@   3005cd0c     cg_servercmds.obj
 0002:00004d10       ??_C@_01NEMOKFLO@?$DN?$AA@ 3005cd10     cg_servercmds.obj
 0002:00004d14       ??_C@_01CELHOKLL@?$HN?$AA@ 3005cd14     cg_servercmds.obj
 0002:00004d18       ??_C@_0CO@OOFJHLNN@?$FO1expected?5?$HL?5found?5?$CFs?5in?5voice?5c@ 3005cd18     cg_servercmds.obj
 0002:00004d48       ??_C@_01HCONENDN@?$HL?$AA@ 3005cd48     cg_servercmds.obj
 0002:00004d4c       ??_C@_0DE@LFCGMCMO@?$FO1expected?5gender?5not?5found?5in?5v@ 3005cd4c     cg_servercmds.obj
 0002:00004d80       ??_C@_06GHFJMDBL@neuter?$AA@ 3005cd80     cg_servercmds.obj
 0002:00004d88       ??_C@_04ICKCIGNO@male?$AA@ 3005cd88     cg_servercmds.obj
 0002:00004d90       ??_C@_06GJLDEJIL@female?$AA@ 3005cd90     cg_servercmds.obj
 0002:00004d98       ??_C@_0DJ@DIHCICBL@?$FO1voice?5chat?5file?5too?5large?3?5?$CFs?5@ 3005cd98     cg_servercmds.obj
 0002:00004dd4       ??_C@_0CB@LCNFPPPE@?$FO1voice?5chat?5file?5not?5found?3?5?$CFs?6@ 3005cdd4     cg_servercmds.obj
 0002:00004df8       ??_C@_0BN@NIPMNCMN@voice?5chat?5memory?5size?5?$DN?5?$CFd?6?$AA@ 3005cdf8     cg_servercmds.obj
 0002:00004e18       ??_C@_0BE@KNDJABAE@scripts?1male5?4voice?$AA@ 3005ce18     cg_servercmds.obj
 0002:00004e2c       ??_C@_0BE@GBJDABJK@scripts?1male4?4voice?$AA@ 3005ce2c     cg_servercmds.obj
 0002:00004e40       ??_C@_0BE@GLFGAIID@scripts?1male3?4voice?$AA@ 3005ce40     cg_servercmds.obj
 0002:00004e54       ??_C@_0BE@KHPMAIBN@scripts?1male2?4voice?$AA@ 3005ce54     cg_servercmds.obj
 0002:00004e68       ??_C@_0BE@CJHDAPPO@scripts?1male1?4voice?$AA@ 3005ce68     cg_servercmds.obj
 0002:00004e7c       ??_C@_0BG@COMLMEN@scripts?1female3?4voice?$AA@ 3005ce7c     cg_servercmds.obj
 0002:00004e94       ??_C@_0BG@MOEGLMND@scripts?1female2?4voice?$AA@ 3005ce94     cg_servercmds.obj
 0002:00004eac       ??_C@_0BG@EAMJLLDA@scripts?1female1?4voice?$AA@ 3005ceac     cg_servercmds.obj
 0002:00004ec4       ??_C@_0O@BPOFCDLG@scripts?1?$CFs?4vc?$AA@ 3005cec4     cg_servercmds.obj
 0002:00004ed4       ??_C@_05GFOLEBJA@?$CFs?1?$CFs?$AA@ 3005ced4     cg_servercmds.obj
 0002:00004edc       ??_C@_0CB@KPHIIGNM@Unknown?5client?5game?5command?3?5?$CFs?6@ 3005cedc     cg_servercmds.obj
 0002:00004f00       ??_C@_0BA@GNMFKLDC@clientLevelShot?$AA@ 3005cf00     cg_servercmds.obj
 0002:00004f10       ??_C@_0M@BLBAMFDN@remapShader?$AA@ 3005cf10     cg_servercmds.obj
 0002:00004f1c       ??_C@_0M@NBIMEKNE@map_restart?$AA@ 3005cf1c     cg_servercmds.obj
 0002:00004f28       ??_C@_05DPGKEEHN@tinfo?$AA@ 3005cf28     cg_servercmds.obj
 0002:00004f30       ??_C@_06KBCJDMLG@scores?$AA@ 3005cf30     cg_servercmds.obj
 0002:00004f38       ??_C@_06FPNOEFND@vtchat?$AA@ 3005cf38     cg_servercmds.obj
 0002:00004f40       ??_C@_05LBAAHPBE@vchat?$AA@ 3005cf40     cg_servercmds.obj
 0002:00004f48       ??_C@_05PMMINOBP@tchat?$AA@ 3005cf48     cg_servercmds.obj
 0002:00004f50       ??_C@_03OFAPEBGM@?$CFs?6?$AA@ 3005cf50     cg_servercmds.obj
 0002:00004f54       ??_C@_04BLJLMHHG@chat?$AA@ 3005cf54     cg_servercmds.obj
 0002:00004f5c       ??_C@_05IJDJACGD@print?$AA@ 3005cf5c     cg_servercmds.obj
 0002:00004f64       ??_C@_02EODNHJKB@cs?$AA@   3005cf64     cg_servercmds.obj
 0002:00004f68       ??_C@_02GFBACKGC@cp?$AA@   3005cf68     cg_servercmds.obj
 0002:00004f6c       ??_C@_06DOEGFMGC@FIGHT?$CB?$AA@ 3005cf6c     cg_servercmds.obj
 0002:00004f74       ??_C@_0P@HFBEHELF@CG_MapRestart?6?$AA@ 3005cf74     cg_servercmds.obj
 0002:00004f84       ??_C@_0DI@NCDIEGIG@CG_ProcessSnapshots?3?5cg?4nextSnap@ 3005cf84     cg_snapshot.obj
 0002:00004fbc       ??_C@_0CF@EPBFNJFD@CG_ProcessSnapshots?3?5cg?4snap?5?$DN?$DN?5@ 3005cfbc     cg_snapshot.obj
 0002:00004fe4       ??_C@_0DA@GODLLJKJ@CG_ProcessSnapshots?3?5Server?5time@ 3005cfe4     cg_snapshot.obj
 0002:00005014       ??_C@_0CO@FFJEMNFE@CG_ProcessSnapshots?3?5n?5?$DM?5cg?4late@ 3005d014     cg_snapshot.obj
 0002:00005044       ??_C@_0CI@JDFDPIEH@CG_TransitionSnapshot?3?5NULL?5cg?4n@ 3005d044     cg_snapshot.obj
 0002:0000506c       ??_C@_0CE@BCLPNDDL@CG_TransitionSnapshot?3?5NULL?5cg?4s@ 3005d06c     cg_snapshot.obj
 0002:00005090       ??_C@_0DI@DABDJKNL@WARNING?3?5CG_ReadNextSnapshot?3?5wa@ 3005d090     cg_snapshot.obj
 0002:000050c8       ??_C@_0BG@GCFGCMGP@Can?8t?5register?5model?6?$AA@ 3005d0c8     cg_view.obj
 0002:000050e0       ??_C@_09FLAEHDCJ@frame?5?$CFi?6?$AA@ 3005d0e0     cg_view.obj
 0002:000050ec       ??_C@_08JKENKHJN@skin?5?$CFi?6?$AA@ 3005d0ec     cg_view.obj
 0002:000050f8       ??_C@_0BD@PLOBIDP@cg?4clientFrame?3?$CFi?6?$AA@ 3005d0f8     cg_view.obj
 0002:0000510c       ??_C@_02NJPGOMH@?$CFf?$AA@ 3005d10c     cg_view.obj
 0002:00005110       __real@c1000000            3005d110     cg_view.obj
 0002:00005114       ??_C@_02PJNFELNH@30?$AA@   3005d114     cg_view.obj
 0002:00005118       __real@c04ca5dc0d03cf26    3005d118     cg_view.obj
 0002:00005120       __real@4040000000000000    3005d120     cg_view.obj
 0002:00005128       __real@44000000            3005d128     cg_view.obj
 0002:0000512c       __real@43e10000            3005d12c     cg_view.obj
 0002:00005130       __real@43160000            3005d130     cg_view.obj
 0002:00005134       __real@40c00000            3005d134     cg_view.obj
 0002:00005138       __real@43c80000            3005d138     cg_view.obj
 0002:00005140       __real@4052c00000000000    3005d140     cg_view.obj
 0002:00005148       __real@43200000            3005d148     cg_view.obj
 0002:00005150       __real@3fe8000000000000    3005d150     cg_weapons.obj
 0002:00005158       __real@c0c00000            3005d158     cg_weapons.obj
 0002:0000515c       __real@41d00000            3005d15c     cg_weapons.obj
 0002:00005160       ??_C@_0BI@CJNPJIJG@models?1weaphits?1bfg?4md3?$AA@ 3005d160     cg_weapons.obj
 0002:00005178       ??_C@_0N@EKABNDDO@bfgExplosion?$AA@ 3005d178     cg_weapons.obj
 0002:00005188       ??_C@_0BP@PEJEDJFL@sound?1weapons?1bfg?1bfg_fire?4wav?$AA@ 3005d188     cg_weapons.obj
 0002:000051a8       ??_C@_0BO@DKJAPIPN@sound?1weapons?1bfg?1bfg_hum?4wav?$AA@ 3005d1a8     cg_weapons.obj
 0002:000051c8       ??_C@_08IJBDIACA@railCore?$AA@ 3005d1c8     cg_weapons.obj
 0002:000051d4       ??_C@_0O@HDLAOPGI@railExplosion?$AA@ 3005d1d4     cg_weapons.obj
 0002:000051e4       ??_C@_0CB@BJCODCG@sound?1weapons?1railgun?1rg_hum?4wav@ 3005d1e4     cg_weapons.obj
 0002:00005208       ??_C@_08EJMAMOFN@railDisc?$AA@ 3005d208     cg_weapons.obj
 0002:00005214       ??_C@_0BA@JAAHPOLK@plasmaExplosion?$AA@ 3005d214     cg_weapons.obj
 0002:00005224       ??_C@_0CC@NOGOIAAL@sound?1weapons?1plasma?1hyprbf1a?4wa@ 3005d224     cg_weapons.obj
 0002:00005248       ??_C@_0CA@FGEGNBKP@sound?1weapons?1plasma?1lasfly?4wav?$AA@ 3005d248     cg_weapons.obj
 0002:00005268       ??_C@_0BB@LIEJLDGP@grenadeExplosion?$AA@ 3005d268     cg_weapons.obj
 0002:0000527c       ??_C@_0CD@BGNAFJPC@sound?1weapons?1grenade?1grenlf1a?4w@ 3005d27c     cg_weapons.obj
 0002:000052a0       ??_C@_0BJ@IPKCPFEO@models?1ammo?1grenade1?4md3?$AA@ 3005d2a0     cg_weapons.obj
 0002:000052bc       ??_C@_0BA@NABNBOMN@rocketExplosion?$AA@ 3005d2bc     cg_weapons.obj
 0002:000052cc       ??_C@_0CC@OIFCIFP@sound?1weapons?1rocket?1rocklf1a?4wa@ 3005d2cc     cg_weapons.obj
 0002:000052f0       ??_C@_0CB@EAPDKGGC@sound?1weapons?1rocket?1rockfly?4wav@ 3005d2f0     cg_weapons.obj
 0002:00005314       ??_C@_0CD@NCGDEMHJ@sound?1weapons?1shotgun?1sshotf1b?4w@ 3005d314     cg_weapons.obj
 0002:00005338       ??_C@_0BA@DOLAHAKE@bulletExplosion?$AA@ 3005d338     cg_weapons.obj
 0002:00005348       ??_C@_0CG@KIFMNGEH@sound?1weapons?1machinegun?1machgf4@ 3005d348     cg_weapons.obj
 0002:00005370       ??_C@_0CG@GNPLOIMJ@sound?1weapons?1machinegun?1machgf3@ 3005d370     cg_weapons.obj
 0002:00005398       ??_C@_0CG@MLIMODHN@sound?1weapons?1machinegun?1machgf2@ 3005d398     cg_weapons.obj
 0002:000053c0       ??_C@_0CG@PKGEPJOA@sound?1weapons?1machinegun?1machgf1@ 3005d3c0     cg_weapons.obj
 0002:000053e8       ??_C@_0BO@BLENFKPL@models?1ammo?1rocket?1rocket?4md3?$AA@ 3005d3e8     cg_weapons.obj
 0002:00005408       ??_C@_0CE@HCIHIIKF@sound?1weapons?1lightning?1lg_hit3?4@ 3005d408     cg_weapons.obj
 0002:0000542c       ??_C@_0CE@LJNLFLAA@sound?1weapons?1lightning?1lg_hit2?4@ 3005d42c     cg_weapons.obj
 0002:00005450       ??_C@_0CD@KNELMIA@sound?1weapons?1lightning?1lg_hit?4w@ 3005d450     cg_weapons.obj
 0002:00005474       ??_C@_0BM@KLCPGNMA@models?1weaphits?1crackle?4md3?$AA@ 3005d474     cg_weapons.obj
 0002:00005490       ??_C@_0BB@FHMAJPD@lightningBoltNew?$AA@ 3005d490     cg_weapons.obj
 0002:000054a4       ??_C@_0CE@DECINOH@sound?1weapons?1lightning?1lg_fire?4@ 3005d4a4     cg_weapons.obj
 0002:000054c8       ??_C@_0CD@IOHDBJGJ@sound?1weapons?1lightning?1lg_hum?4w@ 3005d4c8     cg_weapons.obj
 0002:000054ec       ??_C@_0BP@HFJKFEMF@sound?1weapons?1melee?1fsthum?4wav?$AA@ 3005d4ec     cg_weapons.obj
 0002:0000550c       ??_C@_0CA@KEKFDEFA@sound?1weapons?1melee?1fstatck?4wav?$AA@ 3005d50c     cg_weapons.obj
 0002:0000552c       ??_C@_0BP@BOHFALII@sound?1weapons?1melee?1fstrun?4wav?$AA@ 3005d52c     cg_weapons.obj
 0002:0000554c       ??_C@_0CJ@PEFFPDCJ@models?1weapons2?1shotgun?1shotgun_@ 3005d54c     cg_weapons.obj
 0002:00005578       ??_C@_09OLHEALFG@_hand?4md3?$AA@ 3005d578     cg_weapons.obj
 0002:00005584       ??_C@_0M@GGMINFPA@_barrel?4md3?$AA@ 3005d584     cg_weapons.obj
 0002:00005590       ??_C@_0L@DAPODOKF@_flash?4md3?$AA@ 3005d590     cg_weapons.obj
 0002:0000559c       ??_C@_0BI@JJFMDMDC@Couldn?8t?5find?5weapon?5?$CFi?$AA@ 3005d59c     cg_weapons.obj
 0002:000055b8       __real@c049000000000000    3005d5b8     cg_weapons.obj
 0002:000055c0       __real@c044000000000000    3005d5c0     cg_weapons.obj
 0002:000055c8       __real@3fc999999999999a    3005d5c8     cg_weapons.obj
 0002:000055d0       __real@427c0000            3005d5d0     cg_weapons.obj
 0002:000055d8       __real@4054000000000000    3005d5d8     cg_weapons.obj
 0002:000055e0       __real@405e000000000000    3005d5e0     cg_weapons.obj
 0002:000055e8       ??_C@_0DH@ECKDIILO@CG_RegisterItemVisuals?3?5itemNum?5@ 3005d5e8     cg_weapons.obj
 0002:00005620       ??_C@_09FNBKMGLL@tag_flash?$AA@ 3005d620     cg_weapons.obj
 0002:0000562c       ??_C@_0L@EKFDHKMA@tag_barrel?$AA@ 3005d62c     cg_weapons.obj
 0002:00005638       ??_C@_0L@FGMMEJDC@tag_weapon?$AA@ 3005d638     cg_weapons.obj
 0002:00005644       __real@44bb8000            3005d644     cg_weapons.obj
 0002:00005648       __real@44400000            3005d648     cg_weapons.obj
 0002:0000564c       __real@41600000            3005d64c     cg_weapons.obj
 0002:00005650       __real@c3340000            3005d650     cg_weapons.obj
 0002:00005658       __real@bfc999999999999a    3005d658     cg_weapons.obj
 0002:00005660       __real@4072c00000000000    3005d660     cg_weapons.obj
 0002:00005668       __real@3f847ae147ae147b    3005d668     cg_weapons.obj
 0002:00005670       ??_C@_0CN@NBNBAPF@CG_FireWeapon?3?5ent?9?$DOweapon?5?$DO?$DN?5WP@ 3005d670     cg_weapons.obj
 0002:000056a0       __real@442f0000            3005d6a0     cg_weapons.obj
 0002:000056a4       __real@42480000            3005d6a4     cg_weapons.obj
 0002:000056a8       __real@47800000            3005d6a8     q_math.obj
 0002:000056ac       ??_C@_0BK@JDDBNDOP@Q_fabs?$CIinv_denom?$CJ?5?$CB?$DN?50?40f?$AA@ 3005d6ac     q_math.obj
 0002:000056c8       ??_C@_0DD@HJOIBKLP@d?3?2distr?2games_src?2quake3?91?432b?2@ 3005d6c8     q_math.obj
 0002:00005700       __real@4066c16c16c16c17    3005d700     q_math.obj
 0002:00005708       __real@3c8efa35            3005d708     q_math.obj
 0002:0000570c       ??_C@_0BI@KPLEBEJF@ERROR?3?5?$CFs?0?5line?5?$CFd?3?5?$CFs?6?$AA@ 3005d70c     q_shared.obj
 0002:00005724       ??_C@_0BK@DJMKDJBL@WARNING?3?5?$CFs?0?5line?5?$CFd?3?5?$CFs?6?$AA@ 3005d724     q_shared.obj
 0002:00005740       ??_C@_0BF@BFEJCABG@MatchToken?3?5?$CFs?5?$CB?$DN?5?$CFs?$AA@ 3005d740     q_shared.obj
 0002:00005758       ??_C@_01PKGAHCOL@?$CJ?$AA@ 3005d758     q_shared.obj
 0002:0000575c       ??_C@_01ODHLEDKK@?$CI?$AA@ 3005d75c     q_shared.obj
 0002:00005760       ??_C@_0BJ@OLBOPICM@Q_strncpyz?3?5destsize?5?$DM?51?$AA@ 3005d760     q_shared.obj
 0002:0000577c       ??_C@_0BF@BJHHBLMD@Q_strncpyz?3?5NULL?5src?$AA@ 3005d77c     q_shared.obj
 0002:00005794       ??_C@_0BG@EKAPNPCH@Q_strncpyz?3?5NULL?5dest?$AA@ 3005d794     q_shared.obj
 0002:000057ac       ??_C@_0BN@EFOOAHFL@Q_strcat?3?5already?5overflowed?$AA@ 3005d7ac     q_shared.obj
 0002:000057cc       ??_C@_0CD@GIPJKOOD@Com_sprintf?3?5overflow?5of?5?$CFi?5in?5?$CF@ 3005d7cc     q_shared.obj
 0002:000057f0       ??_C@_0CC@GMEFDOKA@Com_sprintf?3?5overflowed?5bigbuffe@ 3005d7f0     q_shared.obj
 0002:00005814       ??_C@_0CG@FLHABLN@Info_ValueForKey?3?5oversize?5infos@ 3005d814     q_shared.obj
 0002:0000583c       ??_C@_0CE@HMPLGKDK@Info_RemoveKey?3?5oversize?5infostr@ 3005d83c     q_shared.obj
 0002:00005860       ??_C@_0CI@CPIEPBLO@Info_RemoveKey_Big?3?5oversize?5inf@ 3005d860     q_shared.obj
 0002:00005888       ??_C@_0BN@CAOBGKLE@Info?5string?5length?5exceeded?6?$AA@ 3005d888     q_shared.obj
 0002:000058a8       ??_C@_06NELKLDPM@?2?$CFs?2?$CFs?$AA@ 3005d8a8     q_shared.obj
 0002:000058b0       ??_C@_0CD@MGFMEBLE@Can?8t?5use?5keys?5or?5values?5with?5a?5@ 3005d8b0     q_shared.obj
 0002:000058d4       ??_C@_0CL@JCFAGLFD@Can?8t?5use?5keys?5or?5values?5with?5a?5@ 3005d8d4     q_shared.obj
 0002:00005900       ??_C@_0CD@JIDDAEOO@Can?8t?5use?5keys?5or?5values?5with?5a?5@ 3005d900     q_shared.obj
 0002:00005924       ??_C@_0CJ@CEEBDGNA@Info_SetValueForKey?3?5oversize?5in@ 3005d924     q_shared.obj
 0002:00005950       ??_C@_0CB@EMDOOGBI@BIG?5Info?5string?5length?5exceeded?6@ 3005d950     q_shared.obj
 0002:00005974       ??_C@_0L@JDDHILPC@fadeAmount?$AA@ 3005d974     ui_shared.obj
 0002:00005980       ??_C@_09LGBLEGN@fadeCycle?$AA@ 3005d980     ui_shared.obj
 0002:0000598c       ??_C@_09DPBPOIDH@fadeClamp?$AA@ 3005d98c     ui_shared.obj
 0002:00005998       ??_C@_05EIEHMANA@popup?$AA@ 3005d998     ui_shared.obj
 0002:000059a0       ??_C@_07BNAIEIKL@itemDef?$AA@ 3005d9a0     ui_shared.obj
 0002:000059a8       ??_C@_09LMHPKFJB@soundLoop?$AA@ 3005d9a8     ui_shared.obj
 0002:000059b4       ??_C@_0BB@FOHPFLED@outOfBoundsClick?$AA@ 3005d9b4     ui_shared.obj
 0002:000059c8       ??_C@_0N@EEPADJLO@disablecolor?$AA@ 3005d9c8     ui_shared.obj
 0002:000059d8       ??_C@_0L@OKFLOHAM@focuscolor?$AA@ 3005d9d8     ui_shared.obj
 0002:000059e4       ??_C@_0L@NBMNMLHL@borderSize?$AA@ 3005d9e4     ui_shared.obj
 0002:000059f0       ??_C@_05IIPJAONP@onESC?$AA@ 3005d9f0     ui_shared.obj
 0002:000059f8       ??_C@_07LAOJOJAJ@onClose?$AA@ 3005d9f8     ui_shared.obj
 0002:00005a00       ??_C@_06CJGNFCEB@onOpen?$AA@ 3005da00     ui_shared.obj
 0002:00005a08       ??_C@_0L@GIACNHMO@fullscreen?$AA@ 3005da08     ui_shared.obj
 0002:00005a14       ??_C@_04EFPADHIC@font?$AA@ 3005da14     ui_shared.obj
 0002:00005a1c       ??_C@_0M@IHJKFHF@doubleclick?$AA@ 3005da1c     ui_shared.obj
 0002:00005a28       ??_C@_09DHDJHDLH@cinematic?$AA@ 3005da28     ui_shared.obj
 0002:00005a34       ??_C@_08BDDCOCNI@hideCvar?$AA@ 3005da34     ui_shared.obj
 0002:00005a40       ??_C@_08LNBEMJIA@showCvar?$AA@ 3005da40     ui_shared.obj
 0002:00005a4c       ??_C@_0M@FBHLBFCC@disableCvar?$AA@ 3005da4c     ui_shared.obj
 0002:00005a58       ??_C@_08KBIDCBHN@cvarTest?$AA@ 3005da58     ui_shared.obj
 0002:00005a64       ??_C@_0L@LCDHKNEJ@enableCvar?$AA@ 3005da64     ui_shared.obj
 0002:00005a70       ??_C@_0O@DACAJCLK@ownerdrawFlag?$AA@ 3005da70     ui_shared.obj
 0002:00005a80       ??_C@_0O@BGFKBLBI@addColorRange?$AA@ 3005da80     ui_shared.obj
 0002:00005a90       ??_C@_0O@IKNDJMDK@cvarFloatList?$AA@ 3005da90     ui_shared.obj
 0002:00005aa0       ??_C@_0M@GOKMFACI@cvarStrList?$AA@ 3005daa0     ui_shared.obj
 0002:00005aac       ??_C@_09CGGKHKAP@cvarFloat?$AA@ 3005daac     ui_shared.obj
 0002:00005ab8       ??_C@_0L@NOGKCHFE@focusSound?$AA@ 3005dab8     ui_shared.obj
 0002:00005ac4       ??_C@_0O@HPCOAMJM@maxPaintChars?$AA@ 3005dac4     ui_shared.obj
 0002:00005ad4       ??_C@_08IHGPPBOI@maxChars?$AA@ 3005dad4     ui_shared.obj
 0002:00005ae0       ??_C@_04PNAHEAFM@cvar?$AA@ 3005dae0     ui_shared.obj
 0002:00005ae8       ??_C@_07BELCMIIP@special?$AA@ 3005dae8     ui_shared.obj
 0002:00005af0       ??_C@_06DDLLCOJG@action?$AA@ 3005daf0     ui_shared.obj
 0002:00005af8       ??_C@_0O@GFPABKKP@mouseExitText?$AA@ 3005daf8     ui_shared.obj
 0002:00005b08       ??_C@_0P@BCEPHLNB@mouseEnterText?$AA@ 3005db08     ui_shared.obj
 0002:00005b18       ??_C@_09OIHCIOIA@mouseExit?$AA@ 3005db18     ui_shared.obj
 0002:00005b24       ??_C@_0L@KAGOMOPN@mouseEnter?$AA@ 3005db24     ui_shared.obj
 0002:00005b30       ??_C@_0L@LMAJDKOE@leaveFocus?$AA@ 3005db30     ui_shared.obj
 0002:00005b3c       ??_C@_07PFEHHELH@onFocus?$AA@ 3005db3c     ui_shared.obj
 0002:00005b44       ??_C@_0L@EGCKCJDC@background?$AA@ 3005db44     ui_shared.obj
 0002:00005b50       ??_C@_0N@LGJOCBPD@outlinecolor?$AA@ 3005db50     ui_shared.obj
 0002:00005b60       ??_C@_0M@CJNAABJD@bordercolor?$AA@ 3005db60     ui_shared.obj
 0002:00005b6c       ??_C@_09MONNBKNO@forecolor?$AA@ 3005db6c     ui_shared.obj
 0002:00005b78       ??_C@_09OPNKCLNO@backcolor?$AA@ 3005db78     ui_shared.obj
 0002:00005b84       ??_C@_09FMCFHDEN@textstyle?$AA@ 3005db84     ui_shared.obj
 0002:00005b90       ??_C@_09BLEIEHKP@textscale?$AA@ 3005db90     ui_shared.obj
 0002:00005b9c       ??_C@_0L@FCLMCIJC@textaligny?$AA@ 3005db9c     ui_shared.obj
 0002:00005ba8       ??_C@_0L@ELKHBJND@textalignx?$AA@ 3005dba8     ui_shared.obj
 0002:00005bb4       ??_C@_09PNBDGNCL@textalign?$AA@ 3005dbb4     ui_shared.obj
 0002:00005bc0       ??_C@_05CBJPDLOK@align?$AA@ 3005dbc0     ui_shared.obj
 0002:00005bc8       ??_C@_09HGLBOMNF@ownerdraw?$AA@ 3005dbc8     ui_shared.obj
 0002:00005bd4       ??_C@_07DPDAEJMK@visible?$AA@ 3005dbd4     ui_shared.obj
 0002:00005bdc       ??_C@_0L@BAAMOEHP@bordersize?$AA@ 3005dbdc     ui_shared.obj
 0002:00005be8       ??_C@_06ODFLABIG@border?$AA@ 3005dbe8     ui_shared.obj
 0002:00005bf0       ??_C@_07HIFEPIJN@columns?$AA@ 3005dbf0     ui_shared.obj
 0002:00005bf8       ??_C@_0M@HBNIAHKL@elementtype?$AA@ 3005dbf8     ui_shared.obj
 0002:00005c04       ??_C@_06GEEPENGB@feeder?$AA@ 3005dc04     ui_shared.obj
 0002:00005c0c       ??_C@_0O@MNJDKOBB@elementheight?$AA@ 3005dc0c     ui_shared.obj
 0002:00005c1c       ??_C@_0N@MILKKPGL@elementwidth?$AA@ 3005dc1c     ui_shared.obj
 0002:00005c2c       ??_C@_04GPMDFGEJ@type?$AA@ 3005dc2c     ui_shared.obj
 0002:00005c34       ??_C@_0BB@EIBMEDHI@horizontalscroll?$AA@ 3005dc34     ui_shared.obj
 0002:00005c48       ??_C@_0M@HHKOOJO@autowrapped?$AA@ 3005dc48     ui_shared.obj
 0002:00005c54       ??_C@_07FJHHECNJ@wrapped?$AA@ 3005dc54     ui_shared.obj
 0002:00005c5c       ??_C@_0O@FDEIBLKE@notselectable?$AA@ 3005dc5c     ui_shared.obj
 0002:00005c6c       ??_C@_0L@GFEIECKE@decoration?$AA@ 3005dc6c     ui_shared.obj
 0002:00005c78       ??_C@_05IAKJCFIM@style?$AA@ 3005dc78     ui_shared.obj
 0002:00005c80       ??_C@_04LHPFHFPH@rect?$AA@ 3005dc80     ui_shared.obj
 0002:00005c88       ??_C@_0M@HHMGANAM@model_angle?$AA@ 3005dc88     ui_shared.obj
 0002:00005c94       ??_C@_0P@NOKHMHPD@model_rotation?$AA@ 3005dc94     ui_shared.obj
 0002:00005ca4       ??_C@_0L@NMCIJLPA@model_fovy?$AA@ 3005dca4     ui_shared.obj
 0002:00005cb0       ??_C@_0L@MFDDKKLB@model_fovx?$AA@ 3005dcb0     ui_shared.obj
 0002:00005cbc       ??_C@_0N@LHLPLFLG@model_origin?$AA@ 3005dcbc     ui_shared.obj
 0002:00005ccc       ??_C@_0N@HLFJAKEA@asset_shader?$AA@ 3005dccc     ui_shared.obj
 0002:00005cdc       ??_C@_0M@DKAIGAGN@asset_model?$AA@ 3005dcdc     ui_shared.obj
 0002:00005ce8       ??_C@_05MGJOOGAJ@group?$AA@ 3005dce8     ui_shared.obj
 0002:00005cf0       ??_C@_04CIMGMMMG@text?$AA@ 3005dcf0     ui_shared.obj
 0002:00005cf8       ??_C@_04MEMAJGDJ@name?$AA@ 3005dcf8     ui_shared.obj
 0002:00005d00       ??_C@_0M@HDIJIOFC@cl_freelook?$AA@ 3005dd00     ui_shared.obj
 0002:00005d0c       ??_C@_08BEMLPELN@m_filter?$AA@ 3005dd0c     ui_shared.obj
 0002:00005d18       ??_C@_0O@CDIHIFMG@joy_threshold?$AA@ 3005dd18     ui_shared.obj
 0002:00005d28       ??_C@_0M@MJEIGFNL@in_joystick?$AA@ 3005dd28     ui_shared.obj
 0002:00005d34       ??_C@_0M@JFLMCFNC@sensitivity?$AA@ 3005dd34     ui_shared.obj
 0002:00005d40       ??_C@_07JIEGLHEC@m_pitch?$AA@ 3005dd40     ui_shared.obj
 0002:00005d48       ??_C@_06HFMKGFEH@cl_run?$AA@ 3005dd48     ui_shared.obj
 0002:00005d54       ??_C@_0N@NFNJCLFL@messagemode4?$AA@ 3005dd54     ui_shared.obj
 0002:00005d64       ??_C@_0N@JKJILNJM@messagemode3?$AA@ 3005dd64     ui_shared.obj
 0002:00005d74       ??_C@_0N@IDIDIMNN@messagemode2?$AA@ 3005dd74     ui_shared.obj
 0002:00005d84       ??_C@_0M@JINOELJH@messagemode?$AA@ 3005dd84     ui_shared.obj
 0002:00005d90       ??_C@_0L@JEAJCAAH@scoresDown?$AA@ 3005dd90     ui_shared.obj
 0002:00005d9c       ??_C@_08NILIEBDN@scoresUp?$AA@ 3005dd9c     ui_shared.obj
 0002:00005da8       ??_C@_0O@BNPKDDEF@tauntGauntlet?$AA@ 3005dda8     ui_shared.obj
 0002:00005db8       ??_C@_0BB@DHLHLJJP@tauntDeathInsult?$AA@ 3005ddb8     ui_shared.obj
 0002:00005dcc       ??_C@_0L@OFGCNOGN@tauntTaunt?$AA@ 3005ddcc     ui_shared.obj
 0002:00005dd8       ??_C@_0M@FHJJKLIB@tauntPraise?$AA@ 3005ddd8     ui_shared.obj
 0002:00005de4       ??_C@_0BA@LAKLAIKA@tauntKillInsult?$AA@ 3005dde4     ui_shared.obj
 0002:00005df4       ??_C@_0M@HEJOPHDA@taskSuicide?$AA@ 3005ddf4     ui_shared.obj
 0002:00005e00       ??_C@_0M@NPBCACOK@taskOwnFlag?$AA@ 3005de00     ui_shared.obj
 0002:00005e0c       ??_C@_0L@JKHNIMGE@taskEscort?$AA@ 3005de0c     ui_shared.obj
 0002:00005e18       ??_C@_0N@DNLIECKN@taskRetrieve?$AA@ 3005de18     ui_shared.obj
 0002:00005e28       ??_C@_0L@HALHAPMG@taskFollow?$AA@ 3005de28     ui_shared.obj
 0002:00005e34       ??_C@_08OELCHPPI@taskCamp?$AA@ 3005de34     ui_shared.obj
 0002:00005e40       ??_C@_0L@HNDPADH@taskPatrol?$AA@ 3005de40     ui_shared.obj
 0002:00005e4c       ??_C@_0M@JPJGJJPF@taskDefense?$AA@ 3005de4c     ui_shared.obj
 0002:00005e58       ??_C@_0M@PDBEJPDO@taskOffense?$AA@ 3005de58     ui_shared.obj
 0002:00005e64       ??_C@_09PEFBKJOE@denyOrder?$AA@ 3005de64     ui_shared.obj
 0002:00005e70       ??_C@_0N@KJLGMAFH@confirmOrder?$AA@ 3005de70     ui_shared.obj
 0002:00005e80       ??_C@_09DIHAGAEB@nextOrder?$AA@ 3005de80     ui_shared.obj
 0002:00005e8c       ??_C@_0P@GJIGAACM@nextTeamMember?$AA@ 3005de8c     ui_shared.obj
 0002:00005e9c       ??_C@_0P@NMPIEJIB@prevTeamMember?$AA@ 3005de9c     ui_shared.obj
 0002:00005eac       ??_C@_08DDALFEDF@?$CLbutton4?$AA@ 3005deac     ui_shared.obj
 0002:00005eb8       ??_C@_08HMEKMCPC@?$CLbutton3?$AA@ 3005deb8     ui_shared.obj
 0002:00005ec4       ??_C@_07MAODEHGM@?$CLattack?$AA@ 3005dec4     ui_shared.obj
 0002:00005ecc       ??_C@_09EAGNIMIH@weapon?513?$AA@ 3005decc     ui_shared.obj
 0002:00005ed8       ??_C@_09FJHGLNMG@weapon?512?$AA@ 3005ded8     ui_shared.obj
 0002:00005ee4       ??_C@_09HCFLOOAF@weapon?511?$AA@ 3005dee4     ui_shared.obj
 0002:00005ef0       ??_C@_09GLEANPEE@weapon?510?$AA@ 3005def0     ui_shared.obj
 0002:00005efc       ??_C@_08MFIOAKPE@weapon?59?$AA@ 3005defc     ui_shared.obj
 0002:00005f08       ??_C@_08NMJFDLLF@weapon?58?$AA@ 3005df08     ui_shared.obj
 0002:00005f14       ??_C@_08FLANCHHK@weapon?57?$AA@ 3005df14     ui_shared.obj
 0002:00005f20       ??_C@_08ECBGBGDL@weapon?56?$AA@ 3005df20     ui_shared.obj
 0002:00005f2c       ??_C@_08GJDLEFPI@weapon?55?$AA@ 3005df2c     ui_shared.obj
 0002:00005f38       ??_C@_08HACAHELJ@weapon?54?$AA@ 3005df38     ui_shared.obj
 0002:00005f44       ??_C@_08DPGBOCHO@weapon?53?$AA@ 3005df44     ui_shared.obj
 0002:00005f50       ??_C@_08CGHKNDDP@weapon?52?$AA@ 3005df50     ui_shared.obj
 0002:00005f5c       ??_C@_08NFHIAPM@weapon?51?$AA@ 3005df5c     ui_shared.obj
 0002:00005f68       ??_C@_0L@FHIBDANG@centerview?$AA@ 3005df68     ui_shared.obj
 0002:00005f74       ??_C@_06OBEGBCAL@?$CLmlook?$AA@ 3005df74     ui_shared.obj
 0002:00005f7c       ??_C@_09KCKOGCLI@?$CLlookdown?$AA@ 3005df7c     ui_shared.obj
 0002:00005f88       ??_C@_07BDFIGFL@?$CLlookup?$AA@ 3005df88     ui_shared.obj
 0002:00005f90       ??_C@_07CHKKNAEO@?$CLstrafe?$AA@ 3005df90     ui_shared.obj
 0002:00005f98       ??_C@_06NGIHBNMB@?$CLright?$AA@ 3005df98     ui_shared.obj
 0002:00005fa0       ??_C@_05HEGFDNLE@?$CLleft?$AA@ 3005dfa0     ui_shared.obj
 0002:00005fa8       ??_C@_09HNJJMOJG@?$CLmovedown?$AA@ 3005dfa8     ui_shared.obj
 0002:00005fb4       ??_C@_07CKGNAPCP@?$CLmoveup?$AA@ 3005dfb4     ui_shared.obj
 0002:00005fbc       ??_C@_0L@FMBJCMEG@?$CLmoveright?$AA@ 3005dfbc     ui_shared.obj
 0002:00005fc8       ??_C@_09IPJNFGKP@?$CLmoveleft?$AA@ 3005dfc8     ui_shared.obj
 0002:00005fd4       ??_C@_05IPKGNIPH@?$CLback?$AA@ 3005dfd4     ui_shared.obj
 0002:00005fdc       ??_C@_08KKEOHAPB@?$CLforward?$AA@ 3005dfdc     ui_shared.obj
 0002:00005fe8       ??_C@_06JIDIHCBO@?$CLspeed?$AA@ 3005dfe8     ui_shared.obj
 0002:00005ff0       ??_C@_08GFFBPDLD@?$CLbutton2?$AA@ 3005dff0     ui_shared.obj
 0002:00005ffc       ??_C@_05KJPHCDKJ@orbit?$AA@ 3005dffc     ui_shared.obj
 0002:00006004       ??_C@_0L@NDOCJLDE@playlooped?$AA@ 3005e004     ui_shared.obj
 0002:00006010       ??_C@_04GBHMDDO@play?$AA@  3005e010     ui_shared.obj
 0002:00006018       ??_C@_04MGEIEJAD@exec?$AA@ 3005e018     ui_shared.obj
 0002:00006020       ??_C@_07DFOFNCMO@setcvar?$AA@ 3005e020     ui_shared.obj
 0002:00006028       ??_C@_0L@KGLELNDP@transition?$AA@ 3005e028     ui_shared.obj
 0002:00006034       ??_C@_0O@DDHOJBLA@setplayerhead?$AA@ 3005e034     ui_shared.obj
 0002:00006044       ??_C@_0P@COHLPKKB@setplayermodel?$AA@ 3005e044     ui_shared.obj
 0002:00006054       ??_C@_08OKIAJKBO@setfocus?$AA@ 3005e054     ui_shared.obj
 0002:00006060       ??_C@_0N@KMLJLNON@setteamcolor?$AA@ 3005e060     ui_shared.obj
 0002:00006070       ??_C@_0N@EBBIOPHN@setitemcolor?$AA@ 3005e070     ui_shared.obj
 0002:00006080       ??_C@_0O@FOIIKEEB@setbackground?$AA@ 3005e080     ui_shared.obj
 0002:00006090       ??_C@_08FBOLLCAN@setasset?$AA@ 3005e090     ui_shared.obj
 0002:0000609c       ??_C@_05LBOHBHFK@close?$AA@ 3005e09c     ui_shared.obj
 0002:000060a4       ??_C@_0BA@JLPGECPM@conditionalopen?$AA@ 3005e0a4     ui_shared.obj
 0002:000060b4       ??_C@_04PMOCAHAA@open?$AA@ 3005e0b4     ui_shared.obj
 0002:000060bc       ??_C@_08OKIEAMBM@setcolor?$AA@ 3005e0bc     ui_shared.obj
 0002:000060c8       ??_C@_04IBOFHAPJ@hide?$AA@ 3005e0c8     ui_shared.obj
 0002:000060d0       ??_C@_04FKMICODN@show?$AA@ 3005e0d0     ui_shared.obj
 0002:000060d8       ??_C@_07BJADIKJG@fadeout?$AA@ 3005e0d8     ui_shared.obj
 0002:000060e0       ??_C@_06JFGPOFJL@fadein?$AA@ 3005e0e0     ui_shared.obj
 0002:000060e8       ??_C@_0CD@LBKPCJLM@UI_Alloc?3?5Failure?4?5Out?5of?5memory@ 3005e0e8     ui_shared.obj
 0002:0000610c       ??_C@_0DG@OMGKABNP@Memory?5Pool?5is?5?$CF?41f?$CF?$CF?5full?0?5?$CFi?5b@ 3005e10c     ui_shared.obj
 0002:00006144       __real@49800000            3005e144     ui_shared.obj
 0002:00006148       ??_C@_0DG@MABFDHIF@String?5Pool?5is?5?$CF?41f?$CF?$CF?5full?0?5?$CFi?5b@ 3005e148     ui_shared.obj
 0002:00006180       __real@48c00000            3005e180     ui_shared.obj
 0002:00006184       ??_C@_0BC@DKLFONDB@?9?9?9?9?9?9?9?9?9?9?9?9?9?9?9?9?6?$AA@ 3005e184     ui_shared.obj
 0002:00006198       ??_C@_0BJ@GAPDFKFM@Memory?1String?5Pool?5Info?6?$AA@ 3005e198     ui_shared.obj
 0002:000061b4       ??_C@_0BM@DJGMFAMK@?$FO3WARNING?3?5?$CFs?0?5line?5?$CFd?3?5?$CFs?6?$AA@ 3005e1b4     ui_shared.obj
 0002:000061d0       ??_C@_0BK@OKFEFFGN@?$FO1ERROR?3?5?$CFs?0?5line?5?$CFd?3?5?$CFs?6?$AA@ 3005e1d0     ui_shared.obj
 0002:000061ec       ??_C@_0BN@CKJPOGNB@expected?5float?5but?5found?5?$CFs?6?$AA@ 3005e1ec     ui_shared.obj
 0002:0000620c       ??_C@_0BP@FLADEANJ@expected?5integer?5but?5found?5?$CFs?6?$AA@ 3005e20c     ui_shared.obj
 0002:0000622c       ??_C@_01CLKCMJKC@?5?$AA@   3005e22c     ui_shared.obj
 0002:00006230       ??_C@_04OEDFLLKD@?$CC?$CFs?$CC?$AA@ 3005e230     ui_shared.obj
 0002:00006238       ??_C@_05LKKGNBCL@?$CFs?5?$DL?5?$AA@ 3005e238     ui_shared.obj
 0002:00006240       __real@4058000000000000    3005e240     ui_shared.obj
 0002:00006248       ??_C@_0BI@MLGEDDNA@slider?5handle?5key?5exit?6?$AA@ 3005e248     ui_shared.obj
 0002:00006260       ??_C@_0M@FHKEBODE@screenshot?6?$AA@ 3005e260     ui_shared.obj
 0002:0000626c       ??_C@_02JINPPBEP@No?$AA@   3005e26c     ui_shared.obj
 0002:00006270       ??_C@_03CCLAEDDF@Yes?$AA@  3005e270     ui_shared.obj
 0002:00006274       ??_C@_0M@LMHCNBPD@in_restart?6?$AA@ 3005e274     ui_shared.obj
 0002:00006280       ??_C@_03BBKEAIF@?$DP?$DP?$DP?$AA@ 3005e280     ui_shared.obj
 0002:00006284       ??_C@_04FJKIFICP@?5or?5?$AA@ 3005e284     ui_shared.obj
 0002:0000628c       ??_C@_05DJCKAPIL@FIXME?$AA@ 3005e28c     ui_shared.obj
 0002:00006294       __real@3f4ccccd            3005e294     ui_shared.obj
 0002:00006298       __real@402e000000000000    3005e298     ui_shared.obj
 0002:000062a0       ??_C@_0BO@GKGLOPGG@end?5of?5file?5inside?5menu?5item?6?$AA@ 3005e2a0     ui_shared.obj
 0002:000062c0       ??_C@_0CE@OIGKMGKE@couldn?8t?5parse?5menu?5item?5keyword@ 3005e2c0     ui_shared.obj
 0002:000062e4       ??_C@_0BN@JHFMAPJL@unknown?5menu?5item?5keyword?5?$CFs?$AA@ 3005e2e4     ui_shared.obj
 0002:00006304       ??_C@_04GHJNJNPO@main?$AA@ 3005e304     ui_shared.obj
 0002:0000630c       ??_C@_0BP@HJCDHJDP@couldn?8t?5parse?5menu?5keyword?5?$CFs?$AA@ 3005e30c     ui_shared.obj
 0002:0000632c       ??_C@_0BI@PALCAEGK@unknown?5menu?5keyword?5?$CFs?$AA@ 3005e32c     ui_shared.obj
 0002:00006344       ??_C@_0BJ@MPIMCBOA@end?5of?5file?5inside?5menu?6?$AA@ 3005e344     ui_shared.obj
 0002:00006360       ??_C@_07KLAFGBNN@fps?3?5?$CFf?$AA@ 3005e360     ui_shared.obj
 0002:00006368       ??_C@_0P@NFGNABCI@string?5?$CB?$DN?5NULL?$AA@ 3005e368     LIBCMTD:vsprintf.obj
 0002:00006378       ??_C@_0L@MDILGHEC@vsprintf?4c?$AA@ 3005e378     LIBCMTD:vsprintf.obj
 0002:00006384       ??_C@_0P@NHGFNCDP@format?5?$CB?$DN?5NULL?$AA@ 3005e384     LIBCMTD:vsprintf.obj
 0002:000063f0       ??_C@_02PHMGELLB@?6?6?$AA@ 3005e3f0     LIBCMTD:assert.obj
 0002:000063f4       ??_C@_01EEMJAFIK@?6?$AA@   3005e3f4     LIBCMTD:assert.obj
 0002:000063f8       ??_C@_03KHICJKCI@?4?4?4?$AA@ 3005e3f8     LIBCMTD:assert.obj
 0002:000063fc       ??_C@_0CF@GOGNBNAK@Microsoft?5Visual?5C?$CL?$CL?5Runtime?5Lib@ 3005e3fc     LIBCMTD:assert.obj
 0002:00006424       ??_C@_0DN@EBBNMLME@?$CIPress?5Retry?5to?5debug?5the?5applic@ 3005e424     LIBCMTD:assert.obj
 0002:00006468       ??_C@_0HA@OJHAGA@For?5information?5on?5how?5your?5prog@ 3005e468     LIBCMTD:assert.obj
 0002:000064d8       ??_C@_0N@MEECIJGN@Expression?3?5?$AA@ 3005e4d8     LIBCMTD:assert.obj
 0002:000064e8       ??_C@_06FIEBOLOH@Line?3?5?$AA@ 3005e4e8     LIBCMTD:assert.obj
 0002:000064f0       ??_C@_06IGPBOHMJ@File?3?5?$AA@ 3005e4f0     LIBCMTD:assert.obj
 0002:000064f8       ??_C@_0BH@DNAGHKFM@?$DMprogram?5name?5unknown?$DO?$AA@ 3005e4f8     LIBCMTD:assert.obj
 0002:00006510       ??_C@_09KLGCKDOD@Program?3?5?$AA@ 3005e510     LIBCMTD:assert.obj
 0002:0000651c       ??_C@_0BC@LAIDCHCH@Assertion?5failed?$CB?$AA@ 3005e51c     LIBCMTD:assert.obj
 0002:00006530       ??_C@_09IFKEODFF@dllcrt0?4c?$AA@ 3005e530     LIBCMTD:dllcrt0.obj
 0002:00006550       __real@4150017ec0000000    3005e550     LIBCMTD:testfdiv.obj
 0002:00006558       __real@4147ffff80000000    3005e558     LIBCMTD:testfdiv.obj
 0002:00006560       ??_C@_0BK@NHEOCAHP@IsProcessorFeaturePresent?$AA@ 3005e560     LIBCMTD:testfdiv.obj
 0002:0000657c       ??_C@_08CPNIBGIE@KERNEL32?$AA@ 3005e57c     LIBCMTD:testfdiv.obj
 0002:00006588       ??_C@_05KLBDPFGC@e?$CL000?$AA@ 3005e588     LIBCMTD:cvt.obj
 0002:00006598       __DEFAULT_CW_in_mem        3005e598     LIBCMTD:common.obj
 0002:0000659a       __pi_by_2_to_61            3005e59a     LIBCMTD:common.obj
 0002:000065d4       ??_C@_0L@KDOEJCKC@_nextafter?$AA@ 3005e5d4     LIBCMTD:fpexcept.obj
 0002:000065e0       ??_C@_05JGDBENOH@_logb?$AA@ 3005e5e0     LIBCMTD:fpexcept.obj
 0002:000065e8       ??_C@_03ONILCKOB@_yn?$AA@  3005e5e8     LIBCMTD:fpexcept.obj
 0002:000065ec       ??_C@_03NAKIGLHK@_y1?$AA@  3005e5ec     LIBCMTD:fpexcept.obj
 0002:000065f0       ??_C@_03MJLDFKDL@_y0?$AA@  3005e5f0     LIBCMTD:fpexcept.obj
 0002:000065f4       ??_C@_05GKKHEGJL@frexp?$AA@ 3005e5f4     LIBCMTD:fpexcept.obj
 0002:000065fc       ??_C@_04KEPJIHGP@fmod?$AA@ 3005e5fc     LIBCMTD:fpexcept.obj
 0002:00006604       ??_C@_06MEIMCGCF@_hypot?$AA@ 3005e604     LIBCMTD:fpexcept.obj
 0002:0000660c       ??_C@_05KBKMEMPO@_cabs?$AA@ 3005e60c     LIBCMTD:fpexcept.obj
 0002:00006614       ??_C@_05CEJMAHNP@ldexp?$AA@ 3005e614     LIBCMTD:fpexcept.obj
 0002:0000661c       ??_C@_04EHEDPDJG@modf?$AA@ 3005e61c     LIBCMTD:fpexcept.obj
 0002:00006624       ??_C@_04ODHECPBC@fabs?$AA@ 3005e624     LIBCMTD:fpexcept.obj
 0002:0000662c       ??_C@_05PBJFFIGL@floor?$AA@ 3005e62c     LIBCMTD:fpexcept.obj
 0002:00006634       ??_C@_04GFPJNGEK@ceil?$AA@ 3005e634     LIBCMTD:fpexcept.obj
 0002:0000663c       ??_C@_03IIINPABG@tan?$AA@  3005e63c     LIBCMTD:fpexcept.obj
 0002:00006640       ??_C@_03LALBNOCG@cos?$AA@  3005e640     LIBCMTD:fpexcept.obj
 0002:00006644       ??_C@_03BLEJJJBH@sin?$AA@  3005e644     LIBCMTD:fpexcept.obj
 0002:00006648       ??_C@_04EIAKFFMI@sqrt?$AA@ 3005e648     LIBCMTD:fpexcept.obj
 0002:00006650       ??_C@_05KNGEOGJB@atan2?$AA@ 3005e650     LIBCMTD:fpexcept.obj
 0002:00006658       ??_C@_04MLLJIGOK@atan?$AA@ 3005e658     LIBCMTD:fpexcept.obj
 0002:00006660       ??_C@_04PDIFKINK@acos?$AA@ 3005e660     LIBCMTD:fpexcept.obj
 0002:00006668       ??_C@_04FIHNOPOL@asin?$AA@ 3005e668     LIBCMTD:fpexcept.obj
 0002:00006670       ??_C@_04FJHINJAO@tanh?$AA@ 3005e670     LIBCMTD:fpexcept.obj
 0002:00006678       ??_C@_04HPJJNFIM@cosh?$AA@ 3005e678     LIBCMTD:fpexcept.obj
 0002:00006680       ??_C@_04COOMCNPB@sinh?$AA@ 3005e680     LIBCMTD:fpexcept.obj
 0002:00006688       ??_C@_05HGHHAHAP@log10?$AA@ 3005e688     LIBCMTD:fpexcept.obj
 0002:00006690       ??_C@_03MGHMBJCF@log?$AA@  3005e690     LIBCMTD:fpexcept.obj
 0002:00006694       ??_C@_03JGHBODFD@pow?$AA@  3005e694     LIBCMTD:fpexcept.obj
 0002:00006698       ??_C@_03KHJOGHMM@exp?$AA@  3005e698     LIBCMTD:fpexcept.obj
 0002:0000669c       ??_C@_09BLOOPMDK@isctype?4c?$AA@ 3005e69c     LIBCMTD:isctype.obj
 0002:000066a8       ??_C@_0BJ@IAKBGELC@?$CIunsigned?$CJ?$CIc?5?$CL?51?$CJ?5?$DM?$DN?5256?$AA@ 3005e6a8     LIBCMTD:isctype.obj
 0002:00006848       ??_C@_07LCBHPJJN@LC_TIME?$AA@ 3005e848     LIBCMTD:setlocal.obj
 0002:00006850       ??_C@_0L@DLHIECNL@LC_NUMERIC?$AA@ 3005e850     LIBCMTD:setlocal.obj
 0002:0000685c       ??_C@_0M@MIENIKLA@LC_MONETARY?$AA@ 3005e85c     LIBCMTD:setlocal.obj
 0002:00006868       ??_C@_08EADHIDAD@LC_CTYPE?$AA@ 3005e868     LIBCMTD:setlocal.obj
 0002:00006874       ??_C@_0L@KFJHEKIK@LC_COLLATE?$AA@ 3005e874     LIBCMTD:setlocal.obj
 0002:00006880       ??_C@_06NEFDFEKB@LC_ALL?$AA@ 3005e880     LIBCMTD:setlocal.obj
 0002:00006894       ??_C@_0L@LEECJGMI@setlocal?4c?$AA@ 3005e894     LIBCMTD:setlocal.obj
 0002:000068ac       ??_C@_01ICJEACDI@?$DL?$AA@ 3005e8ac     LIBCMTD:setlocal.obj
 0002:000068b0       ??_C@_02BALPLPBG@?$DN?$DL?$AA@ 3005e8b0     LIBCMTD:setlocal.obj
 0002:000068b4       ??_C@_03EGDHDPFD@_?4?0?$AA@ 3005e8b4     LIBCMTD:setlocal.obj
 0002:000068b8       ??_C@_01LFCBOECM@?4?$AA@   3005e8b8     LIBCMTD:setlocal.obj
 0002:000068bc       ??_C@_01IDAFKMJL@_?$AA@    3005e8bc     LIBCMTD:setlocal.obj
 0002:000068c0       ??_C@_0L@JKCACIOJ@tidtable?4c?$AA@ 3005e8c0     LIBCMTD:tidtable.obj
 0002:000068cc       ??_C@_07PEJMOBNF@FlsFree?$AA@ 3005e8cc     LIBCMTD:tidtable.obj
 0002:000068d4       ??_C@_0M@JCPCPOEF@FlsSetValue?$AA@ 3005e8d4     LIBCMTD:tidtable.obj
 0002:000068e0       ??_C@_0M@GDNOONDI@FlsGetValue?$AA@ 3005e8e0     LIBCMTD:tidtable.obj
 0002:000068ec       ??_C@_08KNHFBNJ@FlsAlloc?$AA@ 3005e8ec     LIBCMTD:tidtable.obj
 0002:000068f8       ??_C@_0N@MDJJJHMB@kernel32?4dll?$AA@ 3005e8f8     LIBCMTD:tidtable.obj
 0002:00006920       ??_C@_0DP@FICHPIPH@?$CI?$CCinconsistent?5IOB?5fields?$CC?0?5stre@ 3005e920     LIBCMTD:_flsbuf.obj
 0002:00006960       ??_C@_09DHJHPHJP@_flsbuf?4c?$AA@ 3005e960     LIBCMTD:_flsbuf.obj
 0002:0000696c       ??_C@_0M@CMNAFCJK@str?5?$CB?$DN?5NULL?$AA@ 3005e96c     LIBCMTD:_flsbuf.obj
 0002:00006978       ___lookuptable             3005e978     LIBCMTD:output.obj
 0002:000069d4       ??_C@_1O@CEDCILHN@?$AA?$CI?$AAn?$AAu?$AAl?$AAl?$AA?$CJ?$AA?$AA@ 3005e9d4     LIBCMTD:output.obj
 0002:000069e4       ??_C@_06OJHGLDPL@?$CInull?$CJ?$AA@ 3005e9e4     LIBCMTD:output.obj
 0002:000069ec       ??_C@_08MEPFMIND@output?4c?$AA@ 3005e9ec     LIBCMTD:output.obj
 0002:000069f8       ??_C@_0P@LGFCLPDP@ch?5?$CB?$DN?5_T?$CI?8?20?8?$CJ?$AA@ 3005e9f8     LIBCMTD:output.obj
 0002:00006a08       ??_C@_0BB@NAGLCMLI@Assertion?5Failed?$AA@ 3005ea08     LIBCMTD:dbgrpt.obj
 0002:00006a1c       ??_C@_05NAOIJFC@Error?$AA@ 3005ea1c     LIBCMTD:dbgrpt.obj
 0002:00006a24       ??_C@_07KGMMFLDN@Warning?$AA@ 3005ea24     LIBCMTD:dbgrpt.obj
 0002:00006a2c       ??_C@_08ODMAMGBE@dbgrpt?4c?$AA@ 3005ea2c     LIBCMTD:dbgrpt.obj
 0002:00006a44       ??_C@_0M@IPILFDFN@?$CFs?$CI?$CFd?$CJ?5?3?5?$CFs?$AA@ 3005ea44     LIBCMTD:dbgrpt.obj
 0002:00006a50       ??_C@_01LIIJDEN@?$AN?$AA@  3005ea50     LIBCMTD:dbgrpt.obj
 0002:00006a54       ??_C@_0BD@CAENFOHP@Assertion?5failed?3?5?$AA@ 3005ea54     LIBCMTD:dbgrpt.obj
 0002:00006a68       ??_C@_0CL@EACFGMNB@_CrtDbgReport?3?5String?5too?5long?5o@ 3005ea68     LIBCMTD:dbgrpt.obj
 0002:00006a94       ??_C@_0DC@HLHDIIKH@Second?5Chance?5Assertion?5Failed?3?5@ 3005ea94     LIBCMTD:dbgrpt.obj
 0002:00006ac8       ??_C@_09FOPFMPEJ@wsprintfA?$AA@ 3005eac8     LIBCMTD:dbgrpt.obj
 0002:00006ad4       ??_C@_0L@GMPLCCII@user32?4dll?$AA@ 3005ead4     LIBCMTD:dbgrpt.obj
 0002:00006aec       ??_C@_0CD@EBCGLDDL@Microsoft?5Visual?5C?$CL?$CL?5Debug?5Libra@ 3005eaec     LIBCMTD:dbgrpt.obj
 0002:00006b10       ??_C@_0FD@IIKNDPHJ@Debug?5?$CFs?$CB?6?6Program?3?5?$CFs?$CFs?$CFs?$CFs?$CFs?$CFs@ 3005eb10     LIBCMTD:dbgrpt.obj
 0002:00006b64       ??_C@_09OFBFHMBK@?6Module?3?5?$AA@ 3005eb64     LIBCMTD:dbgrpt.obj
 0002:00006b70       ??_C@_07OPHPPLBG@?6File?3?5?$AA@ 3005eb70     LIBCMTD:dbgrpt.obj
 0002:00006b78       ??_C@_07DBMPPHDI@?6Line?3?5?$AA@ 3005eb78     LIBCMTD:dbgrpt.obj
 0002:00006b80       ??_C@_0HD@GNBNFCCL@?6?6For?5information?5on?5how?5your?5pr@ 3005eb80     LIBCMTD:dbgrpt.obj
 0002:00006bf4       ??_C@_0BG@IHOEIIEJ@szUserMessage?5?$CB?$DN?5NULL?$AA@ 3005ebf4     LIBCMTD:dbgrpt.obj
 0002:00006c78       ??_C@_05EOHGHCHD@exp10?$AA@ 3005ec78     LIBCMTD:libm_error.obj
 0002:00006c80       ??_C@_04HPAFEEIN@exp2?$AA@ 3005ec80     LIBCMTD:libm_error.obj
 0002:00006c88       ??_C@_04KGLCPMCP@log2?$AA@ 3005ec88     LIBCMTD:libm_error.obj
 0002:00006c90       ??_C@_0N@FFJGBINN@AuthenticAMD?$AA@ 3005ec90     LIBCMTD:cpu_disp.obj
 0002:00006cec       ??_C@_0P@MIGLKIOC@CorExitProcess?$AA@ 3005ecec     LIBCMTD:crt0dat.obj
 0002:00006cfc       ??_C@_0M@MBOPBNBK@mscoree?4dll?$AA@ 3005ecfc     LIBCMTD:crt0dat.obj
 0002:00006d08       ??_C@_08FKHPDPAC@winsig?4c?$AA@ 3005ed08     LIBCMTD:winsig.obj
 0002:00006d44       ??_C@_0BI@DFKBFLJE@GetProcessWindowStation?$AA@ 3005ed44     LIBCMTD:crtmbox.obj
 0002:00006d5c       ??_C@_0BK@CIDNPOGP@GetUserObjectInformationA?$AA@ 3005ed5c     LIBCMTD:crtmbox.obj
 0002:00006d78       ??_C@_0BD@HHGDFDBJ@GetLastActivePopup?$AA@ 3005ed78     LIBCMTD:crtmbox.obj
 0002:00006d8c       ??_C@_0BA@HNOPNCHB@GetActiveWindow?$AA@ 3005ed8c     LIBCMTD:crtmbox.obj
 0002:00006d9c       ??_C@_0M@CHKKJDAI@MessageBoxA?$AA@ 3005ed9c     LIBCMTD:crtmbox.obj
 0002:00006dd0       ??_C@_09JMJGGMME@fprintf?4c?$AA@ 3005edd0     LIBCMTD:fprintf.obj
 0002:00006dec       ??_C@_09KGBNCNDN@setvbuf?4c?$AA@ 3005edec     LIBCMTD:setvbuf.obj
 0002:00006e04       ??_C@_07PNHPCIEC@_file?4c?$AA@ 3005ee04     LIBCMTD:_file.obj
 0002:00006e1c       ??_C@_07FEAFKIIG@a_map?4c?$AA@ 3005ee1c     LIBCMTD:a_map.obj
 0002:00006e24       ??_C@_13NOLLCAOD@?$AA?$AA?$AA?$AA@ 3005ee24     LIBCMTD:a_map.obj
 0002:00006e4c       ??_C@_06PJIGMIJB@Client?$AA@ 3005ee4c     LIBCMTD:dbgheap.obj
 0002:00006e54       ??_C@_06KMEJCCGM@Ignore?$AA@ 3005ee54     LIBCMTD:dbgheap.obj
 0002:00006e5c       ??_C@_03OGPFLFLO@CRT?$AA@  3005ee5c     LIBCMTD:dbgheap.obj
 0002:00006e60       ??_C@_06EFAGIKOH@Normal?$AA@ 3005ee60     LIBCMTD:dbgheap.obj
 0002:00006e68       ??_C@_04HJMOFLDF@Free?$AA@ 3005ee68     LIBCMTD:dbgheap.obj
 0002:00006e7c       ??_C@_0DC@JEMAGEKG@Error?3?5memory?5allocation?3?5bad?5me@ 3005ee7c     LIBCMTD:dbgheap.obj
 0002:00006eb0       ??_C@_0CF@BICKFLAF@Invalid?5allocation?5size?3?5?$CFIu?5byt@ 3005eeb0     LIBCMTD:dbgheap.obj
 0002:00006ed8       ??_C@_0CB@CCLOLAHO@Client?5hook?5allocation?5failure?4?6@ 3005eed8     LIBCMTD:dbgheap.obj
 0002:00006efc       ??_C@_0DF@BBEGIFEK@Client?5hook?5allocation?5failure?5a@ 3005eefc     LIBCMTD:dbgheap.obj
 0002:00006f34       ??_C@_09DPMMACIH@dbgheap?4c?$AA@ 3005ef34     LIBCMTD:dbgheap.obj
 0002:00006f40       ??_C@_0BC@FKEPGOPH@_CrtCheckMemory?$CI?$CJ?$AA@ 3005ef40     LIBCMTD:dbgheap.obj
 0002:00006f64       ??_C@_0BK@DJDKJKNJ@_pFirstBlock?5?$DN?$DN?5pOldBlock?$AA@ 3005ef64     LIBCMTD:dbgheap.obj
 0002:00006f80       ??_C@_0BJ@PGMLBCKP@_pLastBlock?5?$DN?$DN?5pOldBlock?$AA@ 3005ef80     LIBCMTD:dbgheap.obj
 0002:00006f9c       ??_C@_0DC@LIEEBBFH@fRealloc?5?$HM?$HM?5?$CI?$CBfRealloc?5?$CG?$CG?5pNewBl@ 3005ef9c     LIBCMTD:dbgheap.obj
 0002:00006fd0       ??_C@_0EF@BKJNHFDP@pOldBlock?9?$DOnLine?5?$DN?$DN?5IGNORE_LINE?5@ 3005efd0     LIBCMTD:dbgheap.obj
 0002:00007018       ??_C@_0CC@MCCNOMLK@_CrtIsValidHeapPointer?$CIpUserData@ 3005f018     LIBCMTD:dbgheap.obj
 0002:00007040       ??_C@_0EM@LGFLMAGJ@The?5Block?5at?50x?$CFp?5was?5allocated?5@ 3005f040     LIBCMTD:dbgheap.obj
 0002:0000708c       ??_C@_0CO@KPNFNEPA@Allocation?5too?5large?5or?5negative@ 3005f08c     LIBCMTD:dbgheap.obj
 0002:000070bc       ??_C@_0CE@DOFMDOL@Client?5hook?5re?9allocation?5failur@ 3005f0bc     LIBCMTD:dbgheap.obj
 0002:000070e0       ??_C@_0DI@KKJPDPGM@Client?5hook?5re?9allocation?5failur@ 3005f0e0     LIBCMTD:dbgheap.obj
 0002:00007134       ??_C@_0BG@JDINNDDC@_pFirstBlock?5?$DN?$DN?5pHead?$AA@ 3005f134     LIBCMTD:dbgheap.obj
 0002:0000714c       ??_C@_0BF@LMGMGAEG@_pLastBlock?5?$DN?$DN?5pHead?$AA@ 3005f14c     LIBCMTD:dbgheap.obj
 0002:00007164       ??_C@_0BO@LGCGBMOH@pHead?9?$DOnBlockUse?5?$DN?$DN?5nBlockUse?$AA@ 3005f164     LIBCMTD:dbgheap.obj
 0002:00007184       ??_C@_0DN@GKKPDMLN@pHead?9?$DOnLine?5?$DN?$DN?5IGNORE_LINE?5?$CG?$CG?5p@ 3005f184     LIBCMTD:dbgheap.obj
 0002:000071c4       ??_C@_0CI@CMGHMNIC@DAMAGE?3?5after?5?$CFhs?5block?5?$CI?$CD?$CFd?$CJ?5at@ 3005f1c4     LIBCMTD:dbgheap.obj
 0002:000071ec       ??_C@_0CJ@OHOOBLKI@DAMAGE?3?5before?5?$CFhs?5block?5?$CI?$CD?$CFd?$CJ?5a@ 3005f1ec     LIBCMTD:dbgheap.obj
 0002:00007218       ??_C@_0CH@IAGMNLOM@_BLOCK_TYPE_IS_VALID?$CIpHead?9?$DOnBlo@ 3005f218     LIBCMTD:dbgheap.obj
 0002:00007240       ??_C@_0BL@KEIPLFAC@Client?5hook?5free?5failure?4?6?$AA@ 3005f240     LIBCMTD:dbgheap.obj
 0002:00007260       ??_C@_0EJ@HEIBCIMJ@The?5Block?5at?50x?$CFp?5was?5allocated?5@ 3005f260     LIBCMTD:dbgheap.obj
 0002:000072cc       ??_C@_0CI@JMLBEDHJ@?$CFhs?5located?5at?50x?$CFp?5is?5?$CFIu?5bytes@ 3005f2cc     LIBCMTD:dbgheap.obj
 0002:000072f4       ??_C@_0CA@FGFAGAOM@?$CFhs?5allocated?5at?5file?5?$CFhs?$CI?$CFd?$CJ?4?6?$AA@ 3005f2f4     LIBCMTD:dbgheap.obj
 0002:00007314       ??_C@_0CH@JKKAOBEK@DAMAGE?3?5on?5top?5of?5Free?5block?5at?5@ 3005f314     LIBCMTD:dbgheap.obj
 0002:0000733c       ??_C@_07OHKEFPKJ@DAMAGED?$AA@ 3005f33c     LIBCMTD:dbgheap.obj
 0002:00007344       ??_C@_0CL@HNNNMKMJ@_heapchk?5fails?5with?5unknown?5retu@ 3005f344     LIBCMTD:dbgheap.obj
 0002:00007370       ??_C@_0CC@MFFCHFHO@_heapchk?5fails?5with?5_HEAPBADPTR?4@ 3005f370     LIBCMTD:dbgheap.obj
 0002:00007394       ??_C@_0CC@MJGLGBDG@_heapchk?5fails?5with?5_HEAPBADEND?4@ 3005f394     LIBCMTD:dbgheap.obj
 0002:000073b8       ??_C@_0CD@CPKEAPBD@_heapchk?5fails?5with?5_HEAPBADNODE@ 3005f3b8     LIBCMTD:dbgheap.obj
 0002:000073dc       ??_C@_0CE@MKKHMBMK@_heapchk?5fails?5with?5_HEAPBADBEGI@ 3005f3dc     LIBCMTD:dbgheap.obj
 0002:0000743c       ??_C@_0CB@EAAIGELO@Bad?5memory?5block?5found?5at?50x?$CFp?4?6@ 3005f43c     LIBCMTD:dbgheap.obj
 0002:00007460       ??_C@_0CI@KDKEAJEJ@_CrtMemCheckPoint?3?5NULL?5state?5po@ 3005f460     LIBCMTD:dbgheap.obj
 0002:00007494       ??_C@_0CI@ENCLCMLG@_CrtMemDifference?3?5NULL?5state?5po@ 3005f494     LIBCMTD:dbgheap.obj
 0002:000074bc       ??_C@_0BH@GFGKJDCO@Object?5dump?5complete?4?6?$AA@ 3005f4bc     LIBCMTD:dbgheap.obj
 0002:000074d4       ??_C@_0DA@MDLBNIBM@crt?5block?5at?50x?$CFp?0?5subtype?5?$CFx?0?5?$CF@ 3005f4d4     LIBCMTD:dbgheap.obj
 0002:00007504       ??_C@_0CH@FAGDDGPN@normal?5block?5at?50x?$CFp?0?5?$CFIu?5bytes?5@ 3005f504     LIBCMTD:dbgheap.obj
 0002:0000752c       ??_C@_0DD@GHNAAKBB@client?5block?5at?50x?$CFp?0?5subtype?5?$CFx@ 3005f52c     LIBCMTD:dbgheap.obj
 0002:00007560       ??_C@_06PKLGBFGM@?$HL?$CFld?$HN?5?$AA@ 3005f560     LIBCMTD:dbgheap.obj
 0002:00007568       ??_C@_0L@JMEFFCCJ@?$CFhs?$CI?$CFd?$CJ?5?3?5?$AA@ 3005f568     LIBCMTD:dbgheap.obj
 0002:00007574       ??_C@_0BE@OIEFNFL@?$CDFile?5Error?$CD?$CI?$CFd?$CJ?5?3?5?$AA@ 3005f574     LIBCMTD:dbgheap.obj
 0002:00007588       ??_C@_0BE@KCIPKCIA@Dumping?5objects?5?9?$DO?6?$AA@ 3005f588     LIBCMTD:dbgheap.obj
 0002:000075ac       ??_C@_0BA@HJBKCELP@?5Data?3?5?$DM?$CFs?$DO?5?$CFs?6?$AA@ 3005f5ac     LIBCMTD:dbgheap.obj
 0002:000075bc       ??_C@_05MKKEDADM@?$CF?42X?5?$AA@ 3005f5bc     LIBCMTD:dbgheap.obj
 0002:000075c4       ??_C@_0BI@JBFPOEJA@Detected?5memory?5leaks?$CB?6?$AA@ 3005f5c4     LIBCMTD:dbgheap.obj
 0002:000075dc       ??_C@_0BP@DEDHGGGI@Total?5allocations?3?5?$CFId?5bytes?4?6?$AA@ 3005f5dc     LIBCMTD:dbgheap.obj
 0002:000075fc       ??_C@_0CB@BLHDAFNE@Largest?5number?5used?3?5?$CFId?5bytes?4?6@ 3005f5fc     LIBCMTD:dbgheap.obj
 0002:00007620       ??_C@_0BO@DACNIABB@?$CFId?5bytes?5in?5?$CFId?5?$CFhs?5Blocks?4?6?$AA@ 3005f620     LIBCMTD:dbgheap.obj
 0002:00007640       ??_C@_0CC@GFBJAAAH@?$CI?$CCoffset?5must?5be?5within?5size?$CC?0?50@ 3005f640     LIBCMTD:dbgheap.obj
 0002:00007664       ??_C@_0CF@PGBEDOC@?$CI?$CCalignment?5must?5be?5a?5power?5of?52@ 3005f664     LIBCMTD:dbgheap.obj
 0002:0000768c       ??_C@_0DL@PGHMMKNE@Damage?5before?50x?$CFp?5which?5was?5all@ 3005f68c     LIBCMTD:dbgheap.obj
 0002:000076c8       ??_C@_0EI@NDNJMAJK@The?5block?5at?50x?$CFp?5was?5not?5alloca@ 3005f6c8     LIBCMTD:dbgheap.obj
 0002:00007710       ??_C@_0EF@PGELACII@The?5block?5at?50x?$CFp?5was?5not?5alloca@ 3005f710     LIBCMTD:dbgheap.obj
 0002:00007758       ??_C@_08MAFBHINM@ioinit?4c?$AA@ 3005f758     LIBCMTD:ioinit.obj
 0002:00007764       ??_C@_09HCDLHOJP@stdenvp?4c?$AA@ 3005f764     LIBCMTD:stdenvp.obj
 0002:00007770       ??_C@_09IKILHJIC@stdargv?4c?$AA@ 3005f770     LIBCMTD:stdargv.obj
 0002:0000777c       ??_C@_07BPGNOCOG@a_env?4c?$AA@ 3005f77c     LIBCMTD:a_env.obj
 0002:000077a4       ??_C@_0P@GGKDKEEG@runtime?5error?5?$AA@ 3005f7a4     LIBCMTD:crt0msg.obj
 0002:000077b4       ??_C@_02PCIJFNDE@?$AN?6?$AA@ 3005f7b4     LIBCMTD:crt0msg.obj
 0002:000077b8       ??_C@_0O@MJNIPGOH@TLOSS?5error?$AN?6?$AA@ 3005f7b8     LIBCMTD:crt0msg.obj
 0002:000077c8       ??_C@_0N@BONNPDHF@SING?5error?$AN?6?$AA@ 3005f7c8     LIBCMTD:crt0msg.obj
 0002:000077d8       ??_C@_0P@MBDAJNE@DOMAIN?5error?$AN?6?$AA@ 3005f7d8     LIBCMTD:crt0msg.obj
 0002:000077e8       ??_C@_0KC@BDDGGBEJ@R6029?$AN?6?9?5This?5application?5cannot@ 3005f7e8     LIBCMTD:crt0msg.obj
 0002:0000788c       ??_C@_0CF@KJDAIALP@R6028?$AN?6?9?5unable?5to?5initialize?5he@ 3005f88c     LIBCMTD:crt0msg.obj
 0002:000078b4       ??_C@_0DF@GAKBPDFP@R6027?$AN?6?9?5not?5enough?5space?5for?5lo@ 3005f8b4     LIBCMTD:crt0msg.obj
 0002:000078ec       ??_C@_0DF@IBLNNAIG@R6026?$AN?6?9?5not?5enough?5space?5for?5st@ 3005f8ec     LIBCMTD:crt0msg.obj
 0002:00007924       ??_C@_0CG@IOHKGFNJ@R6025?$AN?6?9?5pure?5virtual?5function?5c@ 3005f924     LIBCMTD:crt0msg.obj
 0002:0000794c       ??_C@_0DF@JIJJFJDC@R6024?$AN?6?9?5not?5enough?5space?5for?5_o@ 3005f94c     LIBCMTD:crt0msg.obj
 0002:00007984       ??_C@_0CJ@EGEJHFME@R6019?$AN?6?9?5unable?5to?5open?5console?5@ 3005f984     LIBCMTD:crt0msg.obj
 0002:000079b0       ??_C@_0CB@GNHNIELH@R6018?$AN?6?9?5unexpected?5heap?5error?$AN?6@ 3005f9b0     LIBCMTD:crt0msg.obj
 0002:000079d4       ??_C@_0CN@FOLDKNG@R6017?$AN?6?9?5unexpected?5multithread?5@ 3005f9d4     LIBCMTD:crt0msg.obj
 0002:00007a04       ??_C@_0CM@FAHFJNHO@R6016?$AN?6?9?5not?5enough?5space?5for?5th@ 3005fa04     LIBCMTD:crt0msg.obj
 0002:00007a30       ??_C@_0JG@LBKMGKLD@?$AN?6This?5application?5has?5requested@ 3005fa30     LIBCMTD:crt0msg.obj
 0002:00007ac8       ??_C@_0CM@FLCNIPKK@R6009?$AN?6?9?5not?5enough?5space?5for?5en@ 3005fac8     LIBCMTD:crt0msg.obj
 0002:00007af4       ??_C@_0CK@KMMJOAPP@R6008?$AN?6?9?5not?5enough?5space?5for?5ar@ 3005faf4     LIBCMTD:crt0msg.obj
 0002:00007b20       ??_C@_0CF@HOHMHDEK@R6002?$AN?6?9?5floating?5point?5not?5load@ 3005fb20     LIBCMTD:crt0msg.obj
 0002:00007b48       ??_C@_0BK@OFGJDLJJ@Runtime?5Error?$CB?6?6Program?3?5?$AA@ 3005fb48     LIBCMTD:crt0msg.obj
 0002:00007b68       ___newctype                3005fb68     LIBCMTD:ctype.obj
 0002:00007e68       __wctype                   3005fe68     LIBCMTD:ctype.obj
 0002:0000806c       ??_C@_07GPNABLBE@a_str?4c?$AA@ 3006006c     LIBCMTD:a_str.obj
 0002:00008084       ??_C@_08JCCMCCIL@HH?3mm?3ss?$AA@ 30060084     LIBCMTD:strftime.obj
 0002:00008090       ??_C@_0BE@CKGJFCPC@dddd?0?5MMMM?5dd?0?5yyyy?$AA@ 30060090     LIBCMTD:strftime.obj
 0002:000080a4       ??_C@_08BPBNCDIB@MM?1dd?1yy?$AA@ 300600a4     LIBCMTD:strftime.obj
 0002:000080b0       ??_C@_02CJNFDJBF@PM?$AA@   300600b0     LIBCMTD:strftime.obj
 0002:000080b4       ??_C@_02DEDBPAFC@AM?$AA@   300600b4     LIBCMTD:strftime.obj
 0002:000080b8       ??_C@_08EDHMEBNP@December?$AA@ 300600b8     LIBCMTD:strftime.obj
 0002:000080c4       ??_C@_08HCHEGEOA@November?$AA@ 300600c4     LIBCMTD:strftime.obj
 0002:000080d0       ??_C@_07JJNFCEND@October?$AA@ 300600d0     LIBCMTD:strftime.obj
 0002:000080d8       ??_C@_09BHHEALKD@September?$AA@ 300600d8     LIBCMTD:strftime.obj
 0002:000080e4       ??_C@_06LBBHFDDG@August?$AA@ 300600e4     LIBCMTD:strftime.obj
 0002:000080ec       ??_C@_04MIEPOIFP@July?$AA@ 300600ec     LIBCMTD:strftime.obj
 0002:000080f4       ??_C@_04CNLMGBGM@June?$AA@ 300600f4     LIBCMTD:strftime.obj
 0002:000080fc       ??_C@_05DMJDNLEJ@April?$AA@ 300600fc     LIBCMTD:strftime.obj
 0002:00008104       ??_C@_05HPCKOFNC@March?$AA@ 30060104     LIBCMTD:strftime.obj
 0002:0000810c       ??_C@_08GNJGEPFN@February?$AA@ 3006010c     LIBCMTD:strftime.obj
 0002:00008118       ??_C@_07CGJPFGJA@January?$AA@ 30060118     LIBCMTD:strftime.obj
 0002:00008120       ??_C@_03MKABNOCG@Dec?$AA@  30060120     LIBCMTD:strftime.obj
 0002:00008124       ??_C@_03JPJOFNIA@Nov?$AA@  30060124     LIBCMTD:strftime.obj
 0002:00008128       ??_C@_03BMAOKBAD@Oct?$AA@  30060128     LIBCMTD:strftime.obj
 0002:0000812c       ??_C@_03GGCAPAJC@Sep?$AA@  3006012c     LIBCMTD:strftime.obj
 0002:00008130       ??_C@_03IFJFEIGA@Aug?$AA@  30060130     LIBCMTD:strftime.obj
 0002:00008134       ??_C@_03LBGABGKK@Jul?$AA@  30060134     LIBCMTD:strftime.obj
 0002:00008138       ??_C@_03IDFGHECI@Jun?$AA@  30060138     LIBCMTD:strftime.obj
 0002:0000813c       ??_C@_03CNMDKL@May?$AA@    3006013c     LIBCMTD:strftime.obj
 0002:00008140       ??_C@_03LEOLGMJP@Apr?$AA@  30060140     LIBCMTD:strftime.obj
 0002:00008144       ??_C@_03ODNJBKGA@Mar?$AA@  30060144     LIBCMTD:strftime.obj
 0002:00008148       ??_C@_03HJBDCHOM@Feb?$AA@  30060148     LIBCMTD:strftime.obj
 0002:0000814c       ??_C@_03JIHJHPIE@Jan?$AA@  3006014c     LIBCMTD:strftime.obj
 0002:00008150       ??_C@_08INBOOONO@Saturday?$AA@ 30060150     LIBCMTD:strftime.obj
 0002:0000815c       ??_C@_06JECMNKMI@Friday?$AA@ 3006015c     LIBCMTD:strftime.obj
 0002:00008164       ??_C@_08HACCIKIA@Thursday?$AA@ 30060164     LIBCMTD:strftime.obj
 0002:00008170       ??_C@_09DLIGFAKA@Wednesday?$AA@ 30060170     LIBCMTD:strftime.obj
 0002:0000817c       ??_C@_07BAAGCFCM@Tuesday?$AA@ 3006017c     LIBCMTD:strftime.obj
 0002:00008184       ??_C@_06JLEDEDGH@Monday?$AA@ 30060184     LIBCMTD:strftime.obj
 0002:0000818c       ??_C@_06OOPIFAJ@Sunday?$AA@ 3006018c     LIBCMTD:strftime.obj
 0002:00008194       ??_C@_03FEFJNEK@Sat?$AA@   30060194     LIBCMTD:strftime.obj
 0002:00008198       ??_C@_03IDIOELNC@Fri?$AA@  30060198     LIBCMTD:strftime.obj
 0002:0000819c       ??_C@_03IOFIKPDN@Thu?$AA@  3006019c     LIBCMTD:strftime.obj
 0002:000081a0       ??_C@_03MHOMLAJA@Wed?$AA@  300601a0     LIBCMTD:strftime.obj
 0002:000081a4       ??_C@_03NAGEINEP@Tue?$AA@  300601a4     LIBCMTD:strftime.obj
 0002:000081a8       ??_C@_03PDAGKDH@Mon?$AA@   300601a8     LIBCMTD:strftime.obj
 0002:000081ac       ??_C@_03KOEHGMDN@Sun?$AA@  300601ac     LIBCMTD:strftime.obj
 0002:000081b0       ??_C@_0L@OCEOFAIF@strftime?4c?$AA@ 300601b0     LIBCMTD:strftime.obj
 0002:000081bc       ??_C@_0DJ@BLPIACFC@?$CI?$CCInvalid?5MBCS?5character?5sequenc@ 300601bc     LIBCMTD:strftime.obj
 0002:000081f8       ??_C@_0DD@GLPHLKIC@?$CI?$CCZero?5length?5output?5buffer?5pass@ 300601f8     LIBCMTD:strftime.obj
 0002:0000822c       ??_C@_0DL@LLHFCBKO@?$CI?$CCInvalid?5MBCS?5character?5sequenc@ 3006022c     LIBCMTD:strftime.obj
 0002:00008268       ??_C@_0EC@CJNAOFBG@?$CI?$CCInvalid?5MBCS?5character?5sequenc@ 30060268     LIBCMTD:strftime.obj
 0002:000082ac       ??_C@_03EBAPMIKO@a?1p?$AA@ 300602ac     LIBCMTD:strftime.obj
 0002:000082b0       ??_C@_05JAMEPDIN@am?1pm?$AA@ 300602b0     LIBCMTD:strftime.obj
 0002:000082c4       ??_C@_0L@IOJADHBB@inittime?4c?$AA@ 300602c4     LIBCMTD:inittime.obj
 0002:000082d0       ??_C@_09MECGNAGI@initnum?4c?$AA@ 300602d0     LIBCMTD:initnum.obj
 0002:000082dc       ??_C@_09HKFHICAL@initmon?4c?$AA@ 300602dc     LIBCMTD:initmon.obj
 0002:000082e8       ??_C@_0L@GBAGBCPL@initctyp?4c?$AA@ 300602e8     LIBCMTD:initctyp.obj
 0002:000082f4       ??_C@_07CKDBCAPD@mlock?4c?$AA@ 300602f4     LIBCMTD:mlock.obj
 0002:00008310       ___rgLocInfo               30060310     LIBCMTD:getqloc.obj
 0002:000087b4       ??_C@_08PKBIPKE@Paraguay?$AA@ 300607b4     LIBCMTD:getqloc.obj
 0002:000087c0       ??_C@_07GHBIBIBP@Uruguay?$AA@ 300607c0     LIBCMTD:getqloc.obj
 0002:000087c8       ??_C@_05HBNKAPDN@Chile?$AA@ 300607c8     LIBCMTD:getqloc.obj
 0002:000087d0       ??_C@_07FEIFIPNF@Ecuador?$AA@ 300607d0     LIBCMTD:getqloc.obj
 0002:000087d8       ??_C@_09PGNFPGME@Argentina?$AA@ 300607d8     LIBCMTD:getqloc.obj
 0002:000087e4       ??_C@_04IALPBJF@Peru?$AA@  300607e4     LIBCMTD:getqloc.obj
 0002:000087ec       ??_C@_08IJPLNLKH@Colombia?$AA@ 300607ec     LIBCMTD:getqloc.obj
 0002:000087f8       ??_C@_09IDMFKCN@Venezuela?$AA@ 300607f8     LIBCMTD:getqloc.obj
 0002:00008804       ??_C@_0BD@DNEJOGOK@Dominican?5Republic?$AA@ 30060804     LIBCMTD:getqloc.obj
 0002:00008818       ??_C@_0N@LPINDNDB@South?5Africa?$AA@ 30060818     LIBCMTD:getqloc.obj
 0002:00008828       ??_C@_06BLJPEOBG@Panama?$AA@ 30060828     LIBCMTD:getqloc.obj
 0002:00008830       ??_C@_0L@BOCNDGON@Luxembourg?$AA@ 30060830     LIBCMTD:getqloc.obj
 0002:0000883c       ??_C@_0L@CONEHKA@Costa?5Rica?$AA@ 3006083c     LIBCMTD:getqloc.obj
 0002:00008848       ??_C@_0M@KGBPELAM@Switzerland?$AA@ 30060848     LIBCMTD:getqloc.obj
 0002:00008854       ??_C@_09FJGLIMAG@Guatemala?$AA@ 30060854     LIBCMTD:getqloc.obj
 0002:00008860       ??_C@_06ECHIPDMK@Canada?$AA@ 30060860     LIBCMTD:getqloc.obj
 0002:00008868       ??_C@_0BG@CCEBNPGH@Spanish?5?9?5Modern?5Sort?$AA@ 30060868     LIBCMTD:getqloc.obj
 0002:00008880       ??_C@_09EFGJAPAD@Australia?$AA@ 30060880     LIBCMTD:getqloc.obj
 0002:0000888c       ??_C@_07NEKHPBCG@English?$AA@ 3006088c     LIBCMTD:getqloc.obj
 0002:00008894       ??_C@_07LKIIOGFH@Austria?$AA@ 30060894     LIBCMTD:getqloc.obj
 0002:0000889c       ??_C@_06EDDDIONA@German?$AA@ 3006089c     LIBCMTD:getqloc.obj
 0002:000088a4       ??_C@_07LIIIOFOA@Belgium?$AA@ 300608a4     LIBCMTD:getqloc.obj
 0002:000088ac       ??_C@_06DIAOLLEH@Mexico?$AA@ 300608ac     LIBCMTD:getqloc.obj
 0002:000088b4       ??_C@_07PFALJOGE@Spanish?$AA@ 300608b4     LIBCMTD:getqloc.obj
 0002:000088bc       ??_C@_06FFOOPAJB@Basque?$AA@ 300608bc     LIBCMTD:getqloc.obj
 0002:000088c4       ??_C@_06DGHNDJFJ@Sweden?$AA@ 300608c4     LIBCMTD:getqloc.obj
 0002:000088cc       ??_C@_07OBINPKFN@Swedish?$AA@ 300608cc     LIBCMTD:getqloc.obj
 0002:000088d4       ??_C@_07NCOIHDGC@Iceland?$AA@ 300608d4     LIBCMTD:getqloc.obj
 0002:000088dc       ??_C@_09JHBBDDIA@Icelandic?$AA@ 300608dc     LIBCMTD:getqloc.obj
 0002:000088e8       ??_C@_06COBCPIFO@France?$AA@ 300608e8     LIBCMTD:getqloc.obj
 0002:000088f0       ??_C@_06GODMCAND@French?$AA@ 300608f0     LIBCMTD:getqloc.obj
 0002:000088f8       ??_C@_07MFHPMOED@Finland?$AA@ 300608f8     LIBCMTD:getqloc.obj
 0002:00008900       ??_C@_07MCEAMKOD@Finnish?$AA@ 30060900     LIBCMTD:getqloc.obj
 0002:00008908       ??_C@_05CBHOCCK@Spain?$AA@ 30060908     LIBCMTD:getqloc.obj
 0002:00008910       ??_C@_0BL@GIOEGDHB@Spanish?5?9?5Traditional?5Sort?$AA@ 30060910     LIBCMTD:getqloc.obj
 0002:0000892c       ___rglangidNotDefault      3006092c     LIBCMTD:getqloc.obj
 0002:00008940       ___rg_country              30060940     LIBCMTD:getqloc.obj
 0002:000089f8       ??_C@_0O@FMJNFNKE@united?9states?$AA@ 300609f8     LIBCMTD:getqloc.obj
 0002:00008a08       ??_C@_0P@NDHFFKCA@united?9kingdom?$AA@ 30060a08     LIBCMTD:getqloc.obj
 0002:00008a18       ??_C@_0BC@HHDADLGF@trinidad?5?$CG?5tobago?$AA@ 30060a18     LIBCMTD:getqloc.obj
 0002:00008a2c       ??_C@_0M@IOAEBDAC@south?9korea?$AA@ 30060a2c     LIBCMTD:getqloc.obj
 0002:00008a38       ??_C@_0N@FIELFKIJ@south?9africa?$AA@ 30060a38     LIBCMTD:getqloc.obj
 0002:00008a48       ??_C@_0M@OPNDHCMC@south?5korea?$AA@ 30060a48     LIBCMTD:getqloc.obj
 0002:00008a54       ??_C@_0N@MDEOEPFI@south?5africa?$AA@ 30060a54     LIBCMTD:getqloc.obj
 0002:00008a64       ??_C@_06FKAPCJLB@slovak?$AA@ 30060a64     LIBCMTD:getqloc.obj
 0002:00008a6c       ??_C@_0M@EFJANOAL@puerto?9rico?$AA@ 30060a6c     LIBCMTD:getqloc.obj
 0002:00008a78       ??_C@_08PGOJKDAI@pr?9china?$AA@ 30060a78     LIBCMTD:getqloc.obj
 0002:00008a84       ??_C@_08JHDOMCMI@pr?5china?$AA@ 30060a84     LIBCMTD:getqloc.obj
 0002:00008a90       ??_C@_02JHCHFBLL@nz?$AA@   30060a90     LIBCMTD:getqloc.obj
 0002:00008a94       ??_C@_0M@LINHDHKP@new?9zealand?$AA@ 30060a94     LIBCMTD:getqloc.obj
 0002:00008aa0       ??_C@_09IIIPPBDB@hong?9kong?$AA@ 30060aa0     LIBCMTD:getqloc.obj
 0002:00008aac       ??_C@_07HJLCKBG@holland?$AA@ 30060aac     LIBCMTD:getqloc.obj
 0002:00008ab4       ??_C@_0O@LEHGMHAG@great?5britain?$AA@ 30060ab4     LIBCMTD:getqloc.obj
 0002:00008ac4       ??_C@_07FACOMELA@england?$AA@ 30060ac4     LIBCMTD:getqloc.obj
 0002:00008acc       ??_C@_05JIHCEICB@czech?$AA@ 30060acc     LIBCMTD:getqloc.obj
 0002:00008ad4       ??_C@_05BBJOBLGB@china?$AA@ 30060ad4     LIBCMTD:getqloc.obj
 0002:00008adc       ??_C@_07GPKPHICP@britain?$AA@ 30060adc     LIBCMTD:getqloc.obj
 0002:00008ae4       ??_C@_07MHIPBHMG@america?$AA@ 30060ae4     LIBCMTD:getqloc.obj
 0002:00008af0       ___rg_language             30060af0     LIBCMTD:getqloc.obj
 0002:00008cf8       ??_C@_03KIALPMKC@usa?$AA@  30060cf8     LIBCMTD:getqloc.obj
 0002:00008cfc       ??_C@_02FGJGKGGD@us?$AA@   30060cfc     LIBCMTD:getqloc.obj
 0002:00008d00       ??_C@_02NEINDODK@uk?$AA@   30060d00     LIBCMTD:getqloc.obj
 0002:00008d04       ??_C@_05JMPCFJFJ@swiss?$AA@ 30060d04     LIBCMTD:getqloc.obj
 0002:00008d0c       ??_C@_0BA@HLOCPIOD@swedish?9finland?$AA@ 30060d0c     LIBCMTD:getqloc.obj
 0002:00008d1c       ??_C@_0BC@PKCNIABK@spanish?9venezuela?$AA@ 30060d1c     LIBCMTD:getqloc.obj
 0002:00008d30       ??_C@_0BA@GBHHMIJI@spanish?9uruguay?$AA@ 30060d30     LIBCMTD:getqloc.obj
 0002:00008d40       ??_C@_0BE@BHDOHPMC@spanish?9puerto?5rico?$AA@ 30060d40     LIBCMTD:getqloc.obj
 0002:00008d54       ??_C@_0N@KMOIDGGN@spanish?9peru?$AA@ 30060d54     LIBCMTD:getqloc.obj
 0002:00008d64       ??_C@_0BB@HMHLPGPH@spanish?9paraguay?$AA@ 30060d64     LIBCMTD:getqloc.obj
 0002:00008d78       ??_C@_0P@MCPKNGFD@spanish?9panama?$AA@ 30060d78     LIBCMTD:getqloc.obj
 0002:00008d88       ??_C@_0BC@IHOHGAIL@spanish?9nicaragua?$AA@ 30060d88     LIBCMTD:getqloc.obj
 0002:00008d9c       ??_C@_0P@KLMJDNFJ@spanish?9modern?$AA@ 30060d9c     LIBCMTD:getqloc.obj
 0002:00008dac       ??_C@_0BA@BPAPGBCM@spanish?9mexican?$AA@ 30060dac     LIBCMTD:getqloc.obj
 0002:00008dbc       ??_C@_0BB@PDECHHHE@spanish?9honduras?$AA@ 30060dbc     LIBCMTD:getqloc.obj
 0002:00008dd0       ??_C@_0BC@KLHKFGDB@spanish?9guatemala?$AA@ 30060dd0     LIBCMTD:getqloc.obj
 0002:00008de4       ??_C@_0BE@MFOOKJAI@spanish?9el?5salvador?$AA@ 30060de4     LIBCMTD:getqloc.obj
 0002:00008df8       ??_C@_0BA@FCOKFPFC@spanish?9ecuador?$AA@ 30060df8     LIBCMTD:getqloc.obj
 0002:00008e08       ??_C@_0BL@PLMGIMOO@spanish?9dominican?5republic?$AA@ 30060e08     LIBCMTD:getqloc.obj
 0002:00008e24       ??_C@_0BD@HLGDNMHB@spanish?9costa?5rica?$AA@ 30060e24     LIBCMTD:getqloc.obj
 0002:00008e38       ??_C@_0BB@PKCBKCPE@spanish?9colombia?$AA@ 30060e38     LIBCMTD:getqloc.obj
 0002:00008e4c       ??_C@_0O@MCBIJGNE@spanish?9chile?$AA@ 30060e4c     LIBCMTD:getqloc.obj
 0002:00008e5c       ??_C@_0BA@BEFEIGJJ@spanish?9bolivia?$AA@ 30060e5c     LIBCMTD:getqloc.obj
 0002:00008e6c       ??_C@_0BC@EMECMPD@spanish?9argentina?$AA@ 30060e6c     LIBCMTD:getqloc.obj
 0002:00008e80       ??_C@_0BF@EALFLENP@portuguese?9brazilian?$AA@ 30060e80     LIBCMTD:getqloc.obj
 0002:00008e98       ??_C@_0BC@HBLEBLNN@norwegian?9nynorsk?$AA@ 30060e98     LIBCMTD:getqloc.obj
 0002:00008eac       ??_C@_0BB@HMACDDCK@norwegian?9bokmal?$AA@ 30060eac     LIBCMTD:getqloc.obj
 0002:00008ec0       ??_C@_09BAFFPPHE@norwegian?$AA@ 30060ec0     LIBCMTD:getqloc.obj
 0002:00008ecc       ??_C@_0O@EAJFJDFG@italian?9swiss?$AA@ 30060ecc     LIBCMTD:getqloc.obj
 0002:00008edc       ??_C@_0O@CNOMPGD@irish?9english?$AA@ 30060edc     LIBCMTD:getqloc.obj
 0002:00008eec       ??_C@_0N@EDHBGCKG@german?9swiss?$AA@ 30060eec     LIBCMTD:getqloc.obj
 0002:00008efc       ??_C@_0BC@JACMHNBP@german?9luxembourg?$AA@ 30060efc     LIBCMTD:getqloc.obj
 0002:00008f10       ??_C@_0BE@HBGMGFEG@german?9lichtenstein?$AA@ 30060f10     LIBCMTD:getqloc.obj
 0002:00008f24       ??_C@_0BA@HKKBIBKL@german?9austrian?$AA@ 30060f24     LIBCMTD:getqloc.obj
 0002:00008f34       ??_C@_0N@GCAEPEBK@french?9swiss?$AA@ 30060f34     LIBCMTD:getqloc.obj
 0002:00008f44       ??_C@_0BC@DJFJJCK@french?9luxembourg?$AA@ 30060f44     LIBCMTD:getqloc.obj
 0002:00008f58       ??_C@_0BA@NNCEDFIC@french?9canadian?$AA@ 30060f58     LIBCMTD:getqloc.obj
 0002:00008f68       ??_C@_0P@CMPOCLM@french?9belgian?$AA@ 30060f68     LIBCMTD:getqloc.obj
 0002:00008f78       ??_C@_0M@GHHDJOK@english?9usa?$AA@ 30060f78     LIBCMTD:getqloc.obj
 0002:00008f84       ??_C@_0L@PLDJKEIL@english?9us?$AA@ 30060f84     LIBCMTD:getqloc.obj
 0002:00008f90       ??_C@_0L@HJCCDMNC@english?9uk?$AA@ 30060f90     LIBCMTD:getqloc.obj
 0002:00008f9c       ??_C@_0BK@CKLIAGJB@english?9trinidad?5y?5tobago?$AA@ 30060f9c     LIBCMTD:getqloc.obj
 0002:00008fb8       ??_C@_0BF@JMJMGNNF@english?9south?5africa?$AA@ 30060fb8     LIBCMTD:getqloc.obj
 0002:00008fd0       ??_C@_0L@DKIIFDFD@english?9nz?$AA@ 30060fd0     LIBCMTD:getqloc.obj
 0002:00008fdc       ??_C@_0BA@ONHGJCLH@english?9jamaica?$AA@ 30060fdc     LIBCMTD:getqloc.obj
 0002:00008fec       ??_C@_0M@HJBGHOPO@english?9ire?$AA@ 30060fec     LIBCMTD:getqloc.obj
 0002:00008ff8       ??_C@_0BC@LFEKMIFB@english?9caribbean?$AA@ 30060ff8     LIBCMTD:getqloc.obj
 0002:0000900c       ??_C@_0M@OLDPFKHI@english?9can?$AA@ 3006100c     LIBCMTD:getqloc.obj
 0002:00009018       ??_C@_0P@OMDEHBMP@english?9belize?$AA@ 30061018     LIBCMTD:getqloc.obj
 0002:00009028       ??_C@_0M@KFHFPFED@english?9aus?$AA@ 30061028     LIBCMTD:getqloc.obj
 0002:00009034       ??_C@_0BB@MNMBKDFE@english?9american?$AA@ 30061034     LIBCMTD:getqloc.obj
 0002:00009048       ??_C@_0O@KIDLNNBA@dutch?9belgian?$AA@ 30061048     LIBCMTD:getqloc.obj
 0002:00009058       ??_C@_0BE@JBKABBMH@chinese?9traditional?$AA@ 30061058     LIBCMTD:getqloc.obj
 0002:0000906c       ??_C@_0BC@MJJMPKCG@chinese?9singapore?$AA@ 3006106c     LIBCMTD:getqloc.obj
 0002:00009080       ??_C@_0BD@FDKADDCP@chinese?9simplified?$AA@ 30061080     LIBCMTD:getqloc.obj
 0002:00009094       ??_C@_0BB@DBEFDDME@chinese?9hongkong?$AA@ 30061094     LIBCMTD:getqloc.obj
 0002:000090a8       ??_C@_07DHNMFMCI@chinese?$AA@ 300610a8     LIBCMTD:getqloc.obj
 0002:000090b0       ??_C@_03FNDDCHI@chi?$AA@   300610b0     LIBCMTD:getqloc.obj
 0002:000090b4       ??_C@_03BMMIADDJ@chh?$AA@  300610b4     LIBCMTD:getqloc.obj
 0002:000090b8       ??_C@_08OAIPJDGI@canadian?$AA@ 300610b8     LIBCMTD:getqloc.obj
 0002:000090c4       ??_C@_07HBPMNPNJ@belgian?$AA@ 300610c4     LIBCMTD:getqloc.obj
 0002:000090cc       ??_C@_0L@OEKOPBEL@australian?$AA@ 300610cc     LIBCMTD:getqloc.obj
 0002:000090d8       ??_C@_0BB@MEIMBEDG@american?9english?$AA@ 300610d8     LIBCMTD:getqloc.obj
 0002:000090ec       ??_C@_0BB@DFMDPDGB@american?5english?$AA@ 300610ec     LIBCMTD:getqloc.obj
 0002:00009100       ??_C@_08IJLOKOLL@american?$AA@ 30061100     LIBCMTD:getqloc.obj
 0002:0000910c       ??_C@_0BC@NFIEMBLL@Norwegian?9Nynorsk?$AA@ 3006110c     LIBCMTD:getqloc.obj
 0002:00009120       ??_C@_03NFKLAGEF@OCP?$AA@  30061120     LIBCMTD:getqloc.obj
 0002:00009124       ??_C@_03DFHEHBHG@ACP?$AA@  30061124     LIBCMTD:getqloc.obj
 0002:00009134       ??_C@_09KJLOAKHC@mbctype?4c?$AA@ 30061134     LIBCMTD:mbctype.obj
 0002:0000916c       ??_C@_09PKAEMGHJ@_getbuf?4c?$AA@ 3006116c     LIBCMTD:_getbuf.obj
 0002:00009178       ??_C@_0CP@PEILCOHB@f?3?2vs70builds?23077?2vc?2crtbld?2crt@ 30061178     LIBCMTD:snprintf.obj
 0002:000091a8       ??_C@_0DA@KHEJFFIK@f?3?2vs70builds?23077?2vc?2crtbld?2crt@ 300611a8     LIBCMTD:vsnprint.obj
 0002:000091e4       ??_C@_08GNMOIKDK@onexit?4c?$AA@ 300611e4     LIBCMTD:onexit.obj
 0002:000091fc       ??_C@_09IFKHNCOH@_sftbuf?4c?$AA@ 300611fc     LIBCMTD:_sftbuf.obj
 0002:00009208       ??_C@_0BH@HIGALIFJ@flag?5?$DN?$DN?50?5?$HM?$HM?5flag?5?$DN?$DN?51?$AA@ 30061208     LIBCMTD:_sftbuf.obj
 0002:00009220       ??_C@_0L@CKFHAPLH@_freebuf?4c?$AA@ 30061220     LIBCMTD:_freebuf.obj
 0002:0000922c       ??_C@_0P@FELNCIKG@stream?5?$CB?$DN?5NULL?$AA@ 3006122c     LIBCMTD:_freebuf.obj
 0002:00009250       ??_C@_0KA@JEHFIFGP@A?5buffer?5overrun?5has?5been?5detect@ 30061250     LIBCMTD:secfail.obj
 0002:000092f0       ??_C@_0BJ@MDEKIEOJ@Buffer?5overrun?5detected?$CB?$AA@ 300612f0     LIBCMTD:secfail.obj
 0002:00009310       ??_C@_0LB@BPLHHLFD@A?5security?5error?5of?5unknown?5caus@ 30061310     LIBCMTD:secfail.obj
 0002:000093c4       ??_C@_0CD@GMKACBEK@Unknown?5security?5failure?5detecte@ 300613c4     LIBCMTD:secfail.obj
 0002:000093f4       ??_C@_0L@KBNGFDKM@convrtcp?4c?$AA@ 300613f4     LIBCMTD:convrtcp.obj
 0002:0000945c       ??_C@_09FNBBCGGI@sprintf?4c?$AA@ 3006145c     LIBCMTD:sprintf.obj
 0002:00009468       ??_C@_0CG@PKBDLMEO@InitializeCriticalSectionAndSpin@ 30061468     LIBCMTD:initcrit.obj
 0002:0000949c       ??_C@_06IMKFLFPG@1?$CDQNAN?$AA@ 3006149c     LIBCMTD:x10fout.obj
 0002:000094a4       ??_C@_05DNEBIAHO@1?$CDINF?$AA@ 300614a4     LIBCMTD:x10fout.obj
 0002:000094ac       ??_C@_05PHHOCPM@1?$CDIND?$AA@ 300614ac     LIBCMTD:x10fout.obj
 0002:000094b4       ??_C@_06PGGFOGJG@1?$CDSNAN?$AA@ 300614b4     LIBCMTD:x10fout.obj
 0002:000094bc       ___dnames                  300614bc     LIBCMTD:timeset.obj
 0002:000094d4       ___mnames                  300614d4     LIBCMTD:timeset.obj
 0002:0000951c       ??_C@_07LOOFNDIO@tzset?4c?$AA@ 3006151c     LIBCMTD:tzset.obj
 0002:00009524       ??_C@_02CLFPBFFP@TZ?$AA@   30061524     LIBCMTD:tzset.obj
 0002:00009544       ??_C@_0L@DILIPMN@inithelp?4c?$AA@ 30061544     LIBCMTD:inithelp.obj
 0002:00009550       ??_C@_09MGNHMPHC@osfinfo?4c?$AA@ 30061550     LIBCMTD:osfinfo.obj
 0002:000095a4       ??_C@_08BDNGOBJJ@fclose?4c?$AA@ 300615a4     LIBCMTD:fclose.obj
 0002:000095cc       ??_C@_07NIBBAFJP@w_loc?4c?$AA@ 300615cc     LIBCMTD:w_loc.obj
 0002:000095e4       ??_C@_07GCMFDNDD@a_loc?4c?$AA@ 300615e4     LIBCMTD:a_loc.obj
 0002:0000960c       ??_C@_0L@CELCHBFJ@wtombenv?4c?$AA@ 3006160c     LIBCMTD:wtombenv.obj
 0002:00009618       ??_C@_07KLPPCEPH@a_cmp?4c?$AA@ 30061618     LIBCMTD:a_cmp.obj
 0002:00009620       ??_C@_0DN@NFIMOOFE@cchCount1?$DN?$DN0?5?$CG?$CG?5cchCount2?$DN?$DN1?5?$HM?$HM?5@ 30061620     LIBCMTD:a_cmp.obj
 0002:00009678       ??_C@_08BMJILFKN@setenv?4c?$AA@ 30061678     LIBCMTD:setenv.obj
 0002:00009684       ??_C@_05MAJJAKPI@FALSE?$AA@ 30061684     LIBCMTD:setenv.obj
 0002:000096e4       ___rtc_iaa                 300616e4     LIBCMTD:initsect.obj
 0002:000096e8       ___rtc_izz                 300616e8     LIBCMTD:initsect.obj
 0002:000096ec       ___rtc_taa                 300616ec     LIBCMTD:initsect.obj
 0002:000096f0       ___rtc_tzz                 300616f0     LIBCMTD:initsect.obj
 0002:000096f4       __IMPORT_DESCRIPTOR_KERNEL32 300616f4     kernel32:KERNEL32.dll
 0002:00009708       __NULL_IMPORT_DESCRIPTOR   30061708     kernel32:KERNEL32.dll
 0003:00000000       ___xc_a                    30062000     LIBCMTD:crt0init.obj
 0003:00000008       ___xc_z                    30062008     LIBCMTD:crt0init.obj
 0003:0000000c       ___xi_a                    3006200c     LIBCMTD:crt0init.obj
 0003:00000020       ___xi_z                    30062020     LIBCMTD:crt0init.obj
 0003:00000024       ___xp_a                    30062024     LIBCMTD:crt0init.obj
 0003:0000002c       ___xp_z                    3006202c     LIBCMTD:crt0init.obj
 0003:00000030       ___xt_a                    30062030     LIBCMTD:crt0init.obj
 0003:00000034       ___xt_z                    30062034     LIBCMTD:crt0init.obj
 0003:00000040       _bg_itemlist               30062040     bg_misc.obj
 0003:000007c4       _bg_numItems               300627c4     bg_misc.obj
 0003:000007c8       _eventnames                300627c8     bg_misc.obj
 0003:000008f8       _pm_stopspeed              300628f8     bg_pmove.obj
 0003:000008fc       _pm_duckScale              300628fc     bg_pmove.obj
 0003:00000900       _pm_swimScale              30062900     bg_pmove.obj
 0003:00000904       _pm_wadeScale              30062904     bg_pmove.obj
 0003:00000908       _pm_accelerate             30062908     bg_pmove.obj
 0003:0000090c       _pm_airaccelerate          3006290c     bg_pmove.obj
 0003:00000910       _pm_wateraccelerate        30062910     bg_pmove.obj
 0003:00000914       _pm_flyaccelerate          30062914     bg_pmove.obj
 0003:00000918       _pm_friction               30062918     bg_pmove.obj
 0003:0000091c       _pm_waterfriction          3006291c     bg_pmove.obj
 0003:00000920       _pm_flightfriction         30062920     bg_pmove.obj
 0003:00000924       _pm_spectatorfriction      30062924     bg_pmove.obj
 0003:000009e0       _drawTeamOverlayModificationCount 300629e0     cg_draw.obj
 0003:000011c8       _forceModelModificationCount 300631c8     cg_main.obj
 0003:00001910       _cl_numparticles           30063910     cg_marks.obj
 0003:00001918       _cg_customSoundNames       30063918     cg_players.obj
 0003:000019d8       _axisDefault               300639d8     q_math.obj
 0003:000019fc       _colorBlack                300639fc     q_math.obj
 0003:00001a0c       _colorRed                  30063a0c     q_math.obj
 0003:00001a1c       _colorGreen                30063a1c     q_math.obj
 0003:00001a2c       _colorBlue                 30063a2c     q_math.obj
 0003:00001a3c       _colorYellow               30063a3c     q_math.obj
 0003:00001a4c       _colorMagenta              30063a4c     q_math.obj
 0003:00001a5c       _colorCyan                 30063a5c     q_math.obj
 0003:00001a6c       _colorWhite                30063a6c     q_math.obj
 0003:00001a7c       _colorLtGrey               30063a7c     q_math.obj
 0003:00001a8c       _colorMdGrey               30063a8c     q_math.obj
 0003:00001a9c       _colorDkGrey               30063a9c     q_math.obj
 0003:00001ab0       _g_color_table             30063ab0     q_math.obj
 0003:00001b30       _bytedirs                  30063b30     q_math.obj
 0003:000022c8       ?__LINE__Var@?1??ProjectPointOnPlane@@9@9 300642c8     q_math.obj
 0003:000022d8       _commandList               300642d8     ui_shared.obj
 0003:00002380       _scriptCommandCount        30064380     ui_shared.obj
 0003:00002998       _itemParseKeywords         30064998     ui_shared.obj
 0003:00002c90       _menuParseKeywords         30064c90     ui_shared.obj
 0003:00002dec       __fltused                  30064dec     LIBCMTD:fpinit.obj
 0003:00002df0       __ldused                   30064df0     LIBCMTD:fpinit.obj
 0003:00002df4       __FPinit                   30064df4     LIBCMTD:fpinit.obj
 0003:00002df8       __FPmtinit                 30064df8     LIBCMTD:fpinit.obj
 0003:00002dfc       __FPmtterm                 30064dfc     LIBCMTD:fpinit.obj
 0003:00002e80       __aexit_rtn                30064e80     LIBCMTD:dllcrt0.obj
 0003:00002e84       __cfltcvt_tab              30064e84     LIBCMTD:cmiscdat.obj
 0003:00002ea0       __indefinite               30064ea0     LIBCMTD:87disp.obj
 0003:00002eaa       __piby2                    30064eaa     LIBCMTD:87disp.obj
 0003:00002fb8       __d_inf                    30064fb8     LIBCMTD:util.obj
 0003:00002fc0       __d_ind                    30064fc0     LIBCMTD:util.obj
 0003:00002fc8       __d_max                    30064fc8     LIBCMTD:util.obj
 0003:00002fd0       __d_min                    30064fd0     LIBCMTD:util.obj
 0003:00002fd8       __d_mzero                  30064fd8     LIBCMTD:util.obj
 0003:00003000       ___initiallocinfo          30065000     LIBCMTD:setlocal.obj
 0003:00003054       ___ptlocinfo               30065054     LIBCMTD:setlocal.obj
 0003:00003190       ___lc_category             30065190     LIBCMTD:setlocal.obj
 0003:000031d8       ___tlsindex                300651d8     LIBCMTD:tidtable.obj
 0003:000031e0       ___nullstring              300651e0     LIBCMTD:output.obj
 0003:000031e4       ___wnullstring             300651e4     LIBCMTD:output.obj
 0003:000031e8       __crtAssertBusy            300651e8     LIBCMTD:dbgrpt.obj
 0003:000031ec       __CrtDbgMode               300651ec     LIBCMTD:dbgrpt.obj
 0003:000031f8       __CrtDbgFile               300651f8     LIBCMTD:dbgrpt.obj
 0003:00003210       __pmatherr                 30065210     LIBCMTD:libm_error.obj
 0003:00003220       __OP_ATAN2jmptab           30065220     LIBCMTD:87triga.obj
 0003:00003270       __iob                      30065270     LIBCMTD:_file.obj
 0003:000034f0       ___security_cookie         300654f0     LIBCMTD:seccook.obj
 0003:000034f4       __crtDbgFlag               300654f4     LIBCMTD:dbgheap.obj
 0003:000034fc       __crtBreakAlloc            300654fc     LIBCMTD:dbgheap.obj
 0003:00003518       ___badioinfo               30065518     LIBCMTD:ioinit.obj
 0003:0000353c       __amblksiz                 3006553c     LIBCMTD:heapinit.obj
 0003:00003540       __XcptActTab               30065540     LIBCMTD:winxfltr.obj
 0003:000035b8       __First_FPE_Indx           300655b8     LIBCMTD:winxfltr.obj
 0003:000035bc       __Num_FPE                  300655bc     LIBCMTD:winxfltr.obj
 0003:000035c0       __XcptActTabSize           300655c0     LIBCMTD:winxfltr.obj
 0003:000035c4       __XcptActTabCount          300655c4     LIBCMTD:winxfltr.obj
 0003:000035c8       __NLG_Destination          300655c8     LIBCMTD:exsup.obj
 0003:00003670       ___mb_cur_max              30065670     LIBCMTD:nlsdata1.obj
 0003:00003674       ___decimal_point           30065674     LIBCMTD:nlsdata1.obj
 0003:00003678       ___decimal_point_length    30065678     LIBCMTD:nlsdata1.obj
 0003:00003818       __matherr_flag             30065818     LIBCMTD:matherr.obj
 0003:0000381c       __pctype                   3006581c     LIBCMTD:ctype.obj
 0003:00003820       __pwctype                  30065820     LIBCMTD:ctype.obj
 0003:00003824       ___lc_time_curr            30065824     LIBCMTD:strftime.obj
 0003:00003828       ___lc_time_c               30065828     LIBCMTD:strftime.obj
 0003:000038e0       ___lconv_static_decimal    300658e0     LIBCMTD:lconv.obj
 0003:000038e4       ___lconv_c                 300658e4     LIBCMTD:lconv.obj
 0003:00003914       ___lconv                   30065914     LIBCMTD:lconv.obj
 0003:00003a38       ___lc_clike                30065a38     LIBCMTD:nlsdata2.obj
 0003:00003b40       __pfnAllocHook             30065b40     LIBCMTD:dbghook.obj
 0003:00003b48       __timezone                 30065b48     LIBCMTD:timeset.obj
 0003:00003b4c       __daylight                 30065b4c     LIBCMTD:timeset.obj
 0003:00003b50       __dstbias                  30065b50     LIBCMTD:timeset.obj
 0003:00003bd8       __tzname                   30065bd8     LIBCMTD:timeset.obj
 0003:00003c00       __pow10pos                 30065c00     LIBCMTD:constpow.obj
 0003:00003d60       __pow10neg                 30065d60     LIBCMTD:constpow.obj
 0003:00003ebc       __lpdays                   30065ebc     LIBCMTD:days.obj
 0003:00003ef0       __days                     30065ef0     LIBCMTD:days.obj
 0003:00003f40       _c_pmove                   30065f40     bg_pmove.obj
 0003:00006474       _initparticles             30068474     cg_marks.obj
 0003:00006db0       _vec3_origin               30068db0     q_math.obj
 0003:00181014       _DC                        301e3014     ui_shared.obj
 0003:00181028       _menuCount                 301e3028     ui_shared.obj
 0003:0018102c       _openMenuCount             301e302c     ui_shared.obj
 0003:00181044       ___fastflag                301e3044     LIBCMTD:fpinit.obj
 0003:00181048       __adjust_fdiv              301e3048     LIBCMTD:fpinit.obj
 0003:00181050       __aenvptr                  301e3050     LIBCMTD:dllcrt0.obj
 0003:00181054       __wenvptr                  301e3054     LIBCMTD:dllcrt0.obj
 0003:00181058       ___error_mode              301e3058     LIBCMTD:dllcrt0.obj
 0003:0018105c       ___app_type                301e305c     LIBCMTD:dllcrt0.obj
 0003:0018106c       _gpFlsAlloc                301e306c     LIBCMTD:tidtable.obj
 0003:00181070       _gpFlsGetValue             301e3070     LIBCMTD:tidtable.obj
 0003:00181074       _gpFlsSetValue             301e3074     LIBCMTD:tidtable.obj
 0003:00181078       _gpFlsFree                 301e3078     LIBCMTD:tidtable.obj
 0003:00181080       __umaskval                 301e3080     LIBCMTD:crt0dat.obj
 0003:00181084       __osplatform               301e3084     LIBCMTD:crt0dat.obj
 0003:00181088       __osver                    301e3088     LIBCMTD:crt0dat.obj
 0003:0018108c       __winver                   301e308c     LIBCMTD:crt0dat.obj
 0003:00181090       __winmajor                 301e3090     LIBCMTD:crt0dat.obj
 0003:00181094       __winminor                 301e3094     LIBCMTD:crt0dat.obj
 0003:00181098       ___argc                    301e3098     LIBCMTD:crt0dat.obj
 0003:0018109c       ___argv                    301e309c     LIBCMTD:crt0dat.obj
 0003:001810a0       ___wargv                   301e30a0     LIBCMTD:crt0dat.obj
 0003:001810a4       __environ                  301e30a4     LIBCMTD:crt0dat.obj
 0003:001810a8       ___initenv                 301e30a8     LIBCMTD:crt0dat.obj
 0003:001810ac       __wenviron                 301e30ac     LIBCMTD:crt0dat.obj
 0003:001810b0       ___winitenv                301e30b0     LIBCMTD:crt0dat.obj
 0003:001810b4       __pgmptr                   301e30b4     LIBCMTD:crt0dat.obj
 0003:001810b8       __wpgmptr                  301e30b8     LIBCMTD:crt0dat.obj
 0003:001810bc       __exitflag                 301e30bc     LIBCMTD:crt0dat.obj
 0003:001810c0       __C_Termination_Done       301e30c0     LIBCMTD:crt0dat.obj
 0003:001810c4       __C_Exit_Done              301e30c4     LIBCMTD:crt0dat.obj
 0003:001810f4       __cflush                   301e30f4     LIBCMTD:_file.obj
 0003:00181224       __adbgmsg                  301e3224     LIBCMTD:crt0msg.obj
 0003:0018122c       ___lconv_static_null       301e322c     LIBCMTD:lconv.obj
 0003:00181230       ___lc_time_intl            301e3230     LIBCMTD:inittime.obj
 0003:00181234       ___lconv_intl              301e3234     LIBCMTD:initmon.obj
 0003:00181388       ___lc_handle               301e3388     LIBCMTD:nlsdata2.obj
 0003:001813a0       ___lc_codepage             301e33a0     LIBCMTD:nlsdata2.obj
 0003:001813a4       ___lc_collate_cp           301e33a4     LIBCMTD:nlsdata2.obj
 0003:001813a8       ___lc_id                   301e33a8     LIBCMTD:nlsdata3.obj
 0003:001813f4       __stdbuf                   301e33f4     LIBCMTD:_sftbuf.obj
 0003:00181400       __newmode                  301e3400     LIBCMTD:_newmode.obj
 0003:00181404       ?_pnhHeap@@3P6AHI@ZA       301e3404     LIBCMTD:handler.obj
 0003:00181540       _itemParseKeywordHash      301e3540     <common>
 0003:00181d40       _Menus                     301e3d40     <common>
 0003:0018be40       _g_nameBind1               301ede40     <common>
 0003:0018be60       _g_nameBind2               301ede60     <common>
 0003:0018be80       _menuParseKeywordHash      301ede80     <common>
 0003:0018c680       _menuStack                 301ee680     <common>
 0003:0018c6c0       _headModelVoiceChat        301ee6c0     <common>
 0003:0018d7c0       _voiceChatLists            301ef7c0     <common>
 0003:003b6200       _voiceChatBuffer           30418200     <common>
 0003:003b8900       _cg_freeMarkPolys          3041a900     <common>
 0003:003b8904       _active_particles          3041a904     <common>
 0003:003b8920       _cg_markPolys              3041a920     <common>
 0003:003ca920       _oldtime                   3042c920     <common>
 0003:003ca930       _rup                       3042c930     <common>
 0003:003ca940       _particles                 3042c940     <common>
 0003:003e9940       _rright                    3044b940     <common>
 0003:003e994c       _free_particles            3044b94c     <common>
 0003:003e9950       _rforward                  3044b950     <common>
 0003:003e9960       _pvright                   3044b960     <common>
 0003:003e9970       _pvforward                 3044b970     <common>
 0003:003e9980       _cg_activeMarkPolys        3044b980     <common>
 0003:003e9aa0       _pvup                      3044baa0     <common>
 0003:003e9ac0       _cg_trueLightning          3044bac0     <common>
 0003:003e9be0       _cg_weapons                3044bbe0     <common>
 0003:003ea460       _cg_timescaleFadeEnd       3044c460     <common>
 0003:003ea580       _cg_drawTeamOverlay        3044c580     <common>
 0003:003ea6a0       _cg_gun_y                  3044c6a0     <common>
 0003:003ea7c0       _cg_oldRail                3044c7c0     <common>
 0003:003ea8e0       _cg_noTaunt                3044c8e0     <common>
 0003:003eaa00       _cg_animSpeed              3044ca00     <common>
 0003:003eab20       _cg_stats                  3044cb20     <common>
 0003:003eac40       _cg_drawRewards            3044cc40     <common>
 0003:003ead60       _cg_scorePlum              3044cd60     <common>
 0003:003eae80       _cgs                       3044ce80     <common>
 0003:004105a0       _cg_drawFPS                304725a0     <common>
 0003:004106c0       _cg_thirdPerson            304726c0     <common>
 0003:004107e0       _cg_zoomFov                304727e0     <common>
 0003:00410900       _cg_drawCrosshair          30472900     <common>
 0003:00410a20       _cg_cameraOrbitDelay       30472a20     <common>
 0003:00410b40       _cg_shadows                30472b40     <common>
 0003:00410c60       _cg_debugAnim              30472c60     <common>
 0003:00410d80       _cg_timescale              30472d80     <common>
 0003:00410ea0       _cg_addMarks               30472ea0     <common>
 0003:00410fc0       _cg_gun_z                  30472fc0     <common>
 0003:004110e0       _pmove_msec                304730e0     <common>
 0003:00411200       _cg_autoswitch             30473200     <common>
 0003:00411320       _cg_noVoiceText            30473320     <common>
 0003:00411440       _cg_drawStatus             30473440     <common>
 0003:00411560       _cg_drawSnapshot           30473560     <common>
 0003:00411680       _cg_gun_frame              30473680     <common>
 0003:004117a0       _cg_runpitch               304737a0     <common>
 0003:004118c0       _cg_railTrailTime          304738c0     <common>
 0003:004119e0       _cg_drawTimer              304739e0     <common>
 0003:00411b00       _cg_drawFriend             30473b00     <common>
 0003:00411c20       _cg_draw2D                 30473c20     <common>
 0003:00411d40       _cg_gun_x                  30473d40     <common>
 0003:00411e60       _cg_drawAmmoWarning        30473e60     <common>
 0003:00411f80       _cg_debugPosition          30473f80     <common>
 0003:004120a0       _cg_cameraMode             304740a0     <common>
 0003:004121c0       _cg_bigFont                304741c0     <common>
 0003:004122e0       _cg_drawGun                304742e0     <common>
 0003:00412400       _cg_swingSpeed             30474400     <common>
 0003:00412520       _cg_centertime             30474520     <common>
 0003:00412640       _cg_forceModel             30474640     <common>
 0003:00412760       _cg_items                  30474760     <common>
 0003:00413f60       _cg_crosshairHealth        30475f60     <common>
 0003:00414080       _cg_noProjectileTrail      30476080     <common>
 0003:004141a0       _cg_crosshairY             304761a0     <common>
 0003:004142c0       _cg_draw3dIcons            304762c0     <common>
 0003:004143e0       _cg_simpleItems            304763e0     <common>
 0003:00414500       _cg_hudFiles               30476500     <common>
 0003:00414620       _cg_tracerChance           30476620     <common>
 0003:00414740       _cg_thirdPersonRange       30476740     <common>
 0003:00414860       _cg_oldPlasma              30476860     <common>
 0003:00414980       _cg_debugEvents            30476980     <common>
 0003:00414aa0       _cg_stereoSeparation       30476aa0     <common>
 0003:00414bc0       _cg_smoothClients          30476bc0     <common>
 0003:00414ce0       _cg_bobroll                30476ce0     <common>
 0003:00414e00       _cg_ignore                 30476e00     <common>
 0003:00414f20       _cg_smallFont              30476f20     <common>
 0003:00415040       _cg_drawCrosshairNames     30477040     <common>
 0003:00415160       _cg_crosshairX             30477160     <common>
 0003:00415280       _cg_footsteps              30477280     <common>
 0003:004153a0       _cg_noVoiceChats           304773a0     <common>
 0003:004154c0       _cg_teamChatTime           304774c0     <common>
 0003:004155e0       _cg_nopredict              304775e0     <common>
 0003:00415700       _cg_buildScript            30477700     <common>
 0003:00415820       _cg_synchronousClients     30477820     <common>
 0003:00415940       _cg_drawAttacker           30477940     <common>
 0003:00415a60       _cg_bobpitch               30477a60     <common>
 0003:00415b80       _cg_lagometer              30477b80     <common>
 0003:00415ca0       _cg_errorDecay             30477ca0     <common>
 0003:00415dc0       _cg_teamChatHeight         30477dc0     <common>
 0003:00415ee0       _cg_pmove_msec             30477ee0     <common>
 0003:00416000       _cg_runroll                30478000     <common>
 0003:00416120       _cg                        30478120     <common>
 0003:00434960       _cg_gibs                   30496960     <common>
 0003:00434a80       _cg_cameraOrbit            30496a80     <common>
 0003:00434ba0       _cg_bobup                  30496ba0     <common>
 0003:00434cc0       _cg_tracerWidth            30496cc0     <common>
 0003:00434de0       _cg_timescaleFadeSpeed     30496de0     <common>
 0003:00434f00       _cg_entities               30496f00     <common>
 0003:004eaf00       _pmove_fixed               3054cf00     <common>
 0003:004eb020       _cg_teamOverlayUserinfo    3054d020     <common>
 0003:004eb140       _cg_brassTime              3054d140     <common>
 0003:004eb260       _cg_blood                  3054d260     <common>
 0003:004eb380       _cg_teamChatsOnly          3054d380     <common>
 0003:004eb4a0       _cg_viewsize               3054d4a0     <common>
 0003:004eb5c0       _cg_deferPlayers           3054d5c0     <common>
 0003:004eb6e0       _cg_showmiss               3054d6e0     <common>
 0003:004eb800       _cg_noPlayerAnims          3054d800     <common>
 0003:004eb920       _cg_crosshairSize          3054d920     <common>
 0003:004eba40       _cg_drawIcons              3054da40     <common>
 0003:004ebb60       _cg_oldRocket              3054db60     <common>
 0003:004ebc80       _cg_predictItems           3054dc80     <common>
 0003:004ebda0       _cg_fov                    3054dda0     <common>
 0003:004ebec0       _cg_paused                 3054dec0     <common>
 0003:004ebfe0       _cg_thirdPersonAngle       3054dfe0     <common>
 0003:004ec100       _cg_tracerLength           3054e100     <common>
 0003:004ec220       _cg_localEntities          3054e220     <common>
 0003:00510a20       _cg_freeLocalEntities      30572a20     <common>
 0003:00510a40       _cg_activeLocalEntities    30572a40     <common>
 0003:00510b80       _lagometer                 30572b80     <common>
 0003:005111a0       _sortedTeamPlayers         305731a0     <common>
 0003:00511220       _teamChat1                 30573220     <common>
 0003:00511320       _numSortedTeamPlayers      30573320     <common>
 0003:00511340       _systemChat                30573340     <common>
 0003:00511440       _teamChat2                 30573440     <common>
 0003:00511540       _pml                       30573540     <common>
 0003:005115cc       _pm                        305735cc     <common>
 0003:005115d0       ___sbh_initialized         305735d0     <common>
 0003:005115d4       ___sbh_pHeaderDefer        305735d4     <common>
 0003:005115d8       ___sbh_cntHeaderList       305735d8     <common>
 0003:005115dc       ___sbh_pHeaderList         305735dc     <common>
 0003:005115e0       ___sbh_threshold           305735e0     <common>
 0003:005115e4       ___sbh_pHeaderScan         305735e4     <common>
 0003:005115e8       ___sbh_sizeHeaderList      305735e8     <common>
 0003:005115ec       ___sbh_indGroupDefer       305735ec     <common>
 0003:005115f0       ___mblcid                  305735f0     <common>
 0003:005115f4       ___ptmbcinfo               305735f4     <common>
 0003:005115f8       ___ismbcodepage            305735f8     <common>
 0003:00511600       __mbctype                  30573600     <common>
 0003:00511704       ___mbcodepage              30573704     <common>
 0003:00511710       ___mbulinfo                30573710     <common>
 0003:00511720       __mbcasemap                30573720     <common>
 0003:00511820       ___ctype1                  30573820     <common>
 0003:00511824       ___ctype1_refcount         30573824     <common>
 0003:00511828       ___lconv_mon_refcount      30573828     <common>
 0003:0051182c       ___lconv_intl_refcount     3057382c     <common>
 0003:00511830       ___lconv_num_refcount      30573830     <common>
 0003:00511834       __crtheap                  30573834     <common>
 0003:00511838       ___active_heap             30573838     <common>
 0003:0051183c       __nhandle                  3057383c     <common>
 0003:00511840       ___pioinfo                 30573840     <common>
 0003:00511940       __pfnDumpClient            30573940     <common>
 0003:00511944       ___piob                    30573944     <common>
 0003:00511960       __bufin                    30573960     <common>
 0003:00512960       __nstream                  30574960     <common>
 0003:00512964       ___env_initialized         30574964     <common>
 0003:00512968       ___onexitend               30574968     <common>
 0003:0051296c       ___onexitbegin             3057496c     <common>
 0003:00512970       ___mbctype_initialized     30574970     <common>
 0003:00512974       ___use_sse2_mathfcns       30574974     <common>
 0003:00512978       ___sse2_available          30574978     <common>
 0003:0051297c       __pfnReportHook            3057497c     <common>
 0003:00512980       __pReportHookList          30574980     <common>
 0003:00512984       ___setlc_active            30574984     <common>
 0003:00512988       ___unguarded_readlc_active 30574988     <common>
 0003:0051298c       __acmdln                   3057498c     <common>
 0003:00512990       __pRawDllMain              30574990     <common>

 entry point at        0001:0003b590

 Static symbols

 0001:00001880       _PM_WaterJumpMove          30002880 f   bg_pmove.obj
 0001:00001900       _PM_WaterMove              30002900 f   bg_pmove.obj
 0001:00001b40       _VectorLength              30002b40 f   bg_pmove.obj
 0001:00001b90       _PM_Friction               30002b90 f   bg_pmove.obj
 0001:00001d50       _PM_Accelerate             30002d50 f   bg_pmove.obj
 0001:00001e20       _PM_CmdScale               30002e20 f   bg_pmove.obj
 0001:00001f10       _PM_CheckWaterJump         30002f10 f   bg_pmove.obj
 0001:000020b0       _PM_FlyMove                300030b0 f   bg_pmove.obj
 0001:000021c0       _PM_AirMove                300031c0 f   bg_pmove.obj
 0001:00002340       _PM_SetMovementDir         30003340 f   bg_pmove.obj
 0001:00002510       _PM_GrappleMove            30003510 f   bg_pmove.obj
 0001:00002670       _PM_WalkMove               30003670 f   bg_pmove.obj
 0001:00002a40       _PM_CheckJump              30003a40 f   bg_pmove.obj
 0001:00002b50       _PM_ForceLegsAnim          30003b50 f   bg_pmove.obj
 0001:00002b80       _PM_StartLegsAnim          30003b80 f   bg_pmove.obj
 0001:00002be0       _PM_DeadMove               30003be0 f   bg_pmove.obj
 0001:00002cc0       _PM_NoclipMove             30003cc0 f   bg_pmove.obj
 0001:00002f60       _PM_GroundTrace            30003f60 f   bg_pmove.obj
 0001:00003270       _PM_CrashLand              30004270 f   bg_pmove.obj
 0001:00003470       _PM_FootstepForSurface     30004470 f   bg_pmove.obj
 0001:000034b0       _PM_CorrectAllSolid        300044b0 f   bg_pmove.obj
 0001:000036a0       _PM_GroundTraceMissed      300046a0 f   bg_pmove.obj
 0001:000037f0       _PM_SetWaterLevel          300047f0 f   bg_pmove.obj
 0001:00003960       _PM_CheckDuck              30004960 f   bg_pmove.obj
 0001:00003c30       _PM_Footsteps              30004c30 f   bg_pmove.obj
 0001:00003ea0       _PM_ContinueLegsAnim       30004ea0 f   bg_pmove.obj
 0001:00003ef0       _PM_WaterEvents            30004ef0 f   bg_pmove.obj
 0001:00003f90       _PM_TorsoAnimation         30004f90 f   bg_pmove.obj
 0001:00003fe0       _PM_ContinueTorsoAnim      30004fe0 f   bg_pmove.obj
 0001:00004030       _PM_StartTorsoAnim         30005030 f   bg_pmove.obj
 0001:00004080       _PM_Weapon                 30005080 f   bg_pmove.obj
 0001:000044c0       _PM_BeginWeaponChange      300054c0 f   bg_pmove.obj
 0001:00004550       _PM_FinishWeaponChange     30005550 f   bg_pmove.obj
 0001:000045f0       _PM_Animate                300055f0 f   bg_pmove.obj
 0001:00004640       _PM_DropTimers             30005640 f   bg_pmove.obj
 0001:00005060       _CrossProduct              30006060 f   bg_slidemove.obj
 0001:00005550       _CG_SizeUp_f               30006550 f   cg_consolecmds.obj
 0001:00005590       _CG_SizeDown_f             30006590 f   cg_consolecmds.obj
 0001:000055d0       _CG_Viewpos_f              300065d0 f   cg_consolecmds.obj
 0001:00005620       _CG_ScoresDown_f           30006620 f   cg_consolecmds.obj
 0001:00005690       _CG_ScoresUp_f             30006690 f   cg_consolecmds.obj
 0001:000056c0       _CG_TellTarget_f           300066c0 f   cg_consolecmds.obj
 0001:00005730       _CG_TellAttacker_f         30006730 f   cg_consolecmds.obj
 0001:000057a0       _CG_VoiceTellTarget_f      300067a0 f   cg_consolecmds.obj
 0001:00005810       _CG_VoiceTellAttacker_f    30006810 f   cg_consolecmds.obj
 0001:00005880       _CG_StartOrbit_f           30006880 f   cg_consolecmds.obj
 0001:000062e0       _CG_Draw2D                 300072e0 f   cg_draw.obj
 0001:000063d0       _CG_DrawStatusBar          300073d0 f   cg_draw.obj
 0001:000067b0       _CG_DrawField              300077b0 f   cg_draw.obj
 0001:000069b0       _CG_DrawStatusBarHead      300079b0 f   cg_draw.obj
 0001:00006cf0       _CG_DrawStatusBarFlag      30007cf0 f   cg_draw.obj
 0001:00006d30       _CG_DrawUpperRight         30007d30 f   cg_draw.obj
 0001:00006dd0       _CG_DrawAttacker           30007dd0 f   cg_draw.obj
 0001:00006f10       _CG_DrawSnapshot           30007f10 f   cg_draw.obj
 0001:00006fa0       _CG_DrawFPS                30007fa0 f   cg_draw.obj
 0001:000070b0       _CG_DrawTimer              300080b0 f   cg_draw.obj
 0001:00007180       _CG_DrawTeamOverlay        30008180 f   cg_draw.obj
 0001:000076c0       _CG_DrawLowerRight         300086c0 f   cg_draw.obj
 0001:00007720       _CG_DrawScores             30008720 f   cg_draw.obj
 0001:00007d90       _CG_DrawPowerups           30008d90 f   cg_draw.obj
 0001:00008160       _CG_DrawLowerLeft          30009160 f   cg_draw.obj
 0001:000081c0       _CG_DrawPickupItem         300091c0 f   cg_draw.obj
 0001:000082a0       _CG_DrawTeamInfo           300092a0 f   cg_draw.obj
 0001:000084c0       _CG_DrawHoldableItem       300094c0 f   cg_draw.obj
 0001:00008520       _CG_DrawReward             30009520 f   cg_draw.obj
 0001:00008740       _CG_DrawLagometer          30009740 f   cg_draw.obj
 0001:00008b00       _CG_DrawDisconnect         30009b00 f   cg_draw.obj
 0001:00008bd0       _CG_DrawCenterString       30009bd0 f   cg_draw.obj
 0001:00008d70       _CG_DrawCrosshair          30009d70 f   cg_draw.obj
 0001:00008f00       _CG_DrawCrosshairNames     30009f00 f   cg_draw.obj
 0001:00008fe0       _CG_ScanForCrosshairEntity 30009fe0 f   cg_draw.obj
 0001:000090c0       _CG_DrawSpectator          3000a0c0 f   cg_draw.obj
 0001:00009140       _CG_DrawVote               3000a140 f   cg_draw.obj
 0001:000091f0       _CG_DrawTeamVote           3000a1f0 f   cg_draw.obj
 0001:000092f0       _CG_DrawScoreboard         3000a2f0 f   cg_draw.obj
 0001:00009310       _CG_DrawIntermission       3000a310 f   cg_draw.obj
 0001:00009350       _CG_DrawFollow             3000a350 f   cg_draw.obj
 0001:00009420       _CG_DrawAmmoWarning        3000a420 f   cg_draw.obj
 0001:000094a0       _CG_DrawWarmup             3000a4a0 f   cg_draw.obj
 0001:00009840       _CG_DrawTourneyScoreboard  3000a840 f   cg_draw.obj
 0001:0000a060       _CG_TileClearBox           3000b060 f   cg_drawtools.obj
 0001:0000a430       _UI_DrawBannerString2      3000b430 f   cg_drawtools.obj
 0001:0000a8a0       _UI_DrawProportionalString2 3000b8a0 f   cg_drawtools.obj
 0001:0000c830       _CG_CalcEntityLerpPositions 3000d830 f   cg_ents.obj
 0001:0000c940       _CG_InterpolateEntityPosition 3000d940 f   cg_ents.obj
 0001:0000ca80       _CG_AddCEntity             3000da80 f   cg_ents.obj
 0001:0000cbb0       _CG_EntityEffects          3000dbb0 f   cg_ents.obj
 0001:0000ccc0       _CG_General                3000dcc0 f   cg_ents.obj
 0001:0000cdd0       _CG_Speaker                3000ddd0 f   cg_ents.obj
 0001:0000ce90       _CG_Item                   3000de90 f   cg_ents.obj
 0001:0000d4f0       _CG_Missile                3000e4f0 f   cg_ents.obj
 0001:0000d7b0       _CG_Grapple                3000e7b0 f   cg_ents.obj
 0001:0000d920       _CG_Mover                  3000e920 f   cg_ents.obj
 0001:0000da60       _CG_Portal                 3000ea60 f   cg_ents.obj
 0001:0000dba0       _CrossProduct              3000eba0 f   cg_ents.obj
 0001:0000dc10       _CG_TeamBase               3000ec10 f   cg_ents.obj
 0001:0000f520       _CG_Obituary               30010520 f   cg_event.obj
 0001:0000fa70       _CG_UseItem                30010a70 f   cg_event.obj
 0001:0000fb90       _CG_ItemPickup             30010b90 f   cg_event.obj
 0001:00010410       _CG_DrawLoadingIcons       30011410 f   cg_info.obj
 0001:000110e0       _VectorLength              300120e0 f   cg_localents.obj
 0001:00011130       _CrossProduct              30012130 f   cg_localents.obj
 0001:000112c0       _CG_AddMoveScaleFade       300122c0 f   cg_localents.obj
 0001:00011410       _CG_AddScaleFade           30012410 f   cg_localents.obj
 0001:000114f0       _CG_AddFallScaleFade       300124f0 f   cg_localents.obj
 0001:000115f0       _CG_AddExplosion           300125f0 f   cg_localents.obj
 0001:000116d0       _CG_AddSpriteExplosion     300126d0 f   cg_localents.obj
 0001:00011b40       _CG_ForceModelChange       30012b40 f   cg_main.obj
 0001:00012130       _CG_RegisterSounds         30013130 f   cg_main.obj
 0001:000129b0       _CG_RegisterItemSounds     300139b0 f   cg_main.obj
 0001:00012ad0       _CG_RegisterGraphics       30013ad0 f   cg_main.obj
 0001:00013370       _CG_RegisterClients        30014370 f   cg_main.obj
 0001:00013a30       _CrossProduct              30014a30 f   cg_marks.obj
 0001:00016060       _Distance                  30017060 f   cg_marks.obj
 0001:000160b0       _VectorLength              300170b0 f   cg_marks.obj
 0001:00019190       _CG_ColorFromString        3001a190 f   cg_players.obj
 0001:00019230       _CG_LoadClientInfo         3001a230 f   cg_players.obj
 0001:00019560       _CG_RegisterClientModelname 3001a560 f   cg_players.obj
 0001:000199d0       _CG_ParseAnimationFile     3001a9d0 f   cg_players.obj
 0001:0001a220       _CG_FindClientHeadFile     3001b220 f   cg_players.obj
 0001:0001a470       _CG_FileExists             3001b470 f   cg_players.obj
 0001:0001a4b0       _CG_RegisterClientSkin     3001b4b0 f   cg_players.obj
 0001:0001a610       _CG_FindClientModelFile    3001b610 f   cg_players.obj
 0001:0001a850       _CG_ScanForExistingClientInfo 3001b850 f   cg_players.obj
 0001:0001a9c0       _CG_CopyClientInfoModel    3001b9c0 f   cg_players.obj
 0001:0001ab00       _CG_SetDeferredClientInfo  3001bb00 f   cg_players.obj
 0001:0001b3d0       _CG_PlayerAnimation        3001c3d0 f   cg_players.obj
 0001:0001b530       _CG_RunLerpFrame           3001c530 f   cg_players.obj
 0001:0001b7b0       _CG_SetLerpFrameAnimation  3001c7b0 f   cg_players.obj
 0001:0001b840       _CG_PlayerAngles           3001c840 f   cg_players.obj
 0001:0001bbe0       _CG_SwingAngles            3001cbe0 f   cg_players.obj
 0001:0001bdc0       _CG_AddPainTwitch          3001cdc0 f   cg_players.obj
 0001:0001be40       _CG_PlayerPowerups         3001ce40 f   cg_players.obj
 0001:0001c070       _CG_HasteTrail             3001d070 f   cg_players.obj
 0001:0001c170       _CG_TrailItem              3001d170 f   cg_players.obj
 0001:0001c290       _CG_PlayerFlag             3001d290 f   cg_players.obj
 0001:0001c6f0       _CG_PlayerSprites          3001d6f0 f   cg_players.obj
 0001:0001c880       _CG_PlayerFloatSprite      3001d880 f   cg_players.obj
 0001:0001c950       _CG_PlayerShadow           3001d950 f   cg_players.obj
 0001:0001caa0       _CG_PlayerSplash           3001daa0 f   cg_players.obj
 0001:0001cf30       _CG_ClearLerpFrame         3001df30 f   cg_players.obj
 0001:0001d360       _VectorLength              3001e360 f   cg_playerstate.obj
 0001:0001dbe0       _pushReward                3001ebe0 f   cg_playerstate.obj
 0001:0001df10       _CG_ClipMoveToEntities     3001ef10 f   cg_predict.obj
 0001:0001e820       _VectorCompare             3001f820 f   cg_predict.obj
 0001:0001e880       _VectorLength              3001f880 f   cg_predict.obj
 0001:0001e8d0       _CG_InterpolatePlayerState 3001f8d0 f   cg_predict.obj
 0001:0001ea80       _CG_TouchTriggerPrediction 3001fa80 f   cg_predict.obj
 0001:0001ebd0       _CG_TouchItem              3001fbd0 f   cg_predict.obj
 0001:0001f340       _CG_DrawClientScore        30020340 f   cg_scoreboard.obj
 0001:0001f9a0       _CG_TeamScoreboard         300209a0 f   cg_scoreboard.obj
 0001:0001fd50       _CG_CenterGiantLine        30020d50 f   cg_scoreboard.obj
 0001:00020dc0       _CG_ServerCommand          30021dc0 f   cg_servercmds.obj
 0001:000210d0       _CG_ParseScores            300220d0 f   cg_servercmds.obj
 0001:00021420       _CG_ParseTeamInfo          30022420 f   cg_servercmds.obj
 0001:00021570       _CG_ConfigStringModified   30022570 f   cg_servercmds.obj
 0001:00021880       _CG_ParseWarmup            30022880 f   cg_servercmds.obj
 0001:000218f0       _CG_AddToTeamChat          300228f0 f   cg_servercmds.obj
 0001:00021b20       _CG_MapRestart             30022b20 f   cg_servercmds.obj
 0001:00021be0       _CG_RemoveChatEscapeChar   30022be0 f   cg_servercmds.obj
 0001:00021d50       _CG_ResetEntity            30022d50 f   cg_snapshot.obj
 0001:00021f60       _CG_TransitionSnapshot     30022f60 f   cg_snapshot.obj
 0001:00022140       _CG_TransitionEntity       30023140 f   cg_snapshot.obj
 0001:000221b0       _CG_SetNextSnap            300231b0 f   cg_snapshot.obj
 0001:00022330       _CG_ReadNextSnapshot       30023330 f   cg_snapshot.obj
 0001:00023960       _CG_AddTestModel           30024960 f   cg_view.obj
 0001:00023ad0       _CG_DamageBlendBlob        30024ad0 f   cg_view.obj
 0001:00023c80       _CG_CalcViewValues         30024c80 f   cg_view.obj
 0001:00023f10       _CG_CalcVrect              30024f10 f   cg_view.obj
 0001:00024000       _CG_OffsetThirdPersonView  30025000 f   cg_view.obj
 0001:00024350       _CG_OffsetFirstPersonView  30025350 f   cg_view.obj
 0001:00024740       _CG_StepOffset             30025740 f   cg_view.obj
 0001:00024790       _CG_CalcFov                30025790 f   cg_view.obj
 0001:000249d0       _CG_PowerupTimerSounds     300259d0 f   cg_view.obj
 0001:00024a80       _CG_PlayBufferedSounds     30025a80 f   cg_view.obj
 0001:000253d0       _Distance                  300263d0 f   cg_weapons.obj
 0001:00025420       _VectorLength              30026420 f   cg_weapons.obj
 0001:00025d00       _CG_MachineGunEjectBrass   30026d00 f   cg_weapons.obj
 0001:00026080       _CG_ShotgunEjectBrass      30027080 f   cg_weapons.obj
 0001:00026470       _CG_RocketTrail            30027470 f   cg_weapons.obj
 0001:00026600       _CG_PlasmaTrail            30027600 f   cg_weapons.obj
 0001:00026a30       _CG_GrenadeTrail           30027a30 f   cg_weapons.obj
 0001:00027110       _CG_LightningBolt          30028110 f   cg_weapons.obj
 0001:00027590       _CG_SpawnRailTrail         30028590 f   cg_weapons.obj
 0001:00027600       _CG_MachinegunSpinAngle    30028600 f   cg_weapons.obj
 0001:000276f0       _CG_AddWeaponWithPowerups  300286f0 f   cg_weapons.obj
 0001:00027aa0       _CG_MapTorsoToWeaponFrame  30028aa0 f   cg_weapons.obj
 0001:00027b50       _CG_CalculateWeaponPosition 30028b50 f   cg_weapons.obj
 0001:00027fd0       _CG_WeaponSelectable       30028fd0 f   cg_weapons.obj
 0001:00028930       _CG_ShotgunPattern         30029930 f   cg_weapons.obj
 0001:00028a60       _CrossProduct              30029a60 f   cg_weapons.obj
 0001:00028ad0       _CG_ShotgunPellet          30029ad0 f   cg_weapons.obj
 0001:00029190       _CG_CalcMuzzlePoint        3002a190 f   cg_weapons.obj
 0001:00029790       _CrossProduct              3002a790 f   q_math.obj
 0001:0002a5e0       _VectorLength              3002b5e0 f   q_math.obj
 0001:0002b7c0       _SkipWhitespace            3002c7c0 f   q_shared.obj
 0001:0002cb60       _hashForString             3002db60 f   ui_shared.obj
 0001:0002e600       _Menu_RunCloseScript       3002f600 f   ui_shared.obj
 0001:00031530       _Scroll_ListBox_AutoFunc   30032530 f   ui_shared.obj
 0001:000315d0       _Scroll_ListBox_ThumbFunc  300325d0 f   ui_shared.obj
 0001:00031870       _Scroll_Slider_ThumbFunc   30032870 f   ui_shared.obj
 0001:00032040       _Display_CloseCinematics   30033040 f   ui_shared.obj
 0001:00032090       _Menu_CloseCinematics      30033090 f   ui_shared.obj
 0001:00032130       _Window_CloseCinematic     30033130 f   ui_shared.obj
 0001:00032900       _Item_CorrectedTextRect    30033900 f   ui_shared.obj
 0001:00033cc0       _Controls_GetKeyAssignment 30034cc0 f   ui_shared.obj
 0001:00038fe0       _Menu_CacheContents        30039fe0 f   ui_shared.obj
 0001:00039080       _Window_CacheContents      3003a080 f   ui_shared.obj
 0001:000390e0       _Item_CacheContents        3003a0e0 f   ui_shared.obj
 0001:00039110       _Menu_OverActiveItem       3003a110 f   ui_shared.obj
 0001:0003a2a0       _$$$00001                  3003b2a0 f   LIBCMTD:strchr.obj
 0001:0003ba80       __cftoe2                   3003ca80 f   LIBCMTD:cvt.obj
 0001:0003bc70       __cftof2                   3003cc70 f   LIBCMTD:cvt.obj
 0001:0003bf10       __shift                    3003cf10 f   LIBCMTD:cvt.obj
 0001:0003c033       _$$$00003                  3003d033 f   LIBCMTD:87disp.obj
 0001:0003d480       __get_fname                3003e480 f   LIBCMTD:fpexcept.obj
 0001:0003dc10       ___updatetlocinfo_lk       3003ec10 f   LIBCMTD:setlocal.obj
 0001:0003e000       __setlocale_lk             3003f000 f   LIBCMTD:setlocal.obj
 0001:0003e3b0       __setlocale_set_cat        3003f3b0 f   LIBCMTD:setlocal.obj
 0001:0003e780       __setlocale_get_all        3003f780 f   LIBCMTD:setlocal.obj
 0001:00040250       _write_char                30041250 f   LIBCMTD:output.obj
 0001:000402f0       _write_multi_char          300412f0 f   LIBCMTD:output.obj
 0001:00040330       _write_string              30041330 f   LIBCMTD:output.obj
 0001:000403a0       _get_int_arg               300413a0 f   LIBCMTD:output.obj
 0001:000403c0       _get_int64_arg             300413c0 f   LIBCMTD:output.obj
 0001:000403e0       _get_short_arg             300413e0 f   LIBCMTD:output.obj
 0001:00040bd0       _CrtMessageWindow          30041bd0 f   LIBCMTD:dbgrpt.obj
 0001:00041a00       _has_osfxsr_set            30042a00 f   LIBCMTD:cpu_disp.obj
 0001:00041bd0       _$$$00001                  30042bd0 f   LIBCMTD:87triga.obj
 0001:00042000       _doexit                    30043000 f   LIBCMTD:crt0dat.obj
 0001:000421a0       __initterm                 300431a0 f   LIBCMTD:crt0dat.obj
 0001:000421d0       __initterm_e               300431d0 f   LIBCMTD:crt0dat.obj
 0001:00042480       _ctrlevent_capture@4       30043480 f   LIBCMTD:winsig.obj
 0001:000427b0       _siglookup                 300437b0 f   LIBCMTD:winsig.obj
 0001:000429f0       _xtoa                      300439f0 f   LIBCMTD:xtoa.obj
 0001:00042b70       _x64toa@20                 30043b70 f   LIBCMTD:xtoa.obj
 0001:00042f70       _flsall                    30043f70 f   LIBCMTD:fflush.obj
 0001:000435e0       _report_failure            300445e0 f   LIBCMTD:secchk.obj
 0001:00043bc0       _strncnt                   30044bc0 f   LIBCMTD:a_map.obj
 0001:000441c0       _realloc_help              300451c0 f   LIBCMTD:dbgheap.obj
 0001:00044f00       _CheckBytes                30045f00 f   LIBCMTD:dbgheap.obj
 0001:00045c50       __printMemBlockData        30046c50 f   LIBCMTD:dbgheap.obj
 0001:00046a70       _parse_cmdline             30047a70 f   LIBCMTD:stdargv.obj
 0001:00047450       _xcptlookup                30048450 f   LIBCMTD:winxfltr.obj
 0001:000474bc       $$$00001                   300484bc f   LIBCMTD:exsup.obj
 0001:000474dc       __unwind_handler           300484dc f   LIBCMTD:exsup.obj
 0001:000474dc       $$$00003                   300484dc f   LIBCMTD:exsup.obj
 0001:000474fe       $$$00005                   300484fe f   LIBCMTD:exsup.obj
 0001:00047566       $$$00007                   30048566 f   LIBCMTD:exsup.obj
 0001:000475aa       $$$00011                   300485aa f   LIBCMTD:exsup.obj
 0001:000476b5       $$$00003                   300486b5 f   LIBCMTD:exsup3.obj
 0001:00047a70       __abstract_cw              30048a70 f   LIBCMTD:ieee87.obj
 0001:00047bc0       __hw_cw                    30048bc0 f   LIBCMTD:ieee87.obj
 0001:00047d20       __abstract_sw              30048d20 f   LIBCMTD:ieee87.obj
 0001:0004a070       __expandtime               3004b070 f   LIBCMTD:strftime.obj
 0001:0004a650       __store_str                3004b650 f   LIBCMTD:strftime.obj
 0001:0004a6a0       __store_num                3004b6a0 f   LIBCMTD:strftime.obj
 0001:0004a750       __store_number             3004b750 f   LIBCMTD:strftime.obj
 0001:0004a800       __store_winword            3004b800 f   LIBCMTD:strftime.obj
 0001:0004b160       __get_lc_time              3004c160 f   LIBCMTD:inittime.obj
 0001:0004bca0       _fix_grouping              3004cca0 f   LIBCMTD:initnum.obj
 0001:0004c140       _fix_grouping              3004d140 f   LIBCMTD:initmon.obj
 0001:0004cd40       _TranslateName             3004dd40 f   LIBCMTD:getqloc.obj
 0001:0004cdd0       _GetLcidFromLangCountry    3004ddd0 f   LIBCMTD:getqloc.obj
 0001:0004ce90       _LangCountryEnumProc@4     3004de90 f   LIBCMTD:getqloc.obj
 0001:0004d210       _GetLcidFromLanguage       3004e210 f   LIBCMTD:getqloc.obj
 0001:0004d280       _LanguageEnumProc@4        3004e280 f   LIBCMTD:getqloc.obj
 0001:0004d3d0       _GetLcidFromCountry        3004e3d0 f   LIBCMTD:getqloc.obj
 0001:0004d420       _CountryEnumProc@4         3004e420 f   LIBCMTD:getqloc.obj
 0001:0004d4f0       _GetLcidFromDefault        3004e4f0 f   LIBCMTD:getqloc.obj
 0001:0004d520       _ProcessCodePage           3004e520 f   LIBCMTD:getqloc.obj
 0001:0004d5d0       _TestDefaultCountry        3004e5d0 f   LIBCMTD:getqloc.obj
 0001:0004d620       _TestDefaultLanguage       3004e620 f   LIBCMTD:getqloc.obj
 0001:0004d6c0       _crtGetLocaleInfoA@16      3004e6c0 f   LIBCMTD:getqloc.obj
 0001:0004d850       _LcidFromHexString         3004e850 f   LIBCMTD:getqloc.obj
 0001:0004d8d0       _GetPrimaryLen             3004e8d0 f   LIBCMTD:getqloc.obj
 0001:0004dbe0       _getSystemCP               3004ebe0 f   LIBCMTD:mbctype.obj
 0001:0004dc40       __setmbcp_lk               3004ec40 f   LIBCMTD:mbctype.obj
 0001:0004df30       _CPtoLCID                  3004ef30 f   LIBCMTD:mbctype.obj
 0001:0004dfb0       _setSBCS                   3004efb0 f   LIBCMTD:mbctype.obj
 0001:0004e030       _setSBUpLow                3004f030 f   LIBCMTD:mbctype.obj
 0001:0004ee90       __onexit_lk                3004fe90 f   LIBCMTD:onexit.obj
 0001:00052170       ___crtInitCritSecNoSpinCount@8 30053170 f   LIBCMTD:initcrit.obj
 0001:00053330       __tzset_lk                 30054330 f   LIBCMTD:tzset.obj
 0001:000537c0       __isindst_lk               300547c0 f   LIBCMTD:tzset.obj
 0001:00053a90       _cvtdate                   30054a90 f   LIBCMTD:tzset.obj
 0001:000559a0       _strncnt                   300569a0 f   LIBCMTD:a_cmp.obj
 0001:00055d70       _findenv                   30056d70 f   LIBCMTD:setenv.obj
 0001:00055df0       _copy_environ              30056df0 f   LIBCMTD:setenv.obj
